 ftdi_ser

 Timestamp is 54f4635d (Mon Mar 02 13:19:25 2015)

 Preferred load address is 10000000

 Start         Length     Name                   Class
 0001:00000000 0000dd30H .rdata                  CODE
 0001:0000dd30 00000038H .rdata$debug            CODE
 0001:0000dd70 00000004H .rdata$sxdata           CODE
 0001:0000dd74 00017a02H .text                   CODE
 0001:00025778 0000016cH .xdata$x                CODE
 0001:000258e4 0000003cH .idata$2                CODE
 0001:00025920 00000014H .idata$3                CODE
 0001:00025934 00000160H .idata$4                CODE
 0001:00025a94 00000032H .idata$6                CODE
 0001:00025ad0 00000156H .edata                  CODE
 0002:00000000 00000160H .idata$5                DATA
 0002:00000160 00000568H .data                   DATA
 0002:000006e0 00001778H .bss                    DATA
 0003:00000000 00000058H .rsrc$01                DATA
 0003:00000060 00000328H .rsrc$02                DATA

  Address         Publics by Value              Rva+Base       Lib:Object

 0000:00000001       ___safe_se_handler_count   00000001     <absolute>
 0001:000002e8       ??_C@_0O@LCBLIIOL@IRP_MJ_CREATE?$AA@ 100012e8     mdd.obj
 0001:000002f8       ??_C@_0BJ@MMKIHFHH@IRP_MJ_CREATE_NAMED_PIPE?$AA@ 100012f8     mdd.obj
 0001:00000314       ??_C@_0N@FMCDOLCP@IRP_MJ_CLOSE?$AA@ 10001314     mdd.obj
 0001:00000324       ??_C@_0M@LJKCMGIA@IRP_MJ_READ?$AA@ 10001324     mdd.obj
 0001:00000330       ??_C@_0N@DLJAMLBI@IRP_MJ_WRITE?$AA@ 10001330     mdd.obj
 0001:00000340       ??_C@_0BJ@FPMLIFJJ@IRP_MJ_QUERY_INFORMATION?$AA@ 10001340     mdd.obj
 0001:0000035c       ??_C@_0BH@GNAPBNMO@IRP_MJ_SET_INFORMATION?$AA@ 1000135c     mdd.obj
 0001:00000374       ??_C@_0BA@LFPMCNA@IRP_MJ_QUERY_EA?$AA@ 10001374     mdd.obj
 0001:00000384       ??_C@_0O@FPNILENL@IRP_MJ_SET_EA?$AA@ 10001384     mdd.obj
 0001:00000394       ??_C@_0BF@CBDAKCPM@IRP_MJ_FLUSH_BUFFERS?$AA@ 10001394     mdd.obj
 0001:000003ac       ??_C@_0CA@FDGJPBOD@IRP_MJ_QUERY_VOLUME_INFORMATION?$AA@ 100013ac     mdd.obj
 0001:000003cc       ??_C@_0BO@CJJMMMF@IRP_MJ_SET_VOLUME_INFORMATION?$AA@ 100013cc     mdd.obj
 0001:000003ec       ??_C@_0BJ@NCGIANAN@IRP_MJ_DIRECTORY_CONTROL?$AA@ 100013ec     mdd.obj
 0001:00000408       ??_C@_0BL@MFHGBIDL@IRP_MJ_FILE_SYSTEM_CONTROL?$AA@ 10001408     mdd.obj
 0001:00000424       ??_C@_0BG@HAFCIBGJ@IRP_MJ_DEVICE_CONTROL?$AA@ 10001424     mdd.obj
 0001:0000043c       ??_C@_0BP@ODEFGAEK@IRP_MJ_INTERNAL_DEVICE_CONTROL?$AA@ 1000143c     mdd.obj
 0001:0000045c       ??_C@_0BA@CDMDNOAC@IRP_MJ_SHUTDOWN?$AA@ 1000145c     mdd.obj
 0001:0000046c       ??_C@_0BE@LODBBEFP@IRP_MJ_LOCK_CONTROL?$AA@ 1000146c     mdd.obj
 0001:00000480       ??_C@_0P@JJLCIODE@IRP_MJ_CLEANUP?$AA@ 10001480     mdd.obj
 0001:00000490       ??_C@_0BH@CKPKPKHL@IRP_MJ_CREATE_MAILSLOT?$AA@ 10001490     mdd.obj
 0001:000004a8       ??_C@_0BG@MIODHPEN@IRP_MJ_QUERY_SECURITY?$AA@ 100014a8     mdd.obj
 0001:000004c0       ??_C@_0BE@MPINJCAP@IRP_MJ_SET_SECURITY?$AA@ 100014c0     mdd.obj
 0001:000004d4       ??_C@_0N@BGEEMFOO@IRP_MJ_POWER?$AA@ 100014d4     mdd.obj
 0001:000004e4       ??_C@_0BG@JHIMGJML@IRP_MJ_SYSTEM_CONTROL?$AA@ 100014e4     mdd.obj
 0001:000004fc       ??_C@_0BF@HOMHCDN@IRP_MJ_DEVICE_CHANGE?$AA@ 100014fc     mdd.obj
 0001:00000514       ??_C@_0BD@MDBGANBO@IRP_MJ_QUERY_QUOTA?$AA@ 10001514     mdd.obj
 0001:00000528       ??_C@_0BB@MFPKCKFI@IRP_MJ_SET_QUOTA?$AA@ 10001528     mdd.obj
 0001:0000053c       ??_C@_0L@EACGAIIF@IRP_MJ_PNP?$AA@ 1000153c     mdd.obj
 0001:00000548       ??_C@_0BE@LNOGIHJB@IRP_MN_START_DEVICE?$AA@ 10001548     mdd.obj
 0001:0000055c       ??_C@_0BL@BKMKKOEG@IRP_MN_QUERY_REMOVE_DEVICE?$AA@ 1000155c     mdd.obj
 0001:00000578       ??_C@_0BF@CIDCHGNK@IRP_MN_REMOVE_DEVICE?$AA@ 10001578     mdd.obj
 0001:00000590       ??_C@_0BM@NHOBKHFC@IRP_MN_CANCEL_REMOVE_DEVICE?$AA@ 10001590     mdd.obj
 0001:000005ac       ??_C@_0BD@OKOEKPNG@IRP_MN_STOP_DEVICE?$AA@ 100015ac     mdd.obj
 0001:000005c0       ??_C@_0BJ@DBBODAKD@IRP_MN_QUERY_STOP_DEVICE?$AA@ 100015c0     mdd.obj
 0001:000005dc       ??_C@_0BK@IHBBLJPI@IRP_MN_CANCEL_STOP_DEVICE?$AA@ 100015dc     mdd.obj
 0001:000005f8       ??_C@_0BO@EDNJKJCF@IRP_MN_QUERY_DEVICE_RELATIONS?$AA@ 100015f8     mdd.obj
 0001:00000618       ??_C@_0BH@NJFMIPMO@IRP_MN_QUERY_INTERFACE?$AA@ 10001618     mdd.obj
 0001:00000630       ??_C@_0BK@FNPJPCCF@IRP_MN_QUERY_CAPABILITIES?$AA@ 10001630     mdd.obj
 0001:0000064c       ??_C@_0BH@BAILDNEP@IRP_MN_QUERY_RESOURCES?$AA@ 1000164c     mdd.obj
 0001:00000664       ??_C@_0CD@MPPOHAEF@IRP_MN_QUERY_RESOURCE_REQUIREMEN@ 10001664     mdd.obj
 0001:00000688       ??_C@_0BJ@KBKMPMKH@IRP_MN_QUERY_DEVICE_TEXT?$AA@ 10001688     mdd.obj
 0001:000006a4       ??_C@_0CE@FFGNIHMK@IRP_MN_FILTER_RESOURCE_REQUIREME@ 100016a4     mdd.obj
 0001:000006c8       ??_C@_00CNPNBAHC@?$AA@     100016c8     mdd.obj
 0001:000006cc       ??_C@_0BD@KCLCONNF@IRP_MN_READ_CONFIG?$AA@ 100016cc     mdd.obj
 0001:000006e0       ??_C@_0BE@MNGKLJHO@IRP_MN_WRITE_CONFIG?$AA@ 100016e0     mdd.obj
 0001:000006f4       ??_C@_0N@KBDCJDGM@IRP_MN_EJECT?$AA@ 100016f4     mdd.obj
 0001:00000704       ??_C@_0BA@JCIHPHAO@IRP_MN_SET_LOCK?$AA@ 10001704     mdd.obj
 0001:00000714       ??_C@_0BA@MPOLLMHD@IRP_MN_QUERY_ID?$AA@ 10001714     mdd.obj
 0001:00000724       ??_C@_0BO@CLJGNPDL@IRP_MN_QUERY_PNP_DEVICE_STATE?$AA@ 10001724     mdd.obj
 0001:00000744       ??_C@_0BN@FKLLPNEA@IRP_MN_QUERY_BUS_INFORMATION?$AA@ 10001744     mdd.obj
 0001:00000764       ??_C@_0CB@EEGIBKLH@IRP_MN_DEVICE_USAGE_NOTIFICATION@ 10001764     mdd.obj
 0001:00000788       ??_C@_0BI@JJMGKCHF@IRP_MN_SURPRISE_REMOVAL?$AA@ 10001788     mdd.obj
 0001:000007a0       ??_C@_0BH@EHCPJIHK@PowerSystemUnspecified?$AA@ 100017a0     mdd.obj
 0001:000007b8       ??_C@_0BD@IGOFMIAA@PowerSystemWorking?$AA@ 100017b8     mdd.obj
 0001:000007cc       ??_C@_0BF@ODKMAJGJ@PowerSystemSleeping1?$AA@ 100017cc     mdd.obj
 0001:000007e4       ??_C@_0BF@MIIBFKKK@PowerSystemSleeping2?$AA@ 100017e4     mdd.obj
 0001:000007fc       ??_C@_0BF@NBJKGLOL@PowerSystemSleeping3?$AA@ 100017fc     mdd.obj
 0001:00000814       ??_C@_0BF@BLIMNHBE@PowerSystemHibernate?$AA@ 10001814     mdd.obj
 0001:0000082c       ??_C@_0BE@MHPMHFJA@PowerSystemShutdown?$AA@ 1000182c     mdd.obj
 0001:00000840       ??_C@_0BD@IFAENNPE@PowerSystemMaximum?$AA@ 10001840     mdd.obj
 0001:00000854       ??_C@_0BH@GKBPJHKE@PowerDeviceUnspecified?$AA@ 10001854     mdd.obj
 0001:0000086c       ??_C@_0O@GCKIBLHO@PowerDeviceD0?$AA@ 1000186c     mdd.obj
 0001:0000087c       ??_C@_0O@HLLDCKDP@PowerDeviceD1?$AA@ 1000187c     mdd.obj
 0001:0000088c       ??_C@_0O@FAJOHJPM@PowerDeviceD2?$AA@ 1000188c     mdd.obj
 0001:0000089c       ??_C@_0O@EJIFEILN@PowerDeviceD3?$AA@ 1000189c     mdd.obj
 0001:000008ac       ??_C@_0BD@ODMBHIPK@PowerDeviceMaximum?$AA@ 100018ac     mdd.obj
 0001:000008c0       ??_C@_0BP@FLGKAAJA@IOCTL_FT_GET_CONFIG_DESCRIPTOR?$AA@ 100018c0     mdd.obj
 0001:000008e0       ??_C@_0BG@DOCNNGHC@IOCTL_FT_RESET_DEVICE?$AA@ 100018e0     mdd.obj
 0001:000008f8       ??_C@_0BE@FABLCAED@IOCTL_FT_RESET_PIPE?$AA@ 100018f8     mdd.obj
 0001:0000090c       ??_C@_0BB@FBCNPIH@IOCTL_FT_READ_EE?$AA@ 1000190c     mdd.obj
 0001:00000920       ??_C@_0BC@OHPDLGEF@IOCTL_FT_WRITE_EE?$AA@ 10001920     mdd.obj
 0001:00000934       ??_C@_0BC@ELCPKCGN@IOCTL_FT_ERASE_EE?$AA@ 10001934     mdd.obj
 0001:00000948       ??_C@_0CA@IODMOPHM@IOCTL_FT_SET_EVENT_NOTIFICATION?$AA@ 10001948     mdd.obj
 0001:00000968       ??_C@_0BK@EJDPMNCO@IOCTL_FT_GET_EVENT_STATUS?$AA@ 10001968     mdd.obj
 0001:00000984       ??_C@_0BE@EMGAIAOB@IOCTL_FT_GET_STATUS?$AA@ 10001984     mdd.obj
 0001:00000998       ??_C@_0BF@JGFBPKNP@IOCTL_FT_SET_DIVISOR?$AA@ 10001998     mdd.obj
 0001:000009b0       ??_C@_0BL@HCANEGKH@IOCTL_FT_GET_SERIAL_NUMBER?$AA@ 100019b0     mdd.obj
 0001:000009cc       ??_C@_0BJ@OLKCOGMM@IOCTL_FT_GET_DESCRIPTION?$AA@ 100019cc     mdd.obj
 0001:000009e8       ??_C@_0BJ@JDPGMLEJ@IOCTL_FT_GET_LOCATION_ID?$AA@ 100019e8     mdd.obj
 0001:00000a04       ??_C@_0BH@EJPDLGOK@IOCTL_FT_SET_BAUD_RATE?$AA@ 10001a04     mdd.obj
 0001:00000a1c       ??_C@_0BK@PFEMHFKC@IOCTL_FT_SET_LINE_CONTROL?$AA@ 10001a1c     mdd.obj
 0001:00000a38       ??_C@_0BG@IENJBHAC@IOCTL_FT_SET_BREAK_ON?$AA@ 10001a38     mdd.obj
 0001:00000a50       ??_C@_0BH@EGLKABAA@IOCTL_FT_SET_BREAK_OFF?$AA@ 10001a50     mdd.obj
 0001:00000a68       ??_C@_0BG@KHIOGLNM@IOCTL_FT_SET_TIMEOUTS?$AA@ 10001a68     mdd.obj
 0001:00000a80       ??_C@_0BG@NDDAKHJA@IOCTL_FT_GET_TIMEOUTS?$AA@ 10001a80     mdd.obj
 0001:00000a98       ??_C@_0BB@BCOMHHON@IOCTL_FT_SET_DTR?$AA@ 10001a98     mdd.obj
 0001:00000aac       ??_C@_0BB@CNJGOAAI@IOCTL_FT_CLR_DTR?$AA@ 10001aac     mdd.obj
 0001:00000ac0       ??_C@_0BB@HOIFEOOP@IOCTL_FT_SET_RTS?$AA@ 10001ac0     mdd.obj
 0001:00000ad4       ??_C@_0BB@EBPPNJAK@IOCTL_FT_CLR_RTS?$AA@ 10001ad4     mdd.obj
 0001:00000ae8       ??_C@_0BH@LNMCHPLE@IOCTL_FT_SET_WAIT_MASK?$AA@ 10001ae8     mdd.obj
 0001:00000b00       ??_C@_0BG@MMDPJEA@IOCTL_FT_WAIT_ON_MASK?$AA@ 10001b00     mdd.obj
 0001:00000b18       ??_C@_0P@OECEKIHJ@IOCTL_FT_PURGE?$AA@ 10001b18     mdd.obj
 0001:00000b28       ??_C@_0BD@PODBMED@IOCTL_FT_GET_CHARS?$AA@ 10001b28     mdd.obj
 0001:00000b3c       ??_C@_0BD@CBKGDNNB@IOCTL_FT_SET_CHARS?$AA@ 10001b3c     mdd.obj
 0001:00000b50       ??_C@_0BK@LFGFOKIB@IOCTL_FT_SET_FLOW_CONTROL?$AA@ 10001b50     mdd.obj
 0001:00000b6c       ??_C@_0BJ@DLMGBINJ@IOCTL_FT_GET_MODEMSTATUS?$AA@ 10001b6c     mdd.obj
 0001:00000b88       ??_C@_0BJ@OOGKBGBB@IOCTL_FT_GET_QUEUESTATUS?$AA@ 10001b88     mdd.obj
 0001:00000ba4       ??_C@_0BL@NHFHHAA@IOCTL_FT_SET_LATENCY_TIMER?$AA@ 10001ba4     mdd.obj
 0001:00000bc0       ??_C@_0BL@CIHOPMBO@IOCTL_FT_GET_LATENCY_TIMER?$AA@ 10001bc0     mdd.obj
 0001:00000bdc       ??_C@_0BG@GNIFFKPL@IOCTL_FT_SET_BIT_MODE?$AA@ 10001bdc     mdd.obj
 0001:00000bf4       ??_C@_0BG@BJDLJGLH@IOCTL_FT_GET_BIT_MODE?$AA@ 10001bf4     mdd.obj
 0001:00000c0c       ??_C@_0BM@CNPPBJDK@IOCTL_FT_SET_USB_PARAMETERS?$AA@ 10001c0c     mdd.obj
 0001:00000c28       ??_C@_0BI@IGFHGNPP@IOCTL_FT_SET_EVENT_MASK?$AA@ 10001c28     mdd.obj
 0001:00000c40       ??_C@_0BE@IBOFEHFE@IOCTL_FT_WAIT_EVENT?$AA@ 10001c40     mdd.obj
 0001:00000c54       ??_C@_0BF@NJHOHKAI@IOCTL_FT_CLEAR_ERROR?$AA@ 10001c54     mdd.obj
 0001:00000c6c       ??_C@_0BD@JPHFIMKM@IOCTL_FT_SET_STATE?$AA@ 10001c6c     mdd.obj
 0001:00000c80       ??_C@_0BD@LBDAKNDO@IOCTL_FT_GET_STATE?$AA@ 10001c80     mdd.obj
 0001:00000c94       ??_C@_0BJ@NCPCPEG@IOCTL_FT_GET_DEVICE_INFO?$AA@ 10001c94     mdd.obj
 0001:00000cb0       ??_C@_0BG@BCAAJPHH@IOCTL_FT_STOP_IN_TASK?$AA@ 10001cb0     mdd.obj
 0001:00000cc8       ??_C@_0BJ@PKEBDLPL@IOCTL_FT_RESTART_IN_TASK?$AA@ 10001cc8     mdd.obj
 0001:00000ce4       ??_C@_0CE@GEOHMJN@IOCTL_FT_SET_RESET_PIPE_RETRY_CO@ 10001ce4     mdd.obj
 0001:00000d08       ??_C@_1MA@IKEHAPG@?$AAc?$AA?3?$AA?2?$AAw?$AAi?$AAn?$AAc?$AAe?$AA8?$AA0?$AA0?$AA?2?$AAo?$AAs?$AAd?$AAe?$AAs?$AAi?$AAg?$AAn?$AAs?$AA?2?$AAv?$AAc?$AAp?$AAo?$AAs?$AAc?$AAe?$AAp?$AAc?$AA?2@ 10001d08     mdd.obj
 0001:00000dc8       ??_C@_1BA@LEPJIIOK@?$AAU?$AAn?$AAk?$AAn?$AAo?$AAw?$AAn?$AA?$AA@ 10001dc8     mdd.obj
 0001:00000dd8       ??_C@_1FK@FNONLNGN@?$AA?$CF?$AAs?$AA?3?$AA?5?$AAD?$AAE?$AAB?$AAU?$AAG?$AAC?$AAH?$AAK?$AA?5?$AAf?$AAa?$AAi?$AAl?$AAe?$AAd?$AA?5?$AAi?$AAn?$AA?5?$AAf?$AAi?$AAl?$AAe?$AA?5?$AA?$CF?$AAs?$AA?5?$AAa@ 10001dd8     mdd.obj
 0001:00000e34       ??_C@_1DK@BHNGFHBN@?$AAs?$AAe?$AAr?$AAi?$AAa?$AAl?$AA?5?$AAp?$AAo?$AAr?$AAt?$AA?5?$AAp?$AAr?$AAo?$AAc?$AAe?$AAs?$AAs?$AA?5?$AAa?$AAt?$AAt?$AAa?$AAc?$AAh?$AA?$AN?$AA?6?$AA?$AA@ 10001e34     mdd.obj
 0001:00000e70       ??_C@_1O@OEJLCMKK@?$AA?$CF?$AAd?$AA?3?$AA?5?$AA?$CF?$AAs?$AA?$AA@ 10001e70     mdd.obj
 0001:00000e80       ??_C@_1DA@LGJDGOIM@?$AAp?$AAr?$AAo?$AAc?$AAe?$AAs?$AAs?$AA?5?$AAd?$AAe?$AAt?$AAa?$AAc?$AAh?$AA?5?$AAc?$AAa?$AAl?$AAl?$AAe?$AAd?$AA?$AN?$AA?6?$AA?$AA@ 10001e80     mdd.obj
 0001:00000eb0       ??_C@_1EE@GKGAJBJP@?$AAD?$AAo?$AAP?$AAu?$AAt?$AAB?$AAy?$AAt?$AAe?$AAs?$AA?5?$AAw?$AAa?$AAi?$AAt?$AA?5?$AAf?$AAo?$AAr?$AA?5?$AAC?$AAr?$AAi?$AAt?$AAS?$AAe?$AAc?$AA?5?$AA?$CF?$AAx?$AA?4?$AA?$AN@ 10001eb0     mdd.obj
 0001:00000ef4       ??_C@_1DK@JKMHGAMG@?$AAD?$AAo?$AAP?$AAu?$AAt?$AAB?$AAy?$AAt?$AAe?$AAs?$AA?5?$AAg?$AAo?$AAt?$AA?5?$AAC?$AAr?$AAi?$AAt?$AAS?$AAe?$AAc?$AA?5?$AA?$CF?$AAx?$AA?4?$AA?$AN?$AA?6?$AA?$AA@ 10001ef4     mdd.obj
 0001:00000f30       ??_C@_1EI@PHLIHGKN@?$AAD?$AAe?$AAv?$AAi?$AAc?$AAe?$AA?5?$AAc?$AAl?$AAo?$AAs?$AAe?$AAd?$AA?$CB?$AA?5?$AAQ?$AAu?$AAi?$AAt?$AA?5?$AAt?$AAr?$AAa?$AAn?$AAs?$AAm?$AAi?$AAs?$AAs?$AAi?$AAo?$AAn@ 10001f30     mdd.obj
 0001:00000f78       ??_C@_1FC@IBKKBMKO@?$AAS?$AAe?$AAr?$AAi?$AAa?$AAl?$AAE?$AAv?$AAe?$AAn?$AAt?$AAH?$AAa?$AAn?$AAd?$AAl?$AAe?$AAr?$AA?3?$AA?5?$AA?$CF?$AAd?$AA?5?$AAs?$AAe?$AAn?$AAt?$AA?5?$AAu?$AAp?$AA?9?$AAt@ 10001f78     mdd.obj
 0001:00000fcc       ??_C@_1BG@OPJKPKO@?$AAR?$AAT?$AAS?$AA?5?$AAs?$AAe?$AAt?$AA?4?$AA?$AN?$AA?6?$AA?$AA@ 10001fcc     mdd.obj
 0001:00000fe4       ??_C@_1DC@KIHGPOMJ@?$AAX?$AAO?$AAF?$AAF?$AA?8?$AAe?$AAd?$AA?0?$AA?5?$AAs?$AAe?$AAn?$AAd?$AA?5?$AAn?$AAo?$AAt?$AAh?$AAi?$AAn?$AAg?$AA?4?$AA?$AN?$AA?6?$AA?$AA@ 10001fe4     mdd.obj
 0001:00001018       ??_C@_1GC@MPMHAODJ@?$AAT?$AAx?$AAR?$AAe?$AAa?$AAd?$AA?5?$AA?$DN?$AA?5?$AA?$CF?$AAd?$AA?0?$AA?5?$AAT?$AAx?$AAL?$AAe?$AAn?$AAg?$AAt?$AAh?$AA?5?$AA?$DN?$AA?5?$AA?$CF?$AAd?$AA?0?$AA?5?$AAT?$AAx?$AAB?$AAy@ 10002018     mdd.obj
 0001:0000107c       ??_C@_1DC@FONCMGND@?$AAA?$AAb?$AAo?$AAu?$AAt?$AA?5?$AAt?$AAo?$AA?5?$AAc?$AAo?$AAp?$AAy?$AA?5?$AA?$CF?$AAd?$AA?5?$AAb?$AAy?$AAt?$AAe?$AAs?$AA?$AN?$AA?6?$AA?$AA@ 1000207c     mdd.obj
 0001:000010b0       ??_C@_1DI@GGPGJBLB@?$AA?$CF?$AAd?$AA?5?$AAb?$AAy?$AAt?$AAe?$AAs?$AA?5?$AAa?$AAc?$AAt?$AAu?$AAa?$AAl?$AAl?$AAy?$AA?5?$AAc?$AAo?$AAp?$AAi?$AAe?$AAd?$AA?4?$AA?$AN?$AA?6?$AA?$AA@ 100020b0     mdd.obj
 0001:000010e8       ??_C@_1EO@IFEAHMMF@?$AAT?$AAr?$AAa?$AAn?$AAs?$AAm?$AAi?$AAs?$AAs?$AAi?$AAo?$AAn?$AA?5?$AAc?$AAo?$AAm?$AAp?$AAl?$AAe?$AAt?$AAe?$AA?0?$AA?5?$AA?$CF?$AAd?$AA?5?$AAb?$AAy?$AAt?$AAe?$AAs?$AA?5@ 100020e8     mdd.obj
 0001:00001138       ??_C@_1EG@PNOECNFM@?$AAD?$AAo?$AAP?$AAu?$AAt?$AAB?$AAy?$AAt?$AAe?$AAs?$AA?5?$AAr?$AAe?$AAl?$AAe?$AAa?$AAs?$AAe?$AAd?$AA?5?$AAC?$AAr?$AAi?$AAt?$AAS?$AAe?$AAc?$AA?3?$AA?5?$AA?$CF?$AAx?$AA?4@ 10002138     mdd.obj
 0001:00001180       ??_C@_1EE@PGFICLOP@?$AA?$CL?$AAS?$AAe?$AAr?$AAi?$AAa?$AAl?$AAE?$AAv?$AAe?$AAn?$AAt?$AAH?$AAa?$AAn?$AAd?$AAl?$AAe?$AAr?$AA?0?$AA?5?$AAp?$AAH?$AAe?$AAa?$AAd?$AA?5?$AA0?$AAx?$AA?$CF?$AAX?$AA?$AN@ 10002180     mdd.obj
 0001:000011c4       ??_C@_1CC@GADAIIGI@?$AAE?$AAx?$AAi?$AAt?$AAi?$AAn?$AAg?$AA?5?$AAt?$AAh?$AAr?$AAe?$AAa?$AAd?$AA?$AN?$AA?6?$AA?$AA@ 100021c4     mdd.obj
 0001:000011e8       ??_C@_1EI@MHGBBLDA@?$AAS?$AAe?$AAr?$AAi?$AAa?$AAl?$AAE?$AAv?$AAe?$AAn?$AAt?$AAH?$AAa?$AAn?$AAd?$AAl?$AAe?$AAr?$AA?0?$AA?5?$AAN?$AAo?$AA?5?$AAI?$AAn?$AAt?$AAe?$AAr?$AAr?$AAu?$AAp?$AAt@ 100021e8     mdd.obj
 0001:00001230       ??_C@_1EM@PPCKGCIP@?$AAS?$AAe?$AAr?$AAi?$AAa?$AAl?$AAE?$AAv?$AAe?$AAn?$AAt?$AAH?$AAa?$AAn?$AAd?$AAl?$AAe?$AAr?$AA?0?$AA?5?$AAI?$AAn?$AAt?$AAe?$AAr?$AAr?$AAu?$AAp?$AAt?$AAs?$AA?5?$AA0@ 10002230     mdd.obj
 0001:0000127c       ??_C@_1BG@NHAMELLH@?$AAR?$AAx?$AA?5?$AAE?$AAv?$AAe?$AAn?$AAt?$AA?$AN?$AA?6?$AA?$AA@ 1000227c     mdd.obj
 0001:00001294       ??_C@_1CE@NDNCGIIC@?$AAT?$AAo?$AAs?$AAs?$AAe?$AAd?$AA?5?$AA?$CF?$AAd?$AA?5?$AAb?$AAy?$AAt?$AAe?$AAs?$AA?$AN?$AA?6?$AA?$AA@ 10002294     mdd.obj
 0001:000012b8       ??_C@_1HG@EGFFDKNF@?$AAA?$AAf?$AAt?$AAe?$AAr?$AA?5?$AAH?$AAW?$AAG?$AAe?$AAt?$AAB?$AAy?$AAt?$AAe?$AAs?$AA?0?$AA?5?$AAF?$AAi?$AAf?$AAo?$AA?$CI?$AAR?$AA?$DN?$AA?$CF?$AAd?$AA?0?$AAW?$AA?$DN?$AA?$CF?$AAd@ 100022b8     mdd.obj
 0001:00001330       ??_C@_1CA@EJJJJNNE@?$AAR?$AAe?$AAc?$AAe?$AAi?$AAv?$AAe?$AAd?$AA?5?$AAX?$AAO?$AAF?$AAF?$AA?$AN?$AA?6?$AA?$AA@ 10002330     mdd.obj
 0001:00001350       ??_C@_1BO@EEIJDLJ@?$AAR?$AAe?$AAc?$AAe?$AAi?$AAv?$AAe?$AAd?$AA?5?$AAX?$AAO?$AAN?$AA?$AN?$AA?6?$AA?$AA@ 10002350     mdd.obj
 0001:00001370       ??_C@_1EK@FLILIJBB@?$AAD?$AAT?$AAR?$AA_?$AAC?$AAO?$AAN?$AAT?$AAR?$AAO?$AAL?$AA_?$AAH?$AAA?$AAN?$AAD?$AAS?$AAH?$AAA?$AAK?$AAE?$AA?5?$AAC?$AAl?$AAe?$AAa?$AAr?$AAi?$AAn?$AAg?$AA?5?$AAD@ 10002370     mdd.obj
 0001:000013c0       ??_C@_1EK@LMCHJDFJ@?$AAR?$AAT?$AAS?$AA_?$AAC?$AAO?$AAN?$AAT?$AAR?$AAO?$AAL?$AA_?$AAH?$AAA?$AAN?$AAD?$AAS?$AAH?$AAA?$AAK?$AAE?$AA?5?$AAC?$AAl?$AAe?$AAa?$AAr?$AAi?$AAn?$AAg?$AA?5?$AAR@ 100023c0     mdd.obj
 0001:0000140c       ??_C@_1BO@CNGNDNHF@?$AAS?$AAe?$AAn?$AAd?$AAi?$AAn?$AAg?$AA?5?$AAX?$AAO?$AAF?$AAF?$AA?$AN?$AA?6?$AA?$AA@ 1000240c     mdd.obj
 0001:0000142c       ??_C@_1CK@CPCFPBFI@?$AAO?$AAt?$AAh?$AAe?$AAr?$AA?5?$AAE?$AAv?$AAe?$AAn?$AAt?$AA?0?$AA?5?$AAi?$AAt?$AA?3?$AA?$CF?$AAx?$AA?$AN?$AA?6?$AA?$AA@ 1000242c     mdd.obj
 0001:00001458       ??_C@_1CI@EJHAPNLK@?$AAL?$AAi?$AAn?$AAe?$AA?5?$AAE?$AAv?$AAe?$AAn?$AAt?$AA?0?$AA?5?$AAi?$AAt?$AA?3?$AA?$CF?$AAx?$AA?$AN?$AA?6?$AA?$AA@ 10002458     mdd.obj
 0001:00001480       ??_C@_1FI@GGFBGELP@?$AA?9?$AAS?$AAe?$AAr?$AAi?$AAa?$AAl?$AAE?$AAv?$AAe?$AAn?$AAt?$AAH?$AAa?$AAn?$AAd?$AAl?$AAe?$AAr?$AA?0?$AA?5?$AAF?$AAi?$AAf?$AAo?$AA?$CI?$AAR?$AA?$DN?$AA?$CF?$AAd?$AA?0?$AAW@ 10002480     mdd.obj
 0001:000014d8       ??_C@_1EE@JPBAFGIH@?$AAE?$AAn?$AAt?$AAe?$AAr?$AAe?$AAd?$AA?5?$AAS?$AAe?$AAr?$AAi?$AAa?$AAl?$AAD?$AAi?$AAs?$AAp?$AAa?$AAt?$AAc?$AAh?$AAT?$AAh?$AAr?$AAe?$AAa?$AAd?$AA?5?$AA?$CF?$AAX?$AA?$AN@ 100024d8     mdd.obj
 0001:00001520       ??_C@_1EI@IJEBFPL@?$AAS?$AAp?$AAi?$AAn?$AAn?$AAi?$AAn?$AAg?$AA?5?$AAi?$AAn?$AA?5?$AAd?$AAi?$AAs?$AAp?$AAa?$AAt?$AAc?$AAh?$AA?5?$AAt?$AAh?$AAr?$AAe?$AAa?$AAd?$AA?5?$AA?$CF?$AAX?$AA?5?$AA?$CF@ 10002520     mdd.obj
 0001:00001568       ??_C@_1BO@CNJNPPHP@?$AAE?$AAv?$AAe?$AAn?$AAt?$AA?5?$AA?$CF?$AAX?$AA?0?$AA?5?$AA?$CF?$AAd?$AA?$AN?$AA?6?$AA?$AA@ 10002568     mdd.obj
 0001:00001588       ??_C@_1EE@NKOOKCAI@?$AAS?$AAe?$AAr?$AAi?$AAa?$AAl?$AAD?$AAi?$AAs?$AAp?$AAa?$AAt?$AAc?$AAh?$AAT?$AAh?$AAr?$AAe?$AAa?$AAd?$AA?5?$AA?$CF?$AAx?$AA?5?$AAe?$AAx?$AAi?$AAt?$AAi?$AAn?$AAg?$AA?$AN@ 10002588     mdd.obj
 0001:000015cc       ??_C@_1CI@MPKANNOJ@?$AAS?$AAp?$AAi?$AAn?$AAn?$AAi?$AAn?$AAg?$AA?5?$AAt?$AAh?$AAr?$AAe?$AAa?$AAd?$AA?$CF?$AAX?$AA?6?$AA?$AN?$AA?$AA@ 100025cc     mdd.obj
 0001:000015f8       ??_C@_1EM@FFMAHOCG@?$AAE?$AAr?$AAr?$AAo?$AAr?$AA?5?$AAc?$AAr?$AAe?$AAa?$AAt?$AAi?$AAn?$AAg?$AA?5?$AAd?$AAi?$AAs?$AAp?$AAa?$AAt?$AAc?$AAh?$AA?5?$AAt?$AAh?$AAr?$AAe?$AAa?$AAd?$AA?5?$AA?$CI@ 100025f8     mdd.obj
 0001:00001644       ??_C@_1DI@KMMMNJHO@?$AAC?$AAr?$AAe?$AAa?$AAt?$AAe?$AAd?$AA?5?$AAr?$AAe?$AAc?$AAe?$AAi?$AAv?$AAe?$AA?5?$AAt?$AAh?$AAr?$AAe?$AAa?$AAd?$AA?5?$AA?$CF?$AAX?$AA?$AN?$AA?6?$AA?$AA@ 10002644     mdd.obj
 0001:00001680       ??_C@_1EI@JFKDHKHE@?$AA?$AN?$AA?6?$AAT?$AAr?$AAy?$AAi?$AAn?$AAg?$AA?5?$AAt?$AAo?$AA?5?$AAc?$AAl?$AAo?$AAs?$AAe?$AA?5?$AAd?$AAi?$AAs?$AAp?$AAa?$AAt?$AAc?$AAh?$AA?5?$AAt?$AAh?$AAr?$AAe?$AAa@ 10002680     mdd.obj
 0001:000016c8       ??_C@_1EI@FHNFOMPC@?$AA?$AN?$AA?6?$AAT?$AAr?$AAy?$AAi?$AAn?$AAg?$AA?5?$AAt?$AAo?$AA?5?$AAs?$AAi?$AAg?$AAn?$AAa?$AAl?$AA?5?$AAs?$AAe?$AAr?$AAi?$AAa?$AAl?$AA?5?$AAt?$AAh?$AAr?$AAe?$AAa?$AAd@ 100026c8     mdd.obj
 0001:00001710       ??_C@_1DO@BPPHAKCP@?$AA?$AN?$AA?6?$AAT?$AAr?$AAy?$AAi?$AAn?$AAg?$AA?5?$AAt?$AAo?$AA?5?$AAc?$AAa?$AAl?$AAl?$AA?5?$AAC?$AAl?$AAo?$AAs?$AAe?$AAH?$AAa?$AAn?$AAd?$AAl?$AAe?$AA?$AN?$AA?6?$AA?$AA@ 10002710     mdd.obj
 0001:00001750       ??_C@_1DM@NEFLPBFN@?$AA?$AN?$AA?6?$AAR?$AAe?$AAt?$AAu?$AAr?$AAn?$AAe?$AAd?$AA?5?$AAf?$AAr?$AAo?$AAm?$AA?5?$AAC?$AAl?$AAo?$AAs?$AAe?$AAH?$AAa?$AAn?$AAd?$AAl?$AAe?$AA?$AN?$AA?6?$AA?$AA@ 10002750     mdd.obj
 0001:00001790       ??_C@_1FG@GEFMJHJN@?$AAI?$AAO?$AAC?$AAT?$AAL?$AA?3?$AAD?$AAT?$AAR?$AA_?$AAC?$AAO?$AAN?$AAT?$AAR?$AAO?$AAL?$AA_?$AAH?$AAA?$AAN?$AAD?$AAS?$AAH?$AAA?$AAK?$AAE?$AA?5?$AAC?$AAl?$AAe?$AAa@ 10002790     mdd.obj
 0001:000017e8       ??_C@_1FE@MINNMIFE@?$AAI?$AAO?$AAC?$AAT?$AAL?$AA?3?$AAD?$AAT?$AAR?$AA_?$AAC?$AAO?$AAN?$AAT?$AAR?$AAO?$AAL?$AA_?$AAH?$AAA?$AAN?$AAD?$AAS?$AAH?$AAA?$AAK?$AAE?$AA?5?$AAS?$AAe?$AAt?$AAt@ 100027e8     mdd.obj
 0001:00001840       ??_C@_1FG@IDPAINNF@?$AAI?$AAO?$AAC?$AAT?$AAL?$AA?3?$AAR?$AAT?$AAS?$AA_?$AAC?$AAO?$AAN?$AAT?$AAR?$AAO?$AAL?$AA_?$AAH?$AAA?$AAN?$AAD?$AAS?$AAH?$AAA?$AAK?$AAE?$AA?5?$AAC?$AAl?$AAe?$AAa@ 10002840     mdd.obj
 0001:00001898       ??_C@_1FE@DAKNODMA@?$AAI?$AAO?$AAC?$AAT?$AAL?$AA?3?$AAR?$AAT?$AAS?$AA_?$AAC?$AAO?$AAN?$AAT?$AAR?$AAO?$AAL?$AA_?$AAH?$AAA?$AAN?$AAD?$AAS?$AAH?$AAA?$AAK?$AAE?$AA?5?$AAS?$AAe?$AAt?$AAt@ 10002898     mdd.obj
 0001:000018ec       ??_C@_1BI@GFHIOEJL@?$AA?$CL?$AAC?$AAO?$AAM?$AA_?$AAI?$AAn?$AAi?$AAt?$AA?$AN?$AA?6?$AA?$AA@ 100028ec     mdd.obj
 0001:00001904       ??_C@_1DM@MMPBEIDB@?$AAC?$AAO?$AAM?$AA_?$AAI?$AAn?$AAi?$AAt?$AA?0?$AA?5?$AAl?$AAp?$AAv?$AAB?$AAu?$AAs?$AAC?$AAo?$AAn?$AAt?$AAe?$AAx?$AAt?$AA?5?$AA?$DN?$AA?5?$AA?$CF?$AAp?$AA?6?$AA?$AA@ 10002904     mdd.obj
 0001:00001940       ??_C@_1HG@FCOJGPAE@?$AAE?$AAr?$AAr?$AAo?$AAr?$AA?5?$AAa?$AAl?$AAl?$AAo?$AAc?$AAa?$AAt?$AAi?$AAn?$AAg?$AA?5?$AAm?$AAe?$AAm?$AAo?$AAr?$AAy?$AA?5?$AAf?$AAo?$AAr?$AA?5?$AAp?$AAS?$AAe?$AAr@ 10002940     mdd.obj
 0001:000019b8       ??_C@_1FO@NFNODHBL@?$AAE?$AAr?$AAr?$AAo?$AAr?$AA?5?$AAl?$AAp?$AAv?$AAB?$AAu?$AAs?$AAC?$AAo?$AAn?$AAt?$AAe?$AAx?$AAt?$AA?5?$AA?$DN?$AA?$DN?$AA?5?$AAN?$AAU?$AAL?$AAL?$AA?0?$AA?5?$AAC?$AAO?$AAM@ 100029b8     mdd.obj
 0001:00001a18       ??_C@_1EA@GHGHHBKP@?$AAl?$AAp?$AAv?$AAB?$AAu?$AAs?$AAC?$AAo?$AAn?$AAt?$AAe?$AAx?$AAt?$AA?5?$AAO?$AAK?$AA?0?$AA?5?$AAC?$AAO?$AAM?$AA_?$AAI?$AAn?$AAi?$AAt?$AA?4?$AA?4?$AA?4?$AA?6?$AA?$AN?$AA?$AA@ 10002a18     mdd.obj
 0001:00001a58       ??_C@_1FA@BECDDKGM@?$AAE?$AAr?$AAr?$AAo?$AAr?$AA?5?$AAc?$AAr?$AAe?$AAa?$AAt?$AAi?$AAn?$AAg?$AA?5?$AAe?$AAv?$AAe?$AAn?$AAt?$AA?0?$AA?5?$AAC?$AAO?$AAM?$AA_?$AAI?$AAn?$AAi?$AAt?$AA?5?$AAf@ 10002a58     mdd.obj
 0001:00001aa8       ??_C@_1CC@OIKDCOFG@?$AAT?$AAr?$AAy?$AA?5?$AAt?$AAo?$AA?5?$AAo?$AAp?$AAe?$AAn?$AA?5?$AA?$CF?$AAs?$AA?$AN?$AA?6?$AA?$AA@ 10002aa8     mdd.obj
 0001:00001ad0       ??_C@_1FK@GNPHIAEF@?$AAF?$AAa?$AAi?$AAl?$AAe?$AAd?$AA?5?$AAt?$AAo?$AA?5?$AAo?$AAp?$AAe?$AAn?$AA?5?$AAd?$AAe?$AAv?$AAk?$AAe?$AAy?$AAp?$AAa?$AAt?$AAh?$AA?0?$AA?5?$AAC?$AAO?$AAM?$AA_?$AAI@ 10002ad0     mdd.obj
 0001:00001b2c       ??_C@_1CC@KMPFMANC@?$AAD?$AAe?$AAv?$AAi?$AAc?$AAe?$AAA?$AAr?$AAr?$AAa?$AAy?$AAI?$AAn?$AAd?$AAe?$AAx?$AA?$AA@ 10002b2c     mdd.obj
 0001:00001b50       ??_C@_1HA@FDKKDCHL@?$AAF?$AAa?$AAi?$AAl?$AAe?$AAd?$AA?5?$AAt?$AAo?$AA?5?$AAg?$AAe?$AAt?$AA?5?$AAD?$AAe?$AAv?$AAi?$AAc?$AAe?$AAA?$AAr?$AAr?$AAa?$AAy?$AAI?$AAn?$AAd?$AAe?$AAx?$AA?5?$AAv@ 10002b50     mdd.obj
 0001:00001bc0       ??_C@_1BI@BHLBGEOK@?$AAP?$AAr?$AAi?$AAo?$AAr?$AAi?$AAt?$AAy?$AA2?$AA5?$AA6?$AA?$AA@ 10002bc0     mdd.obj
 0001:00001bd8       ??_C@_1GI@IGAGBKDE@?$AAF?$AAa?$AAi?$AAl?$AAe?$AAd?$AA?5?$AAt?$AAo?$AA?5?$AAg?$AAe?$AAt?$AA?5?$AAP?$AAr?$AAi?$AAo?$AAr?$AAi?$AAt?$AAy?$AA2?$AA5?$AA6?$AA?5?$AAv?$AAa?$AAl?$AAu?$AAe?$AA?0@ 10002bd8     mdd.obj
 0001:00001c40       ??_C@_1BM@EFMMMFDH@?$AAD?$AAe?$AAv?$AAI?$AAn?$AAd?$AAe?$AAx?$AA?5?$AA?$CF?$AAX?$AA?$AN?$AA?6?$AA?$AA@ 10002c40     mdd.obj
 0001:00001c60       ??_C@_1FI@OHFMJBNJ@?$AAE?$AAr?$AAr?$AAo?$AAr?$AA?5?$AAi?$AAn?$AA?5?$AAG?$AAe?$AAt?$AAS?$AAe?$AAr?$AAi?$AAa?$AAl?$AAO?$AAb?$AAj?$AAe?$AAc?$AAt?$AA?0?$AA?5?$AAC?$AAO?$AAM?$AA_?$AAI?$AAn@ 10002c60     mdd.obj
 0001:00001cb8       ??_C@_1EA@DFMKFADA@?$AAA?$AAb?$AAo?$AAu?$AAt?$AA?5?$AAt?$AAo?$AA?5?$AAc?$AAa?$AAl?$AAl?$AA?5?$AAH?$AAW?$AAI?$AAn?$AAi?$AAt?$AA?$CI?$AA?$CF?$AAs?$AA?0?$AA0?$AAx?$AA?$CF?$AAX?$AA?$CJ?$AA?$AN?$AA?6?$AA?$AA@ 10002cb8     mdd.obj
 0001:00001cf8       ??_C@_1GG@LFOFGOL@?$AAH?$AAa?$AAr?$AAd?$AAw?$AAa?$AAr?$AAe?$AA?5?$AAd?$AAo?$AAe?$AAs?$AAn?$AA?8?$AAt?$AA?5?$AAi?$AAn?$AAi?$AAt?$AA?5?$AAc?$AAo?$AAr?$AAr?$AAe?$AAc?$AAt?$AAl?$AAy?$AA?0@ 10002cf8     mdd.obj
 0001:00001d60       ??_C@_1DE@CLLKJMN@?$AAB?$AAa?$AAc?$AAk?$AA?5?$AAf?$AAr?$AAo?$AAm?$AA?5?$AAh?$AAa?$AAr?$AAd?$AAw?$AAa?$AAr?$AAe?$AA?5?$AAi?$AAn?$AAi?$AAt?$AA?$AN?$AA?6?$AA?$AA@ 10002d60     mdd.obj
 0001:00001d98       ??_C@_1GG@FCOIFIDD@?$AAE?$AAr?$AAr?$AAo?$AAr?$AA?5?$AAa?$AAl?$AAl?$AAo?$AAc?$AAa?$AAt?$AAi?$AAn?$AAg?$AA?5?$AAr?$AAe?$AAc?$AAe?$AAi?$AAv?$AAe?$AA?5?$AAb?$AAu?$AAf?$AAf?$AAe?$AAr?$AA?0@ 10002d98     mdd.obj
 0001:00001e00       ??_C@_1CC@POKINGEF@?$AAR?$AAx?$AAH?$AAe?$AAa?$AAd?$AA?5?$AAi?$AAn?$AAi?$AAt?$AA?8?$AAe?$AAd?$AA?$AN?$AA?6?$AA?$AA@ 10002e00     mdd.obj
 0001:00001e28       ??_C@_1EI@FNCKFJMM@?$AAR?$AAx?$AAB?$AAu?$AAf?$AAf?$AAe?$AAr?$AA?5?$AAi?$AAn?$AAi?$AAt?$AA?8?$AAe?$AAd?$AA?5?$AAw?$AAi?$AAt?$AAh?$AA?5?$AAs?$AAt?$AAa?$AAr?$AAt?$AA?5?$AAa?$AAt?$AA?5?$AA?$CF@ 10002e28     mdd.obj
 0001:00001e70       ??_C@_1BI@NFEFLGML@?$AA?9?$AAC?$AAO?$AAM?$AA_?$AAI?$AAn?$AAi?$AAt?$AA?$AN?$AA?6?$AA?$AA@ 10002e70     mdd.obj
 0001:00001e88       ??_C@_1FM@OGLFDPL@?$AA?$CL?$AAC?$AAO?$AAM?$AA_?$AAO?$AAp?$AAe?$AAn?$AA?5?$AAh?$AAa?$AAn?$AAd?$AAl?$AAe?$AA?5?$AAx?$AA?$CF?$AAX?$AA?0?$AA?5?$AAa?$AAc?$AAc?$AAe?$AAs?$AAs?$AA?5?$AAx?$AA?$CF?$AAX@ 10002e88     mdd.obj
 0001:00001ee8       ??_C@_1EK@IHGIHNNE@?$AAO?$AAp?$AAe?$AAn?$AA?5?$AAa?$AAt?$AAt?$AAe?$AAm?$AAp?$AAt?$AAe?$AAd?$AA?5?$AAo?$AAn?$AA?5?$AAu?$AAn?$AAi?$AAn?$AAi?$AAt?$AAe?$AAd?$AA?5?$AAd?$AAe?$AAv?$AAi?$AAc@ 10002ee8     mdd.obj
 0001:00001f38       ??_C@_1HA@GJBLLAJC@?$AAO?$AAp?$AAe?$AAn?$AA?5?$AAr?$AAe?$AAq?$AAu?$AAe?$AAs?$AAt?$AAe?$AAd?$AA?5?$AAa?$AAc?$AAc?$AAe?$AAs?$AAs?$AA?5?$AA?$CF?$AAx?$AA?0?$AA?5?$AAh?$AAa?$AAn?$AAd?$AAl?$AAe@ 10002f38     mdd.obj
 0001:00001fa8       ??_C@_1HC@GGJLMGKF@?$AAE?$AAr?$AAr?$AAo?$AAr?$AA?5?$AAa?$AAl?$AAl?$AAo?$AAc?$AAa?$AAt?$AAi?$AAn?$AAg?$AA?5?$AAm?$AAe?$AAm?$AAo?$AAr?$AAy?$AA?5?$AAf?$AAo?$AAr?$AA?5?$AAp?$AAO?$AAp?$AAe@ 10002fa8     mdd.obj
 0001:00002020       ??_C@_1GC@CLBBDJNN@?$AAC?$AAO?$AAM?$AA_?$AAO?$AAp?$AAe?$AAn?$AA?3?$AA?5?$AAA?$AAc?$AAc?$AAe?$AAs?$AAs?$AA?5?$AAp?$AAe?$AAr?$AAm?$AAi?$AAs?$AAs?$AAi?$AAo?$AAn?$AA?5?$AAh?$AAa?$AAn?$AAd@ 10003020     mdd.obj
 0001:00002088       ??_C@_1EK@MCEDHMPN@?$AAC?$AAO?$AAM?$AA_?$AAO?$AAp?$AAe?$AAn?$AA?3?$AA?5?$AAF?$AAi?$AAr?$AAs?$AAt?$AA?5?$AAo?$AAp?$AAe?$AAn?$AA?5?$AA?3?$AA?5?$AAD?$AAo?$AA?5?$AAI?$AAn?$AAi?$AAt?$AA?5?$AAx@ 10003088     mdd.obj
 0001:000020d8       ??_C@_1FA@GFAOJBEN@?$AAC?$AAO?$AAM?$AA_?$AAO?$AAp?$AAe?$AAn?$AA?3?$AA?5?$AAS?$AAt?$AAa?$AAr?$AAt?$AAi?$AAn?$AAg?$AA?5?$AAD?$AAi?$AAs?$AAp?$AAa?$AAt?$AAc?$AAh?$AAT?$AAh?$AAr?$AAe?$AAa@ 100030d8     mdd.obj
 0001:00002128       ??_C@_1FG@FDKJAEDJ@?$AAC?$AAO?$AAM?$AA_?$AAO?$AAp?$AAe?$AAn?$AA?3?$AA?5?$AAF?$AAa?$AAi?$AAl?$AAe?$AAd?$AA?5?$AAS?$AAt?$AAa?$AAr?$AAt?$AAD?$AAi?$AAs?$AAp?$AAa?$AAt?$AAc?$AAh?$AAT?$AAh@ 10003128     mdd.obj
 0001:00002180       ??_C@_1CE@HHPKLFBI@?$AAH?$AAW?$AA?5?$AAO?$AAp?$AAe?$AAn?$AA?5?$AAf?$AAa?$AAi?$AAl?$AAe?$AAd?$AA?4?$AA?$AN?$AA?6?$AA?$AA@ 10003180     mdd.obj
 0001:000021a8       ??_C@_1EK@MFLOMJPC@?$AA?9?$AAC?$AAO?$AAM?$AA_?$AAO?$AAp?$AAe?$AAn?$AA?5?$AAh?$AAa?$AAn?$AAd?$AAl?$AAe?$AA?5?$AAx?$AA?$CF?$AAX?$AA?0?$AA?5?$AAx?$AA?$CF?$AAX?$AA?0?$AA?5?$AAR?$AAe?$AAf?$AA?5?$AAx@ 100031a8     mdd.obj
 0001:000021f4       ??_C@_1BK@FMFILLAC@?$AA?$CL?$AAC?$AAO?$AAM?$AA_?$AAC?$AAl?$AAo?$AAs?$AAe?$AA?$AN?$AA?6?$AA?$AA@ 100031f4     mdd.obj
 0001:00002210       ??_C@_1BI@CPEANALD@?$AA?$DO?$AAC?$AAO?$AAM?$AA_?$AAC?$AAl?$AAo?$AAs?$AAe?$AA?6?$AA?$AA@ 10003210     mdd.obj
 0001:00002228       ??_C@_1EK@JBKGBIGA@?$AA?$CB?$AA?$CB?$AAC?$AAO?$AAM?$AA_?$AAC?$AAl?$AAo?$AAs?$AAe?$AA?3?$AA?5?$AAp?$AAS?$AAe?$AAr?$AAi?$AAa?$AAl?$AAH?$AAe?$AAa?$AAd?$AA?5?$AA?$DN?$AA?$DN?$AA?5?$AAN?$AAU?$AAL?$AAL@ 10003228     mdd.obj
 0001:00002278       ??_C@_1JK@JHJOGNCH@?$AAC?$AAO?$AAM?$AA_?$AAC?$AAl?$AAo?$AAs?$AAe?$AA?3?$AA?5?$AA?$CI?$AA?$CF?$AAd?$AA?5?$AAh?$AAa?$AAn?$AAd?$AAl?$AAe?$AAs?$AA?$CJ?$AA?5?$AAt?$AAo?$AAt?$AAa?$AAl?$AA?5?$AAR?$AAX@ 10003278     mdd.obj
 0001:00002318       ??_C@_1EO@OBGHLNIN@?$AAC?$AAO?$AAM?$AA_?$AAC?$AAl?$AAo?$AAs?$AAe?$AA?3?$AA?5?$AA?$CF?$AAd?$AA?5?$AAu?$AAs?$AAe?$AAr?$AAs?$AA?5?$AAi?$AAn?$AA?5?$AAM?$AAD?$AAD?$AA?5?$AAf?$AAu?$AAn?$AAc?$AAt@ 10003318     mdd.obj
 0001:00002368       ??_C@_1HC@IJEHCFNA@?$AAC?$AAO?$AAM?$AA_?$AAC?$AAl?$AAo?$AAs?$AAe?$AA?3?$AA?5?$AAW?$AAa?$AAi?$AAt?$AAe?$AAd?$AA?5?$AA2?$AAs?$AA?5?$AAf?$AAo?$AAr?$AA?5?$AAs?$AAe?$AAr?$AAi?$AAa?$AAl?$AA?5@ 10003368     mdd.obj
 0001:000023dc       ??_C@_1DA@EPLPIONK@?$AAA?$AAb?$AAo?$AAu?$AAt?$AA?5?$AAt?$AAo?$AA?5?$AAc?$AAa?$AAl?$AAl?$AA?5?$AAH?$AAW?$AAC?$AAl?$AAo?$AAs?$AAe?$AA?$AN?$AA?6?$AA?$AA@ 100033dc     mdd.obj
 0001:0000240c       ??_C@_1DA@HIJABIAN@?$AAR?$AAe?$AAt?$AAu?$AAr?$AAn?$AAe?$AAd?$AA?5?$AAf?$AAr?$AAo?$AAm?$AA?5?$AAH?$AAW?$AAC?$AAl?$AAo?$AAs?$AAe?$AA?$AN?$AA?6?$AA?$AA@ 1000340c     mdd.obj
 0001:00002440       ??_C@_1EO@KHAJIML@?$AAC?$AAO?$AAM?$AA_?$AAC?$AAl?$AAo?$AAs?$AAe?$AA?5?$AA?3?$AA?5?$AAS?$AAt?$AAo?$AAp?$AAp?$AAi?$AAn?$AAg?$AA?5?$AAD?$AAi?$AAs?$AAp?$AAa?$AAt?$AAc?$AAh?$AA?5?$AAT?$AAh@ 10003440     mdd.obj
 0001:00002490       ??_C@_1FA@FDHIAIFB@?$AAC?$AAO?$AAM?$AA_?$AAC?$AAl?$AAo?$AAs?$AAe?$AA?3?$AA?5?$AAC?$AAl?$AAo?$AAs?$AAe?$AAd?$AA?5?$AAa?$AAc?$AAc?$AAe?$AAs?$AAs?$AA?5?$AAo?$AAw?$AAn?$AAe?$AAr?$AA?5?$AAh@ 10003490     mdd.obj
 0001:000024e0       ??_C@_1EE@HJGCIAAB@?$AA?$CB?$AA?$CB?$AAC?$AAl?$AAo?$AAs?$AAe?$AA?5?$AAo?$AAf?$AA?5?$AAn?$AAo?$AAn?$AA?9?$AAo?$AAp?$AAe?$AAn?$AA?5?$AAs?$AAe?$AAr?$AAi?$AAa?$AAl?$AA?5?$AAp?$AAo?$AAr?$AAt?$AA?$AN@ 100034e0     mdd.obj
 0001:00002524       ??_C@_1BK@GDIGGGLD@?$AA?9?$AAC?$AAO?$AAM?$AA_?$AAC?$AAl?$AAo?$AAs?$AAe?$AA?$AN?$AA?6?$AA?$AA@ 10003524     mdd.obj
 0001:00002540       ??_C@_1CE@GDEBELBJ@?$AA?$CL?$AAP?$AAr?$AAo?$AAc?$AAe?$AAs?$AAs?$AAE?$AAx?$AAi?$AAt?$AAi?$AAn?$AAg?$AA?$AN?$AA?6?$AA?$AA@ 10003540     mdd.obj
 0001:00002568       ??_C@_1FE@DFEILEFJ@?$AA?$CB?$AA?$CB?$AAP?$AAr?$AAo?$AAc?$AAe?$AAs?$AAs?$AAE?$AAx?$AAi?$AAt?$AAi?$AAn?$AAg?$AA?3?$AA?5?$AAp?$AAS?$AAe?$AAr?$AAi?$AAa?$AAl?$AAH?$AAe?$AAa?$AAd?$AA?5?$AA?$DN?$AA?$DN@ 10003568     mdd.obj
 0001:000025c0       ??_C@_1KA@EBBKPACJ@?$AAP?$AAr?$AAo?$AAc?$AAe?$AAs?$AAs?$AAC?$AAl?$AAo?$AAs?$AAe?$AA?3?$AA?5?$AA?$CI?$AA?$CF?$AAd?$AA?5?$AAh?$AAa?$AAn?$AAd?$AAl?$AAe?$AAs?$AA?$CJ?$AA?5?$AAt?$AAo?$AAt?$AAa?$AAl@ 100035c0     mdd.obj
 0001:00002660       ??_C@_1FI@EHPKKKJN@?$AAP?$AAr?$AAo?$AAc?$AAe?$AAs?$AAs?$AAE?$AAx?$AAi?$AAt?$AAi?$AAn?$AAg?$AA?3?$AA?5?$AA?$CF?$AAd?$AA?5?$AAu?$AAs?$AAe?$AAr?$AAs?$AA?5?$AAi?$AAn?$AA?5?$AAM?$AAD?$AAD?$AA?5@ 10003660     mdd.obj
 0001:000026b8       ??_C@_1HM@BIAPEHED@?$AAP?$AAr?$AAo?$AAc?$AAe?$AAs?$AAs?$AAE?$AAx?$AAi?$AAt?$AAi?$AAn?$AAg?$AA?3?$AA?5?$AAW?$AAa?$AAi?$AAt?$AAe?$AAd?$AA?5?$AA2?$AAs?$AA?5?$AAf?$AAo?$AAr?$AA?5?$AAs?$AAe@ 100036b8     mdd.obj
 0001:00002734       ??_C@_1CE@KKIBLMOF@?$AA?9?$AAP?$AAr?$AAo?$AAc?$AAe?$AAs?$AAs?$AAE?$AAx?$AAi?$AAt?$AAi?$AAn?$AAg?$AA?$AN?$AA?6?$AA?$AA@ 10003734     mdd.obj
 0001:00002758       ??_C@_1BM@ODDOENCJ@?$AA?$CL?$AAC?$AAO?$AAM?$AA_?$AAD?$AAe?$AAi?$AAn?$AAi?$AAt?$AA?$AN?$AA?6?$AA?$AA@ 10003758     mdd.obj
 0001:00002778       ??_C@_1EI@FADDJAGG@?$AAC?$AAO?$AAM?$AA_?$AAD?$AAe?$AAi?$AAn?$AAi?$AAt?$AA?5?$AAc?$AAa?$AAn?$AA?8?$AAt?$AA?5?$AAf?$AAi?$AAn?$AAd?$AA?5?$AAp?$AAS?$AAe?$AAr?$AAi?$AAa?$AAl?$AAH?$AAe?$AAa@ 10003778     mdd.obj
 0001:000027c0       ??_C@_1EA@JDMAPCPA@?$AA?5?$AAD?$AAe?$AAi?$AAn?$AAi?$AAt?$AA?5?$AA?9?$AA?5?$AAC?$AAl?$AAo?$AAs?$AAi?$AAn?$AAg?$AA?5?$AAH?$AAa?$AAn?$AAd?$AAl?$AAe?$AA?5?$AA0?$AAx?$AA?$CF?$AAX?$AA?$AN?$AA?6?$AA?$AA@ 100037c0     mdd.obj
 0001:00002800       ??_C@_1DC@PMGMNFPK@?$AAA?$AAb?$AAo?$AAu?$AAt?$AA?5?$AAt?$AAo?$AA?5?$AAc?$AAa?$AAl?$AAl?$AA?5?$AAH?$AAW?$AAD?$AAe?$AAi?$AAn?$AAi?$AAt?$AA?$AN?$AA?6?$AA?$AA@ 10003800     mdd.obj
 0001:00002834       ??_C@_1DC@CLHJIHHM@?$AAR?$AAe?$AAt?$AAu?$AAr?$AAn?$AAe?$AAd?$AA?5?$AAf?$AAr?$AAo?$AAm?$AA?5?$AAH?$AAW?$AAD?$AAe?$AAi?$AAn?$AAi?$AAt?$AA?$AN?$AA?6?$AA?$AA@ 10003834     mdd.obj
 0001:00002868       ??_C@_1BM@OGICEDGH@?$AA?9?$AAC?$AAO?$AAM?$AA_?$AAD?$AAe?$AAi?$AAn?$AAi?$AAt?$AA?$AN?$AA?6?$AA?$AA@ 10003868     mdd.obj
 0001:00002884       ??_C@_1DE@HFOANDEN@?$AA?$CL?$AAC?$AAO?$AAM?$AA_?$AAR?$AAE?$AAA?$AAD?$AA?$CI?$AA0?$AAx?$AA?$CF?$AAX?$AA?0?$AA0?$AAx?$AA?$CF?$AAX?$AA?0?$AA?$CF?$AAd?$AA?$CJ?$AA?$AN?$AA?6?$AA?$AA@ 10003884     mdd.obj
 0001:000028b8       ??_C@_1EE@JCLKGIBD@?$AAC?$AAO?$AAM?$AA_?$AAR?$AAE?$AAA?$AAD?$AA?0?$AA?5?$AAE?$AAr?$AAr?$AAo?$AAr?$AA?3?$AA?5?$AAH?$AAa?$AAn?$AAd?$AAl?$AAe?$AA?5?$AAi?$AAs?$AA?5?$AAN?$AAU?$AAL?$AAL?$AA?$AN@ 100038b8     mdd.obj
 0001:00002900       ??_C@_1GE@IIMCKPP@?$AAC?$AAO?$AAM?$AA_?$AAR?$AAE?$AAA?$AAD?$AA?0?$AA?5?$AAU?$AAn?$AAp?$AAl?$AAu?$AAg?$AAg?$AAe?$AAd?$AA?5?$AAd?$AAe?$AAv?$AAi?$AAc?$AAe?$AA?5?$AAo?$AAr?$AA?5?$AAd?$AAe@ 10003900     mdd.obj
 0001:00002964       ??_C@_1DI@CKPKPEIH@?$AAC?$AAO?$AAM?$AA_?$AAR?$AAE?$AAA?$AAD?$AA?0?$AA?5?$AAd?$AAe?$AAv?$AAi?$AAc?$AAe?$AA?5?$AAn?$AAo?$AAt?$AA?5?$AAo?$AAp?$AAe?$AAn?$AA?$AN?$AA?6?$AA?$AA@ 10003964     mdd.obj
 0001:000029a0       ??_C@_1FE@BNFDNPPG@?$AAC?$AAO?$AAM?$AA_?$AAR?$AAe?$AAa?$AAd?$AA?3?$AA?5?$AAA?$AAc?$AAc?$AAe?$AAs?$AAs?$AA?5?$AAp?$AAe?$AAr?$AAm?$AAi?$AAs?$AAs?$AAi?$AAo?$AAn?$AA?5?$AAf?$AAa?$AAi?$AAl@ 100039a0     mdd.obj
 0001:000029f4       ??_C@_1CE@PICJNKFA@?$AAT?$AAo?$AAt?$AAa?$AAl?$AAT?$AAi?$AAm?$AAe?$AAo?$AAu?$AAt?$AA?3?$AA?$CF?$AAd?$AA?$AN?$AA?6?$AA?$AA@ 100039f4     mdd.obj
 0001:00002a18       ??_C@_1FC@CGIHBGNN@?$AAT?$AAo?$AAp?$AA?5?$AAo?$AAf?$AA?5?$AAL?$AAo?$AAo?$AAp?$AA?5?$AAF?$AAi?$AAf?$AAo?$AA?$CI?$AAR?$AA?$DN?$AA?$CF?$AAd?$AA?0?$AAW?$AA?$DN?$AA?$CF?$AAd?$AA?0?$AAL?$AA?$DN?$AA?$CF?$AAd?$AA?0@ 10003a18     mdd.obj
 0001:00002a6c       ??_C@_1CK@GLIEOMOP@?$AAA?$AAb?$AAo?$AAu?$AAt?$AA?5?$AAt?$AAo?$AA?5?$AAw?$AAa?$AAi?$AAt?$AA?5?$AA?$CF?$AAd?$AAm?$AAs?$AA?$AN?$AA?6?$AA?$AA@ 10003a6c     mdd.obj
 0001:00002a98       ??_C@_1DG@NGGANINM@?$AAC?$AAO?$AAM?$AA_?$AAR?$AAe?$AAa?$AAd?$AA?5?$AA?9?$AA?5?$AAA?$AAb?$AAo?$AAr?$AAt?$AAi?$AAn?$AAg?$AA?5?$AAr?$AAe?$AAa?$AAd?$AA?$AN?$AA?6?$AA?$AA@ 10003a98     mdd.obj
 0001:00002ad0       ??_C@_1DO@LAJCOFEP@?$AAC?$AAO?$AAM?$AA_?$AAR?$AAe?$AAa?$AAd?$AA?5?$AA?9?$AA?5?$AAd?$AAe?$AAv?$AAi?$AAc?$AAe?$AA?5?$AAw?$AAa?$AAs?$AA?5?$AAc?$AAl?$AAo?$AAs?$AAe?$AAd?$AA?6?$AA?$AN?$AA?$AA@ 10003ad0     mdd.obj
 0001:00002b10       ??_C@_1BM@LDMNCPPP@?$AAS?$AAe?$AAn?$AAd?$AAi?$AAn?$AAg?$AA?5?$AAX?$AAO?$AAN?$AA?$AN?$AA?6?$AA?$AA@ 10003b10     mdd.obj
 0001:00002b30       ??_C@_1EI@PFOBJKJM@?$AAR?$AAT?$AAS?$AA_?$AAC?$AAO?$AAN?$AAT?$AAR?$AAO?$AAL?$AA_?$AAH?$AAA?$AAN?$AAD?$AAS?$AAH?$AAA?$AAK?$AAE?$AA?5?$AAS?$AAe?$AAt?$AAt?$AAi?$AAn?$AAg?$AA?5?$AAR?$AAT@ 10003b30     mdd.obj
 0001:00002b78       ??_C@_1EI@NJBLBAI@?$AAD?$AAT?$AAR?$AA_?$AAC?$AAO?$AAN?$AAT?$AAR?$AAO?$AAL?$AA_?$AAH?$AAA?$AAN?$AAD?$AAS?$AAH?$AAA?$AAK?$AAE?$AA?5?$AAS?$AAe?$AAt?$AAt?$AAi?$AAn?$AAg?$AA?5?$AAD?$AAT@ 10003b78     mdd.obj
 0001:00002bc0       ??_C@_1CO@BMKNIMFL@?$AAR?$AAe?$AAc?$AAe?$AAi?$AAv?$AAe?$AAB?$AAy?$AAt?$AAe?$AAs?$AA?5?$AAe?$AAx?$AAi?$AAt?$AAi?$AAn?$AAg?$AA?$AN?$AA?6?$AA?$AA@ 10003bc0     mdd.obj
 0001:00002bf0       ??_C@_1GI@KJLFCJIJ@?$AA?9?$AAC?$AAO?$AAM?$AA_?$AAR?$AAE?$AAA?$AAD?$AA?3?$AA?5?$AAr?$AAe?$AAt?$AAu?$AAr?$AAn?$AAi?$AAn?$AAg?$AA?5?$AA?$CF?$AAd?$AA?5?$AA?$CI?$AAt?$AAo?$AAt?$AAa?$AAl?$AA?5?$AA?$CF@ 10003bf0     mdd.obj
 0001:00002c58       ??_C@_1DK@NPDDAOLJ@?$AA?$CL?$AAC?$AAO?$AAM?$AA_?$AAW?$AAR?$AAI?$AAT?$AAE?$AA?$CI?$AA0?$AAx?$AA?$CF?$AAX?$AA?0?$AA?5?$AA0?$AAx?$AA?$CF?$AAX?$AA?0?$AA?5?$AA?$CF?$AAd?$AA?$CJ?$AA?$AN?$AA?6?$AA?$AA@ 10003c58     mdd.obj
 0001:00002c98       ??_C@_1GG@PMJCHLGF@?$AAC?$AAO?$AAM?$AA_?$AAW?$AAR?$AAI?$AAT?$AAE?$AA?0?$AA?5?$AAU?$AAn?$AAp?$AAl?$AAu?$AAg?$AAg?$AAe?$AAd?$AA?5?$AAd?$AAe?$AAv?$AAi?$AAc?$AAe?$AA?5?$AAo?$AAr?$AA?5?$AAd@ 10003c98     mdd.obj
 0001:00002d00       ??_C@_1DK@PMCNIBAH@?$AAC?$AAO?$AAM?$AA_?$AAW?$AAR?$AAI?$AAT?$AAE?$AA?0?$AA?5?$AAd?$AAe?$AAv?$AAi?$AAc?$AAe?$AA?5?$AAn?$AAo?$AAt?$AA?5?$AAo?$AAp?$AAe?$AAn?$AA?$AN?$AA?6?$AA?$AA@ 10003d00     mdd.obj
 0001:00002d40       ??_C@_1FG@IAEGGCHL@?$AAC?$AAO?$AAM?$AA_?$AAW?$AAr?$AAi?$AAt?$AAe?$AA?3?$AA?5?$AAA?$AAc?$AAc?$AAe?$AAs?$AAs?$AA?5?$AAp?$AAe?$AAr?$AAm?$AAi?$AAs?$AAs?$AAi?$AAo?$AAn?$AA?5?$AAf?$AAa?$AAi@ 10003d40     mdd.obj
 0001:00002d98       ??_C@_1DM@JLPMFDMF@?$AAC?$AAO?$AAM?$AA_?$AAW?$AAR?$AAI?$AAT?$AAE?$AA?0?$AA?5?$AAb?$AAa?$AAd?$AA?5?$AAr?$AAe?$AAa?$AAd?$AA?5?$AAp?$AAo?$AAi?$AAn?$AAt?$AAe?$AAr?$AA?$AN?$AA?6?$AA?$AA@ 10003d98     mdd.obj
 0001:00002dd8       ??_C@_1GC@BNCJFOA@?$AAC?$AAO?$AAM?$AA_?$AAW?$AAr?$AAi?$AAt?$AAe?$AA?5?$AAC?$AAe?$AAA?$AAl?$AAl?$AAo?$AAc?$AAA?$AAs?$AAy?$AAn?$AAc?$AAh?$AAr?$AAo?$AAn?$AAo?$AAu?$AAs?$AAB?$AAu?$AAf@ 10003dd8     mdd.obj
 0001:00002e40       ??_C@_1HC@EIECOKLC@?$AAc?$AA?3?$AA?2?$AAw?$AAi?$AAn?$AAc?$AAe?$AA8?$AA0?$AA0?$AA?2?$AAo?$AAs?$AAd?$AAe?$AAs?$AAi?$AAg?$AAn?$AAs?$AA?2?$AAv?$AAc?$AAp?$AAo?$AAs?$AAc?$AAe?$AAp?$AAc?$AA?2@ 10003e40     mdd.obj
 0001:00002eb8       ??_C@_1EC@FLKHHNEC@?$AAC?$AAO?$AAM?$AA_?$AAW?$AAr?$AAi?$AAt?$AAe?$AA?5?$AAw?$AAa?$AAi?$AAt?$AA?5?$AAf?$AAo?$AAr?$AA?5?$AAC?$AAr?$AAi?$AAt?$AAS?$AAe?$AAc?$AA?5?$AA?$CF?$AAx?$AA?4?$AA?$AN?$AA?6@ 10003eb8     mdd.obj
 0001:00002efc       ??_C@_1DI@CAEOCHGO@?$AAC?$AAO?$AAM?$AA_?$AAW?$AAr?$AAi?$AAt?$AAe?$AA?5?$AAG?$AAo?$AAt?$AA?5?$AAC?$AAr?$AAi?$AAt?$AAS?$AAe?$AAc?$AA?5?$AA?$CF?$AAx?$AA?4?$AA?$AN?$AA?6?$AA?$AA@ 10003efc     mdd.obj
 0001:00002f34       ??_C@_1DI@DJLNOFJH@?$AAC?$AAO?$AAM?$AA_?$AAW?$AAr?$AAi?$AAt?$AAe?$AA?5?$AAg?$AAo?$AAt?$AA?5?$AAC?$AAr?$AAi?$AAt?$AAS?$AAe?$AAc?$AA?5?$AA?$CF?$AAx?$AA?4?$AA?$AN?$AA?6?$AA?$AA@ 10003f34     mdd.obj
 0001:00002f70       ??_C@_1EE@GAMOAJJK@?$AAC?$AAO?$AAM?$AA_?$AAW?$AAr?$AAi?$AAt?$AAe?$AA?5?$AAr?$AAe?$AAl?$AAe?$AAa?$AAs?$AAe?$AAd?$AA?5?$AAC?$AAr?$AAi?$AAt?$AAS?$AAe?$AAc?$AA?3?$AA?5?$AA?$CF?$AAx?$AA?4?$AA?$AN@ 10003f70     mdd.obj
 0001:00002fb8       ??_C@_1GK@PCKMKKFI@?$AAC?$AAO?$AAM?$AA_?$AAW?$AAr?$AAi?$AAt?$AAe?$AA?5?$AAw?$AAa?$AAi?$AAt?$AA?5?$AAf?$AAo?$AAr?$AA?5?$AAt?$AAr?$AAa?$AAn?$AAs?$AAm?$AAi?$AAs?$AAs?$AAi?$AAo?$AAn?$AA?5@ 10003fb8     mdd.obj
 0001:00003024       ??_C@_1DK@IBJJCGOP@?$AAC?$AAO?$AAM?$AA_?$AAW?$AAr?$AAi?$AAt?$AAe?$AA?5?$AA?9?$AA?5?$AAA?$AAb?$AAo?$AAr?$AAt?$AAi?$AAn?$AAg?$AA?5?$AAw?$AAr?$AAi?$AAt?$AAe?$AA?$AN?$AA?6?$AA?$AA@ 10004024     mdd.obj
 0001:00003060       ??_C@_1EA@JJCCGAEK@?$AAC?$AAO?$AAM?$AA_?$AAW?$AAr?$AAi?$AAt?$AAe?$AA?5?$AA?9?$AA?5?$AAd?$AAe?$AAv?$AAi?$AAc?$AAe?$AA?5?$AAw?$AAa?$AAs?$AA?5?$AAc?$AAl?$AAo?$AAs?$AAe?$AAd?$AA?6?$AA?$AN?$AA?$AA@ 10004060     mdd.obj
 0001:000030a0       ??_C@_1FE@LGJDMHNB@?$AAC?$AAO?$AAM?$AA_?$AAW?$AAr?$AAi?$AAt?$AAe?$AA?5?$AAr?$AAe?$AAl?$AAe?$AAa?$AAs?$AAe?$AAd?$AA?5?$AAC?$AAr?$AAi?$AAt?$AAS?$AAe?$AAc?$AA?3?$AA?5?$AA?$CF?$AAx?$AA?4?$AA?5@ 100040a0     mdd.obj
 0001:000030f4       ??_C@_1DG@PKENKCNO@?$AA?9?$AAC?$AAO?$AAM?$AA_?$AAW?$AAR?$AAI?$AAT?$AAE?$AA?0?$AA?5?$AAr?$AAe?$AAt?$AAu?$AAr?$AAn?$AAi?$AAn?$AAg?$AA?5?$AA?$CF?$AAd?$AA?6?$AA?$AN?$AA?$AA@ 100040f4     mdd.obj
 0001:0000312c       ??_C@_1BM@KPCOGPII@?$AA?$DO?$AAC?$AAO?$AAM?$AA_?$AAP?$AAo?$AAw?$AAe?$AAr?$AAU?$AAp?$AA?6?$AA?$AA@ 1000412c     mdd.obj
 0001:00003148       ??_C@_1EO@NMNMJGIA@?$AA?$DO?$AAC?$AAO?$AAM?$AA_?$AAP?$AAo?$AAw?$AAe?$AAr?$AAU?$AAp?$AA?4?$AA?5?$AAE?$AAr?$AAr?$AAo?$AAr?$AA?5?$AAp?$AAH?$AAW?$AAI?$AAH?$AAe?$AAa?$AAd?$AA?5?$AA?$DN?$AA?$DN?$AA?5@ 10004148     mdd.obj
 0001:00003198       ??_C@_1CA@NAGNEGF@?$AA?$DO?$AAC?$AAO?$AAM?$AA_?$AAP?$AAo?$AAw?$AAe?$AAr?$AAD?$AAo?$AAw?$AAn?$AA?6?$AA?$AA@ 10004198     mdd.obj
 0001:000031b8       ??_C@_1EI@CENKJDJK@?$AA?$CL?$AAW?$AAa?$AAi?$AAt?$AAC?$AAo?$AAm?$AAm?$AAE?$AAv?$AAe?$AAn?$AAt?$AA?5?$AAx?$AA?$CF?$AAX?$AA?5?$AAx?$AA?$CF?$AAX?$AA?0?$AA?5?$AAp?$AAM?$AAa?$AAs?$AAk?$AA?5?$AAx?$AA?$CF@ 100041b8     mdd.obj
 0001:00003200       ??_C@_1FM@MENBDCNM@?$AA?9?$AAW?$AAa?$AAi?$AAt?$AAC?$AAo?$AAm?$AAm?$AAE?$AAv?$AAe?$AAn?$AAt?$AA?5?$AA?9?$AA?5?$AAd?$AAe?$AAv?$AAi?$AAc?$AAe?$AA?5?$AAn?$AAo?$AAt?$AA?5?$AAo?$AAp?$AAe?$AAn@ 10004200     mdd.obj
 0001:00003260       ??_C@_1EM@NBPFGEAJ@?$AA?9?$AAW?$AAa?$AAi?$AAt?$AAC?$AAo?$AAm?$AAm?$AAE?$AAv?$AAe?$AAn?$AAt?$AA?5?$AA?9?$AA?5?$AAM?$AAa?$AAs?$AAk?$AA?5?$AAa?$AAl?$AAr?$AAe?$AAa?$AAd?$AAy?$AA?5?$AAc?$AAl@ 10004260     mdd.obj
 0001:000032b0       ??_C@_1GI@MFJIILJA@?$AA?5?$AAW?$AAa?$AAi?$AAt?$AAC?$AAo?$AAm?$AAm?$AAE?$AAv?$AAe?$AAn?$AAt?$AA?5?$AA?9?$AA?5?$AAE?$AAv?$AAe?$AAn?$AAt?$AAs?$AA?5?$AA0?$AAx?$AA?$CF?$AAX?$AA?0?$AA?5?$AAM?$AAa@ 100042b0     mdd.obj
 0001:00003318       ??_C@_1EI@FGBADKHH@?$AA?5?$AAW?$AAa?$AAi?$AAt?$AAC?$AAo?$AAm?$AAm?$AAE?$AAv?$AAe?$AAn?$AAt?$AA?5?$AA?9?$AA?5?$AAM?$AAa?$AAs?$AAk?$AA?5?$AAw?$AAa?$AAs?$AA?5?$AAc?$AAl?$AAe?$AAa?$AAr?$AAe@ 10004318     mdd.obj
 0001:00003360       ??_C@_1EK@BIALANPL@?$AA?9?$AAW?$AAa?$AAi?$AAt?$AAC?$AAo?$AAm?$AAm?$AAE?$AAv?$AAe?$AAn?$AAt?$AA?5?$AA?9?$AA?5?$AAd?$AAe?$AAv?$AAi?$AAc?$AAe?$AA?5?$AAw?$AAa?$AAs?$AA?5?$AAc?$AAl?$AAo?$AAs@ 10004360     mdd.obj
 0001:000033b0       ??_C@_1EO@HJMBEPIE@?$AA?9?$AAW?$AAa?$AAi?$AAt?$AAC?$AAo?$AAm?$AAm?$AAE?$AAv?$AAe?$AAn?$AAt?$AA?5?$AA?9?$AA?5?$AA?$CK?$AAp?$AAf?$AAd?$AAw?$AAE?$AAv?$AAe?$AAn?$AAt?$AAM?$AAa?$AAs?$AAk?$AA?5@ 100043b0     mdd.obj
 0001:00003400       ??_C@_1FC@CHEKKMIP@?$AA?5?$AAE?$AAv?$AAa?$AAl?$AAu?$AAa?$AAt?$AAe?$AAE?$AAv?$AAe?$AAn?$AAt?$AAF?$AAl?$AAa?$AAg?$AA?5?$AA?9?$AA?5?$AAd?$AAe?$AAv?$AAi?$AAc?$AAe?$AA?5?$AAw?$AAa?$AAs?$AA?5@ 10004400     mdd.obj
 0001:00003458       ??_C@_1FI@GNEBOJFH@?$AA?5?$AAC?$AAo?$AAm?$AAm?$AAE?$AAv?$AAe?$AAn?$AAt?$AA?5?$AA?9?$AA?5?$AAE?$AAv?$AAe?$AAn?$AAt?$AA?5?$AA0?$AAx?$AA?$CF?$AAX?$AA?0?$AA?5?$AAG?$AAl?$AAo?$AAb?$AAa?$AAl?$AA?5@ 10004458     mdd.obj
 0001:000034b0       ??_C@_1GM@NOKKMADJ@?$AA?5?$AAC?$AAo?$AAm?$AAm?$AAE?$AAv?$AAe?$AAn?$AAt?$AA?5?$AA?9?$AA?5?$AAE?$AAv?$AAe?$AAn?$AAt?$AA?5?$AA0?$AAx?$AA?$CF?$AAX?$AA?0?$AA?5?$AAH?$AAa?$AAn?$AAd?$AAl?$AAe?$AA?5@ 100044b0     mdd.obj
 0001:00003520       ??_C@_1FI@OMADJLMN@?$AA?5?$AAC?$AAO?$AAM?$AA_?$AAI?$AAO?$AAC?$AAo?$AAn?$AAt?$AAr?$AAo?$AAl?$AA?5?$AA?9?$AA?5?$AAE?$AAr?$AAr?$AAo?$AAr?$AA?5?$AAp?$AAO?$AAp?$AAe?$AAn?$AAH?$AAe?$AAa?$AAd@ 10004520     mdd.obj
 0001:00003578       ??_C@_1GK@BPHGGHEJ@?$AA?$CL?$AAC?$AAO?$AAM?$AA_?$AAI?$AAO?$AAC?$AAo?$AAn?$AAt?$AAr?$AAo?$AAl?$AA?$CI?$AA0?$AAx?$AA?$CF?$AAX?$AA?0?$AA?5?$AA?$CF?$AAd?$AA?0?$AA?5?$AA0?$AAx?$AA?$CF?$AAX?$AA?0?$AA?5?$AA?$CF@ 10004578     mdd.obj
 0001:000035e8       ??_C@_1GO@LMOKINEG@?$AAC?$AAO?$AAM?$AA_?$AAI?$AAO?$AAC?$AAo?$AAn?$AAt?$AAr?$AAo?$AAl?$AA?0?$AA?5?$AAU?$AAn?$AAp?$AAl?$AAu?$AAg?$AAg?$AAe?$AAd?$AA?5?$AAd?$AAe?$AAv?$AAi?$AAc?$AAe?$AA?5@ 100045e8     mdd.obj
 0001:00003658       ??_C@_1EK@GAFFJFEI@?$AA?5?$AAC?$AAO?$AAM?$AA_?$AAI?$AAO?$AAC?$AAo?$AAn?$AAt?$AAr?$AAo?$AAl?$AA?5?$AA?9?$AA?5?$AAd?$AAe?$AAv?$AAi?$AAc?$AAe?$AA?5?$AAw?$AAa?$AAs?$AA?5?$AAc?$AAl?$AAo?$AAs@ 10004658     mdd.obj
 0001:000036a4       ??_C@_1CM@DKOMLJNL@?$AAP?$AAr?$AAo?$AAc?$AAe?$AAs?$AAs?$AA?5?$AAi?$AAs?$AA?5?$AAe?$AAx?$AAi?$AAt?$AAi?$AAn?$AAg?$AA?4?$AA?$AN?$AA?6?$AA?$AA@ 100046a4     mdd.obj
 0001:000036d0       ??_C@_1GI@OFPAKAHG@?$AAC?$AAO?$AAM?$AA_?$AAI?$AAo?$AAc?$AAt?$AAl?$AA?3?$AA?5?$AAI?$AAo?$AAc?$AAt?$AAl?$AA?5?$AA?$CF?$AAx?$AA?5?$AAa?$AAc?$AAc?$AAe?$AAs?$AAs?$AA?5?$AAp?$AAe?$AAr?$AAm?$AAi@ 100046d0     mdd.obj
 0001:00003738       ??_C@_1DK@NGIHOHIF@?$AA?5?$AAI?$AAO?$AAC?$AAT?$AAL?$AA_?$AAS?$AAE?$AAR?$AAI?$AAA?$AAL?$AA_?$AAS?$AAE?$AAT?$AA_?$AAB?$AAR?$AAE?$AAA?$AAK?$AA_?$AAO?$AAN?$AA?$AN?$AA?6?$AA?$AA@ 10004738     mdd.obj
 0001:00003774       ??_C@_1DM@GNACIDMB@?$AA?5?$AAI?$AAO?$AAC?$AAT?$AAL?$AA_?$AAS?$AAE?$AAR?$AAI?$AAA?$AAL?$AA_?$AAS?$AAE?$AAT?$AA_?$AAB?$AAR?$AAE?$AAA?$AAK?$AA_?$AAO?$AAF?$AAF?$AA?$AN?$AA?6?$AA?$AA@ 10004774     mdd.obj
 0001:000037b0       ??_C@_1DA@NGELBLAF@?$AA?5?$AAI?$AAO?$AAC?$AAT?$AAL?$AA_?$AAS?$AAE?$AAR?$AAI?$AAA?$AAL?$AA_?$AAS?$AAE?$AAT?$AA_?$AAD?$AAT?$AAR?$AA?$AN?$AA?6?$AA?$AA@ 100047b0     mdd.obj
 0001:000037e0       ??_C@_1DA@JNBPMBCJ@?$AA?5?$AAI?$AAO?$AAC?$AAT?$AAL?$AA_?$AAS?$AAE?$AAR?$AAI?$AAA?$AAL?$AA_?$AAC?$AAL?$AAR?$AA_?$AAD?$AAT?$AAR?$AA?$AN?$AA?6?$AA?$AA@ 100047e0     mdd.obj
 0001:00003810       ??_C@_1DA@PJMEFDIH@?$AA?5?$AAI?$AAO?$AAC?$AAT?$AAL?$AA_?$AAS?$AAE?$AAR?$AAI?$AAA?$AAL?$AA_?$AAS?$AAE?$AAT?$AA_?$AAR?$AAT?$AAS?$AA?$AN?$AA?6?$AA?$AA@ 10004810     mdd.obj
 0001:00003840       ??_C@_1DA@LCJAIJKL@?$AA?5?$AAI?$AAO?$AAC?$AAT?$AAL?$AA_?$AAS?$AAE?$AAR?$AAI?$AAA?$AAL?$AA_?$AAC?$AAL?$AAR?$AA_?$AAR?$AAT?$AAS?$AA?$AN?$AA?6?$AA?$AA@ 10004840     mdd.obj
 0001:00003870       ??_C@_1DC@OONFCAKE@?$AA?5?$AAI?$AAO?$AAC?$AAT?$AAL?$AA_?$AAS?$AAE?$AAR?$AAI?$AAA?$AAL?$AA_?$AAS?$AAE?$AAT?$AA_?$AAX?$AAO?$AAF?$AAF?$AA?$AN?$AA?6?$AA?$AA@ 10004870     mdd.obj
 0001:000038a4       ??_C@_1DA@CLADOFAD@?$AA?5?$AAI?$AAO?$AAC?$AAT?$AAL?$AA_?$AAS?$AAE?$AAR?$AAI?$AAA?$AAL?$AA_?$AAS?$AAE?$AAT?$AA_?$AAX?$AAO?$AAN?$AA?$AN?$AA?6?$AA?$AA@ 100048a4     mdd.obj
 0001:000038d4       ??_C@_1DM@BJAAJCOJ@?$AA?5?$AAI?$AAO?$AAC?$AAT?$AAL?$AA_?$AAS?$AAE?$AAR?$AAI?$AAA?$AAL?$AA_?$AAG?$AAE?$AAT?$AA_?$AAW?$AAA?$AAI?$AAT?$AA_?$AAM?$AAA?$AAS?$AAK?$AA?$AN?$AA?6?$AA?$AA@ 100048d4     mdd.obj
 0001:00003910       ??_C@_1CK@EJMDEGNB@?$AA?5?$AAI?$AAn?$AAv?$AAa?$AAl?$AAi?$AAd?$AA?5?$AAp?$AAa?$AAr?$AAa?$AAm?$AAe?$AAt?$AAe?$AAr?$AA?$AN?$AA?6?$AA?$AA@ 10004910     mdd.obj
 0001:00003940       ??_C@_1EG@JONHGGFH@?$AA?5?$AAI?$AAO?$AAC?$AAT?$AAL?$AA_?$AAS?$AAE?$AAR?$AAI?$AAA?$AAL?$AA_?$AAS?$AAE?$AAT?$AA_?$AAW?$AAA?$AAI?$AAT?$AA_?$AAM?$AAA?$AAS?$AAK?$AA?5?$AA0?$AAx?$AA?$CF?$AAX@ 10004940     mdd.obj
 0001:00003988       ??_C@_1EK@BIBFMIMA@?$AA?5?$AAS?$AAe?$AAt?$AAW?$AAa?$AAi?$AAt?$AAM?$AAa?$AAs?$AAk?$AA?5?$AA?9?$AA?5?$AAh?$AAa?$AAn?$AAd?$AAl?$AAe?$AA?5?$AAx?$AA?$CF?$AAX?$AA?5?$AAm?$AAa?$AAs?$AAk?$AA?5?$AAx@ 10004988     mdd.obj
 0001:000039d8       ??_C@_1FG@BOKINKK@?$AA?5?$AAS?$AAe?$AAt?$AAW?$AAa?$AAi?$AAt?$AAM?$AAa?$AAs?$AAk?$AA?5?$AA?9?$AA?5?$AAm?$AAa?$AAs?$AAk?$AA?5?$AAx?$AA?$CF?$AAX?$AA?0?$AA?5?$AAg?$AAl?$AAo?$AAb?$AAa?$AAl?$AA?5@ 100049d8     mdd.obj
 0001:00003a30       ??_C@_1DK@MHHDNLMO@?$AA?5?$AAI?$AAO?$AAC?$AAT?$AAL?$AA_?$AAS?$AAE?$AAR?$AAI?$AAA?$AAL?$AA_?$AAW?$AAA?$AAI?$AAT?$AA_?$AAO?$AAN?$AA_?$AAM?$AAA?$AAS?$AAK?$AA?$AN?$AA?6?$AA?$AA@ 10004a30     mdd.obj
 0001:00003a70       ??_C@_1FE@DCNACOPO@?$AA?5?$AAC?$AAO?$AAM?$AA_?$AAI?$AAO?$AAC?$AAo?$AAn?$AAt?$AAr?$AAo?$AAl?$AA?5?$AA?9?$AA?5?$AAE?$AAr?$AAr?$AAo?$AAr?$AA?5?$AAi?$AAn?$AA?5?$AAW?$AAa?$AAi?$AAt?$AAC?$AAo@ 10004a70     mdd.obj
 0001:00003ac4       ??_C@_1DO@GPNOPFOC@?$AA?5?$AAI?$AAO?$AAC?$AAT?$AAL?$AA_?$AAS?$AAE?$AAR?$AAI?$AAA?$AAL?$AA_?$AAG?$AAE?$AAT?$AA_?$AAC?$AAO?$AAM?$AAM?$AAS?$AAT?$AAA?$AAT?$AAU?$AAS?$AA?$AN?$AA?6?$AA?$AA@ 10004ac4     mdd.obj
 0001:00003b08       ??_C@_1EA@IBDHDHLD@?$AA?5?$AAI?$AAO?$AAC?$AAT?$AAL?$AA_?$AAS?$AAE?$AAR?$AAI?$AAA?$AAL?$AA_?$AAG?$AAE?$AAT?$AA_?$AAM?$AAO?$AAD?$AAE?$AAM?$AAS?$AAT?$AAA?$AAT?$AAU?$AAS?$AA?$AN?$AA?6?$AA?$AA@ 10004b08     mdd.obj
 0001:00003b48       ??_C@_1DO@COBPCJBD@?$AA?5?$AAI?$AAO?$AAC?$AAT?$AAL?$AA_?$AAS?$AAE?$AAR?$AAI?$AAA?$AAL?$AA_?$AAG?$AAE?$AAT?$AA_?$AAP?$AAR?$AAO?$AAP?$AAE?$AAR?$AAT?$AAI?$AAE?$AAS?$AA?$AN?$AA?6?$AA?$AA@ 10004b48     mdd.obj
 0001:00003b88       ??_C@_1GE@COCIEMAI@?$AA?5?$AAI?$AAO?$AAC?$AAT?$AAL?$AA_?$AAS?$AAE?$AAR?$AAI?$AAA?$AAL?$AA_?$AAS?$AAE?$AAT?$AA_?$AAC?$AAO?$AAM?$AAM?$AAT?$AAI?$AAM?$AAE?$AAO?$AAU?$AAT?$AAS?$AA?5?$AA?$CI@ 10004b88     mdd.obj
 0001:00003bec       ??_C@_1DK@FGFBKMCP@?$AA?5?$AAI?$AAO?$AAC?$AAT?$AAL?$AA_?$AAS?$AAE?$AAR?$AAI?$AAA?$AAL?$AA_?$AAG?$AAE?$AAT?$AA_?$AAT?$AAI?$AAM?$AAE?$AAO?$AAU?$AAT?$AAS?$AA?$AN?$AA?6?$AA?$AA@ 10004bec     mdd.obj
 0001:00003c28       ??_C@_1DG@NONFKDMH@?$AA?5?$AAI?$AAO?$AAC?$AAT?$AAL?$AA_?$AAS?$AAE?$AAR?$AAI?$AAA?$AAL?$AA_?$AAP?$AAU?$AAR?$AAG?$AAE?$AA?5?$AA0?$AAx?$AA?$CF?$AAX?$AA?$AN?$AA?6?$AA?$AA@ 10004c28     mdd.obj
 0001:00003c60       ??_C@_1FE@LCKDINPA@?$AA?5?$AAF?$AAl?$AAu?$AAs?$AAh?$AAi?$AAn?$AAg?$AA?5?$AA?$CF?$AAd?$AA?5?$AAb?$AAy?$AAt?$AAe?$AAs?$AA?5?$AAf?$AAr?$AAo?$AAm?$AA?5?$AAt?$AAh?$AAe?$AA?5?$AAr?$AAe?$AAa?$AAd@ 10004c60     mdd.obj
 0001:00003cb8       ??_C@_1EO@NAIOPLFA@?$AA?5?$AAI?$AAO?$AAC?$AAT?$AAL?$AA_?$AAS?$AAE?$AAR?$AAI?$AAA?$AAL?$AA_?$AAS?$AAE?$AAT?$AA_?$AAQ?$AAU?$AAE?$AAU?$AAE?$AA_?$AAS?$AAI?$AAZ?$AAE?$AA?5?$AA?$CI?$AA?$CF?$AAd@ 10004cb8     mdd.obj
 0001:00003d08       ??_C@_1EI@KIHCPENE@?$AA?5?$AAI?$AAO?$AAC?$AAT?$AAL?$AA_?$AAS?$AAE?$AAR?$AAI?$AAA?$AAL?$AA_?$AAI?$AAM?$AAM?$AAE?$AAD?$AAI?$AAA?$AAT?$AAE?$AA_?$AAC?$AAH?$AAA?$AAR?$AA?5?$AA0?$AAx?$AA?$CF@ 10004d08     mdd.obj
 0001:00003d50       ??_C@_1DA@MBKJPAMD@?$AA?5?$AAI?$AAO?$AAC?$AAT?$AAL?$AA_?$AAS?$AAE?$AAR?$AAI?$AAA?$AAL?$AA_?$AAG?$AAE?$AAT?$AA_?$AAD?$AAC?$AAB?$AA?$AN?$AA?6?$AA?$AA@ 10004d50     mdd.obj
 0001:00003d80       ??_C@_1DA@GPICLALP@?$AA?5?$AAI?$AAO?$AAC?$AAT?$AAL?$AA_?$AAS?$AAE?$AAR?$AAI?$AAA?$AAL?$AA_?$AAS?$AAE?$AAT?$AA_?$AAD?$AAC?$AAB?$AA?$AN?$AA?6?$AA?$AA@ 10004d80     mdd.obj
 0001:00003db0       ??_C@_1CG@IAPBOCP@?$AA?5?$AAA?$AAp?$AAp?$AAl?$AAy?$AAD?$AAC?$AAB?$AA?5?$AAf?$AAa?$AAi?$AAl?$AAe?$AAd?$AA?$AN?$AA?6?$AA?$AA@ 10004db0     mdd.obj
 0001:00003dd8       ??_C@_1CE@NOAPAGNI@?$AAI?$AAO?$AAC?$AAT?$AAL?$AA?5?$AAE?$AAn?$AAa?$AAb?$AAl?$AAe?$AA?5?$AAI?$AAR?$AA?$AN?$AA?6?$AA?$AA@ 10004dd8     mdd.obj
 0001:00003dfc       ??_C@_1CC@LGNHCIBI@?$AAI?$AAR?$AA?5?$AAm?$AAo?$AAd?$AAe?$AA?5?$AAf?$AAa?$AAi?$AAl?$AAe?$AAd?$AA?$AN?$AA?6?$AA?$AA@ 10004dfc     mdd.obj
 0001:00003e20       ??_C@_1CG@MLMOPDDN@?$AAI?$AAO?$AAC?$AAT?$AAL?$AA?5?$AAD?$AAi?$AAs?$AAa?$AAb?$AAl?$AAe?$AA?5?$AAI?$AAR?$AA?$AN?$AA?6?$AA?$AA@ 10004e20     mdd.obj
 0001:00003e48       ??_C@_1CM@ENDIALIE@?$AA?5?$AAI?$AAn?$AAv?$AAa?$AAl?$AAi?$AAd?$AA?5?$AAi?$AAo?$AAc?$AAt?$AAl?$AA?5?$AA0?$AAx?$AA?$CF?$AAX?$AA?$AN?$AA?6?$AA?$AA@ 10004e48     mdd.obj
 0001:00003e74       ??_C@_1BA@JFDCMKFN@?$AAS?$AAu?$AAc?$AAc?$AAe?$AAs?$AAs?$AA?$AA@ 10004e74     mdd.obj
 0001:00003e84       ??_C@_1M@ILHOPKA@?$AAE?$AAr?$AAr?$AAo?$AAr?$AA?$AA@ 10004e84     mdd.obj
 0001:00003e90       ??_C@_1EM@GAPNEPLB@?$AA?9?$AAC?$AAO?$AAM?$AA_?$AAI?$AAO?$AAC?$AAo?$AAn?$AAt?$AAr?$AAo?$AAl?$AA?5?$AA?$CF?$AAs?$AA?5?$AAE?$AAc?$AAo?$AAd?$AAe?$AA?$DN?$AA?$CF?$AAd?$AA?5?$AA?$CI?$AAl?$AAe?$AAn?$AA?$DN@ 10004e90     mdd.obj
 0001:00003ee0       _IoVTbl                    10004ee0     ftdi_ser.obj
 0001:00004208       ??_C@_1DI@KFJKHKDI@?$AA?$DO?$AAF?$AAT?$AAD?$AAI?$AAW?$AAr?$AAi?$AAt?$AAe?$AAT?$AAr?$AAa?$AAn?$AAs?$AAf?$AAe?$AAr?$AAC?$AAo?$AAm?$AAp?$AAl?$AAe?$AAt?$AAe?$AA?6?$AA?$AA@ 10005208     ftdi_ser.obj
 0001:00004240       ??_C@_1DG@KGMCLKFK@?$AA?$CK?$AA?$CK?$AA?$CK?$AA?5?$AAS?$AAe?$AAt?$AAE?$AAv?$AAe?$AAn?$AAt?$AA?5?$AAE?$AAR?$AAR?$AAO?$AAR?$AA?3?$AA?$CF?$AAd?$AA?5?$AA?$CK?$AA?$CK?$AA?$CK?$AA?6?$AA?$AA@ 10005240     ftdi_ser.obj
 0001:00004278       ??_C@_1FI@BPFNGHAP@?$AA?$CK?$AA?$CK?$AA?$CK?$AA?5?$AAF?$AAT?$AAD?$AAI?$AAW?$AAr?$AAi?$AAt?$AAe?$AAT?$AAr?$AAa?$AAn?$AAs?$AAf?$AAe?$AAr?$AAC?$AAo?$AAm?$AAp?$AAl?$AAe?$AAt?$AAe?$AA?5?$AAE?$AAR@ 10005278     ftdi_ser.obj
 0001:000042d0       ??_C@_1DI@JOLAFNJG@?$AA?$DM?$AAF?$AAT?$AAD?$AAI?$AAW?$AAr?$AAi?$AAt?$AAe?$AAT?$AAr?$AAa?$AAn?$AAs?$AAf?$AAe?$AAr?$AAC?$AAo?$AAm?$AAp?$AAl?$AAe?$AAt?$AAe?$AA?6?$AA?$AA@ 100052d0     ftdi_ser.obj
 0001:00004308       ??_C@_1DK@KDDNDDOD@?$AAE?$AAn?$AAt?$AAe?$AAr?$AAe?$AAd?$AA?5?$AAF?$AAT?$AAD?$AAI?$AAE?$AAv?$AAe?$AAn?$AAt?$AAT?$AAh?$AAr?$AAe?$AAa?$AAd?$AA?5?$AA?$CF?$AAX?$AA?$AN?$AA?6?$AA?$AA@ 10005308     ftdi_ser.obj
 0001:00004348       ??_C@_1EC@IIAKPKJI@?$AAS?$AAp?$AAi?$AAn?$AAn?$AAi?$AAn?$AAg?$AA?5?$AAi?$AAn?$AA?5?$AAd?$AAi?$AAs?$AAp?$AAa?$AAt?$AAc?$AAh?$AA?5?$AAt?$AAh?$AAr?$AAe?$AAa?$AAd?$AA?5?$AA?$CF?$AAX?$AA?6?$AA?$AN@ 10005348     ftdi_ser.obj
 0001:0000438c       ??_C@_1DK@MMEIMHPK@?$AAE?$AAv?$AAe?$AAn?$AAt?$AA?5?$AA?$CF?$AAX?$AA?0?$AA?5?$AAI?$AAn?$AAd?$AAe?$AAx?$AA?5?$AA?$CF?$AAd?$AA?0?$AA?5?$AAI?$AAn?$AAt?$AA?5?$AA?$CF?$AAd?$AA?$AN?$AA?6?$AA?$AA@ 1000538c     ftdi_ser.obj
 0001:000043c8       ??_C@_1DK@OJBMLGML@?$AAF?$AAT?$AAD?$AAI?$AAE?$AAv?$AAe?$AAn?$AAt?$AAT?$AAh?$AAr?$AAe?$AAa?$AAd?$AA?5?$AA?$CF?$AAx?$AA?5?$AAe?$AAx?$AAi?$AAt?$AAi?$AAn?$AAg?$AA?$AN?$AA?6?$AA?$AA@ 100053c8     ftdi_ser.obj
 0001:00004408       ??_C@_1EG@LOJAOGIE@?$AAE?$AAr?$AAr?$AAo?$AAr?$AA?5?$AAc?$AAr?$AAe?$AAa?$AAt?$AAi?$AAn?$AAg?$AA?5?$AAE?$AAv?$AAe?$AAn?$AAt?$AA?5?$AAt?$AAh?$AAr?$AAe?$AAa?$AAd?$AA?5?$AA?$CI?$AA?$CF?$AAd?$AA?$CJ@ 10005408     ftdi_ser.obj
 0001:00004450       ??_C@_1DE@HAHCLMBN@?$AAC?$AAr?$AAe?$AAa?$AAt?$AAe?$AAd?$AA?5?$AAE?$AAv?$AAe?$AAn?$AAt?$AA?5?$AAt?$AAh?$AAr?$AAe?$AAa?$AAd?$AA?5?$AA?$CF?$AAX?$AA?$AN?$AA?6?$AA?$AA@ 10005450     ftdi_ser.obj
 0001:00004484       ??_C@_1DC@PAHLGEH@?$AAA?$AAb?$AAo?$AAu?$AAt?$AA?5?$AAt?$AAo?$AA?5?$AAs?$AAe?$AAt?$AA?5?$AAp?$AAr?$AAi?$AAo?$AAr?$AAi?$AAt?$AAy?$AA?4?$AA?$AN?$AA?6?$AA?$AA@ 10005484     ftdi_ser.obj
 0001:000044b8       ??_C@_1CA@DNNLFDGH@?$AAP?$AAr?$AAi?$AAo?$AAr?$AAi?$AAt?$AAy?$AA?5?$AAs?$AAe?$AAt?$AA?4?$AA?$AN?$AA?6?$AA?$AA@ 100054b8     ftdi_ser.obj
 0001:000044d8       ??_C@_1EI@KOGHEFFI@?$AAA?$AAc?$AAt?$AAi?$AAv?$AAe?$AAS?$AAy?$AAn?$AAc?$AA?5?$AAt?$AAh?$AAr?$AAe?$AAa?$AAd?$AA?5?$AA?9?$AA?5?$AAI?$AAn?$AAv?$AAa?$AAl?$AAi?$AAd?$AA?5?$AAh?$AAa?$AAn?$AAd@ 100054d8     ftdi_ser.obj
 0001:00004520       ??_C@_1DM@LNDGNIKN@?$AAI?$AAn?$AAd?$AAi?$AAc?$AAa?$AAt?$AAe?$AAd?$AA?5?$AAR?$AAS?$AA2?$AA3?$AA2?$AA?5?$AAC?$AAa?$AAb?$AAl?$AAe?$AA?5?$AAE?$AAv?$AAe?$AAn?$AAt?$AA?$AN?$AA?6?$AA?$AA@ 10005520     ftdi_ser.obj
 0001:0000455c       ??_C@_1M@DFKENGJN@?$AA?$CF?$AAs?$AA?2?$AA?$CF?$AAs?$AA?$AA@ 1000555c     ftdi_ser.obj
 0001:00004568       ??_C@_1CE@ILLNCEFP@?$AAA?$AAc?$AAt?$AAi?$AAv?$AAe?$AAS?$AAy?$AAn?$AAc?$AAS?$AAe?$AAt?$AAt?$AAi?$AAn?$AAg?$AA?$AA@ 10005568     ftdi_ser.obj
 0001:00004590       ??_C@_1FK@GOPHHIPH@?$AAF?$AAa?$AAi?$AAl?$AAe?$AAd?$AA?5?$AAt?$AAo?$AA?5?$AAg?$AAe?$AAt?$AA?5?$AAr?$AAe?$AAg?$AAi?$AAs?$AAt?$AAr?$AAy?$AA?5?$AAs?$AAe?$AAt?$AAt?$AAi?$AAn?$AAg?$AAs?$AA?5@ 10005590     ftdi_ser.obj
 0001:000045f0       ??_C@_1FK@IJDJMFDF@?$AAA?$AAc?$AAt?$AAi?$AAv?$AAe?$AAS?$AAy?$AAn?$AAc?$AA?5?$AAT?$AAh?$AAr?$AAe?$AAa?$AAd?$AA?5?$AAN?$AAo?$AAt?$AA?5?$AAE?$AAx?$AAi?$AAt?$AAe?$AAd?$AA?5?$AAP?$AAr?$AAo@ 100055f0     ftdi_ser.obj
 0001:00004650       ??_C@_1EA@BIKPCLNL@?$AAF?$AAa?$AAi?$AAl?$AAe?$AAd?$AA?5?$AAt?$AAo?$AA?5?$AAo?$AAp?$AAe?$AAn?$AA?5?$AA?$CF?$AAs?$AA?0?$AA?5?$AAE?$AAr?$AAr?$AAo?$AAr?$AA?5?$AA0?$AAx?$AA?$CF?$AAX?$AA?$AN?$AA?6?$AA?$AA@ 10005650     ftdi_ser.obj
 0001:00004690       ??_C@_17KACEIPNC@?$AAK?$AAe?$AAy?$AA?$AA@ 10005690     ftdi_ser.obj
 0001:00004698       ??_C@_1FG@CBCEGKFJ@?$AAF?$AAa?$AAi?$AAl?$AAe?$AAd?$AA?5?$AAt?$AAo?$AA?5?$AAf?$AAi?$AAn?$AAd?$AA?5?$AAd?$AAa?$AAt?$AAa?$AA?5?$AAa?$AAt?$AA?5?$AA?$CF?$AAs?$AA?2?$AA?$CF?$AAs?$AA?0?$AA?5?$AAE?$AAr@ 10005698     ftdi_ser.obj
 0001:000046f0       ??_C@_1CA@BCJOMFGA@?$AA?$CL?$AAS?$AAe?$AAr?$AAI?$AAn?$AAi?$AAt?$AA?5?$AA?9?$AA?5?$AA?$CF?$AAX?$AA?$AN?$AA?6?$AA?$AA@ 100056f0     ftdi_ser.obj
 0001:00004710       ??_C@_1DG@LHHJOINK@?$AA?$CL?$AAS?$AAe?$AAr?$AAI?$AAn?$AAi?$AAt?$AA?5?$AAI?$AAd?$AAe?$AAn?$AAt?$AAi?$AAf?$AAi?$AAe?$AAr?$AA?5?$AA?9?$AA?5?$AA?$CF?$AAX?$AA?$AN?$AA?6?$AA?$AA@ 10005710     ftdi_ser.obj
 0001:00004748       ??_C@_1HA@FBCOOAMN@?$AAS?$AAe?$AAr?$AAI?$AAn?$AAi?$AAt?$AA?5?$AA?9?$AA?5?$AAU?$AAn?$AAa?$AAb?$AAl?$AAe?$AA?5?$AAt?$AAo?$AA?5?$AAr?$AAe?$AAa?$AAd?$AA?5?$AAr?$AAe?$AAg?$AAi?$AAs?$AAt?$AAr@ 10005748     ftdi_ser.obj
 0001:000047b8       ??_C@_1CA@FLNBNCFP@?$AA?9?$AAS?$AAe?$AAr?$AAI?$AAn?$AAi?$AAt?$AA?5?$AA?9?$AA?5?$AA?$CF?$AAX?$AA?$AN?$AA?6?$AA?$AA@ 100057b8     ftdi_ser.obj
 0001:000047d8       ??_C@_1FM@LHCCMHLB@?$AAE?$AAv?$AAe?$AAn?$AAt?$AAT?$AAh?$AAr?$AAe?$AAa?$AAd?$AA?5?$AAT?$AAh?$AAr?$AAe?$AAa?$AAd?$AA?5?$AAN?$AAo?$AAt?$AA?5?$AAE?$AAx?$AAi?$AAt?$AAe?$AAd?$AA?5?$AAP?$AAr@ 100057d8     ftdi_ser.obj
 0001:00004834       ??_C@_1CM@FJCCIHDC@?$AAI?$AAn?$AAi?$AAt?$AAi?$AAa?$AAl?$AAi?$AAs?$AAe?$AAO?$AAp?$AAe?$AAn?$AAD?$AAe?$AAv?$AAi?$AAc?$AAe?$AA?6?$AA?$AA@ 10005834     ftdi_ser.obj
 0001:00004860       ??_C@_1CM@CAALJEKG@?$AAC?$AAr?$AAe?$AAa?$AAt?$AAe?$AAE?$AAv?$AAe?$AAn?$AAt?$AA?5?$AAe?$AAr?$AAr?$AAo?$AAr?$AA?3?$AA?$CF?$AAd?$AA?6?$AA?$AA@ 10005860     ftdi_ser.obj
 0001:0000488c       ??_C@_1CM@IBCBMLIC@?$AAC?$AAr?$AAe?$AAa?$AAt?$AAe?$AAM?$AAu?$AAt?$AAe?$AAx?$AA?5?$AAe?$AAr?$AAr?$AAo?$AAr?$AA?3?$AA?$CF?$AAd?$AA?6?$AA?$AA@ 1000588c     ftdi_ser.obj
 0001:000048b8       ??_C@_1DM@PFHODMGA@?$AAR?$AAe?$AAa?$AAd?$AA?5?$AAB?$AAu?$AAf?$AAf?$AAe?$AAr?$AA?5?$AAa?$AAl?$AAl?$AAo?$AAc?$AA?5?$AAe?$AAr?$AAr?$AAo?$AAr?$AA?5?$AA?$DN?$AA?5?$AA?$CF?$AAd?$AA?6?$AA?$AA@ 100058b8     ftdi_ser.obj
 0001:000048f4       ??_C@_1BK@GLGKBGNH@?$AAL?$AAa?$AAt?$AAe?$AAn?$AAc?$AAy?$AAT?$AAi?$AAm?$AAe?$AAr?$AA?$AA@ 100058f4     ftdi_ser.obj
 0001:00004910       ??_C@_1BO@FLELEHKB@?$AAI?$AAn?$AAT?$AAr?$AAa?$AAn?$AAs?$AAf?$AAe?$AAr?$AAS?$AAi?$AAz?$AAe?$AA?$AA@ 10005910     ftdi_ser.obj
 0001:00004930       ??_C@_1CA@CBPLKEPJ@?$AAO?$AAu?$AAt?$AAT?$AAr?$AAa?$AAn?$AAs?$AAf?$AAe?$AAr?$AAS?$AAi?$AAz?$AAe?$AA?$AA@ 10005930     ftdi_ser.obj
 0001:00004950       ??_C@_1BG@IFDFFDLO@?$AAC?$AAo?$AAn?$AAf?$AAi?$AAg?$AAD?$AAa?$AAt?$AAa?$AA?$AA@ 10005950     ftdi_ser.obj
 0001:00004968       ??_C@_1BM@JCMCOHGE@?$AAD?$AAe?$AAv?$AAi?$AAc?$AAe?$AAC?$AAo?$AAn?$AAt?$AAe?$AAx?$AAt?$AA?$AA@ 10005968     ftdi_ser.obj
 0001:00004988       ??_C@_1EC@KMHNPOHP@?$AAF?$AAa?$AAi?$AAl?$AAe?$AAd?$AA?5?$AAt?$AAo?$AA?5?$AAs?$AAe?$AAt?$AA?5?$AAD?$AAe?$AAv?$AAi?$AAc?$AAe?$AA?5?$AAC?$AAo?$AAn?$AAt?$AAe?$AAx?$AAt?$AA?3?$AA?$CF?$AAd?$AA?6@ 10005988     ftdi_ser.obj
 0001:000049cc       ??_C@_1BM@KEONHDCJ@?$AAE?$AAm?$AAu?$AAl?$AAa?$AAt?$AAi?$AAo?$AAn?$AAM?$AAo?$AAd?$AAe?$AA?$AA@ 100059cc     ftdi_ser.obj
 0001:000049e8       ??_C@_1GM@DJGHOPAK@?$AAF?$AAa?$AAi?$AAl?$AAe?$AAd?$AA?5?$AAt?$AAo?$AA?5?$AAi?$AAn?$AAi?$AAt?$AAi?$AAa?$AAl?$AAi?$AAs?$AAe?$AA?5?$AAM?$AAo?$AAd?$AAe?$AAm?$AA?5?$AAe?$AAm?$AAu?$AAl?$AAa@ 100059e8     ftdi_ser.obj
 0001:00004a54       ??_C@_1CG@MMMJBOMI@?$AAm?$AAs?$AAS?$AAl?$AAe?$AAe?$AAp?$AAA?$AAf?$AAt?$AAe?$AAr?$AAB?$AAu?$AAl?$AAk?$AAI?$AAn?$AA?$AA@ 10005a54     ftdi_ser.obj
 0001:00004a80       ??_C@_1EO@INMGKABB@?$AAF?$AAT?$AAD?$AA_?$AAO?$AAp?$AAe?$AAn?$AA?5?$AAE?$AAr?$AAr?$AAo?$AAr?$AA?5?$AA?$CF?$AAd?$AA?5?$AAc?$AAr?$AAe?$AAa?$AAt?$AAi?$AAn?$AAg?$AA?5?$AAB?$AAu?$AAl?$AAk?$AAI@ 10005a80     ftdi_ser.obj
 0001:00004ad0       ??_C@_1CC@NGCCJKHO@?$AAT?$AAh?$AAr?$AAe?$AAa?$AAd?$AA?5?$AAP?$AAr?$AAi?$AAo?$AAr?$AA?3?$AA?$CF?$AAd?$AA?6?$AA?$AA@ 10005ad0     ftdi_ser.obj
 0001:00004af4       ??_C@_1CA@KIFMDICO@?$AAC?$AAo?$AAn?$AAf?$AAi?$AAg?$AAD?$AAa?$AAt?$AAa?$AAF?$AAl?$AAa?$AAg?$AAs?$AA?$AA@ 10005af4     ftdi_ser.obj
 0001:00004b14       ??_C@_1BK@HLLNPFIM@?$AAB?$AAu?$AAl?$AAk?$AAP?$AAr?$AAi?$AAo?$AAr?$AAi?$AAt?$AAy?$AA?$AA@ 10005b14     ftdi_ser.obj
 0001:00004b30       ??_C@_1EE@FONFPEDK@?$AAE?$AAr?$AAr?$AAo?$AAr?$AA?5?$AAs?$AAe?$AAt?$AAt?$AAi?$AAn?$AAg?$AA?5?$AAB?$AAu?$AAl?$AAk?$AA?5?$AAP?$AAr?$AAi?$AAo?$AAr?$AAi?$AAt?$AAy?$AA?5?$AA?$DN?$AA?5?$AA?$CF?$AAd@ 10005b30     ftdi_ser.obj
 0001:00004b74       ??_C@_1DG@GFDDINE@?$AAS?$AAe?$AAt?$AA?5?$AAB?$AAu?$AAl?$AAk?$AA?5?$AAP?$AAr?$AAi?$AAo?$AAr?$AAi?$AAt?$AAy?$AA?5?$AAt?$AAo?$AA?5?$AA?$DN?$AA?5?$AA?$CF?$AAd?$AA?6?$AA?$AA@ 10005b74     ftdi_ser.obj
 0001:00004bac       ??_C@_1DG@HLFDKNBE@?$AAN?$AAo?$AA?5?$AAe?$AAn?$AAt?$AAr?$AAy?$AA?5?$AAf?$AAo?$AAr?$AA?5?$AAB?$AAu?$AAl?$AAk?$AAP?$AAr?$AAi?$AAo?$AAr?$AAi?$AAt?$AAy?$AA?6?$AA?$AA@ 10005bac     ftdi_ser.obj
 0001:00004be4       ??_C@_1BO@HDCCNDFF@?$AAB?$AAu?$AAl?$AAk?$AAP?$AAr?$AAi?$AAo?$AAr?$AAi?$AAt?$AAy?$AAE?$AAx?$AA?$AA@ 10005be4     ftdi_ser.obj
 0001:00004c04       ??_C@_1BM@ONMIKGLP@?$AAB?$AAu?$AAl?$AAk?$AAT?$AAi?$AAm?$AAe?$AAS?$AAl?$AAi?$AAc?$AAe?$AA?$AA@ 10005c04     ftdi_ser.obj
 0001:00004c20       ??_C@_1EI@KMGKNMMN@?$AAE?$AAr?$AAr?$AAo?$AAr?$AA?5?$AAs?$AAe?$AAt?$AAt?$AAi?$AAn?$AAg?$AA?5?$AAB?$AAu?$AAl?$AAk?$AA?5?$AAT?$AAi?$AAm?$AAe?$AA?5?$AAS?$AAl?$AAi?$AAc?$AAe?$AA?5?$AA?$DN?$AA?5@ 10005c20     ftdi_ser.obj
 0001:00004c68       ??_C@_1EC@HHHHLBIM@?$AAS?$AAe?$AAt?$AAt?$AAi?$AAn?$AAg?$AA?5?$AAB?$AAu?$AAl?$AAk?$AA?5?$AAT?$AAi?$AAm?$AAe?$AA?5?$AAS?$AAl?$AAi?$AAc?$AAe?$AA?5?$AAt?$AAo?$AA?5?$AA?$DN?$AA?5?$AA?$CF?$AAd?$AA?6@ 10005c68     ftdi_ser.obj
 0001:00004cac       ??_C@_1DI@JGDLCJMK@?$AAN?$AAo?$AA?5?$AAe?$AAn?$AAt?$AAr?$AAy?$AA?5?$AAf?$AAo?$AAr?$AA?5?$AAB?$AAu?$AAl?$AAk?$AAT?$AAi?$AAm?$AAe?$AAS?$AAl?$AAi?$AAc?$AAe?$AA?6?$AA?$AA@ 10005cac     ftdi_ser.obj
 0001:00004ce8       ??_C@_1FO@BKPPABNH@?$AAC?$AAo?$AAu?$AAl?$AAd?$AA?5?$AAn?$AAo?$AAt?$AA?5?$AAo?$AAp?$AAe?$AAn?$AA?5?$AAr?$AAe?$AAg?$AAi?$AAs?$AAt?$AAr?$AAy?$AA?5?$AAe?$AAn?$AAt?$AAr?$AAy?$AA?5?$AAf?$AAo@ 10005ce8     ftdi_ser.obj
 0001:00004d48       ??_C@_1FI@LCLHOBE@?$AAC?$AAl?$AAe?$AAa?$AAn?$AAu?$AAp?$AAO?$AAp?$AAe?$AAn?$AAD?$AAe?$AAv?$AAi?$AAc?$AAe?$AA?3?$AA?5?$AAF?$AAa?$AAi?$AAl?$AAe?$AAd?$AA?5?$AAt?$AAo?$AA?5?$AAo?$AAp?$AAe@ 10005d48     ftdi_ser.obj
 0001:00004da0       ??_C@_1CI@PJHJHJNH@?$AA?$DO?$AAC?$AAl?$AAe?$AAa?$AAn?$AAu?$AAp?$AAO?$AAp?$AAe?$AAn?$AAD?$AAe?$AAv?$AAi?$AAc?$AAe?$AA?6?$AA?$AA@ 10005da0     ftdi_ser.obj
 0001:00004dc8       ??_C@_1DK@MBIBFBJC@?$AAC?$AAl?$AAo?$AAs?$AAe?$AAH?$AAa?$AAn?$AAd?$AAl?$AAe?$AA?5?$AA?$CI?$AAE?$AAv?$AAe?$AAn?$AAt?$AA?$CJ?$AAe?$AAr?$AAr?$AAo?$AAr?$AA?3?$AA?$CF?$AAd?$AA?6?$AA?$AA@ 10005dc8     ftdi_ser.obj
 0001:00004e08       ??_C@_1FE@KNBDDELK@?$AAC?$AAl?$AAo?$AAs?$AAe?$AAH?$AAa?$AAn?$AAd?$AAl?$AAe?$AA?5?$AA?$CI?$AAR?$AAe?$AAa?$AAd?$AA?5?$AAR?$AAe?$AAq?$AAu?$AAe?$AAs?$AAt?$AA?5?$AAE?$AAv?$AAe?$AAn?$AAt?$AA?$CJ@ 10005e08     ftdi_ser.obj
 0001:00004e5c       ??_C@_1DM@BAAOJNAM@?$AAC?$AAl?$AAo?$AAs?$AAe?$AAH?$AAa?$AAn?$AAd?$AAl?$AAe?$AA?5?$AA?$CI?$AAT?$AAh?$AAr?$AAe?$AAa?$AAd?$AA?$CJ?$AAe?$AAr?$AAr?$AAo?$AAr?$AA?3?$AA?$CF?$AAd?$AA?6?$AA?$AA@ 10005e5c     ftdi_ser.obj
 0001:00004e98       ??_C@_1DK@GAKLAOLG@?$AAC?$AAl?$AAo?$AAs?$AAe?$AAH?$AAa?$AAn?$AAd?$AAl?$AAe?$AA?5?$AA?$CI?$AAM?$AAu?$AAt?$AAe?$AAx?$AA?$CJ?$AAe?$AAr?$AAr?$AAo?$AAr?$AA?3?$AA?$CF?$AAd?$AA?6?$AA?$AA@ 10005e98     ftdi_ser.obj
 0001:00004ed8       ??_C@_1EO@KNFGMDCA@?$AAL?$AAo?$AAc?$AAa?$AAl?$AAF?$AAr?$AAe?$AAe?$AA?5?$AAU?$AAs?$AAe?$AAr?$AA?5?$AAB?$AAu?$AAf?$AAf?$AAe?$AAr?$AA?5?$AAF?$AAa?$AAi?$AAl?$AAe?$AAd?$AA?5?$AAE?$AAr?$AAr@ 10005ed8     ftdi_ser.obj
 0001:00004f28       ??_C@_1GE@PKELNCGB@?$AAL?$AAo?$AAc?$AAa?$AAl?$AAF?$AAr?$AAe?$AAe?$AA?5?$AAM?$AAo?$AAd?$AAe?$AAm?$AA?5?$AAE?$AAm?$AAu?$AAl?$AAa?$AAt?$AAi?$AAo?$AAn?$AA?5?$AAB?$AAu?$AAf?$AAf?$AAe?$AAr@ 10005f28     ftdi_ser.obj
 0001:00004f8c       ??_C@_1CI@HMIBFLBI@?$AA?$DM?$AAC?$AAl?$AAe?$AAa?$AAn?$AAu?$AAp?$AAO?$AAp?$AAe?$AAn?$AAD?$AAe?$AAv?$AAi?$AAc?$AAe?$AA?6?$AA?$AA@ 10005f8c     ftdi_ser.obj
 0001:00004fb4       ??_C@_1BE@FEKPIPNA@?$AA?$DO?$AAS?$AAe?$AAr?$AAO?$AAp?$AAe?$AAn?$AA?6?$AA?$AA@ 10005fb4     ftdi_ser.obj
 0001:00004fc8       ??_C@_1BO@OIAOGKHD@?$AA?$DO?$AAA?$AAl?$AAr?$AAe?$AAa?$AAd?$AAy?$AA?5?$AAO?$AAp?$AAe?$AAn?$AA?6?$AA?$AA@ 10005fc8     ftdi_ser.obj
 0001:00004fe8       ??_C@_1BE@JOGBPJFM@?$AA?$DM?$AAS?$AAe?$AAr?$AAO?$AAp?$AAe?$AAn?$AA?6?$AA?$AA@ 10005fe8     ftdi_ser.obj
 0001:00004ffc       ??_C@_1BG@LJFLNHIJ@?$AA?$DO?$AAS?$AAe?$AAr?$AAC?$AAl?$AAo?$AAs?$AAe?$AA?6?$AA?$AA@ 10005ffc     ftdi_ser.obj
 0001:00005014       ??_C@_1DG@DOIFBNPG@?$AAS?$AAe?$AAr?$AAC?$AAl?$AAo?$AAs?$AAe?$AA?0?$AA?5?$AAc?$AAl?$AAo?$AAs?$AAi?$AAn?$AAg?$AA?5?$AAd?$AAe?$AAv?$AAi?$AAc?$AAe?$AA?$AN?$AA?6?$AA?$AA@ 10006014     ftdi_ser.obj
 0001:0000504c       ??_C@_1DI@IPEJEOAH@?$AAS?$AAe?$AAt?$AAE?$AAv?$AAe?$AAn?$AAt?$AA?5?$AAh?$AAC?$AAl?$AAo?$AAs?$AAe?$AAR?$AAe?$AAa?$AAd?$AAe?$AAr?$AAE?$AAv?$AAe?$AAn?$AAt?$AA?6?$AA?$AA@ 1000604c     ftdi_ser.obj
 0001:00005088       ??_C@_1EE@NGMLODEE@?$AAT?$AAh?$AAr?$AAe?$AAa?$AAd?$AA?5?$AAN?$AAo?$AAt?$AA?5?$AAE?$AAx?$AAi?$AAt?$AAe?$AAd?$AA?5?$AAP?$AAr?$AAo?$AAp?$AAe?$AAr?$AAl?$AAy?$AA?5?$AAE?$AAr?$AAr?$AAo?$AAr@ 10006088     ftdi_ser.obj
 0001:000050cc       ??_C@_1DE@FBCDFANI@?$AAC?$AAl?$AAe?$AAa?$AAn?$AAu?$AAp?$AAO?$AAp?$AAe?$AAn?$AAD?$AAe?$AAv?$AAi?$AAc?$AAe?$AA?5?$AAF?$AAa?$AAi?$AAl?$AAe?$AAd?$AA?6?$AA?$AA@ 100060cc     ftdi_ser.obj
 0001:00005100       ??_C@_1DA@ICHDMNMM@?$AAS?$AAe?$AAr?$AAC?$AAl?$AAo?$AAs?$AAe?$AA?5?$AAf?$AAo?$AAr?$AA?5?$AAd?$AAe?$AAv?$AAi?$AAc?$AAe?$AA?5?$AA?$CF?$AAp?$AA?6?$AA?$AA@ 10006100     ftdi_ser.obj
 0001:00005130       ??_C@_1BG@JHALBOAJ@?$AA?$DM?$AAS?$AAe?$AAr?$AAC?$AAl?$AAo?$AAs?$AAe?$AA?6?$AA?$AA@ 10006130     ftdi_ser.obj
 0001:00005148       ??_C@_1CO@FBINAKOG@?$AA?$DO?$AAS?$AAe?$AAr?$AAR?$AAx?$AAI?$AAn?$AAt?$AAr?$AA?5?$AA?9?$AA?5?$AAl?$AAe?$AAn?$AA?5?$AA?$CF?$AAd?$AA?4?$AA?$AN?$AA?6?$AA?$AA@ 10006148     ftdi_ser.obj
 0001:00005178       ??_C@_1CO@PBHBEGHD@?$AAh?$AAB?$AAu?$AAf?$AAf?$AAe?$AAr?$AAM?$AAu?$AAt?$AAe?$AAx?$AA?5?$AAe?$AAr?$AAr?$AAo?$AAr?$AA?3?$AA?$CF?$AAd?$AA?6?$AA?$AA@ 10006178     ftdi_ser.obj
 0001:000051a8       ??_C@_1EK@NFIABAFN@?$AAU?$AAn?$AAh?$AAa?$AAn?$AAd?$AAl?$AAe?$AAd?$AA?5?$AAB?$AAu?$AAf?$AAf?$AAe?$AAr?$AAM?$AAu?$AAt?$AAe?$AAx?$AA?5?$AAW?$AAa?$AAi?$AAt?$AAR?$AAe?$AAa?$AAs?$AAo?$AAn@ 100061a8     ftdi_ser.obj
 0001:000051f8       ??_C@_1EE@OFPCFJOL@?$AAD?$AAr?$AAo?$AAp?$AAp?$AAi?$AAn?$AAg?$AA?5?$AAN?$AAU?$AAL?$AAL?$AA?5?$AAb?$AAy?$AAt?$AAe?$AA?5?$AAd?$AAu?$AAe?$AA?5?$AAt?$AAo?$AA?5?$AAf?$AAN?$AAu?$AAl?$AAl?$AA?$AN@ 100061f8     ftdi_ser.obj
 0001:0000523c       ??_C@_1BC@JCEPIOOB@?$AAR?$AAX?$AA?5?$AA?$CF?$AAX?$AA?3?$AA?$AN?$AA?6?$AA?$AA@ 1000623c     ftdi_ser.obj
 0001:00005250       ??_C@_1BM@ONDFPGAI@?$AAL?$AAa?$AAs?$AAt?$AA?5?$AAR?$AAX?$AA?5?$AA?$CF?$AAX?$AA?3?$AA?$AN?$AA?6?$AA?$AA@ 10006250     ftdi_ser.obj
 0001:0000526c       ??_C@_1DC@MJGLGIFH@?$AAR?$AAe?$AAa?$AAd?$AAC?$AAo?$AAp?$AAi?$AAe?$AAd?$AA?5?$AAf?$AAr?$AAo?$AAm?$AA?5?$AA?$CF?$AAd?$AA?5?$AAt?$AAo?$AA?5?$AA?$CF?$AAd?$AA?$AA@ 1000626c     ftdi_ser.obj
 0001:000052a0       ??_C@_1EK@DHJPFOIA@?$AAR?$AAX?$AAI?$AAn?$AAt?$AAr?$AA?5?$AA?3?$AA?5?$AA?$CF?$AAd?$AA?5?$AAb?$AAy?$AAt?$AAe?$AAs?$AA?5?$AAl?$AAe?$AAf?$AAt?$AA?5?$AAi?$AAn?$AA?5?$AAF?$AAT?$AAD?$AA?5?$AA?$CI?$AA?$CF@ 100062a0     ftdi_ser.obj
 0001:000052ec       ??_C@_1DM@MFNNGNED@?$AA?9?$AAG?$AAe?$AAt?$AAB?$AAy?$AAt?$AAe?$AAs?$AA?5?$AA?9?$AA?5?$AAr?$AAx?$AA?5?$AA?$CF?$AAd?$AA?0?$AA?5?$AAd?$AAr?$AAo?$AAp?$AA?5?$AA?$CF?$AAd?$AA?4?$AA?$AN?$AA?6?$AA?$AA@ 100062ec     ftdi_ser.obj
 0001:00005328       ??_C@_1EC@LCCJPMFD@?$AAS?$AAe?$AAr?$AAG?$AAe?$AAt?$AAI?$AAn?$AAt?$AAe?$AAr?$AAr?$AAu?$AAp?$AAt?$AAT?$AAy?$AAp?$AAe?$AA?3?$AA?5?$AAI?$AAN?$AAT?$AAR?$AA_?$AAL?$AAI?$AAN?$AAE?$AA?$AN?$AA?6@ 10006328     ftdi_ser.obj
 0001:00005370       ??_C@_1EE@MCCFCCPO@?$AAS?$AAe?$AAr?$AAG?$AAe?$AAt?$AAI?$AAn?$AAt?$AAe?$AAr?$AAr?$AAu?$AAp?$AAt?$AAT?$AAy?$AAp?$AAe?$AA?3?$AA?5?$AAI?$AAN?$AAT?$AAR?$AA_?$AAM?$AAO?$AAD?$AAE?$AAM?$AA?$AN@ 10006370     ftdi_ser.obj
 0001:000053b4       ??_C@_1DO@NACOHOKB@?$AAS?$AAe?$AAr?$AAG?$AAe?$AAt?$AAI?$AAn?$AAt?$AAe?$AAr?$AAr?$AAu?$AAp?$AAt?$AAT?$AAy?$AAp?$AAe?$AA?3?$AA?5?$AAI?$AAN?$AAT?$AAR?$AA_?$AAT?$AAX?$AA?$AN?$AA?6?$AA?$AA@ 100063b4     ftdi_ser.obj
 0001:000053f4       ??_C@_1DO@NNDAAOOG@?$AAS?$AAe?$AAr?$AAG?$AAe?$AAt?$AAI?$AAn?$AAt?$AAe?$AAr?$AAr?$AAu?$AAp?$AAt?$AAT?$AAy?$AAp?$AAe?$AA?3?$AA?5?$AAI?$AAN?$AAT?$AAR?$AA_?$AAR?$AAX?$AA?$AN?$AA?6?$AA?$AA@ 100063f4     ftdi_ser.obj
 0001:00005434       ??_C@_1DM@BMEGOPAM@?$AAM?$AAo?$AAd?$AAe?$AAm?$AA?5?$AAS?$AAt?$AAa?$AAt?$AAu?$AAs?$AA?5?$AA?$CF?$AA2?$AA?4?$AA2?$AAX?$AA?5?$AA?$DM?$AA?$DO?$AA?5?$AA?$CF?$AA2?$AA?4?$AA2?$AAX?$AA?$AN?$AA?6?$AA?$AA@ 10006434     ftdi_ser.obj
 0001:00005470       ??_C@_1CK@KAHJLAMC@?$AAO?$AAu?$AAt?$AAR?$AAe?$AAq?$AAu?$AAe?$AAs?$AAt?$AA?5?$AAe?$AAr?$AAr?$AAo?$AAr?$AA?3?$AA?$CF?$AAd?$AA?6?$AA?$AA@ 10006470     ftdi_ser.obj
 0001:0000549c       ??_C@_1DC@GEKLBHMI@?$AAn?$AAR?$AAe?$AAq?$AAu?$AAe?$AAs?$AAt?$AA?5?$AAR?$AAE?$AAS?$AAE?$AAT?$AAT?$AAI?$AAN?$AAG?$AA?5?$AAP?$AAI?$AAP?$AAE?$AA?6?$AA?$AA@ 1000649c     ftdi_ser.obj
 0001:000054d0       ??_C@_1DE@HHLBBNBE@?$AAB?$AAu?$AAl?$AAk?$AA?5?$AAW?$AAr?$AAi?$AAt?$AAe?$AA?$DN?$AA?$CF?$AAd?$AA?0?$AA?5?$AAL?$AAe?$AAn?$AAg?$AAt?$AAh?$AA?$DN?$AA?$CF?$AAd?$AA?6?$AA?$AA@ 100064d0     ftdi_ser.obj
 0001:00005504       ??_C@_1DK@IHPFKPFO@?$AAB?$AAu?$AAl?$AAk?$AA?5?$AAn?$AAt?$AAS?$AAt?$AAa?$AAt?$AAu?$AAs?$AA?$DN?$AA?$CF?$AAd?$AA?0?$AA?5?$AAE?$AAr?$AAr?$AAo?$AAr?$AA?$DN?$AA?$CF?$AAd?$AA?5?$AA?6?$AA?$AA@ 10006504     ftdi_ser.obj
 0001:00005540       ??_C@_1EE@OAJGDHLJ@?$AAO?$AAu?$AAt?$AAR?$AAe?$AAq?$AAu?$AAe?$AAs?$AAt?$AA?5?$AAR?$AAe?$AAq?$AAu?$AAe?$AAs?$AAt?$AAe?$AAd?$AA?3?$AA?$CF?$AAd?$AA?5?$AAW?$AAr?$AAo?$AAt?$AAe?$AA?3?$AA?$CF?$AAd@ 10006540     ftdi_ser.obj
 0001:00005584       ??_C@_1CE@CDHMNDKP@?$AA?$DO?$AAS?$AAe?$AAr?$AAT?$AAx?$AAI?$AAn?$AAt?$AAr?$AA?5?$AA0?$AAx?$AA?$CF?$AAX?$AA?$AN?$AA?6?$AA?$AA@ 10006584     ftdi_ser.obj
 0001:000055a8       ??_C@_1CM@BMGHKIPN@?$AAT?$AAX?$AA?3?$AA?5?$AAn?$AAo?$AAt?$AAh?$AAi?$AAn?$AAg?$AA?5?$AAt?$AAo?$AA?5?$AAs?$AAe?$AAn?$AAd?$AA?$AN?$AA?6?$AA?$AA@ 100065a8     ftdi_ser.obj
 0001:000055d4       ??_C@_1CM@PNCBOAPJ@?$AA?$DO?$AAW?$AAr?$AAi?$AAt?$AAe?$AA?5?$AAd?$AAw?$AAT?$AAi?$AAm?$AAe?$AAo?$AAu?$AAt?$AA?5?$AA?$CF?$AAd?$AA?$AN?$AA?6?$AA?$AA@ 100065d4     ftdi_ser.obj
 0001:00005600       ??_C@_1CC@LLLGBBIH@?$AA?$DO?$AAO?$AAu?$AAt?$AAR?$AAe?$AAq?$AAu?$AAe?$AAs?$AAt?$AA?5?$AA?$CF?$AAd?$AA?$AN?$AA?6?$AA?$AA@ 10006600     ftdi_ser.obj
 0001:00005628       ??_C@_1GA@OFKAHEBC@?$AAI?$AAs?$AAs?$AAu?$AAe?$AAB?$AAu?$AAl?$AAk?$AAT?$AAr?$AAa?$AAn?$AAs?$AAf?$AAe?$AAr?$AA?5?$AAe?$AAr?$AAr?$AAo?$AAr?$AA?3?$AA?$CF?$AAd?$AA?0?$AA?5?$AA0?$AAx?$AA?$CF?$AAx@ 10006628     ftdi_ser.obj
 0001:00005688       ??_C@_1EC@CAGBGMGJ@?$AA?$CK?$AA?$CK?$AA?$CK?$AA?5?$AAS?$AAe?$AAt?$AAS?$AAe?$AAr?$AAi?$AAa?$AAl?$AAE?$AAv?$AAe?$AAn?$AAt?$AA?5?$AAE?$AAR?$AAR?$AAO?$AAR?$AA?3?$AA?$CF?$AAd?$AA?5?$AA?$CK?$AA?$CK?$AA?$CK?$AA?6@ 10006688     ftdi_ser.obj
 0001:000056d0       ??_C@_1EC@EHLOHMHJ@?$AAS?$AAe?$AAr?$AAT?$AAx?$AAI?$AAn?$AAt?$AAr?$AA?3?$AA?5?$AAE?$AAR?$AAR?$AAO?$AAR?$AA_?$AAI?$AAN?$AAV?$AAA?$AAL?$AAI?$AAD?$AA_?$AAH?$AAA?$AAN?$AAD?$AAL?$AAE?$AA?6@ 100066d0     ftdi_ser.obj
 0001:00005714       ??_C@_1BM@EPBABDBM@?$AAT?$AAx?$AA?5?$AA?$CF?$AAd?$AA?5?$AAo?$AAf?$AA?5?$AA?$CF?$AAd?$AA?$AN?$AA?6?$AA?$AA@ 10006714     ftdi_ser.obj
 0001:00005730       ??_C@_1CE@NCOMHMME@?$AA?$DM?$AAS?$AAe?$AAr?$AAT?$AAx?$AAI?$AAn?$AAt?$AAr?$AA?5?$AA0?$AAx?$AA?$CF?$AAX?$AA?$AN?$AA?6?$AA?$AA@ 10006730     ftdi_ser.obj
 0001:00005758       ??_C@_1GC@OICOCFAO@?$AAS?$AAe?$AAr?$AAP?$AAo?$AAw?$AAe?$AAr?$AAO?$AAf?$AAf?$AA?5?$AA?9?$AA?5?$AAh?$AAa?$AAv?$AAe?$AA?5?$AAw?$AAe?$AA?5?$AAb?$AAe?$AAe?$AAn?$AA?5?$AAs?$AAu?$AAr?$AAp?$AAr@ 10006758     ftdi_ser.obj
 0001:000057bc       ??_C@_1CK@PLILIICG@?$AA?$DO?$AAS?$AAe?$AAr?$AAC?$AAl?$AAe?$AAa?$AAr?$AAD?$AAT?$AAR?$AA?0?$AA?5?$AA0?$AAx?$AA?$CF?$AAX?$AA?$AN?$AA?6?$AA?$AA@ 100067bc     ftdi_ser.obj
 0001:000057e8       ??_C@_1CK@GCIJIHLL@?$AA?$DM?$AAS?$AAe?$AAr?$AAC?$AAl?$AAe?$AAa?$AAr?$AAD?$AAT?$AAR?$AA?0?$AA?5?$AA0?$AAx?$AA?$CF?$AAX?$AA?$AN?$AA?6?$AA?$AA@ 100067e8     ftdi_ser.obj
 0001:00005814       ??_C@_1CG@OHCHFIF@?$AA?$DO?$AAS?$AAe?$AAr?$AAS?$AAe?$AAt?$AAD?$AAT?$AAR?$AA?0?$AA?5?$AA0?$AAx?$AA?$CF?$AAX?$AA?$AN?$AA?6?$AA?$AA@ 10006814     ftdi_ser.obj
 0001:0000583c       ??_C@_1CG@MOBCIIAA@?$AA?$DM?$AAS?$AAe?$AAr?$AAS?$AAe?$AAt?$AAD?$AAT?$AAR?$AA?0?$AA?5?$AA0?$AAx?$AA?$CF?$AAX?$AA?$AN?$AA?6?$AA?$AA@ 1000683c     ftdi_ser.obj
 0001:00005864       ??_C@_1CG@OHGLJHOI@?$AA?$DO?$AAS?$AAe?$AAr?$AAC?$AAl?$AAr?$AAR?$AAT?$AAS?$AA?0?$AA?5?$AA0?$AAx?$AA?$CF?$AAX?$AA?$AN?$AA?6?$AA?$AA@ 10006864     ftdi_ser.obj
 0001:0000588c       ??_C@_1CG@CHALGKGN@?$AA?$DM?$AAS?$AAe?$AAr?$AAC?$AAl?$AAr?$AAR?$AAT?$AAS?$AA?0?$AA?5?$AA0?$AAx?$AA?$CF?$AAX?$AA?$AN?$AA?6?$AA?$AA@ 1000688c     ftdi_ser.obj
 0001:000058b4       ??_C@_1CG@KEEDGDKO@?$AA?$DO?$AAS?$AAe?$AAr?$AAS?$AAe?$AAt?$AAR?$AAT?$AAS?$AA?0?$AA?5?$AA0?$AAx?$AA?$CF?$AAX?$AA?$AN?$AA?6?$AA?$AA@ 100068b4     ftdi_ser.obj
 0001:000058dc       ??_C@_1CG@GECDJOCL@?$AA?$DM?$AAS?$AAe?$AAr?$AAS?$AAe?$AAt?$AAR?$AAT?$AAS?$AA?0?$AA?5?$AA0?$AAx?$AA?$CF?$AAX?$AA?$AN?$AA?6?$AA?$AA@ 100068dc     ftdi_ser.obj
 0001:00005904       ??_C@_1CK@BNLABLFO@?$AA?$DO?$AAS?$AAe?$AAr?$AAC?$AAl?$AAr?$AAB?$AAr?$AAe?$AAa?$AAk?$AA?0?$AA?5?$AA0?$AAx?$AA?$CF?$AAX?$AA?$AN?$AA?6?$AA?$AA@ 10006904     ftdi_ser.obj
 0001:00005930       ??_C@_1CK@IELCBEMD@?$AA?$DM?$AAS?$AAe?$AAr?$AAC?$AAl?$AAr?$AAB?$AAr?$AAe?$AAa?$AAk?$AA?0?$AA?5?$AA0?$AAx?$AA?$CF?$AAX?$AA?$AN?$AA?6?$AA?$AA@ 10006930     ftdi_ser.obj
 0001:0000595c       ??_C@_1CK@KDIKHJDD@?$AA?$DO?$AAS?$AAe?$AAr?$AAS?$AAe?$AAt?$AAB?$AAr?$AAe?$AAa?$AAk?$AA?0?$AA?5?$AA0?$AAx?$AA?$CF?$AAX?$AA?$AN?$AA?6?$AA?$AA@ 1000695c     ftdi_ser.obj
 0001:00005988       ??_C@_1CK@DKIIHGKO@?$AA?$DM?$AAS?$AAe?$AAr?$AAS?$AAe?$AAt?$AAB?$AAr?$AAe?$AAa?$AAk?$AA?0?$AA?5?$AA0?$AAx?$AA?$CF?$AAX?$AA?$AN?$AA?6?$AA?$AA@ 10006988     ftdi_ser.obj
 0001:000059b4       ??_C@_1CO@CFACNPDH@?$AA?$CL?$AAS?$AAe?$AAr?$AAX?$AAm?$AAi?$AAt?$AAC?$AAo?$AAm?$AAC?$AAh?$AAa?$AAr?$AA?5?$AA0?$AAx?$AA?$CF?$AAX?$AA?$AN?$AA?6?$AA?$AA@ 100069b4     ftdi_ser.obj
 0001:000059e8       ??_C@_1EG@BHFJEBOE@?$AAX?$AAm?$AAi?$AAt?$AAC?$AAo?$AAm?$AAC?$AAh?$AAa?$AAr?$AA?5?$AAw?$AAa?$AAi?$AAt?$AA?5?$AAf?$AAo?$AAr?$AA?5?$AAC?$AAr?$AAi?$AAt?$AAS?$AAe?$AAc?$AA?5?$AA?$CF?$AAx?$AA?4@ 100069e8     ftdi_ser.obj
 0001:00005a30       ??_C@_1DM@FEOPEELB@?$AAX?$AAm?$AAi?$AAt?$AAC?$AAo?$AAm?$AAC?$AAh?$AAa?$AAr?$AA?5?$AAg?$AAo?$AAt?$AA?5?$AAC?$AAr?$AAi?$AAt?$AAS?$AAe?$AAc?$AA?5?$AA?$CF?$AAx?$AA?4?$AA?$AN?$AA?6?$AA?$AA@ 10006a30     ftdi_ser.obj
 0001:00005a70       ??_C@_1FE@HBAIIDKC@?$AA?$CB?$AA?$CB?$AA?$CB?$AA?5?$AAS?$AAe?$AAr?$AAX?$AAm?$AAi?$AAt?$AAC?$AAo?$AAm?$AAC?$AAh?$AAa?$AAr?$AA?5?$AA0?$AAx?$AA?$CF?$AAX?$AA?5?$AAn?$AAo?$AAt?$AA?5?$AAi?$AAm?$AAp?$AAl@ 10006a70     ftdi_ser.obj
 0001:00005ac8       ??_C@_1EG@GPEINPFO@?$AAX?$AAm?$AAi?$AAt?$AAC?$AAo?$AAm?$AAC?$AAh?$AAa?$AAr?$AA?5?$AAr?$AAe?$AAl?$AAe?$AAa?$AAs?$AAe?$AAd?$AA?5?$AAC?$AAr?$AAi?$AAt?$AAS?$AAe?$AAc?$AA?5?$AA?$CF?$AAx?$AA?4@ 10006ac8     ftdi_ser.obj
 0001:00005b10       ??_C@_1CO@POMGIABM@?$AA?9?$AAS?$AAe?$AAr?$AAX?$AAm?$AAi?$AAt?$AAC?$AAo?$AAm?$AAC?$AAh?$AAa?$AAr?$AA?5?$AA0?$AAx?$AA?$CF?$AAX?$AA?$AN?$AA?6?$AA?$AA@ 10006b10     ftdi_ser.obj
 0001:00005b40       ??_C@_1CK@CBBGJOLI@?$AA?$DO?$AAS?$AAe?$AAr?$AAG?$AAe?$AAt?$AAS?$AAt?$AAa?$AAt?$AAu?$AAs?$AA?5?$AA0?$AAx?$AA?$CF?$AAX?$AA?$AN?$AA?6?$AA?$AA@ 10006b40     ftdi_ser.obj
 0001:00005b6c       ??_C@_1CK@LIBEJBCF@?$AA?$DM?$AAS?$AAe?$AAr?$AAG?$AAe?$AAt?$AAS?$AAt?$AAa?$AAt?$AAu?$AAs?$AA?5?$AA0?$AAx?$AA?$CF?$AAX?$AA?$AN?$AA?6?$AA?$AA@ 10006b6c     ftdi_ser.obj
 0001:00005b98       ??_C@_1CC@BPNHIFLM@?$AA?$DO?$AAS?$AAe?$AAr?$AAR?$AAe?$AAs?$AAe?$AAt?$AA?5?$AA0?$AAx?$AA?$CF?$AAX?$AA?$AN?$AA?6?$AA?$AA@ 10006b98     ftdi_ser.obj
 0001:00005bbc       ??_C@_1CC@FGNDCHNA@?$AA?$DM?$AAS?$AAe?$AAr?$AAR?$AAe?$AAs?$AAe?$AAt?$AA?5?$AA0?$AAx?$AA?$CF?$AAX?$AA?$AN?$AA?6?$AA?$AA@ 10006bbc     ftdi_ser.obj
 0001:00005be0       ??_C@_1DE@LBMCLKEJ@?$AA?$DO?$AAS?$AAe?$AAr?$AAG?$AAe?$AAt?$AAM?$AAo?$AAd?$AAe?$AAm?$AAS?$AAt?$AAa?$AAt?$AAu?$AAs?$AA?5?$AA0?$AAx?$AA?$CF?$AAX?$AA?$AN?$AA?6?$AA?$AA@ 10006be0     ftdi_ser.obj
 0001:00005c18       ??_C@_1EM@LOCGMLJB@?$AA?$DM?$AAS?$AAe?$AAr?$AAG?$AAe?$AAt?$AAM?$AAo?$AAd?$AAe?$AAm?$AAS?$AAt?$AAa?$AAt?$AAu?$AAs?$AA?5?$AA0?$AAx?$AA?$CF?$AAX?$AA?5?$AA?$CI?$AAs?$AAt?$AAa?$AAt?$AA?5?$AAx?$AA?$CF@ 10006c18     ftdi_ser.obj
 0001:00005c64       ??_C@_1CK@ENPOKPNJ@?$AA?$DO?$AAS?$AAe?$AAr?$AAP?$AAu?$AAr?$AAg?$AAe?$AAC?$AAo?$AAm?$AAm?$AA?5?$AA0?$AAx?$AA?$CF?$AAX?$AA?$AN?$AA?6?$AA?$AA@ 10006c64     ftdi_ser.obj
 0001:00005c90       ??_C@_1DC@JCCLIFHN@?$AAP?$AAU?$AAR?$AAG?$AAE?$AA_?$AAR?$AAX?$AA?5?$AA?9?$AA?5?$AAs?$AAt?$AAo?$AAp?$AA?5?$AAi?$AAn?$AA?5?$AAt?$AAa?$AAs?$AAk?$AA?6?$AA?$AA@ 10006c90     ftdi_ser.obj
 0001:00005cc4       ??_C@_1BO@KKDAEKOA@?$AAP?$AAU?$AAR?$AAG?$AAE?$AA_?$AAT?$AAX?$AA?5?$AAD?$AAo?$AAn?$AAe?$AA?6?$AA?$AA@ 10006cc4     ftdi_ser.obj
 0001:00005ce4       ??_C@_1CK@NEPMKAEE@?$AA?$DM?$AAS?$AAe?$AAr?$AAP?$AAu?$AAr?$AAg?$AAe?$AAC?$AAo?$AAm?$AAm?$AA?5?$AA0?$AAx?$AA?$CF?$AAX?$AA?$AN?$AA?6?$AA?$AA@ 10006ce4     ftdi_ser.obj
 0001:00005d10       ??_C@_1CE@NJADOECG@?$AA?$DO?$AAS?$AAe?$AAr?$AAS?$AAe?$AAt?$AAD?$AAC?$AAB?$AA?5?$AA0?$AAx?$AA?$CF?$AAX?$AA?$AN?$AA?6?$AA?$AA@ 10006d10     ftdi_ser.obj
 0001:00005d34       ??_C@_1CE@CIJDELEN@?$AA?$DM?$AAS?$AAe?$AAr?$AAS?$AAe?$AAt?$AAD?$AAC?$AAB?$AA?5?$AA0?$AAx?$AA?$CF?$AAX?$AA?$AN?$AA?6?$AA?$AA@ 10006d34     ftdi_ser.obj
 0001:00005d58       ??_C@_1DE@MNLCJLCN@?$AA?$DO?$AAS?$AAe?$AAr?$AAS?$AAe?$AAt?$AAC?$AAo?$AAm?$AAm?$AAT?$AAi?$AAm?$AAe?$AAo?$AAu?$AAt?$AA?5?$AA0?$AAx?$AA?$CF?$AAX?$AA?$AN?$AA?6?$AA?$AA@ 10006d58     ftdi_ser.obj
 0001:00005d8c       ??_C@_1DE@BOCLGDDH@?$AA?$DM?$AAS?$AAe?$AAr?$AAS?$AAe?$AAt?$AAC?$AAo?$AAm?$AAm?$AAT?$AAi?$AAm?$AAe?$AAo?$AAu?$AAt?$AA?5?$AA0?$AAx?$AA?$CF?$AAX?$AA?$AN?$AA?6?$AA?$AA@ 10006d8c     ftdi_ser.obj
 0001:00005dc0       ??_C@_1CC@JPFEMKEK@?$AA?$CL?$AAS?$AAe?$AAr?$AAI?$AAo?$AAc?$AAt?$AAl?$AA?5?$AA0?$AAx?$AA?$CF?$AAX?$AA?$AN?$AA?6?$AA?$AA@ 10006dc0     ftdi_ser.obj
 0001:00005de8       ??_C@_1HA@LIMBNBIA@?$AAe?$AAx?$AAc?$AAe?$AAp?$AAt?$AAi?$AAo?$AAn?$AA?5?$AAr?$AAe?$AAa?$AAd?$AAi?$AAn?$AAg?$AA?5?$AAp?$AAB?$AAu?$AAf?$AAI?$AAn?$AA?5?$AAi?$AAn?$AA?5?$AAI?$AAO?$AAC?$AAT@ 10006de8     ftdi_ser.obj
 0001:00005e58       ??_C@_1HA@FGMDNPKG@?$AAe?$AAx?$AAc?$AAe?$AAp?$AAt?$AAi?$AAo?$AAn?$AA?5?$AAr?$AAe?$AAa?$AAd?$AAi?$AAn?$AAg?$AA?5?$AAp?$AAB?$AAu?$AAf?$AAI?$AAn?$AA?5?$AAi?$AAn?$AA?5?$AAI?$AAO?$AAC?$AAT@ 10006e58     ftdi_ser.obj
 0001:00005ec8       ??_C@_1GG@PDOBOPGO@?$AAe?$AAx?$AAc?$AAe?$AAp?$AAt?$AAi?$AAo?$AAn?$AA?5?$AAr?$AAe?$AAa?$AAd?$AAi?$AAn?$AAg?$AA?5?$AAp?$AAB?$AAu?$AAf?$AAI?$AAn?$AA?5?$AAi?$AAn?$AA?5?$AAI?$AAO?$AAC?$AAT@ 10006ec8     ftdi_ser.obj
 0001:00005f30       ??_C@_1GG@OOGJMKMK@?$AAe?$AAx?$AAc?$AAe?$AAp?$AAt?$AAi?$AAo?$AAn?$AA?5?$AAr?$AAe?$AAa?$AAd?$AAi?$AAn?$AAg?$AA?5?$AAp?$AAB?$AAu?$AAf?$AAI?$AAn?$AA?5?$AAi?$AAn?$AA?5?$AAI?$AAO?$AAC?$AAT@ 10006f30     ftdi_ser.obj
 0001:00005f98       ??_C@_1CG@JMPKJGDL@?$AA?$DO?$AAI?$AAO?$AAC?$AAT?$AAL?$AA_?$AAF?$AAT?$AA_?$AAS?$AAE?$AAT?$AA_?$AAD?$AAT?$AAR?$AA?6?$AA?$AA@ 10006f98     ftdi_ser.obj
 0001:00005fc0       ??_C@_1FM@PFMODAP@?$AAe?$AAx?$AAc?$AAe?$AAp?$AAt?$AAi?$AAo?$AAn?$AA?5?$AAr?$AAe?$AAa?$AAd?$AAi?$AAn?$AAg?$AA?5?$AAp?$AAB?$AAu?$AAf?$AAI?$AAn?$AA?5?$AAi?$AAn?$AA?5?$AAI?$AAO?$AAC?$AAT@ 10006fc0     ftdi_ser.obj
 0001:0000601c       ??_C@_1CG@FMJKGLLO@?$AA?$DM?$AAI?$AAO?$AAC?$AAT?$AAL?$AA_?$AAF?$AAT?$AA_?$AAS?$AAE?$AAT?$AA_?$AAD?$AAT?$AAR?$AA?6?$AA?$AA@ 1000701c     ftdi_ser.obj
 0001:00006048       ??_C@_1FM@EEGPKHP@?$AAe?$AAx?$AAc?$AAe?$AAp?$AAt?$AAi?$AAo?$AAn?$AA?5?$AAr?$AAe?$AAa?$AAd?$AAi?$AAn?$AAg?$AA?5?$AAp?$AAB?$AAu?$AAf?$AAI?$AAn?$AA?5?$AAi?$AAn?$AA?5?$AAI?$AAO?$AAC?$AAT@ 10007048     ftdi_ser.obj
 0001:000060a8       ??_C@_1FM@OOLAMBAF@?$AAe?$AAx?$AAc?$AAe?$AAp?$AAt?$AAi?$AAo?$AAn?$AA?5?$AAr?$AAe?$AAa?$AAd?$AAi?$AAn?$AAg?$AA?5?$AAp?$AAB?$AAu?$AAf?$AAI?$AAn?$AA?5?$AAi?$AAn?$AA?5?$AAI?$AAO?$AAC?$AAT@ 100070a8     ftdi_ser.obj
 0001:00006108       ??_C@_1FM@OFKKNIHF@?$AAe?$AAx?$AAc?$AAe?$AAp?$AAt?$AAi?$AAo?$AAn?$AA?5?$AAr?$AAe?$AAa?$AAd?$AAi?$AAn?$AAg?$AA?5?$AAp?$AAB?$AAu?$AAf?$AAI?$AAn?$AA?5?$AAi?$AAn?$AA?5?$AAI?$AAO?$AAC?$AAT@ 10007108     ftdi_ser.obj
 0001:00006164       ??_C@_1DE@DGKPEOKI@?$AA?5?$AAU?$AAn?$AAs?$AAu?$AAp?$AAp?$AAo?$AAr?$AAt?$AAe?$AAd?$AA?5?$AAi?$AAo?$AAc?$AAt?$AAl?$AA?5?$AA0?$AAx?$AA?$CF?$AAX?$AA?$AN?$AA?6?$AA?$AA@ 10007164     ftdi_ser.obj
 0001:00006198       ??_C@_1CC@EEFJCMPO@?$AA?9?$AAS?$AAe?$AAr?$AAI?$AAo?$AAc?$AAt?$AAl?$AA?5?$AA0?$AAx?$AA?$CF?$AAX?$AA?$AN?$AA?6?$AA?$AA@ 10007198     ftdi_ser.obj
 0001:000061bc       ??_C@_1DA@OMGLIHFF@?$AAG?$AAe?$AAt?$AAS?$AAe?$AAr?$AAi?$AAa?$AAl?$AAO?$AAb?$AAj?$AAe?$AAc?$AAt?$AA?5?$AAC?$AAa?$AAl?$AAl?$AAe?$AAd?$AA?6?$AA?$AA@ 100071bc     ftdi_ser.obj
 0001:000064a0       ??_C@_1BI@FIOGDOBI@?$AA?$DO?$AAS?$AAo?$AAf?$AAt?$AAR?$AAe?$AAs?$AAe?$AAt?$AA?6?$AA?$AA@ 100074a0     ftdi_utils.obj
 0001:000064b8       ??_C@_1CG@CPECMOOC@?$AAI?$AAn?$AAv?$AAa?$AAl?$AAi?$AAd?$AA?5?$AAp?$AAa?$AAr?$AAa?$AAm?$AAe?$AAt?$AAe?$AAr?$AA?6?$AA?$AA@ 100074b8     ftdi_utils.obj
 0001:000064e0       ??_C@_1EG@CBDBHDNI@?$AAI?$AAs?$AAs?$AAu?$AAe?$AAV?$AAe?$AAn?$AAd?$AAo?$AAr?$AAT?$AAr?$AAa?$AAn?$AAs?$AAf?$AAe?$AAr?$AA?5?$AAE?$AAR?$AAR?$AAO?$AAR?$AA?3?$AA?$CF?$AAd?$AA?5?$AA0?$AAx?$AA?$CF@ 100074e0     ftdi_utils.obj
 0001:00006528       ??_C@_1BO@DNFDGCMP@?$AA?$DM?$AAS?$AAo?$AAf?$AAt?$AAR?$AAe?$AAs?$AAe?$AAt?$AA?3?$AA?$CF?$AAd?$AA?6?$AA?$AA@ 10007528     ftdi_utils.obj
 0001:00006548       ??_C@_1DE@NDEIEHJE@?$AAR?$AAe?$AAs?$AAe?$AAt?$AAP?$AAi?$AAp?$AAe?$AA?5?$AAR?$AAE?$AAS?$AAE?$AAT?$AAT?$AAI?$AAN?$AAG?$AA?5?$AAP?$AAI?$AAP?$AAE?$AA?6?$AA?$AA@ 10007548     ftdi_utils.obj
 0001:0000657c       ??_C@_02BBAPPCCJ@IN?$AA@   1000757c     ftdi_utils.obj
 0001:00006580       ??_C@_03KJGMBMID@OUT?$AA@  10007580     ftdi_utils.obj
 0001:00006584       ??_C@_1DM@CMDINFMP@?$AAR?$AAe?$AAs?$AAe?$AAt?$AAP?$AAi?$AAp?$AAe?$AA?5?$AA?$CF?$AAs?$AA?5?$AAP?$AAI?$AAP?$AAE?$AA?5?$AAE?$AAR?$AAR?$AAO?$AAR?$AA?5?$AA0?$AAx?$AA?$CF?$AAx?$AA?6?$AA?$AA@ 10007584     ftdi_utils.obj
 0001:000065c0       ??_C@_1DG@LCIJCNCP@?$AA?$DO?$AAI?$AAo?$AAE?$AAr?$AAr?$AAo?$AAr?$AAH?$AAa?$AAn?$AAd?$AAl?$AAe?$AAr?$AA?$CI?$AA?$CF?$AAp?$AA?0?$AA?5?$AA0?$AAx?$AA?$CF?$AAx?$AA?$CJ?$AA?6?$AA?$AA@ 100075c0     ftdi_utils.obj
 0001:000065f8       ??_C@_1CC@EDCLNIN@?$AAU?$AAS?$AAB?$AA_?$AAS?$AAT?$AAA?$AAL?$AAL?$AA_?$AAE?$AAR?$AAR?$AAO?$AAR?$AA?6?$AA?$AA@ 100075f8     ftdi_utils.obj
 0001:00006620       ??_C@_1EC@IPINCEGC@?$AAU?$AAS?$AAB?$AA_?$AAD?$AAE?$AAV?$AAI?$AAC?$AAE?$AA_?$AAN?$AAO?$AAT?$AA_?$AAR?$AAE?$AAS?$AAP?$AAO?$AAN?$AAD?$AAI?$AAN?$AAG?$AA_?$AAE?$AAR?$AAR?$AAO?$AAR?$AA?6@ 10007620     ftdi_utils.obj
 0001:00006664       ??_C@_1BK@INEJMLAI@?$AAD?$AAe?$AAa?$AAd?$AA?5?$AAd?$AAe?$AAv?$AAi?$AAc?$AAe?$AA?6?$AA?$AA@ 10007664     ftdi_utils.obj
 0001:00006680       ??_C@_1EO@ECIKCPDJ@?$AAI?$AAo?$AAE?$AAr?$AAr?$AAo?$AAr?$AAH?$AAa?$AAn?$AAd?$AAl?$AAe?$AAr?$AA?3?$AA?5?$AAU?$AAn?$AAh?$AAa?$AAn?$AAd?$AAl?$AAe?$AAd?$AA?5?$AAe?$AAr?$AAr?$AAo?$AAr?$AA?3@ 10007680     ftdi_utils.obj
 0001:000066d0       ??_C@_1CG@KHNNFMCB@?$AAI?$AAn?$AAv?$AAa?$AAl?$AAi?$AAd?$AA?5?$AAP?$AAa?$AAr?$AAa?$AAm?$AAe?$AAt?$AAe?$AAr?$AA?6?$AA?$AA@ 100076d0     ftdi_utils.obj
 0001:000066f8       ??_C@_1CI@PHBFOJGD@?$AA?$DM?$AAI?$AAo?$AAE?$AAr?$AAr?$AAo?$AAr?$AAH?$AAa?$AAn?$AAd?$AAl?$AAe?$AAr?$AA?3?$AA?$CF?$AAd?$AA?6?$AA?$AA@ 100076f8     ftdi_utils.obj
 0001:00006720       ??_C@_1EC@HHKPAJMM@?$AAI?$AAs?$AAs?$AAu?$AAe?$AAV?$AAe?$AAn?$AAd?$AAo?$AAr?$AAT?$AAr?$AAa?$AAn?$AAs?$AAf?$AAe?$AAr?$AA?5?$AAd?$AAe?$AAv?$AAi?$AAc?$AAe?$AA?5?$AAg?$AAo?$AAn?$AAe?$AA?6@ 10007720     ftdi_utils.obj
 0001:00006764       ??_C@_1DG@DIFOFGHM@?$AAF?$AAT?$AA_?$AAG?$AAe?$AAt?$AAM?$AAo?$AAd?$AAe?$AAm?$AAS?$AAt?$AAa?$AAt?$AAu?$AAs?$AA?5?$AAb?$AAu?$AAf?$AA?5?$AA?$DN?$AA?$CF?$AAx?$AA?6?$AA?$AA@ 10007764     ftdi_utils.obj
 0001:000067a0       ??_C@_1EK@GNGBDENA@?$AAF?$AAT?$AA_?$AAG?$AAe?$AAt?$AAM?$AAo?$AAd?$AAe?$AAm?$AAS?$AAt?$AAa?$AAt?$AAu?$AAs?$AA?5?$AAE?$AAr?$AAr?$AAo?$AAr?$AA?5?$AAn?$AAt?$AAS?$AAt?$AAa?$AAt?$AAu?$AAs@ 100077a0     ftdi_utils.obj
 0001:000067ec       ??_C@_1CK@LFMBBJCH@?$AAF?$AAT?$AA_?$AAR?$AAe?$AAs?$AAe?$AAt?$AAH?$AAa?$AAr?$AAd?$AAw?$AAa?$AAr?$AAe?$AA?5?$AAO?$AAK?$AA?6?$AA?$AA@ 100077ec     ftdi_utils.obj
 0001:00006818       ??_C@_1DG@GGEBPPIN@?$AAF?$AAT?$AA_?$AAR?$AAe?$AAs?$AAe?$AAt?$AAH?$AAa?$AAr?$AAd?$AAw?$AAa?$AAr?$AAe?$AA?5?$AAe?$AAr?$AAr?$AAo?$AAr?$AA?3?$AA?$CF?$AAd?$AA?6?$AA?$AA@ 10007818     ftdi_utils.obj
 0001:00006850       ??_C@_1FE@KGBDAPG@?$AAU?$AAn?$AAh?$AAa?$AAn?$AAd?$AAl?$AAe?$AAd?$AA?5?$AAF?$AAT?$AA_?$AAR?$AAe?$AAs?$AAe?$AAt?$AAH?$AAa?$AAr?$AAd?$AAw?$AAa?$AAr?$AAe?$AA?5?$AAW?$AAa?$AAi?$AAt?$AAR@ 10007850     ftdi_utils.obj
 0001:000068a8       ??_C@_1EA@LJFPHIIA@?$AAF?$AAT?$AA_?$AAS?$AAe?$AAt?$AAD?$AAe?$AAv?$AAi?$AAc?$AAe?$AAE?$AAv?$AAe?$AAn?$AAt?$AA?3?$AA?$CF?$AAp?$AA?0?$AA?5?$AAe?$AAv?$AAe?$AAn?$AAt?$AA?5?$AA?$CF?$AAp?$AA?6?$AA?$AA@ 100078a8     ftdi_utils.obj
 0001:000068e8       _gszArrayIndex             100078e8     ftdi_usb.obj
 0001:0000690c       _gszVersion                1000790c     ftdi_usb.obj
 0001:0000691c       _gszVersionNumber          1000791c     ftdi_usb.obj
 0001:00006930       _gcszUnRegisterClientDriverId 10007930     ftdi_usb.obj
 0001:00006964       _gcszUnRegisterClientSettings 10007964     ftdi_usb.obj
 0001:00006998       _gcszFTDIUSBDriverId       10007998     ftdi_usb.obj
 0001:00006c60       ??_C@_1M@FGICDIHG@?$AAO?$AAS?$AA?5?$AA5?$AA?6?$AA?$AA@ 10007c60     ftdi_usb.obj
 0001:00006c6c       ??_C@_1O@IBJPINJN@?$AAO?$AAS?$AA?5?$AAl?$AA5?$AA?6?$AA?$AA@ 10007c6c     ftdi_usb.obj
 0001:00006c7c       ??_C@_17CHLIBJCN@?$AA?$CF?$AAd?$AA?3?$AA?$AA@ 10007c7c     ftdi_usb.obj
 0001:00006c84       ??_C@_1BE@OGCHJGKA@?$AAi?$AAN?$AAu?$AAm?$AA?3?$AA?5?$AA?$CF?$AAd?$AA?6?$AA?$AA@ 10007c84     ftdi_usb.obj
 0001:00006c98       ??_C@_1DE@MGIBGLKG@?$AA?$DO?$AAG?$AAe?$AAt?$AAR?$AAe?$AAg?$AAi?$AAs?$AAt?$AAr?$AAy?$AAI?$AAn?$AAi?$AAt?$AAi?$AAa?$AAl?$AAI?$AAn?$AAd?$AAe?$AAx?$AA?6?$AA?$AA@ 10007c98     ftdi_usb.obj
 0001:00006cd0       ??_C@_1FA@GJFEIMFN@?$AAA?$AAt?$AAt?$AAe?$AAm?$AAp?$AAt?$AAi?$AAn?$AAg?$AA?5?$AAt?$AAo?$AA?5?$AAg?$AAe?$AAt?$AA?5?$AAd?$AAe?$AAs?$AAc?$AAr?$AAi?$AAp?$AAt?$AAi?$AAo?$AAn?$AA?5?$AAi?$AAn@ 10007cd0     ftdi_usb.obj
 0001:00006d20       ??_C@_15GANGMFKL@?$AA?$CF?$AAs?$AA?$AA@ 10007d20     ftdi_usb.obj
 0001:00006d28       ??_C@_1FA@DPPGCDFE@?$AAO?$AAp?$AAe?$AAn?$AAe?$AAd?$AA?5?$AAr?$AAe?$AAg?$AAi?$AAs?$AAt?$AAr?$AAy?$AA?5?$AAk?$AAe?$AAy?$AA?5?$AAf?$AAo?$AAr?$AA?5?$AAd?$AAe?$AAs?$AAc?$AAr?$AAi?$AAp?$AAt@ 10007d28     ftdi_usb.obj
 0001:00006d78       ??_C@_1BK@BPGMFHJH@?$AAI?$AAn?$AAi?$AAt?$AAi?$AAa?$AAl?$AAI?$AAn?$AAd?$AAe?$AAx?$AA?$AA@ 10007d78     ftdi_usb.obj
 0001:00006d98       ??_C@_1EK@BONHHOJB@?$AAG?$AAo?$AAt?$AA?5?$AAd?$AAe?$AAs?$AAc?$AAr?$AAi?$AAp?$AAt?$AAi?$AAo?$AAn?$AA?5?$AAi?$AAn?$AAi?$AAt?$AAi?$AAa?$AAl?$AA?5?$AAi?$AAn?$AAd?$AAe?$AAx?$AA?5?$AAo?$AAf@ 10007d98     ftdi_usb.obj
 0001:00006de8       ??_C@_1GA@EKPIEEEP@?$AAF?$AAA?$AAI?$AAL?$AAE?$AAD?$AA?5?$AAt?$AAo?$AA?5?$AAo?$AAp?$AAe?$AAn?$AA?5?$AAr?$AAe?$AAg?$AAi?$AAs?$AAt?$AAr?$AAy?$AA?5?$AAk?$AAe?$AAy?$AA?5?$AAf?$AAo?$AAr?$AA?5@ 10007de8     ftdi_usb.obj
 0001:00006e48       ??_C@_1DC@JPKJGDH@?$AAE?$AAr?$AAr?$AAo?$AAr?$AA?5?$AAr?$AAe?$AAa?$AAd?$AAi?$AAn?$AAg?$AA?5?$AAv?$AAa?$AAl?$AAu?$AAe?$AA?3?$AA?5?$AA?$CF?$AAX?$AA?6?$AA?$AA@ 10007e48     ftdi_usb.obj
 0001:00006e7c       ??_C@_1DK@NPANAABN@?$AAI?$AAn?$AAi?$AAt?$AAi?$AAa?$AAl?$AA?5?$AAI?$AAn?$AAd?$AAe?$AAx?$AA?5?$AAR?$AAe?$AAg?$AA?5?$AAv?$AAa?$AAl?$AAu?$AAe?$AA?3?$AA?5?$AA?$CF?$AAd?$AA?6?$AA?$AA@ 10007e7c     ftdi_usb.obj
 0001:00006eb8       ??_C@_1DI@GGKIOBOP@?$AAS?$AAe?$AAt?$AAt?$AAi?$AAn?$AAg?$AA?5?$AAI?$AAn?$AAi?$AAt?$AAi?$AAa?$AAl?$AA?5?$AAi?$AAn?$AAd?$AAe?$AAx?$AA?5?$AAt?$AAo?$AA?5?$AA0?$AA?6?$AA?$AA@ 10007eb8     ftdi_usb.obj
 0001:00006ef0       ??_C@_1DE@BFBIJDLM@?$AA?$DM?$AAG?$AAe?$AAt?$AAR?$AAe?$AAg?$AAi?$AAs?$AAt?$AAr?$AAy?$AAI?$AAn?$AAi?$AAt?$AAi?$AAa?$AAl?$AAI?$AAn?$AAd?$AAe?$AAx?$AA?6?$AA?$AA@ 10007ef0     ftdi_usb.obj
 0001:00006f24       ??_C@_1CG@LEJBEHJC@?$AAI?$AAn?$AAi?$AAt?$AAi?$AAa?$AAl?$AAI?$AAn?$AAd?$AAe?$AAx?$AA?5?$AA?$DN?$AA?5?$AA?$CF?$AAd?$AA?6?$AA?$AA@ 10007f24     ftdi_usb.obj
 0001:00006f4c       ??_C@_1BO@LFKIOHPI@?$AAd?$AAr?$AAi?$AAv?$AAe?$AAr?$AAs?$AA?2?$AAa?$AAc?$AAt?$AAi?$AAv?$AAe?$AA?$AA@ 10007f4c     ftdi_usb.obj
 0001:00006f6c       ??_C@_1CE@EBNPANE@?$AAd?$AAr?$AAi?$AAv?$AAe?$AAr?$AAs?$AA?2?$AAa?$AAc?$AAt?$AAi?$AAv?$AAe?$AA?2?$AA?$CF?$AAs?$AA?$AA@ 10007f6c     ftdi_usb.obj
 0001:00006f90       ??_C@_19DINFBLAK@?$AAN?$AAa?$AAm?$AAe?$AA?$AA@ 10007f90     ftdi_usb.obj
 0001:00006f9c       ??_C@_1BC@HPDGIPOA@?$AAV?$AAe?$AAn?$AAd?$AAo?$AAr?$AAI?$AAd?$AA?$AA@ 10007f9c     ftdi_usb.obj
 0001:00006fb0       ??_C@_17OGBPPHLA@?$AAH?$AAn?$AAd?$AA?$AA@ 10007fb0     ftdi_usb.obj
 0001:00006fb8       ??_C@_1BC@CGPKCBFG@?$AAF?$AAu?$AAl?$AAl?$AAN?$AAa?$AAm?$AAe?$AA?$AA@ 10007fb8     ftdi_usb.obj
 0001:00006fcc       ??_C@_1CK@FDCMAFOF@?$AAC?$AAo?$AAm?$AAP?$AAo?$AAr?$AAt?$AA?5?$AAN?$AAu?$AAm?$AAb?$AAe?$AAr?$AA?5?$AA?$DN?$AA?5?$AA?$CF?$AAd?$AA?6?$AA?$AA@ 10007fcc     ftdi_usb.obj
 0001:00006ff8       ??_C@_1BC@OMMMELN@?$AAu?$AAs?$AAb?$AAd?$AA?4?$AAd?$AAl?$AAl?$AA?$AA@ 10007ff8     ftdi_usb.obj
 0001:0000700c       ??_C@_1CM@ECOBGAKP@?$AAC?$AAa?$AAn?$AA?8?$AAt?$AA?5?$AAl?$AAo?$AAa?$AAd?$AA?5?$AAU?$AAS?$AAB?$AAD?$AA?4?$AAD?$AAL?$AAL?$AA?$AN?$AA?6?$AA?$AA@ 1000800c     ftdi_usb.obj
 0001:00007038       ??_C@_1CO@EKLAAELD@?$AA?$DO?$AAU?$AAS?$AAB?$AAI?$AAn?$AAs?$AAt?$AAa?$AAl?$AAl?$AAD?$AAr?$AAi?$AAv?$AAe?$AAr?$AA?$CI?$AA?$CF?$AAs?$AA?$CJ?$AA?6?$AA?$AA@ 10008038     ftdi_usb.obj
 0001:00007068       ??_C@_0BG@LLEHHBLI@?2Release?2FTDIPORT?4INF?$AA@ 10008068     ftdi_usb.obj
 0001:00007080       ??_C@_1CO@OHLKFGFN@?$AAR?$AAe?$AAg?$AAi?$AAs?$AAt?$AAe?$AAr?$AAC?$AAl?$AAi?$AAe?$AAn?$AAt?$AAD?$AAr?$AAi?$AAv?$AAe?$AAr?$AAI?$AAD?$AA?$AA@ 10008080     ftdi_usb.obj
 0001:000070b0       ??_C@_1CO@GPOIHENG@?$AAR?$AAe?$AAg?$AAi?$AAs?$AAt?$AAe?$AAr?$AAC?$AAl?$AAi?$AAe?$AAn?$AAt?$AAS?$AAe?$AAt?$AAt?$AAi?$AAn?$AAg?$AAs?$AA?$AA@ 100080b0     ftdi_usb.obj
 0001:000070e0       ??_C@_1EA@HAKMBDLJ@?$AAR?$AAe?$AAg?$AAi?$AAs?$AAt?$AAe?$AAr?$AAC?$AAl?$AAi?$AAe?$AAn?$AAt?$AAD?$AAr?$AAi?$AAv?$AAe?$AAr?$AAI?$AAD?$AA?5?$AAF?$AAa?$AAi?$AAl?$AA?5?$AA?$CF?$AAd?$AA?6?$AA?$AA@ 100080e0     ftdi_usb.obj
 0001:00007120       ??_C@_1EC@ECHIDBII@?$AAR?$AAe?$AAg?$AAi?$AAs?$AAt?$AAe?$AAr?$AAC?$AAl?$AAi?$AAe?$AAn?$AAt?$AAS?$AAe?$AAt?$AAt?$AAi?$AAn?$AAg?$AAs?$AA1?$AA?5?$AAF?$AAa?$AAi?$AAl?$AA?5?$AA?$CF?$AAd?$AA?6@ 10008120     ftdi_usb.obj
 0001:00007164       ??_C@_1CK@MJMMODAK@?$AAS?$AAt?$AAr?$AAe?$AAa?$AAm?$AAD?$AAr?$AAi?$AAv?$AAe?$AAr?$AAK?$AAe?$AAy?$AA?3?$AA?5?$AA?$CF?$AAs?$AA?6?$AA?$AA@ 10008164     ftdi_usb.obj
 0001:00007190       ??_C@_17DJMMGLBL@?$AAD?$AAl?$AAl?$AA?$AA@ 10008190     ftdi_usb.obj
 0001:00007198       ??_C@_1O@GBAEOCCH@?$AAP?$AAr?$AAe?$AAf?$AAi?$AAx?$AA?$AA@ 10008198     ftdi_usb.obj
 0001:000071a8       ??_C@_1DK@KBKMPNEE@?$AA?$DM?$AAU?$AAS?$AAB?$AAI?$AAn?$AAs?$AAt?$AAa?$AAl?$AAl?$AAD?$AAr?$AAi?$AAv?$AAe?$AAr?$AA?5?$AAf?$AAR?$AAe?$AAt?$AA?5?$AA?$DN?$AA?5?$AA?$CF?$AAd?$AA?6?$AA?$AA@ 100081a8     ftdi_usb.obj
 0001:000071e4       ??_C@_1DA@INFPNDFP@?$AA?$DM?$AAU?$AAS?$AAB?$AAU?$AAn?$AAI?$AAn?$AAs?$AAt?$AAa?$AAl?$AAl?$AAD?$AAr?$AAi?$AAv?$AAe?$AAr?$AA?3?$AA?$CF?$AAd?$AA?6?$AA?$AA@ 100081e4     ftdi_usb.obj
 0001:00007214       ??_C@_1DI@JNKGABM@?$AA?$DO?$AAR?$AAe?$AAm?$AAo?$AAv?$AAe?$AAD?$AAe?$AAv?$AAi?$AAc?$AAe?$AAS?$AAt?$AAr?$AAu?$AAc?$AAt?$AAu?$AAr?$AAe?$AA?$CI?$AA?$CF?$AAp?$AA?$CJ?$AA?6?$AA?$AA@ 10008214     ftdi_usb.obj
 0001:00007250       ??_C@_1EO@HKIFFLKF@?$AAR?$AAe?$AAm?$AAo?$AAv?$AAe?$AAD?$AAe?$AAv?$AAi?$AAc?$AAe?$AAS?$AAt?$AAr?$AAu?$AAc?$AAt?$AAu?$AAr?$AAe?$AA?5?$AAo?$AAn?$AA?5?$AAo?$AAp?$AAe?$AAn?$AA?5?$AAd?$AAe@ 10008250     ftdi_usb.obj
 0001:000072a0       ??_C@_1HM@CMHCAGJO@?$AAc?$AA?3?$AA?2?$AAw?$AAi?$AAn?$AAc?$AAe?$AA8?$AA0?$AA0?$AA?2?$AAo?$AAs?$AAd?$AAe?$AAs?$AAi?$AAg?$AAn?$AAs?$AA?2?$AAv?$AAc?$AAp?$AAo?$AAs?$AAc?$AAe?$AAp?$AAc?$AA?2@ 100082a0     ftdi_usb.obj
 0001:0000731c       ??_C@_1BK@DIMGGMC@?$AAF?$AAT?$AAD?$AAI?$AA_?$AAS?$AAE?$AAR?$AA?4?$AAD?$AAL?$AAL?$AA?$AA@ 1000831c     ftdi_usb.obj
 0001:00007338       ??_C@_1FO@MLCJFIIN@?$AA?$CF?$AAs?$AA?3?$AA?5?$AAC?$AAo?$AAd?$AAe?$AA?5?$AAC?$AAo?$AAv?$AAe?$AAr?$AAa?$AAg?$AAe?$AA?5?$AAT?$AAr?$AAa?$AAp?$AA?5?$AAi?$AAn?$AA?3?$AA?5?$AAf?$AAt?$AAd?$AAi?$AA_@ 10008338     ftdi_usb.obj
 0001:00007398       ??_C@_1GI@DAGMLPDO@?$AAC?$AAl?$AAo?$AAs?$AAe?$AAH?$AAa?$AAn?$AAd?$AAl?$AAe?$AA?$CI?$AAp?$AAU?$AAs?$AAb?$AAF?$AAT?$AAD?$AAI?$AA?9?$AA?$DO?$AAB?$AAu?$AAl?$AAk?$AAI?$AAn?$AA?4?$AAh?$AAE?$AAv@ 10008398     ftdi_usb.obj
 0001:00007400       ??_C@_1GK@LAGEOCHF@?$AAC?$AAl?$AAo?$AAs?$AAe?$AAH?$AAa?$AAn?$AAd?$AAl?$AAe?$AA?$CI?$AAp?$AAU?$AAs?$AAb?$AAF?$AAT?$AAD?$AAI?$AA?9?$AA?$DO?$AAB?$AAu?$AAl?$AAk?$AAO?$AAu?$AAt?$AA?4?$AAh?$AAE@ 10008400     ftdi_usb.obj
 0001:00007470       ??_C@_1GA@DHFDNBJF@?$AAC?$AAl?$AAo?$AAs?$AAe?$AAH?$AAa?$AAn?$AAd?$AAl?$AAe?$AA?$CI?$AAp?$AAU?$AAs?$AAb?$AAF?$AAT?$AAD?$AAI?$AA?9?$AA?$DO?$AAh?$AAE?$AAP?$AA0?$AAE?$AAv?$AAe?$AAn?$AAt?$AA?$CJ@ 10008470     ftdi_usb.obj
 0001:000074d0       ??_C@_1GE@MKHEJJGO@?$AAC?$AAl?$AAo?$AAs?$AAe?$AAH?$AAa?$AAn?$AAd?$AAl?$AAe?$AA?$CI?$AAp?$AAU?$AAs?$AAb?$AAF?$AAT?$AAD?$AAI?$AA?9?$AA?$DO?$AAh?$AAC?$AAl?$AAo?$AAs?$AAe?$AAE?$AAv?$AAe?$AAn@ 100084d0     ftdi_usb.obj
 0001:00007538       ??_C@_1GM@IHDBLKDK@?$AAC?$AAl?$AAo?$AAs?$AAe?$AAH?$AAa?$AAn?$AAd?$AAl?$AAe?$AA?$CI?$AAp?$AAU?$AAs?$AAb?$AAF?$AAT?$AAD?$AAI?$AA?9?$AA?$DO?$AAh?$AAR?$AAe?$AAc?$AAo?$AAn?$AAn?$AAe?$AAc?$AAt@ 10008538     ftdi_usb.obj
 0001:000075a8       ??_C@_1GI@PAKLNBMO@?$AAC?$AAl?$AAo?$AAs?$AAe?$AAH?$AAa?$AAn?$AAd?$AAl?$AAe?$AA?$CI?$AAp?$AAU?$AAs?$AAb?$AAF?$AAT?$AAD?$AAI?$AA?9?$AA?$DO?$AAh?$AAR?$AAe?$AAs?$AAt?$AAa?$AAr?$AAt?$AAE?$AAv@ 100085a8     ftdi_usb.obj
 0001:00007610       ??_C@_1DA@JHKJENMD@?$AA?$DM?$AAR?$AAe?$AAm?$AAo?$AAv?$AAe?$AAD?$AAe?$AAv?$AAi?$AAc?$AAe?$AAS?$AAt?$AAr?$AAu?$AAc?$AAt?$AAu?$AAr?$AAe?$AA?6?$AA?$AA@ 10008610     ftdi_usb.obj
 0001:00007640       ??_C@_1CA@BKNFHCAM@?$AA?$DO?$AAD?$AAe?$AAv?$AAi?$AAc?$AAe?$AAN?$AAo?$AAt?$AAi?$AAf?$AAy?$AA?$AN?$AA?6?$AA?$AA@ 10008640     ftdi_usb.obj
 0001:00007660       ??_C@_1CE@ELNBPOOA@?$AAI?$AAn?$AAv?$AAa?$AAl?$AAi?$AAd?$AA?5?$AAC?$AAo?$AAn?$AAt?$AAe?$AAx?$AAt?$AA?$CB?$AA?6?$AA?$AA@ 10008660     ftdi_usb.obj
 0001:00007688       ??_C@_1HC@GGDPKEBL@?$AAD?$AAe?$AAv?$AAi?$AAc?$AAe?$AAN?$AAo?$AAt?$AAi?$AAf?$AAy?$AA?5?$AAn?$AAo?$AAt?$AA?5?$AAu?$AAs?$AAi?$AAn?$AAg?$AA?5?$AAO?$AAp?$AAe?$AAn?$AAC?$AAS?$AA?5?$AAb?$AAe@ 10008688     ftdi_usb.obj
 0001:000076fc       ??_C@_1CE@LCJFHOGH@?$AAU?$AAS?$AAB?$AA_?$AAC?$AAL?$AAO?$AAS?$AAE?$AA_?$AAD?$AAE?$AAV?$AAI?$AAC?$AAE?$AA?6?$AA?$AA@ 100086fc     ftdi_usb.obj
 0001:00007720       ??_C@_1EM@GMIFBBAN@?$AAD?$AAe?$AAv?$AAi?$AAc?$AAe?$AAN?$AAo?$AAt?$AAi?$AAf?$AAy?$AA?3?$AA?5?$AAd?$AAe?$AAv?$AAi?$AAc?$AAe?$AA?5?$AAi?$AAs?$AA?5?$AAP?$AAE?$AAR?$AAS?$AAI?$AAS?$AAT?$AAE@ 10008720     ftdi_usb.obj
 0001:0000776c       ??_C@_1DO@FFHELMPG@?$AAD?$AAe?$AAv?$AAi?$AAc?$AAe?$AAN?$AAo?$AAt?$AAi?$AAf?$AAy?$AA?3?$AA?5?$AAd?$AAe?$AAv?$AAi?$AAc?$AAe?$AA?5?$AAi?$AAs?$AA?5?$AAo?$AAp?$AAe?$AAn?$AA?$AN?$AA?6?$AA?$AA@ 1000876c     ftdi_usb.obj
 0001:000077b0       ??_C@_1EC@PGBFPAOE@?$AAD?$AAe?$AAv?$AAi?$AAc?$AAe?$AAN?$AAo?$AAt?$AAi?$AAf?$AAy?$AA?3?$AA?5?$AAd?$AAe?$AAv?$AAi?$AAc?$AAe?$AA?5?$AAi?$AAs?$AA?5?$AAc?$AAl?$AAo?$AAs?$AAe?$AAd?$AA?$AN?$AA?6@ 100087b0     ftdi_usb.obj
 0001:000077f4       ??_C@_1DE@MNPLHKGP@?$AAU?$AAn?$AAh?$AAa?$AAn?$AAd?$AAl?$AAe?$AAd?$AA?5?$AAn?$AAo?$AAt?$AAi?$AAf?$AAy?$AA?5?$AAc?$AAo?$AAd?$AAe?$AA?3?$AA?$CF?$AAd?$AA?6?$AA?$AA@ 100087f4     ftdi_usb.obj
 0001:00007828       ??_C@_1FK@FDMLMPJG@?$AAW?$AAa?$AAi?$AAt?$AAi?$AAn?$AAg?$AA?5?$AAf?$AAo?$AAr?$AA?5?$AAC?$AAl?$AAo?$AAs?$AAe?$AAE?$AAv?$AAe?$AAn?$AAt?$AA?5?$AAo?$AAr?$AA?5?$AAR?$AAe?$AAc?$AAo?$AAn?$AAn@ 10008828     ftdi_usb.obj
 0001:00007888       ??_C@_1EE@NMINGIAI@?$AAD?$AAe?$AAv?$AAi?$AAc?$AAe?$AAN?$AAo?$AAt?$AAi?$AAf?$AAy?$AA?5?$AAc?$AAl?$AAo?$AAs?$AAe?$AA?5?$AAf?$AAo?$AAr?$AA?5?$AAd?$AAe?$AAv?$AAi?$AAc?$AAe?$AA?5?$AA?$CF?$AAp@ 10008888     ftdi_usb.obj
 0001:000078d0       ??_C@_1EO@JPMDAFJ@?$AAS?$AAu?$AAr?$AAp?$AAr?$AAi?$AAs?$AAe?$AA?5?$AAr?$AAe?$AAm?$AAo?$AAv?$AAe?$AAd?$AA?5?$AA?9?$AA?$DO?$AA?5?$AAd?$AAe?$AAa?$AAc?$AAt?$AAi?$AAv?$AAa?$AAt?$AAe?$AA?5?$AAd@ 100088d0     ftdi_usb.obj
 0001:00007920       ??_C@_1CE@PEOIOJON@?$AAD?$AAe?$AAa?$AAc?$AAt?$AAi?$AAv?$AAa?$AAt?$AAe?$AAD?$AAe?$AAv?$AAi?$AAc?$AAe?$AA?6?$AA?$AA@ 10008920     ftdi_usb.obj
 0001:00007944       ??_C@_1DI@FLBENACO@?$AAD?$AAe?$AAa?$AAc?$AAt?$AAi?$AAv?$AAa?$AAt?$AAe?$AAD?$AAe?$AAv?$AAi?$AAc?$AAe?$AA?5?$AAe?$AAr?$AAr?$AAo?$AAr?$AA?3?$AA?5?$AA?$CF?$AAd?$AA?6?$AA?$AA@ 10008944     ftdi_usb.obj
 0001:0000797c       ??_C@_1DO@BFNJPPJF@?$AAD?$AAe?$AAa?$AAc?$AAt?$AAi?$AAv?$AAa?$AAt?$AAe?$AAD?$AAe?$AAv?$AAi?$AAc?$AAe?$AA?5?$AAS?$AAU?$AAC?$AAC?$AAE?$AAE?$AAD?$AAE?$AAD?$AA?$CB?$AA?$CB?$AA?$AN?$AA?6?$AA?$AA@ 1000897c     ftdi_usb.obj
 0001:000079bc       ??_C@_1BO@LJHBDGGK@?$AA?$DM?$AAD?$AAe?$AAv?$AAi?$AAc?$AAe?$AAN?$AAo?$AAt?$AAi?$AAf?$AAy?$AA?6?$AA?$AA@ 100089bc     ftdi_usb.obj
 0001:000079dc       ??_C@_1DE@MJFIOPLO@?$AA?$DO?$AAD?$AAe?$AAl?$AAa?$AAy?$AAe?$AAd?$AAD?$AAe?$AAv?$AAi?$AAc?$AAe?$AAD?$AAe?$AAa?$AAc?$AAt?$AAi?$AAv?$AAa?$AAt?$AAe?$AA?6?$AA?$AA@ 100089dc     ftdi_usb.obj
 0001:00007a10       ??_C@_1DM@DAGIBLB@?$AAD?$AAe?$AAa?$AAc?$AAt?$AAi?$AAv?$AAa?$AAt?$AAe?$AAD?$AAe?$AAv?$AAi?$AAc?$AAe?$AA?5?$AAS?$AAU?$AAC?$AAC?$AAE?$AAE?$AAD?$AAE?$AAD?$AA?$CB?$AA?$CB?$AA?6?$AA?$AA@ 10008a10     ftdi_usb.obj
 0001:00007a4c       ??_C@_1DE@BKMBBHKE@?$AA?$DM?$AAD?$AAe?$AAl?$AAa?$AAy?$AAe?$AAd?$AAD?$AAe?$AAv?$AAi?$AAc?$AAe?$AAD?$AAe?$AAa?$AAc?$AAt?$AAi?$AAv?$AAa?$AAt?$AAe?$AA?6?$AA?$AA@ 10008a4c     ftdi_usb.obj
 0001:00007a80       ??_C@_1FE@DAKKNNLP@?$AAC?$AAr?$AAe?$AAa?$AAt?$AAe?$AAB?$AAu?$AAl?$AAk?$AAP?$AAi?$AAp?$AAe?$AAE?$AAv?$AAe?$AAn?$AAt?$AAs?$AA?5?$AAB?$AAu?$AAl?$AAk?$AAI?$AAn?$AA?4?$AAh?$AAE?$AAv?$AAe@ 10008a80     ftdi_usb.obj
 0001:00007ad8       ??_C@_1FI@CIPNPBJK@?$AAC?$AAr?$AAe?$AAa?$AAt?$AAe?$AAB?$AAu?$AAl?$AAk?$AAP?$AAi?$AAp?$AAe?$AAE?$AAv?$AAe?$AAn?$AAt?$AAs?$AA?5?$AAC?$AAr?$AAe?$AAa?$AAt?$AAe?$AAE?$AAv?$AAe?$AAn?$AAt@ 10008ad8     ftdi_usb.obj
 0001:00007b30       ??_C@_1FI@HAODFILC@?$AAC?$AAr?$AAe?$AAa?$AAt?$AAe?$AAB?$AAu?$AAl?$AAk?$AAP?$AAi?$AAp?$AAe?$AAE?$AAv?$AAe?$AAn?$AAt?$AAs?$AA?5?$AAC?$AAr?$AAe?$AAa?$AAt?$AAe?$AAE?$AAv?$AAe?$AAn?$AAt@ 10008b30     ftdi_usb.obj
 0001:00007b88       ??_C@_1BI@DFKEDNPO@?$AAB?$AAu?$AAl?$AAk?$AAI?$AAn?$AAF?$AAl?$AAa?$AAg?$AAs?$AA?$AA@ 10008b88     ftdi_usb.obj
 0001:00007ba0       ??_C@_1BK@KDFGCGI@?$AAB?$AAu?$AAl?$AAk?$AAO?$AAu?$AAt?$AAF?$AAl?$AAa?$AAg?$AAs?$AA?$AA@ 10008ba0     ftdi_usb.obj
 0001:00007bbc       ??_C@_1CA@CFOPMDEA@?$AAS?$AAy?$AAn?$AAc?$AAh?$AAr?$AAo?$AAn?$AAo?$AAu?$AAs?$AAB?$AAu?$AAl?$AAk?$AA?$AA@ 10008bbc     ftdi_usb.obj
 0001:00007be0       ??_C@_1IG@LBKLLBIB@?$AAG?$AAe?$AAt?$AAB?$AAu?$AAl?$AAk?$AAT?$AAr?$AAa?$AAn?$AAs?$AAf?$AAe?$AAr?$AAF?$AAl?$AAa?$AAg?$AAs?$AA?3?$AA?5?$AAF?$AAa?$AAi?$AAl?$AAe?$AAd?$AA?5?$AAt?$AAo?$AA?5@ 10008be0     ftdi_usb.obj
 0001:00007c68       ??_C@_1CA@PBBEBOEE@?$AAM?$AAi?$AAn?$AAW?$AAr?$AAi?$AAt?$AAe?$AAT?$AAi?$AAm?$AAe?$AAo?$AAu?$AAt?$AA?$AA@ 10008c68     ftdi_usb.obj
 0001:00007c88       ??_C@_1BO@ECPAAEBI@?$AAM?$AAi?$AAn?$AAR?$AAe?$AAa?$AAd?$AAT?$AAi?$AAm?$AAe?$AAo?$AAu?$AAt?$AA?$AA@ 10008c88     ftdi_usb.obj
 0001:00007ca8       ??_C@_1M@EENNDIOJ@?$AAI?$AAn?$AAd?$AAe?$AAx?$AA?$AA@ 10008ca8     ftdi_usb.obj
 0001:00007cb4       ??_C@_1CM@NEKFHIBD@?$AAS?$AAe?$AAt?$AAI?$AAn?$AAd?$AAe?$AAx?$AAK?$AAe?$AAy?$AAV?$AAa?$AAl?$AAu?$AAe?$AA?3?$AA?5?$AA?$CF?$AAd?$AA?6?$AA?$AA@ 10008cb4     ftdi_usb.obj
 0001:00007ce0       ??_C@_1CE@JGFBJHKD@?$AA?$DO?$AAS?$AAe?$AAt?$AAU?$AAs?$AAb?$AAI?$AAn?$AAt?$AAe?$AAr?$AAf?$AAa?$AAc?$AAe?$AA?6?$AA?$AA@ 10008ce0     ftdi_usb.obj
 0001:00007d04       ??_C@_1DE@ODBLKBBI@?$AAU?$AAS?$AAB?$AA_?$AAE?$AAN?$AAD?$AAP?$AAO?$AAI?$AAN?$AAT?$AA_?$AAD?$AAE?$AAS?$AAC?$AAR?$AAI?$AAP?$AAT?$AAO?$AAR?$AA?3?$AA?6?$AA?$AA@ 10008d04     ftdi_usb.obj
 0001:00007d38       ??_C@_1DO@LJAHMEFB@?$AA?9?$AA?9?$AA?9?$AA?9?$AA?9?$AA?9?$AA?9?$AA?9?$AA?9?$AA?9?$AA?9?$AA?9?$AA?9?$AA?9?$AA?9?$AA?9?$AA?9?$AA?9?$AA?9?$AA?9?$AA?9?$AA?9?$AA?9?$AA?9?$AA?9?$AA?9?$AA?9?$AA?9?$AA?9?$AA?6?$AA?$AA@ 10008d38     ftdi_usb.obj
 0001:00007d78       ??_C@_1BO@HCAHHBMN@?$AAb?$AAL?$AAe?$AAn?$AAg?$AAt?$AAh?$AA?3?$AA?5?$AA0?$AAx?$AA?$CF?$AAx?$AA?6?$AA?$AA@ 10008d78     ftdi_usb.obj
 0001:00007d98       ??_C@_1CO@BEMPIGAC@?$AAb?$AAD?$AAe?$AAs?$AAc?$AAr?$AAi?$AAp?$AAt?$AAo?$AAr?$AAT?$AAy?$AAp?$AAe?$AA?3?$AA?5?$AA0?$AAx?$AA?$CF?$AAx?$AA?6?$AA?$AA@ 10008d98     ftdi_usb.obj
 0001:00007dc8       ??_C@_1DA@LICFMHAB@?$AAb?$AAE?$AAn?$AAd?$AAp?$AAo?$AAi?$AAn?$AAt?$AAA?$AAd?$AAd?$AAr?$AAe?$AAs?$AAs?$AA?3?$AA?5?$AA0?$AAx?$AA?$CF?$AAx?$AA?6?$AA?$AA@ 10008dc8     ftdi_usb.obj
 0001:00007df8       ??_C@_1CI@GGILJLCD@?$AAb?$AAm?$AAA?$AAt?$AAt?$AAr?$AAi?$AAb?$AAu?$AAt?$AAe?$AAs?$AA?3?$AA?5?$AA0?$AAx?$AA?$CF?$AAx?$AA?6?$AA?$AA@ 10008df8     ftdi_usb.obj
 0001:00007e20       ??_C@_1CM@JPNNBLII@?$AAw?$AAM?$AAa?$AAx?$AAP?$AAa?$AAc?$AAk?$AAe?$AAt?$AAS?$AAi?$AAz?$AAe?$AA?3?$AA?5?$AA0?$AAx?$AA?$CF?$AAx?$AA?6?$AA?$AA@ 10008e20     ftdi_usb.obj
 0001:00007e4c       ??_C@_1CC@JDIIAJHG@?$AAb?$AAI?$AAn?$AAt?$AAe?$AAr?$AAv?$AAa?$AAl?$AA?3?$AA?5?$AA0?$AAx?$AA?$CF?$AAx?$AA?6?$AA?$AA@ 10008e4c     ftdi_usb.obj
 0001:00007e70       ??_C@_13LBAGMAIH@?$AA?6?$AA?$AA@ 10008e70     ftdi_usb.obj
 0001:00007e74       ??_C@_1CO@PNHOBMFN@?$AAO?$AAp?$AAe?$AAn?$AAP?$AAi?$AAp?$AAe?$AA?5?$AAo?$AAu?$AAt?$AA?5?$AAe?$AAr?$AAr?$AAo?$AAr?$AA?3?$AA?$CF?$AAd?$AA?6?$AA?$AA@ 10008e74     ftdi_usb.obj
 0001:00007ea4       ??_C@_1CA@JNOKEDJE@?$AAh?$AAU?$AAs?$AAb?$AAD?$AAe?$AAv?$AAi?$AAc?$AAe?$AA?3?$AA?5?$AA?$CF?$AAp?$AA?6?$AA?$AA@ 10008ea4     ftdi_usb.obj
 0001:00007ec4       ??_C@_1CA@GKPLHPPM@?$AAD?$AAe?$AAs?$AAc?$AAr?$AAi?$AAp?$AAt?$AAo?$AAr?$AA?3?$AA?5?$AA?$CF?$AAp?$AA?6?$AA?$AA@ 10008ec4     ftdi_usb.obj
 0001:00007ee4       ??_C@_1BM@DKOFLPMF@?$AAO?$AAp?$AAe?$AAn?$AAP?$AAi?$AAp?$AAe?$AA?3?$AA?5?$AA?$CF?$AAp?$AA?6?$AA?$AA@ 10008ee4     ftdi_usb.obj
 0001:00007f00       ??_C@_1BG@NFOAAMOK@?$AAh?$AAP?$AAi?$AAp?$AAe?$AA?3?$AA?5?$AA?$CF?$AAp?$AA?6?$AA?$AA@ 10008f00     ftdi_usb.obj
 0001:00007f18       ??_C@_1BK@GEFCAGJG@?$AAO?$AAu?$AAt?$AA?5?$AAP?$AAi?$AAp?$AAe?$AA?5?$AAO?$AAK?$AA?6?$AA?$AA@ 10008f18     ftdi_usb.obj
 0001:00007f34       ??_C@_1CO@HNNMKLJG@?$AAO?$AAp?$AAe?$AAn?$AAP?$AAi?$AAp?$AAe?$AA?5?$AAi?$AAn?$AA?5?$AAe?$AAr?$AAr?$AAo?$AAr?$AA?3?$AA?5?$AA?$CF?$AAd?$AA?6?$AA?$AA@ 10008f34     ftdi_usb.obj
 0001:00007f64       ??_C@_1BI@CFBNMFFK@?$AAI?$AAn?$AA?5?$AAP?$AAi?$AAp?$AAe?$AA?5?$AAO?$AAK?$AA?6?$AA?$AA@ 10008f64     ftdi_usb.obj
 0001:00007f7c       ??_C@_1CK@MKDOHIHK@?$AA?$DM?$AAS?$AAe?$AAt?$AAU?$AAs?$AAb?$AAI?$AAn?$AAt?$AAe?$AAr?$AAf?$AAa?$AAc?$AAe?$AA?3?$AA?$CF?$AAd?$AA?6?$AA?$AA@ 10008f7c     ftdi_usb.obj
 0001:00007fa8       ??_C@_1CK@LDOAFPDH@?$AAL?$AAo?$AAc?$AAa?$AAl?$AAA?$AAl?$AAl?$AAo?$AAc?$AA?5?$AAe?$AAr?$AAr?$AAo?$AAr?$AA?3?$AA?$CF?$AAd?$AA?6?$AA?$AA@ 10008fa8     ftdi_usb.obj
 0001:00007fd8       ??_C@_1EM@OKCFEHJK@?$AAC?$AAr?$AAe?$AAa?$AAt?$AAe?$AAE?$AAv?$AAe?$AAn?$AAt?$AA?5?$AAh?$AAR?$AAe?$AAc?$AAo?$AAn?$AAn?$AAe?$AAc?$AAt?$AAE?$AAv?$AAe?$AAn?$AAt?$AA?5?$AAe?$AAr?$AAr?$AAo@ 10008fd8     ftdi_usb.obj
 0001:00008024       ??_C@_1DC@PLJJFLGO@?$AAS?$AAe?$AAt?$AAU?$AAs?$AAb?$AAI?$AAn?$AAt?$AAe?$AAr?$AAf?$AAa?$AAc?$AAe?$AA?5?$AAf?$AAa?$AAi?$AAl?$AAe?$AAd?$AA?$CB?$AA?6?$AA?$AA@ 10009024     ftdi_usb.obj
 0001:00008058       ??_C@_1DI@DPLCCEFO@?$AA?$DO?$AAU?$AAS?$AAB?$AAD?$AAe?$AAv?$AAi?$AAc?$AAe?$AAA?$AAt?$AAt?$AAa?$AAc?$AAh?$AA?$CI?$AA0?$AAx?$AA?$CF?$AAx?$AA?0?$AA?5?$AA?$CF?$AAs?$AA?$CJ?$AA?6?$AA?$AA@ 10009058     ftdi_usb.obj
 0001:00008090       ??_C@_1FA@HDEAIDHH@?$AAU?$AAS?$AAB?$AAD?$AAe?$AAv?$AAi?$AAc?$AAe?$AAA?$AAt?$AAt?$AAa?$AAc?$AAh?$AA?5?$AA?9?$AA?5?$AA?$CF?$AAd?$AA?5?$AAi?$AAn?$AAt?$AAe?$AAr?$AAf?$AAa?$AAc?$AAe?$AAs?$AA?5@ 10009090     ftdi_usb.obj
 0001:000080e0       ??_C@_1GC@EBILPLOD@?$AAU?$AAS?$AAB?$AAD?$AAe?$AAv?$AAi?$AAc?$AAe?$AAA?$AAt?$AAt?$AAa?$AAc?$AAh?$AA?5?$AA?9?$AA?5?$AAi?$AAn?$AAf?$AAo?$AAr?$AAm?$AAa?$AAt?$AAi?$AAo?$AAn?$AA?5?$AAf?$AAo@ 100090e0     ftdi_usb.obj
 0001:00008148       ??_C@_1FK@BJBEIKNL@?$AAU?$AAS?$AAB?$AAD?$AAe?$AAv?$AAi?$AAc?$AAe?$AAA?$AAt?$AAt?$AAa?$AAc?$AAh?$AA?5?$AA?9?$AA?5?$AAn?$AAo?$AA?5?$AAi?$AAn?$AAt?$AAe?$AAr?$AAf?$AAa?$AAc?$AAe?$AA?5?$AAi@ 10009148     ftdi_usb.obj
 0001:000081a8       ??_C@_1EC@GNDHBFLE@?$AAU?$AAS?$AAB?$AAD?$AAe?$AAv?$AAi?$AAc?$AAe?$AAA?$AAt?$AAt?$AAa?$AAc?$AAh?$AA?5?$AA?9?$AA?5?$AAi?$AAn?$AAt?$AAe?$AAr?$AAf?$AAa?$AAc?$AAe?$AA?5?$AA?$CF?$AAd?$AA?$AN?$AA?6@ 100091a8     ftdi_usb.obj
 0001:000081f0       ??_C@_1EM@KOBKGIFP@?$AAP?$AAe?$AAr?$AAs?$AAi?$AAs?$AAt?$AAe?$AAn?$AAt?$AA?5?$AAd?$AAe?$AAv?$AAi?$AAc?$AAe?$AA?5?$AA?9?$AA?5?$AAr?$AAe?$AAs?$AAu?$AAm?$AAi?$AAn?$AAg?$AA?5?$AAc?$AAo?$AAn@ 100091f0     ftdi_usb.obj
 0001:00008240       ??_C@_1EG@POEMPLJG@?$AAU?$AAS?$AAB?$AAD?$AAe?$AAv?$AAi?$AAc?$AAe?$AAA?$AAt?$AAt?$AAa?$AAc?$AAh?$AA?5?$AA?9?$AA?5?$AAn?$AAo?$AAt?$AA?5?$AAp?$AAe?$AAr?$AAs?$AAi?$AAs?$AAt?$AAe?$AAn?$AAt@ 10009240     ftdi_usb.obj
 0001:00008288       ??_C@_1DC@OKAJBNEJ@?$AAg?$AAs?$AAz?$AAS?$AAt?$AAr?$AAe?$AAa?$AAm?$AAD?$AAr?$AAi?$AAv?$AAe?$AAr?$AAK?$AAe?$AAy?$AA?5?$AA?$DN?$AA?5?$AA?$CF?$AAs?$AA?6?$AA?$AA@ 10009288     ftdi_usb.obj
 0001:000082c0       ??_C@_1FI@DGBDABNL@?$AAD?$AAe?$AAv?$AAi?$AAc?$AAe?$AA?5?$AAn?$AAo?$AAt?$AA?5?$AAi?$AAn?$AAs?$AAt?$AAa?$AAl?$AAl?$AAe?$AAd?$AA?5?$AA?9?$AA?5?$AAf?$AAr?$AAe?$AAe?$AA?5?$AAi?$AAn?$AAd?$AAe@ 100092c0     ftdi_usb.obj
 0001:00008318       ??_C@_1DC@EPJEPNCJ@?$AAF?$AAr?$AAe?$AAe?$AA?5?$AAi?$AAn?$AAd?$AAe?$AAx?$AA?5?$AAn?$AAo?$AAt?$AA?5?$AAf?$AAo?$AAu?$AAn?$AAd?$AA?5?$AA1?$AA?$AN?$AA?6?$AA?$AA@ 10009318     ftdi_usb.obj
 0001:00008350       ??_C@_1EE@JDDJBBPO@?$AAC?$AAr?$AAe?$AAa?$AAt?$AAe?$AAU?$AAn?$AAi?$AAq?$AAu?$AAe?$AAD?$AAr?$AAi?$AAv?$AAe?$AAr?$AAS?$AAe?$AAt?$AAt?$AAi?$AAn?$AAg?$AAs?$AA?5?$AAt?$AAr?$AAu?$AAe?$AA?$AN@ 10009350     ftdi_usb.obj
 0001:00008394       ??_C@_1DC@MBBLPKMK@?$AAF?$AAr?$AAe?$AAe?$AA?5?$AAi?$AAn?$AAd?$AAe?$AAx?$AA?5?$AAn?$AAo?$AAt?$AA?5?$AAf?$AAo?$AAu?$AAn?$AAd?$AA?5?$AA2?$AA?$AN?$AA?6?$AA?$AA@ 10009394     ftdi_usb.obj
 0001:000083c8       ??_C@_19HEPLDNLP@?$AA?$CF?$AAs?$AA?$CF?$AAd?$AA?$AA@ 100093c8     ftdi_usb.obj
 0001:000083d4       ??_C@_1M@KEKDJCFI@?$AA?$CF?$AAs?$AA?$CF?$AAd?$AA?3?$AA?$AA@ 100093d4     ftdi_usb.obj
 0001:000083e0       ??_C@_1BK@GBMCOKGG@?$AAS?$AAe?$AAr?$AAi?$AAa?$AAl?$AAN?$AAu?$AAm?$AAb?$AAe?$AAr?$AA?$AA@ 100093e0     ftdi_usb.obj
 0001:000083fc       ??_C@_1BI@DLMANABL@?$AAD?$AAe?$AAs?$AAc?$AAr?$AAi?$AAp?$AAt?$AAi?$AAo?$AAn?$AA?$AA@ 100093fc     ftdi_usb.obj
 0001:00008414       ??_C@_1BC@IAEGNIJM@?$AAC?$AAh?$AAi?$AAp?$AAT?$AAy?$AAp?$AAe?$AA?$AA@ 10009414     ftdi_usb.obj
 0001:00008428       ??_C@_1BI@IMELEEEO@?$AAF?$AAT?$AA?5?$AAX?$AA?5?$AAS?$AAe?$AAr?$AAi?$AAe?$AAs?$AA?$AA@ 10009428     ftdi_usb.obj
 0001:00008440       ??_C@_1O@NIBEILOD@?$AAF?$AAT?$AA2?$AA3?$AA2?$AAH?$AA?$AA@ 10009440     ftdi_usb.obj
 0001:00008450       ??_C@_1BA@DHHFLCKG@?$AAF?$AAT?$AA4?$AA2?$AA3?$AA2?$AAH?$AA?$AA@ 10009450     ftdi_usb.obj
 0001:00008460       ??_C@_1BA@NIEIBHEG@?$AAF?$AAT?$AA2?$AA2?$AA3?$AA2?$AAH?$AA?$AA@ 10009460     ftdi_usb.obj
 0001:00008470       ??_C@_1O@OHLADMBI@?$AAF?$AAT?$AA2?$AA3?$AA2?$AAR?$AA?$AA@ 10009470     ftdi_usb.obj
 0001:00008480       ??_C@_1O@NLGABICA@?$AAF?$AAT?$AA2?$AA2?$AA3?$AA2?$AA?$AA@ 10009480     ftdi_usb.obj
 0001:00008490       ??_C@_1O@LHKJGLIH@?$AAF?$AAT?$AA2?$AA3?$AA2?$AAB?$AA?$AA@ 10009490     ftdi_usb.obj
 0001:000084a0       ??_C@_1BE@OOJAEBBK@?$AAF?$AAT?$AA8?$AAU?$AA2?$AA3?$AA2?$AAA?$AAM?$AA?$AA@ 100094a0     ftdi_usb.obj
 0001:000084b4       ??_C@_1BC@LKPHGMEE@?$AAU?$AAs?$AAb?$AAS?$AAp?$AAe?$AAe?$AAd?$AA?$AA@ 100094b4     ftdi_usb.obj
 0001:000084c8       ??_C@_1BC@GCEGDIAC@?$AAH?$AAi?$AA?9?$AAS?$AAp?$AAe?$AAe?$AAd?$AA?$AA@ 100094c8     ftdi_usb.obj
 0001:000084dc       ??_C@_1BG@NNDEAGOP@?$AAF?$AAu?$AAl?$AAl?$AA?9?$AAS?$AAp?$AAe?$AAe?$AAd?$AA?$AA@ 100094dc     ftdi_usb.obj
 0001:000084f4       ??_C@_1BE@PJECJHAI@?$AAP?$AAr?$AAo?$AAd?$AAu?$AAc?$AAt?$AAI?$AAd?$AA?$AA@ 100094f4     ftdi_usb.obj
 0001:00008508       ??_C@_1CI@FLHKDGFA@?$AAC?$AAo?$AAm?$AAP?$AAo?$AAr?$AAt?$AA?5?$AAN?$AAa?$AAm?$AAe?$AA?5?$AA?$DN?$AA?5?$AA?$CF?$AAs?$AA?$AN?$AA?6?$AA?$AA@ 10009508     ftdi_usb.obj
 0001:00008530       ??_C@_1EA@JGDBEMKC@?$AAA?$AAc?$AAt?$AAi?$AAv?$AAa?$AAt?$AAe?$AAD?$AAe?$AAv?$AAi?$AAc?$AAe?$AA?5?$AAS?$AAU?$AAC?$AAC?$AAE?$AAE?$AAD?$AAE?$AAD?$AA?5?$AA?9?$AA?5?$AA?$CF?$AAs?$AA?$AN?$AA?6?$AA?$AA@ 10009530     ftdi_usb.obj
 0001:00008570       ??_C@_1DC@JIBCPPOB@?$AAA?$AAc?$AAt?$AAi?$AAv?$AAa?$AAt?$AAe?$AAD?$AAe?$AAv?$AAi?$AAc?$AAe?$AA?5?$AAe?$AAr?$AAr?$AAo?$AAr?$AA?3?$AA?$CF?$AAd?$AA?6?$AA?$AA@ 10009570     ftdi_usb.obj
 0001:000085a4       ??_C@_1DO@JEHCEJLJ@?$AAF?$AAa?$AAi?$AAl?$AAe?$AAd?$AA?5?$AAt?$AAo?$AA?5?$AAi?$AAn?$AAi?$AAt?$AAi?$AAa?$AAl?$AAi?$AAs?$AAe?$AA?5?$AAe?$AAr?$AAr?$AAo?$AAr?$AA?3?$AA?$CF?$AAd?$AA?6?$AA?$AA@ 100095a4     ftdi_usb.obj
 0001:000085e8       ??_C@_1GA@HNIBAAHE@?$AAU?$AAS?$AAB?$AAD?$AAe?$AAv?$AAi?$AAc?$AAe?$AAA?$AAt?$AAt?$AAa?$AAc?$AAh?$AA?5?$AAS?$AAU?$AAC?$AAC?$AAE?$AAE?$AAD?$AAE?$AAD?$AA?5?$AA?9?$AA?5?$AAa?$AAc?$AAc?$AAe@ 100095e8     ftdi_usb.obj
 0001:00008648       ??_C@_1DA@HHOJEAEO@?$AAU?$AAS?$AAB?$AAD?$AAe?$AAv?$AAi?$AAc?$AAe?$AAA?$AAt?$AAt?$AAa?$AAc?$AAh?$AA?5?$AA?9?$AA?5?$AAe?$AAn?$AAd?$AA?$AN?$AA?6?$AA?$AA@ 10009648     ftdi_usb.obj
 0001:00008928       ??_C@_1FG@IMOLFHFP@?$AAF?$AAT?$AA_?$AAL?$AAo?$AAc?$AAa?$AAl?$AAA?$AAl?$AAl?$AAo?$AAc?$AA?$CI?$AA?$CJ?$AA?5?$AAg?$AAL?$AAo?$AAc?$AAa?$AAl?$AAA?$AAl?$AAl?$AAo?$AAc?$AAC?$AAo?$AAu?$AAn?$AAt@ 10009928     BUSBDBG.obj
 0001:00008980       ??_C@_1FE@MABKOFFD@?$AAF?$AAT?$AA_?$AAL?$AAo?$AAc?$AAa?$AAl?$AAF?$AAr?$AAe?$AAe?$AA?$CI?$AA?$CJ?$AA?5?$AAg?$AAL?$AAo?$AAc?$AAa?$AAl?$AAA?$AAl?$AAl?$AAo?$AAc?$AAC?$AAo?$AAu?$AAn?$AAt?$AA?5@ 10009980     BUSBDBG.obj
 0001:00008c88       ??_C@_1DE@PKBMGLPJ@?$AAF?$AAT?$AAD?$AAI?$AAR?$AAe?$AAa?$AAd?$AAT?$AAr?$AAa?$AAn?$AAs?$AAf?$AAe?$AAr?$AAC?$AAo?$AAm?$AAp?$AAl?$AAe?$AAt?$AAe?$AA?6?$AA?$AA@ 10009c88     BULK_IN.obj
 0001:00008cc0       ??_C@_1FG@MAILNNPO@?$AA?$CK?$AA?$CK?$AA?$CK?$AA?5?$AAF?$AAT?$AAD?$AAI?$AAR?$AAe?$AAa?$AAd?$AAT?$AAr?$AAa?$AAn?$AAs?$AAf?$AAe?$AAr?$AAC?$AAo?$AAm?$AAp?$AAl?$AAe?$AAt?$AAe?$AA?5?$AAE?$AAR?$AAR@ 10009cc0     BULK_IN.obj
 0001:00008d18       ??_C@_1CE@MHGMFLCO@?$AAB?$AAU?$AAL?$AAK?$AA?5?$AAI?$AAN?$AA?5?$AAS?$AAT?$AAA?$AAR?$AAT?$AAE?$AAD?$AA?$AN?$AA?6?$AA?$AA@ 10009d18     BULK_IN.obj
 0001:00008d3c       ??_C@_1DA@EDJDAGPG@?$AAE?$AAn?$AAt?$AAe?$AAr?$AAi?$AAn?$AAg?$AA?5?$AAB?$AAu?$AAl?$AAk?$AA?5?$AAs?$AAt?$AAa?$AAt?$AAe?$AA?5?$AA?$CF?$AAd?$AA?6?$AA?$AA@ 10009d3c     BULK_IN.obj
 0001:00008d6c       ??_C@_1CO@KKHHAHM@?$AAB?$AAu?$AAl?$AAk?$AA?5?$AAs?$AAt?$AAa?$AAt?$AAe?$AA?3?$AA?5?$AAB?$AAU?$AAL?$AAK?$AA_?$AAI?$AAN?$AAI?$AAT?$AA?6?$AA?$AA@ 10009d6c     BULK_IN.obj
 0001:00008d9c       ??_C@_1CO@BOIFBFBD@?$AAB?$AAu?$AAl?$AAk?$AA?5?$AAs?$AAt?$AAa?$AAt?$AAe?$AA?3?$AA?5?$AAB?$AAU?$AAL?$AAK?$AA_?$AAW?$AAA?$AAI?$AAT?$AA?6?$AA?$AA@ 10009d9c     BULK_IN.obj
 0001:00008dcc       ??_C@_1DI@NOPKKBFB@?$AAB?$AAU?$AAL?$AAK?$AA?5?$AAF?$AAr?$AAe?$AAe?$AA?5?$AAb?$AAu?$AAf?$AAf?$AAe?$AAr?$AA?5?$AA?9?$AA?5?$AAn?$AAo?$AAr?$AAm?$AAa?$AAl?$AA?$AN?$AA?6?$AA?$AA@ 10009dcc     BULK_IN.obj
 0001:00008e04       ??_C@_1DG@LKCLFJKB@?$AAC?$AAl?$AAo?$AAs?$AAe?$AA?5?$AAB?$AAU?$AAL?$AAK?$AA?5?$AAT?$AAa?$AAs?$AAk?$AA?5?$AAs?$AAi?$AAg?$AAn?$AAa?$AAl?$AAl?$AAe?$AAd?$AA?6?$AA?$AA@ 10009e04     BULK_IN.obj
 0001:00008e3c       ??_C@_1DK@LFDOJKFP@?$AAB?$AAU?$AAL?$AAK?$AA_?$AAI?$AAN?$AA?5?$AA?9?$AA?5?$AAg?$AAo?$AAt?$AA?5?$AAR?$AAE?$AAS?$AAT?$AAA?$AAR?$AAT?$AA?5?$AAE?$AAV?$AAE?$AAN?$AAT?$AA?6?$AA?$AA@ 10009e3c     BULK_IN.obj
 0001:00008e78       ??_C@_1FK@FJLMNJNJ@?$AAB?$AAU?$AAL?$AAK?$AA_?$AAW?$AAA?$AAI?$AAT?$AA?5?$AAU?$AAn?$AAh?$AAa?$AAn?$AAd?$AAl?$AAe?$AAd?$AA?5?$AAr?$AAe?$AAt?$AAu?$AAr?$AAn?$AA?5?$AAc?$AAo?$AAd?$AAe?$AA?0@ 10009e78     BULK_IN.obj
 0001:00008ed8       ??_C@_1FA@JEFGPAHP@?$AAB?$AAU?$AAL?$AAK?$AA?5?$AAF?$AAr?$AAe?$AAe?$AA?5?$AAb?$AAu?$AAf?$AAf?$AAe?$AAr?$AA?5?$AA?9?$AA?5?$AAs?$AAh?$AAo?$AAu?$AAl?$AAd?$AAn?$AA?8?$AAt?$AA?5?$AAg?$AAe?$AAt@ 10009ed8     BULK_IN.obj
 0001:00008f28       ??_C@_1CG@FNELFJJG@?$AAC?$AAl?$AAo?$AAs?$AAi?$AAn?$AAg?$AA?5?$AAB?$AAU?$AAL?$AAK?$AA?5?$AAT?$AAa?$AAs?$AAk?$AA?6?$AA?$AA@ 10009f28     BULK_IN.obj
 0001:00008f50       ??_C@_1CA@GIGPMPP@?$AAB?$AAU?$AAL?$AAK?$AA_?$AAC?$AAO?$AAN?$AAF?$AAI?$AAG?$AAU?$AAR?$AAE?$AA?6?$AA?$AA@ 10009f50     BULK_IN.obj
 0001:00008f70       ??_C@_1CI@CMCLMEKK@?$AAU?$AAs?$AAb?$AAP?$AAa?$AAc?$AAk?$AAe?$AAt?$AAS?$AAi?$AAz?$AAe?$AA?5?$AA?$DN?$AA?5?$AA?$CF?$AAd?$AA?6?$AA?$AA@ 10009f70     BULK_IN.obj
 0001:00008f98       ??_C@_1HE@NPPHLDOG@?$AAB?$AAU?$AAL?$AAK?$AA_?$AAI?$AAN?$AA?5?$AAC?$AAO?$AAN?$AAF?$AAI?$AAG?$AAU?$AAR?$AAE?$AA?5?$AAA?$AAl?$AAl?$AAo?$AAc?$AAa?$AAt?$AAe?$AAd?$AA?5?$AA?$CF?$AAd?$AA?5?$AAf@ 10009f98     BULK_IN.obj
 0001:0000900c       ??_C@_1CK@FHIMLPAO@?$AAB?$AAu?$AAl?$AAk?$AA?5?$AAS?$AAt?$AAa?$AAt?$AAe?$AA?3?$AA?5?$AAB?$AAU?$AAL?$AAK?$AA_?$AAI?$AAN?$AA?6?$AA?$AA@ 1000a00c     BULK_IN.obj
 0001:00009038       ??_C@_1DM@COPDPIAH@?$AAB?$AAU?$AAL?$AAK?$AA_?$AAI?$AAN?$AA?5?$AAw?$AAa?$AAi?$AAt?$AA?5?$AAf?$AAo?$AAr?$AA?5?$AAh?$AAB?$AAu?$AAf?$AAf?$AAe?$AAr?$AAM?$AAu?$AAt?$AAe?$AAx?$AA?$AA@ 1000a038     BULK_IN.obj
 0001:00009074       ??_C@_1CM@IEGANBGI@?$AAB?$AAU?$AAF?$AAF?$AAE?$AAR?$AA?5?$AAS?$AAI?$AAZ?$AAE?$AA?5?$AAC?$AAH?$AAA?$AAN?$AAG?$AAI?$AAN?$AAG?$AA?6?$AA?$AA@ 1000a074     BULK_IN.obj
 0001:000090a0       ??_C@_1DO@BDJKPMBO@?$AAB?$AAU?$AAL?$AAK?$AA_?$AAI?$AAN?$AA?5?$AAW?$AAa?$AAi?$AAt?$AA?5?$AAf?$AAo?$AAr?$AA?5?$AAm?$AAu?$AAt?$AAe?$AAx?$AA?5?$AAf?$AAa?$AAi?$AAl?$AAe?$AAd?$AA?6?$AA?$AA@ 1000a0a0     BULK_IN.obj
 0001:000090e0       ??_C@_1DO@EAANLBMO@?$AAB?$AAU?$AAL?$AAK?$AA_?$AAI?$AAN?$AA?5?$AAr?$AAe?$AAl?$AAe?$AAa?$AAs?$AAi?$AAn?$AAg?$AA?5?$AAh?$AAB?$AAu?$AAf?$AAf?$AAe?$AAr?$AAM?$AAu?$AAt?$AAe?$AAx?$AA?$AA@ 1000a0e0     BULK_IN.obj
 0001:00009120       ??_C@_1CG@PFCEKANG@?$AAr?$AAx?$AAB?$AAy?$AAt?$AAe?$AAs?$AA?5?$AAS?$AAi?$AAg?$AAn?$AAa?$AAl?$AAl?$AAe?$AAd?$AA?6?$AA?$AA@ 1000a120     BULK_IN.obj
 0001:00009148       ??_C@_1FE@NKKEOBJA@?$AAW?$AAA?$AAI?$AAT?$AAI?$AAN?$AAG?$AA?5?$AAF?$AAO?$AAR?$AA?5?$AAF?$AAR?$AAE?$AAE?$AA?5?$AAS?$AAP?$AAA?$AAC?$AAE?$AA?5?$AA?9?$AA?5?$AAb?$AAy?$AAt?$AAe?$AAs?$AA?5?$AAf@ 1000a148     BULK_IN.obj
 0001:000091a0       ??_C@_1FG@CEIJBDGM@?$AAF?$AAa?$AAi?$AAl?$AAe?$AAd?$AA?5?$AAt?$AAo?$AA?5?$AAg?$AAe?$AAt?$AA?5?$AAl?$AAa?$AAt?$AAe?$AAn?$AAc?$AAy?$AA?5?$AA?9?$AA?5?$AAs?$AAu?$AAr?$AAp?$AAr?$AAi?$AAs?$AAe@ 1000a1a0     BULK_IN.obj
 0001:000091f8       ??_C@_1EM@NBMOODEN@?$AAG?$AAo?$AAt?$AA?5?$AAl?$AAa?$AAt?$AAe?$AAn?$AAc?$AAy?$AA?5?$AAt?$AAi?$AAm?$AAe?$AAr?$AA?5?$AA?$DN?$AA?5?$AA?$CF?$AAd?$AA?5?$AA?$CI?$AAs?$AAt?$AAa?$AAt?$AAu?$AAs?$AA?5?$AA?$DN@ 1000a1f8     BULK_IN.obj
 0001:00009244       ??_C@_1CC@DHKFDFN@?$AAB?$AAU?$AAL?$AAK?$AA_?$AAE?$AAR?$AAR?$AAO?$AAR?$AA?5?$AA?$DN?$AA?5?$AA?$CF?$AAd?$AA?6?$AA?$AA@ 1000a244     BULK_IN.obj
 0001:00009268       ??_C@_1DA@IBJHEBKN@?$AAB?$AAu?$AAl?$AAk?$AA?5?$AAs?$AAt?$AAa?$AAt?$AAe?$AA?3?$AA?5?$AAB?$AAU?$AAL?$AAK?$AA_?$AAE?$AAR?$AAR?$AAO?$AAR?$AA?6?$AA?$AA@ 1000a268     BULK_IN.obj
 0001:00009298       ??_C@_1CO@NLBOJBFL@?$AAS?$AAe?$AAt?$AAt?$AAi?$AAn?$AAg?$AA?5?$AAI?$AAn?$AA?5?$AAS?$AAi?$AAz?$AAe?$AA?5?$AAt?$AAo?$AA?5?$AA?$CF?$AAd?$AA?6?$AA?$AA@ 1000a298     BULK_IN.obj
 0001:000092c8       ??_C@_1DO@HLJMGFDN@?$AAB?$AAu?$AAl?$AAk?$AA?5?$AAs?$AAt?$AAa?$AAt?$AAe?$AA?3?$AA?5?$AAB?$AAU?$AAL?$AAK?$AA_?$AAE?$AAR?$AAR?$AAO?$AAR?$AA?5?$AAm?$AAe?$AAm?$AAo?$AAr?$AAy?$AA?6?$AA?$AA@ 1000a2c8     BULK_IN.obj
 0001:00009308       ??_C@_1EA@BHOPEKGL@?$AAB?$AAu?$AAl?$AAk?$AA?5?$AAs?$AAt?$AAa?$AAt?$AAe?$AA?3?$AA?5?$AAB?$AAU?$AAL?$AAK?$AA_?$AAE?$AAR?$AAR?$AAO?$AAR?$AA?5?$AAt?$AAi?$AAm?$AAe?$AAo?$AAu?$AAt?$AA?6?$AA?$AA@ 1000a308     BULK_IN.obj
 0001:00009348       ??_C@_1DC@OOAPPCAP@?$AAD?$AAi?$AAs?$AAc?$AAo?$AAn?$AAn?$AAe?$AAc?$AAt?$AA?5?$AAo?$AAn?$AA?5?$AAo?$AAp?$AAe?$AAn?$AA?5?$AAp?$AAo?$AAr?$AAt?$AA?6?$AA?$AA@ 1000a348     BULK_IN.obj
 0001:0000937c       ??_C@_1DE@OLJDHNHG@?$AAU?$AAn?$AAh?$AAa?$AAn?$AAd?$AAl?$AAe?$AAd?$AA?5?$AAB?$AAU?$AAL?$AAK?$AA_?$AAE?$AAR?$AAR?$AAO?$AAR?$AA?$CI?$AA?$CF?$AAd?$AA?$CJ?$AA?6?$AA?$AA@ 1000a37c     BULK_IN.obj
 0001:000093b0       ??_C@_1DI@FMKBNELE@?$AAB?$AAU?$AAL?$AAK?$AA_?$AAI?$AAN?$AA?5?$AAS?$AAT?$AAO?$AAP?$AA?5?$AAs?$AAt?$AAa?$AAt?$AAe?$AA?5?$AAe?$AAn?$AAt?$AAe?$AAr?$AAe?$AAd?$AA?6?$AA?$AA@ 1000a3b0     BULK_IN.obj
 0001:000093e8       ??_C@_1CO@CFBNMMFC@?$AAB?$AAu?$AAl?$AAk?$AA?5?$AAs?$AAt?$AAa?$AAt?$AAe?$AA?3?$AA?5?$AAB?$AAU?$AAL?$AAK?$AA_?$AAE?$AAX?$AAI?$AAT?$AA?6?$AA?$AA@ 1000a3e8     BULK_IN.obj
 0001:00009418       ??_C@_1HK@PPPCNGHK@?$AAc?$AA?3?$AA?2?$AAw?$AAi?$AAn?$AAc?$AAe?$AA8?$AA0?$AA0?$AA?2?$AAo?$AAs?$AAd?$AAe?$AAs?$AAi?$AAg?$AAn?$AAs?$AA?2?$AAv?$AAc?$AAp?$AAo?$AAs?$AAc?$AAe?$AAp?$AAc?$AA?2@ 1000a418     BULK_IN.obj
 0001:00009498       ??_C@_1FA@HNDDKAEP@?$AAF?$AAT?$AA_?$AAP?$AAr?$AAo?$AAc?$AAe?$AAs?$AAs?$AAB?$AAu?$AAl?$AAk?$AAI?$AAn?$AAE?$AAx?$AA?5?$AAB?$AAy?$AAt?$AAe?$AAs?$AAT?$AAo?$AAP?$AAr?$AAo?$AAc?$AAe?$AAs@ 1000a498     BULK_IN.obj
 0001:000094e8       ??_C@_1CA@FGEFGMNE@?$AAF?$AAT?$AA_?$AAP?$AAr?$AAo?$AAc?$AAe?$AAs?$AAs?$AAR?$AAe?$AAa?$AAd?$AA?6?$AA?$AA@ 1000a4e8     BULK_IN.obj
 0001:00009508       ??_C@_1DG@FEFJBBDM@?$AAF?$AAT?$AA_?$AAP?$AAr?$AAo?$AAc?$AAe?$AAs?$AAs?$AAR?$AAe?$AAa?$AAd?$AA?5?$AAr?$AAx?$AAB?$AAy?$AAt?$AAe?$AAs?$AA?$DN?$AA?$CF?$AAd?$AA?6?$AA?$AA@ 1000a508     BULK_IN.obj
 0001:00009540       ??_C@_1IC@COLEEGIO@?$AAF?$AAT?$AA_?$AAP?$AAr?$AAo?$AAc?$AAe?$AAs?$AAs?$AAR?$AAe?$AAa?$AAd?$AA?5?$AAW?$AAe?$AA?5?$AAw?$AAo?$AAn?$AA?8?$AAt?$AA?5?$AAb?$AAe?$AA?5?$AAa?$AAb?$AAl?$AAe?$AA?5@ 1000a540     BULK_IN.obj
 0001:000095c4       ??_C@_1DG@DCAONPAD@?$AAB?$AAu?$AAl?$AAk?$AAC?$AAo?$AAp?$AAi?$AAe?$AAd?$AA?5?$AAf?$AAr?$AAo?$AAm?$AA?5?$AA?$CF?$AAd?$AA?5?$AAt?$AAo?$AA?5?$AAe?$AAn?$AAd?$AA?6?$AA?$AA@ 1000a5c4     BULK_IN.obj
 0001:000095fc       ??_C@_1CM@PCMKCNKF@?$AAB?$AAu?$AAl?$AAk?$AAC?$AAo?$AAp?$AAi?$AAe?$AAd?$AA?5?$AAf?$AAr?$AAo?$AAm?$AA?5?$AA?$CF?$AAd?$AA?5?$AAt?$AAo?$AA?$AA@ 1000a5fc     BULK_IN.obj
 0001:00009628       ??_C@_19BOGGFFED@?$AA?5?$AA?$CF?$AAd?$AA?6?$AA?$AA@ 1000a628     BULK_IN.obj
 0001:00009638       ??_C@_1FM@CJJAGHFL@?$AAp?$AAD?$AAe?$AAv?$AAE?$AAx?$AAt?$AA?9?$AA?$DO?$AAR?$AAe?$AAa?$AAd?$AAR?$AAe?$AAq?$AAu?$AAe?$AAs?$AAt?$AA?4?$AAd?$AAw?$AAB?$AAy?$AAt?$AAe?$AAs?$AAT?$AAr?$AAa?$AAn@ 1000a638     BULK_IN.obj
 0001:00009698       ??_C@_1EO@JOMBDAAB@?$AAF?$AAT?$AA_?$AAP?$AAr?$AAo?$AAc?$AAe?$AAs?$AAs?$AAR?$AAe?$AAa?$AAd?$AA?5?$AAr?$AAe?$AAl?$AAe?$AAa?$AAs?$AAi?$AAn?$AAg?$AA?5?$AAh?$AAB?$AAu?$AAf?$AAf?$AAe?$AAr@ 1000a698     BULK_IN.obj
 0001:000096e8       ??_C@_1DM@FBIKHFAC@?$AAI?$AAn?$AAR?$AAe?$AAq?$AAu?$AAe?$AAs?$AAt?$AA?5?$AAB?$AAu?$AAl?$AAk?$AAI?$AAn?$AA?4?$AAh?$AAP?$AAi?$AAp?$AAe?$AA?5?$AA?$DN?$AA?5?$AA0?$AAx?$AA?$CF?$AAX?$AA?$AA@ 1000a6e8     BULK_IN.obj
 0001:00009724       ??_C@_1DM@KCIOLKII@?$AA1?$AAB?$AAu?$AAl?$AAk?$AA?5?$AAn?$AAt?$AAS?$AAt?$AAa?$AAt?$AAu?$AAs?$AA?$DN?$AA?$CF?$AAd?$AA?0?$AA?5?$AAE?$AAr?$AAr?$AAo?$AAr?$AA?$DN?$AA?$CF?$AAd?$AA?5?$AA?6?$AA?$AA@ 1000a724     BULK_IN.obj
 0001:00009760       ??_C@_1EA@BAJLIKLC@?$AAI?$AAn?$AAR?$AAe?$AAq?$AAu?$AAe?$AAs?$AAt?$AA?5?$AAR?$AAe?$AAq?$AAu?$AAe?$AAs?$AAt?$AAe?$AAd?$AA?3?$AA?$CF?$AAd?$AA?5?$AAR?$AAe?$AAa?$AAd?$AA?3?$AA?$CF?$AAd?$AA?6?$AA?$AA@ 1000a760     BULK_IN.obj
 0001:000097a0       ??_C@_1BA@JGFNDEFA@?$AAC?$AAo?$AAn?$AAt?$AAr?$AAo?$AAl?$AA?$AA@ 1000a7a0     usbddrv.obj
 0001:000097b0       ??_C@_1M@ENKHJKGF@?$AAI?$AAs?$AAo?$AAc?$AAh?$AA?$AA@ 1000a7b0     usbddrv.obj
 0001:000097bc       ??_C@_19PBJLGAMD@?$AAB?$AAu?$AAl?$AAk?$AA?$AA@ 1000a7bc     usbddrv.obj
 0001:000097c8       ??_C@_1BE@PBKDACKD@?$AAI?$AAn?$AAt?$AAe?$AAr?$AAr?$AAu?$AAp?$AAt?$AA?$AA@ 1000a7c8     usbddrv.obj
 0001:000097dc       ??_C@_1CI@DNFHOJGM@?$AAb?$AAC?$AAo?$AAn?$AAf?$AAi?$AAg?$AAu?$AAr?$AAa?$AAt?$AAi?$AAo?$AAn?$AAV?$AAa?$AAl?$AAu?$AAe?$AA?$AA@ 1000a7dc     usbddrv.obj
 0001:00009804       ??_C@_1BE@BOHEBICI@?$AAn?$AAe?$AAt?$AAu?$AAi?$AA?4?$AAd?$AAl?$AAl?$AA?$AA@ 1000a804     usbddrv.obj
 0001:00009818       ??_C@_1ME@FEPGGMAE@?$AAc?$AA?3?$AA?2?$AAw?$AAi?$AAn?$AAc?$AAe?$AA8?$AA0?$AA0?$AA?2?$AAo?$AAs?$AAd?$AAe?$AAs?$AAi?$AAg?$AAn?$AAs?$AA?2?$AAv?$AAc?$AAp?$AAo?$AAs?$AAc?$AAe?$AAp?$AAc?$AA?2@ 1000a818     usbddrv.obj
 0001:000098dc       ??_C@_1BM@BBLCKOAO@?$AAC?$AAa?$AAn?$AA?8?$AAt?$AA?5?$AAf?$AAi?$AAn?$AAd?$AA?5?$AA?$CF?$AAS?$AA?$AA@ 1000a8dc     usbddrv.obj
 0001:000098f8       ??_C@_1BM@GPFHMAOF@?$AAC?$AAa?$AAn?$AA?8?$AAt?$AA?5?$AAl?$AAo?$AAa?$AAd?$AA?5?$AA?$CF?$AAS?$AA?$AA@ 1000a8f8     usbddrv.obj
 0001:00009914       ??_C@_1BK@DKPDGMAK@?$AAG?$AAe?$AAt?$AAN?$AAe?$AAt?$AAS?$AAt?$AAr?$AAi?$AAn?$AAg?$AA?$AA@ 1000a914     usbddrv.obj
 0001:00009930       ??_C@_1BE@HOHBOCOB@?$AAN?$AAe?$AAt?$AAM?$AAs?$AAg?$AAB?$AAo?$AAx?$AA?$AA@ 1000a930     usbddrv.obj
 0001:00009948       ??_C@_1GG@KJPBJKDL@?$AA?$CB?$AAC?$AAa?$AAl?$AAl?$AAN?$AAe?$AAt?$AAM?$AAs?$AAg?$AAB?$AAo?$AAx?$AA?3?$AA?5?$AAE?$AAr?$AAr?$AAo?$AAr?$AA?5?$AA?$CF?$AAu?$AA?5?$AAi?$AAn?$AA?5?$AAF?$AAo?$AAr?$AAm@ 1000a948     usbddrv.obj
 0001:000099b0       ??_C@_1BM@LKGLNLOM@?$AAG?$AAe?$AAt?$AAD?$AAr?$AAi?$AAv?$AAe?$AAr?$AAN?$AAa?$AAm?$AAe?$AA?$AA@ 1000a9b0     usbddrv.obj
 0001:000099cc       ??_C@_1BM@LLINKHBA@?$AAk?$AA?4?$AAc?$AAo?$AAr?$AAe?$AAd?$AAl?$AAl?$AA?4?$AAd?$AAl?$AAl?$AA?$AA@ 1000a9cc     usbddrv.obj
 0001:000099e8       ??_C@_1CA@GOGEMIHH@?$AAW?$AAa?$AAi?$AAt?$AAF?$AAo?$AAr?$AAA?$AAP?$AAI?$AAR?$AAe?$AAa?$AAd?$AAy?$AA?$AA@ 1000a9e8     usbddrv.obj
 0001:00009a08       ??_C@_1BO@KLPJMMP@?$AAC?$AAe?$AAC?$AAa?$AAl?$AAl?$AAU?$AAs?$AAe?$AAr?$AAP?$AAr?$AAo?$AAc?$AA?$AA@ 1000aa08     usbddrv.obj
 0001:00009a28       ??_C@_1MI@EJDOBAPI@?$AAc?$AA?3?$AA?2?$AAw?$AAi?$AAn?$AAc?$AAe?$AA8?$AA0?$AA0?$AA?2?$AAo?$AAs?$AAd?$AAe?$AAs?$AAi?$AAg?$AAn?$AAs?$AA?2?$AAv?$AAc?$AAp?$AAo?$AAs?$AAc?$AAe?$AAp?$AAc?$AA?2@ 1000aa28     usbddrv.obj
 0001:00009af0       ??_C@_1CI@OHFAEIPC@?$AAG?$AAe?$AAt?$AAN?$AAe?$AAt?$AAS?$AAt?$AAr?$AAi?$AAn?$AAg?$AAS?$AAi?$AAz?$AAe?$AAE?$AAx?$AAt?$AA?$AA@ 1000aaf0     usbddrv.obj
 0001:00009b18       ??_C@_1CA@CCCHBEML@?$AAG?$AAe?$AAt?$AAN?$AAe?$AAt?$AAS?$AAt?$AAr?$AAi?$AAn?$AAg?$AAE?$AAx?$AAt?$AA?$AA@ 1000ab18     usbddrv.obj
 0001:00009b38       ??_C@_1BK@GALBKKNF@?$AAN?$AAe?$AAt?$AAM?$AAs?$AAg?$AAB?$AAo?$AAx?$AAE?$AAx?$AAt?$AA?$AA@ 1000ab38     usbddrv.obj
 0001:00009b54       ??_C@_0BA@KEDJFCNN@CallKVNetMsgBox?$AA@ 1000ab54     usbddrv.obj
 0001:00009b68       ??_C@_1EO@LKHCIDMF@?$AA?$CF?$AAS?$AA?3?$AA?5?$AAE?$AAr?$AAr?$AAo?$AAr?$AA?5?$AA?$CF?$AAu?$AA?5?$AAi?$AAn?$AA?5?$AAF?$AAo?$AAr?$AAm?$AAa?$AAt?$AAM?$AAe?$AAs?$AAs?$AAa?$AAg?$AAe?$AA?0?$AA?5?$AAI@ 1000ab68     usbddrv.obj
 0001:00009bb8       ??_C@_1CC@NJBMOKJL@?$AAG?$AAe?$AAt?$AAD?$AAr?$AAi?$AAv?$AAe?$AAr?$AAN?$AAa?$AAm?$AAe?$AAE?$AAx?$AAt?$AA?$AA@ 1000abb8     usbddrv.obj
 0001:00009bdc       ??_C@_1CG@NKFDJDMC@?$AAU?$AAS?$AAB?$AAD?$AA?3?$AA?5?$AAD?$AAL?$AAL?$AA?5?$AAa?$AAt?$AAt?$AAa?$AAc?$AAh?$AA?$AN?$AA?6?$AA?$AA@ 1000abdc     usbddrv.obj
 0001:00009c04       ??_C@_1DK@PGDDBEHF@?$AA?$CL?$AAU?$AAS?$AAB?$AAD?$AA?3?$AAH?$AAc?$AAd?$AAA?$AAt?$AAt?$AAa?$AAc?$AAh?$AA?0?$AA?5?$AAh?$AAc?$AAd?$AA?3?$AA?5?$AA0?$AAx?$AA?$CF?$AAX?$AA?$AN?$AA?6?$AA?$AA@ 1000ac04     usbddrv.obj
 0001:00009c40       ??_C@_1IO@FBFCBHBE@?$AA?$CB?$AA?$CB?$AA?$CB?$AAE?$AAr?$AAr?$AAo?$AAr?$AA?3?$AA?5?$AAU?$AAS?$AAB?$AAD?$AA?3?$AAH?$AAc?$AAd?$AAA?$AAt?$AAt?$AAa?$AAc?$AAh?$AA?0?$AA?5?$AAl?$AAp?$AAH?$AAc?$AAd?$AAF@ 1000ac40     usbddrv.obj
 0001:00009cd0       ??_C@_1HO@LNELMHIN@?$AAc?$AA?3?$AA?2?$AAw?$AAi?$AAn?$AAc?$AAe?$AA8?$AA0?$AA0?$AA?2?$AAo?$AAs?$AAd?$AAe?$AAs?$AAi?$AAg?$AAn?$AAs?$AA?2?$AAv?$AAc?$AAp?$AAo?$AAs?$AAc?$AAe?$AAp?$AAc?$AA?2@ 1000acd0     usbddrv.obj
 0001:00009d50       ??_C@_1CM@DKJPPKPA@?$AAS?$AAY?$AAS?$AAT?$AAE?$AAM?$AA?1?$AAG?$AAw?$AAe?$AAA?$AAp?$AAi?$AAS?$AAe?$AAt?$AAR?$AAe?$AAa?$AAd?$AAy?$AA?$AA@ 1000ad50     usbddrv.obj
 0001:00009d80       ??_C@_1HA@EPPFJPCN@?$AA?$CB?$AAU?$AAS?$AAB?$AAD?$AA?3?$AAG?$AAe?$AAt?$AAC?$AAl?$AAi?$AAe?$AAn?$AAt?$AAD?$AAr?$AAi?$AAv?$AAe?$AAr?$AAN?$AAa?$AAm?$AAe?$AA?0?$AA?5?$AAe?$AAr?$AAr?$AAo?$AAr@ 1000ad80     usbddrv.obj
 0001:00009df0       ??_C@_1FC@JOPNENNN@?$AA?$CL?$AAU?$AAS?$AAB?$AAD?$AA?3?$AAH?$AAc?$AAd?$AAD?$AAe?$AAv?$AAi?$AAc?$AAe?$AAA?$AAt?$AAt?$AAa?$AAc?$AAh?$AAe?$AAd?$AA?0?$AA?5?$AAI?$AAn?$AAt?$AAe?$AAr?$AAf?$AAa@ 1000adf0     usbddrv.obj
 0001:00009e48       ??_C@_1FO@BAOGJIO@?$AAU?$AAS?$AAB?$AAD?$AA?5?$AAF?$AAT?$AAD?$AAI?$AA?3?$AA?5?$AAL?$AAo?$AAa?$AAd?$AAe?$AAd?$AA?5?$AAd?$AAr?$AAi?$AAv?$AAe?$AAr?$AA?5?$AAf?$AAo?$AAr?$AA?5?$AAa?$AAt?$AAt@ 1000ae48     usbddrv.obj
 0001:00009ea8       ??_C@_1GG@EIKNDLIA@?$AA?$CB?$AAU?$AAS?$AAB?$AAD?$AA?3?$AA?5?$AAC?$AAo?$AAu?$AAl?$AAd?$AA?5?$AAn?$AAo?$AAt?$AA?5?$AAl?$AAo?$AAa?$AAd?$AA?5?$AAd?$AAr?$AAi?$AAv?$AAe?$AAr?$AA?5?$AAf?$AAo?$AAr@ 1000aea8     usbddrv.obj
 0001:00009f10       ??_C@_1EG@IEGPCBAC@?$AA?$CL?$AAU?$AAS?$AAB?$AAD?$AA?3?$AAH?$AAc?$AAd?$AAD?$AAe?$AAv?$AAi?$AAc?$AAe?$AAD?$AAe?$AAt?$AAa?$AAc?$AAh?$AAe?$AAd?$AA?0?$AA?5?$AAp?$AAD?$AAe?$AAv?$AA?3?$AA0?$AAx@ 1000af10     usbddrv.obj
 0001:00009f58       ??_C@_1FI@HNKBGPCB@?$AAU?$AAS?$AAB?$AAD?$AA?3?$AAH?$AAc?$AAd?$AAD?$AAe?$AAv?$AAi?$AAc?$AAe?$AAD?$AAe?$AAt?$AAa?$AAc?$AAh?$AAe?$AAd?$AA?3?$AA?5?$AAC?$AAl?$AAo?$AAs?$AAi?$AAn?$AAg?$AA?5@ 1000af58     usbddrv.obj
 0001:00009fb0       ??_C@_1EA@POGNCOLH@?$AAU?$AAS?$AAB?$AAD?$AA?3?$AA?5?$AAU?$AAn?$AAl?$AAo?$AAa?$AAd?$AAi?$AAn?$AAg?$AA?5?$AAc?$AAl?$AAi?$AAe?$AAn?$AAt?$AA?5?$AAD?$AAL?$AAL?$AA?4?$AA?4?$AA?4?$AA?$AN?$AA?6?$AA?$AA@ 1000afb0     usbddrv.obj
 0001:00009ff0       ??_C@_1DI@PJHFMIMI@?$AAU?$AAS?$AAB?$AAD?$AA?3?$AA?5?$AAC?$AAl?$AAi?$AAe?$AAn?$AAt?$AA?5?$AAD?$AAL?$AAL?$AA?5?$AAu?$AAn?$AAl?$AAo?$AAa?$AAd?$AAe?$AAd?$AA?$AN?$AA?6?$AA?$AA@ 1000aff0     usbddrv.obj
 0001:0000a028       ??_C@_1EK@HGCGGKKO@?$AA?9?$AAU?$AAS?$AAB?$AAD?$AA?3?$AAH?$AAc?$AAd?$AAD?$AAe?$AAv?$AAi?$AAc?$AAe?$AAD?$AAe?$AAt?$AAa?$AAc?$AAh?$AAe?$AAd?$AA?0?$AA?5?$AAp?$AAD?$AAe?$AAv?$AA?3?$AA0?$AAx@ 1000b028     usbddrv.obj
 0001:0000a078       ??_C@_1EG@COIEIOCN@?$AA?$CL?$AAU?$AAS?$AAB?$AAD?$AA?3?$AAL?$AAo?$AAa?$AAd?$AAG?$AAe?$AAn?$AAe?$AAr?$AAi?$AAc?$AAI?$AAn?$AAt?$AAe?$AAr?$AAf?$AAa?$AAc?$AAe?$AAD?$AAr?$AAi?$AAv?$AAe?$AAr@ 1000b078     usbddrv.obj
 0001:0000a0c0       ??_C@_1EG@CCKBBJBG@?$AA?9?$AAU?$AAS?$AAB?$AAD?$AA?3?$AAL?$AAo?$AAa?$AAd?$AAG?$AAe?$AAn?$AAe?$AAr?$AAi?$AAc?$AAI?$AAn?$AAt?$AAe?$AAr?$AAf?$AAa?$AAc?$AAe?$AAD?$AAr?$AAi?$AAv?$AAe?$AAr@ 1000b0c0     usbddrv.obj
 0001:0000a108       ??_C@_13FPGAJAPJ@?$AA?2?$AA?$AA@ 1000b108     usbddrv.obj
 0001:0000a110       ??_C@_1EK@IGMEBOAJ@?$AA?$CL?$AAU?$AAS?$AAB?$AAD?$AA?3?$AAF?$AAi?$AAn?$AAd?$AAI?$AAn?$AAt?$AAe?$AAr?$AAf?$AAa?$AAc?$AAe?$AA?0?$AA?5?$AAi?$AAf?$AA?3?$AA?$CF?$AAu?$AA?0?$AA?5?$AAA?$AAl?$AAt?$AA?3@ 1000b110     usbddrv.obj
 0001:0000a15c       ??_C@_1CM@FGLFOAEA@?$AA?9?$AAU?$AAS?$AAB?$AAD?$AA?3?$AAF?$AAi?$AAn?$AAd?$AAI?$AAn?$AAt?$AAe?$AAr?$AAf?$AAa?$AAc?$AAe?$AA?$AN?$AA?6?$AA?$AA@ 1000b15c     usbddrv.obj
 0001:0000a188       ??_C@_1FG@CLHJAFLK@?$AA?9?$AAU?$AAS?$AAB?$AAD?$AA?3?$AAF?$AAi?$AAn?$AAd?$AAI?$AAn?$AAt?$AAe?$AAr?$AAf?$AAa?$AAc?$AAe?$AA?0?$AA?5?$AAi?$AAn?$AAt?$AAe?$AAr?$AAf?$AAa?$AAc?$AAe?$AA?5?$AAn@ 1000b188     usbddrv.obj
 0001:0000a1e0       ??_C@_1GO@FJJMNEMD@?$AA?$CB?$AAU?$AAS?$AAB?$AAD?$AA?3?$AAT?$AAa?$AAk?$AAe?$AAF?$AAr?$AAa?$AAm?$AAe?$AAL?$AAe?$AAn?$AAg?$AAt?$AAh?$AAC?$AAo?$AAn?$AAt?$AAr?$AAo?$AAl?$AA?5?$AA?9?$AA?5?$AAI@ 1000b1e0     usbddrv.obj
 0001:0000a250       ??_C@_1DO@LFJFBLBA@?$AA?$CL?$AAU?$AAS?$AAB?$AAD?$AA?3?$AAT?$AAa?$AAk?$AAe?$AAF?$AAr?$AAa?$AAm?$AAe?$AAL?$AAe?$AAn?$AAg?$AAt?$AAh?$AAC?$AAo?$AAn?$AAt?$AAr?$AAo?$AAl?$AA?$AN?$AA?6?$AA?$AA@ 1000b250     usbddrv.obj
 0001:0000a290       ??_C@_1DO@LHCPFGLC@?$AA?9?$AAU?$AAS?$AAB?$AAD?$AA?3?$AAT?$AAa?$AAk?$AAe?$AAF?$AAr?$AAa?$AAm?$AAe?$AAL?$AAe?$AAn?$AAg?$AAt?$AAh?$AAC?$AAo?$AAn?$AAt?$AAr?$AAo?$AAl?$AA?$AN?$AA?6?$AA?$AA@ 1000b290     usbddrv.obj
 0001:0000a2d0       ??_C@_1HE@OODJOPFF@?$AA?$CB?$AAU?$AAS?$AAB?$AAD?$AA?3?$AAR?$AAe?$AAl?$AAe?$AAa?$AAs?$AAe?$AAF?$AAr?$AAa?$AAm?$AAe?$AAL?$AAe?$AAn?$AAg?$AAt?$AAh?$AAC?$AAo?$AAn?$AAt?$AAr?$AAo?$AAl?$AA?5@ 1000b2d0     usbddrv.obj
 0001:0000a348       ??_C@_1EE@DFEKMNHF@?$AA?$CL?$AAU?$AAS?$AAB?$AAD?$AA?3?$AAR?$AAe?$AAl?$AAe?$AAa?$AAs?$AAe?$AAF?$AAr?$AAa?$AAm?$AAe?$AAL?$AAe?$AAn?$AAg?$AAt?$AAh?$AAC?$AAo?$AAn?$AAt?$AAr?$AAo?$AAl?$AA?$AN@ 1000b348     usbddrv.obj
 0001:0000a390       ??_C@_1EE@LALGJLPI@?$AA?9?$AAU?$AAS?$AAB?$AAD?$AA?3?$AAR?$AAe?$AAl?$AAe?$AAa?$AAs?$AAe?$AAF?$AAr?$AAa?$AAm?$AAe?$AAL?$AAe?$AAn?$AAg?$AAt?$AAh?$AAC?$AAo?$AAn?$AAt?$AAr?$AAo?$AAl?$AA?$AN@ 1000b390     usbddrv.obj
 0001:0000a3d8       ??_C@_1FO@DLFCJBBO@?$AA?$CB?$AAU?$AAS?$AAB?$AAD?$AA?3?$AAS?$AAe?$AAt?$AAF?$AAr?$AAa?$AAm?$AAe?$AAL?$AAe?$AAn?$AAg?$AAt?$AAh?$AA?5?$AA?9?$AA?5?$AAI?$AAn?$AAv?$AAa?$AAl?$AAi?$AAd?$AA?5?$AAd@ 1000b3d8     usbddrv.obj
 0001:0000a438       ??_C@_1CO@NNKGEKJD@?$AA?$CL?$AAU?$AAS?$AAB?$AAD?$AA?3?$AAS?$AAe?$AAt?$AAF?$AAr?$AAa?$AAm?$AAe?$AAL?$AAe?$AAn?$AAg?$AAt?$AAh?$AA?$AN?$AA?6?$AA?$AA@ 1000b438     usbddrv.obj
 0001:0000a468       ??_C@_1CO@GGCBFLI@?$AA?9?$AAU?$AAS?$AAB?$AAD?$AA?3?$AAS?$AAe?$AAt?$AAF?$AAr?$AAa?$AAm?$AAe?$AAL?$AAe?$AAn?$AAg?$AAt?$AAh?$AA?$AN?$AA?6?$AA?$AA@ 1000b468     usbddrv.obj
 0001:0000a498       ??_C@_1FO@DLJPGFNC@?$AA?$CB?$AAU?$AAS?$AAB?$AAD?$AA?3?$AAG?$AAe?$AAt?$AAF?$AAr?$AAa?$AAm?$AAe?$AAN?$AAu?$AAm?$AAb?$AAe?$AAr?$AA?5?$AA?9?$AA?5?$AAI?$AAn?$AAv?$AAa?$AAl?$AAi?$AAd?$AA?5?$AAd@ 1000b498     usbddrv.obj
 0001:0000a4f8       ??_C@_1CO@EIDPNHAL@?$AA?$CL?$AAU?$AAS?$AAB?$AAD?$AA?3?$AAG?$AAe?$AAt?$AAF?$AAr?$AAa?$AAm?$AAe?$AAN?$AAu?$AAm?$AAb?$AAe?$AAr?$AA?$AN?$AA?6?$AA?$AA@ 1000b4f8     usbddrv.obj
 0001:0000a528       ??_C@_1FO@IIDCDEBD@?$AA?$CB?$AAU?$AAS?$AAB?$AAD?$AA?3?$AAG?$AAe?$AAt?$AAF?$AAr?$AAa?$AAm?$AAe?$AAL?$AAe?$AAn?$AAg?$AAt?$AAh?$AA?5?$AA?9?$AA?5?$AAI?$AAn?$AAv?$AAa?$AAl?$AAi?$AAd?$AA?5?$AAd@ 1000b528     usbddrv.obj
 0001:0000a588       ??_C@_1CO@GKBJBHOI@?$AA?$CL?$AAU?$AAS?$AAB?$AAD?$AA?3?$AAG?$AAe?$AAt?$AAF?$AAr?$AAa?$AAm?$AAe?$AAL?$AAe?$AAn?$AAg?$AAt?$AAh?$AA?$AN?$AA?6?$AA?$AA@ 1000b588     usbddrv.obj
 0001:0000a5b8       ??_C@_1FC@PHEHDKAN@?$AA?$CB?$AAU?$AAS?$AAB?$AAD?$AA?3?$AAO?$AAp?$AAe?$AAn?$AAP?$AAi?$AAp?$AAe?$AA?5?$AA?9?$AA?5?$AAI?$AAn?$AAv?$AAa?$AAl?$AAi?$AAd?$AA?5?$AAd?$AAe?$AAv?$AAi?$AAc?$AAe?$AA?5@ 1000b5b8     usbddrv.obj
 0001:0000a610       ??_C@_1GC@KMAPJHAF@?$AA?$CL?$AAU?$AAS?$AAB?$AAD?$AA?3?$AAO?$AAp?$AAe?$AAn?$AAP?$AAi?$AAp?$AAe?$AA?0?$AA?5?$AAE?$AAP?$AA?3?$AA?5?$AA0?$AAx?$AA?$CF?$AAx?$AA?0?$AA?5?$AAM?$AAa?$AAx?$AAP?$AAk?$AAt@ 1000b610     usbddrv.obj
 0001:0000a678       ??_C@_1EO@GFCNHJIF@?$AA?9?$AAU?$AAS?$AAB?$AAD?$AA?3?$AAO?$AAp?$AAe?$AAn?$AAP?$AAi?$AAp?$AAe?$AA?5?$AA?9?$AA?5?$AAp?$AAi?$AAp?$AAe?$AA?5?$AAi?$AAs?$AA?5?$AAa?$AAl?$AAr?$AAe?$AAa?$AAd?$AAy@ 1000b678     usbddrv.obj
 0001:0000a6c8       ??_C@_1EI@OIMLOJMC@?$AA?9?$AAU?$AAS?$AAB?$AAD?$AA?3?$AAO?$AAp?$AAe?$AAn?$AAP?$AAi?$AAp?$AAe?$AA?5?$AAs?$AAu?$AAc?$AAc?$AAe?$AAs?$AAs?$AA?0?$AA?5?$AAh?$AAP?$AAi?$AAp?$AAe?$AA?5?$AA?$DN?$AA?5@ 1000b6c8     usbddrv.obj
 0001:0000a710       ??_C@_1EC@IGLCGKFP@?$AA?$CB?$AAU?$AAS?$AAB?$AAD?$AA?3?$AAO?$AAp?$AAe?$AAn?$AAP?$AAi?$AAp?$AAe?$AA?5?$AAr?$AAe?$AAt?$AAu?$AAr?$AAn?$AAi?$AAn?$AAg?$AA?5?$AAe?$AAr?$AAr?$AAo?$AAr?$AA?$AN?$AA?6@ 1000b710     usbddrv.obj
 0001:0000a758       ??_C@_1EG@OKEAGJFI@?$AA?$CB?$AAU?$AAS?$AAB?$AAD?$AA?3?$AAC?$AAl?$AAo?$AAs?$AAe?$AAP?$AAi?$AAp?$AAe?$AA?5?$AA?9?$AA?5?$AAI?$AAn?$AAv?$AAa?$AAl?$AAi?$AAd?$AA?5?$AAh?$AAa?$AAn?$AAd?$AAl?$AAe@ 1000b758     usbddrv.obj
 0001:0000a7a0       ??_C@_1DO@JEHFBCPF@?$AA?$CL?$AAU?$AAS?$AAB?$AAD?$AA?3?$AAC?$AAl?$AAo?$AAs?$AAe?$AAP?$AAi?$AAp?$AAe?$AA?0?$AA?5?$AAh?$AAP?$AAi?$AAp?$AAe?$AA?3?$AA?5?$AA0?$AAx?$AA?$CF?$AAX?$AA?$AN?$AA?6?$AA?$AA@ 1000b7a0     usbddrv.obj
 0001:0000a7e0       ??_C@_1EI@INJLKIHD@?$AA?9?$AAU?$AAS?$AAB?$AAD?$AA?3?$AAC?$AAl?$AAo?$AAs?$AAe?$AAP?$AAi?$AAp?$AAe?$AA?0?$AA?5?$AAp?$AAi?$AAp?$AAe?$AA?5?$AAi?$AAs?$AA?5?$AAn?$AAo?$AAt?$AA?5?$AAo?$AAp?$AAe@ 1000b7e0     usbddrv.obj
 0001:0000a828       ??_C@_1CE@FOLNIAFM@?$AA?9?$AAU?$AAS?$AAB?$AAD?$AA?3?$AAC?$AAl?$AAo?$AAs?$AAe?$AAP?$AAi?$AAp?$AAe?$AA?$AN?$AA?6?$AA?$AA@ 1000b828     usbddrv.obj
 0001:0000a850       ??_C@_1EG@BILBANEM@?$AA?$CB?$AAU?$AAS?$AAB?$AAD?$AA?3?$AAR?$AAe?$AAs?$AAe?$AAt?$AAP?$AAi?$AAp?$AAe?$AA?5?$AA?9?$AA?5?$AAI?$AAn?$AAv?$AAa?$AAl?$AAi?$AAd?$AA?5?$AAh?$AAa?$AAn?$AAd?$AAl?$AAe@ 1000b850     usbddrv.obj
 0001:0000a898       ??_C@_1CE@JMDIPGCG@?$AA?$CL?$AAU?$AAS?$AAB?$AAD?$AA?3?$AAR?$AAe?$AAs?$AAe?$AAt?$AAP?$AAi?$AAp?$AAe?$AA?$AN?$AA?6?$AA?$AA@ 1000b898     usbddrv.obj
 0001:0000a8c0       ??_C@_1GC@HNIPCEDM@?$AA?$CB?$AAU?$AAS?$AAB?$AAD?$AA?3?$AAR?$AAe?$AAs?$AAe?$AAt?$AAD?$AAe?$AAf?$AAa?$AAu?$AAl?$AAt?$AAP?$AAi?$AAp?$AAe?$AA?5?$AA?9?$AA?5?$AAI?$AAn?$AAv?$AAa?$AAl?$AAi?$AAd@ 1000b8c0     usbddrv.obj
 0001:0000a928       ??_C@_1FI@OEBGLOJG@?$AA?$CB?$AAU?$AAS?$AAB?$AAD?$AA?3?$AAA?$AAb?$AAo?$AAr?$AAt?$AAP?$AAi?$AAp?$AAe?$AAT?$AAr?$AAa?$AAn?$AAs?$AAf?$AAe?$AAr?$AAs?$AA?5?$AA?9?$AA?5?$AAI?$AAn?$AAv?$AAa?$AAl@ 1000b928     usbddrv.obj
 0001:0000a980       ??_C@_1JA@GGIFGOAG@?$AA?$CL?$AAU?$AAS?$AAB?$AAD?$AA?3?$AAA?$AAb?$AAo?$AAr?$AAt?$AAP?$AAi?$AAp?$AAe?$AAT?$AAr?$AAa?$AAn?$AAs?$AAf?$AAe?$AAr?$AAs?$AA?0?$AA?5?$AAh?$AAP?$AAi?$AAp?$AAe?$AA?3@ 1000b980     usbddrv.obj
 0001:0000aa10       ??_C@_1DG@KCNADDH@?$AA?9?$AAU?$AAS?$AAB?$AAD?$AA?3?$AAA?$AAb?$AAo?$AAr?$AAt?$AAP?$AAi?$AAp?$AAe?$AAT?$AAr?$AAa?$AAn?$AAs?$AAf?$AAe?$AAr?$AAs?$AA?$AN?$AA?6?$AA?$AA@ 1000ba10     usbddrv.obj
 0001:0000aa48       ??_C@_1CK@DBEJJCOM@?$AA?$CL?$AAU?$AAS?$AAB?$AAD?$AA?3?$AAG?$AAe?$AAt?$AAI?$AAn?$AAt?$AAe?$AAr?$AAf?$AAa?$AAc?$AAe?$AA?$AN?$AA?6?$AA?$AA@ 1000ba48     usbddrv.obj
 0001:0000aa74       ??_C@_1CK@LACGCCMO@?$AA?$CL?$AAU?$AAS?$AAB?$AAD?$AA?3?$AAS?$AAe?$AAt?$AAI?$AAn?$AAt?$AAe?$AAr?$AAf?$AAa?$AAc?$AAe?$AA?$AN?$AA?6?$AA?$AA@ 1000ba74     usbddrv.obj
 0001:0000aaa0       ??_C@_1CM@CLOCJEN@?$AA?$CL?$AAU?$AAS?$AAB?$AAD?$AA?3?$AAG?$AAe?$AAt?$AAD?$AAe?$AAs?$AAc?$AAr?$AAi?$AAp?$AAt?$AAo?$AAr?$AA?$AN?$AA?6?$AA?$AA@ 1000baa0     usbddrv.obj
 0001:0000aacc       ??_C@_1CM@GOGNFNIO@?$AA?$CL?$AAU?$AAS?$AAB?$AAD?$AA?3?$AAS?$AAe?$AAt?$AAD?$AAe?$AAs?$AAc?$AAr?$AAi?$AAp?$AAt?$AAo?$AAr?$AA?$AN?$AA?6?$AA?$AA@ 1000bacc     usbddrv.obj
 0001:0000aaf8       ??_C@_1CG@MDDPDJMM@?$AA?$CL?$AAU?$AAS?$AAB?$AAD?$AA?3?$AAS?$AAe?$AAt?$AAF?$AAe?$AAa?$AAt?$AAu?$AAr?$AAe?$AA?$AN?$AA?6?$AA?$AA@ 1000baf8     usbddrv.obj
 0001:0000ab20       ??_C@_1CK@FOOEAIAJ@?$AA?$CL?$AAU?$AAS?$AAB?$AAD?$AA?3?$AAC?$AAl?$AAe?$AAa?$AAr?$AAF?$AAe?$AAa?$AAt?$AAu?$AAr?$AAe?$AA?$AN?$AA?6?$AA?$AA@ 1000bb20     usbddrv.obj
 0001:0000ab4c       ??_C@_1CE@GPDODGGF@?$AA?$CL?$AAU?$AAS?$AAB?$AAD?$AA?3?$AAG?$AAe?$AAt?$AAS?$AAt?$AAa?$AAt?$AAu?$AAs?$AA?$AN?$AA?6?$AA?$AA@ 1000bb4c     usbddrv.obj
 0001:0000ab70       ??_C@_1CE@IHANNNBO@?$AA?$CL?$AAU?$AAS?$AAB?$AAD?$AA?3?$AAS?$AAy?$AAn?$AAc?$AAF?$AAr?$AAa?$AAm?$AAe?$AA?$AN?$AA?6?$AA?$AA@ 1000bb70     usbddrv.obj
 0001:0000ab98       ??_C@_1GA@MGOHOIPN@?$AA?$CB?$AAU?$AAS?$AAB?$AAD?$AA?3?$AAI?$AAs?$AAs?$AAu?$AAe?$AAV?$AAe?$AAn?$AAd?$AAo?$AAr?$AAT?$AAr?$AAa?$AAn?$AAs?$AAf?$AAe?$AAr?$AA?5?$AA?9?$AA?5?$AAI?$AAn?$AAv?$AAa@ 1000bb98     usbddrv.obj
 0001:0000abf8       ??_C@_1DA@HOLFMPAN@?$AAI?$AAV?$AAT?$AA?5?$AAI?$AAn?$AAv?$AAa?$AAl?$AAi?$AAd?$AA?5?$AAH?$AAa?$AAn?$AAd?$AAl?$AAe?$AA?5?$AA?$CF?$AAp?$AA?$AN?$AA?6?$AA?$AA@ 1000bbf8     usbddrv.obj
 0001:0000ac28       ??_C@_1GI@LJKCEECP@?$AA?$CB?$AAU?$AAS?$AAB?$AAD?$AA?3?$AAI?$AAs?$AAs?$AAu?$AAe?$AAV?$AAe?$AAn?$AAd?$AAo?$AAr?$AAT?$AAr?$AAa?$AAn?$AAs?$AAf?$AAe?$AAr?$AA?5?$AA?9?$AA?5?$AAI?$AAn?$AAv?$AAa@ 1000bc28     usbddrv.obj
 0001:0000ac90       ??_C@_1JM@DLOBDEHN@?$AA?$CL?$AAU?$AAS?$AAB?$AAD?$AA?3?$AAI?$AAs?$AAs?$AAu?$AAe?$AAV?$AAe?$AAn?$AAd?$AAo?$AAr?$AAT?$AAr?$AAa?$AAn?$AAs?$AAf?$AAe?$AAr?$AA?0?$AA?5?$AAd?$AAw?$AAF?$AAl?$AAa@ 1000bc90     usbddrv.obj
 0001:0000ad30       ??_C@_1GC@ILDLJAGK@?$AA?$CB?$AAU?$AAS?$AAB?$AAD?$AA?3?$AAI?$AAs?$AAs?$AAu?$AAe?$AAV?$AAe?$AAn?$AAd?$AAo?$AAr?$AAT?$AAr?$AAa?$AAn?$AAs?$AAf?$AAe?$AAr?$AA?5?$AA?9?$AA?5?$AAI?$AAn?$AAv?$AAa@ 1000bd30     usbddrv.obj
 0001:0000ad98       ??_C@_1HG@IKAMJOCN@?$AAI?$AAs?$AAs?$AAu?$AAe?$AAV?$AAe?$AAn?$AAd?$AAo?$AAr?$AAT?$AAr?$AAa?$AAn?$AAs?$AAf?$AAe?$AAr?$AA?5?$AAC?$AAe?$AAA?$AAl?$AAl?$AAo?$AAc?$AAA?$AAs?$AAy?$AAn?$AAc@ 1000bd98     usbddrv.obj
 0001:0000ae10       ??_C@_1FI@KEPJGPBP@?$AA?9?$AAU?$AAS?$AAB?$AAD?$AA?3?$AAI?$AAs?$AAs?$AAu?$AAe?$AAV?$AAe?$AAn?$AAd?$AAo?$AAr?$AAT?$AAr?$AAa?$AAn?$AAs?$AAf?$AAe?$AAr?$AA?0?$AA?5?$AAp?$AAT?$AAr?$AAa?$AAn@ 1000be10     usbddrv.obj
 0001:0000ae68       ??_C@_1FM@MGLHIHNJ@?$AA?$CB?$AAU?$AAS?$AAB?$AAD?$AA?3?$AAI?$AAs?$AAs?$AAu?$AAe?$AAC?$AAo?$AAn?$AAt?$AAr?$AAo?$AAl?$AAT?$AAr?$AAa?$AAn?$AAs?$AAf?$AAe?$AAr?$AA?5?$AA?9?$AA?5?$AAI?$AAn?$AAv@ 1000be68     usbddrv.obj
 0001:0000aec8       ??_C@_1MM@JMLJMGDP@?$AA?$CL?$AAU?$AAS?$AAB?$AAD?$AA?3?$AAI?$AAs?$AAs?$AAu?$AAe?$AAC?$AAo?$AAn?$AAt?$AAr?$AAo?$AAl?$AAT?$AAr?$AAa?$AAn?$AAs?$AAf?$AAe?$AAr?$AA?0?$AA?5?$AAP?$AAi?$AAp?$AAe@ 1000bec8     usbddrv.obj
 0001:0000af98       ??_C@_1HI@FAOFBAFI@?$AAI?$AAs?$AAs?$AAu?$AAe?$AAC?$AAo?$AAn?$AAt?$AAr?$AAo?$AAl?$AAT?$AAr?$AAa?$AAn?$AAs?$AAf?$AAe?$AAr?$AA?5?$AAC?$AAe?$AAA?$AAl?$AAl?$AAo?$AAc?$AAA?$AAs?$AAy?$AAn@ 1000bf98     usbddrv.obj
 0001:0000b010       ??_C@_1FK@JMGJGDAK@?$AA?9?$AAU?$AAS?$AAB?$AAD?$AA?3?$AAI?$AAs?$AAs?$AAu?$AAe?$AAC?$AAo?$AAn?$AAt?$AAr?$AAo?$AAl?$AAT?$AAr?$AAa?$AAn?$AAs?$AAf?$AAe?$AAr?$AA?0?$AA?5?$AAp?$AAT?$AAr?$AAa@ 1000c010     usbddrv.obj
 0001:0000b070       ??_C@_1FG@PAILEIK@?$AA?$CB?$AAU?$AAS?$AAB?$AAD?$AA?3?$AAI?$AAs?$AAs?$AAu?$AAe?$AAB?$AAu?$AAl?$AAk?$AAT?$AAr?$AAa?$AAn?$AAs?$AAf?$AAe?$AAr?$AA?5?$AA?9?$AA?5?$AAI?$AAn?$AAv?$AAa?$AAl?$AAi@ 1000c070     usbddrv.obj
 0001:0000b0c8       ??_C@_1KG@KDBCJIKH@?$AA?$CL?$AAU?$AAS?$AAB?$AAD?$AA?3?$AAI?$AAs?$AAs?$AAu?$AAe?$AAB?$AAu?$AAl?$AAk?$AAT?$AAr?$AAa?$AAn?$AAs?$AAf?$AAe?$AAr?$AA?0?$AA?5?$AAp?$AAi?$AAp?$AAe?$AA?3?$AA?$CF?$AAX@ 1000c0c8     usbddrv.obj
 0001:0000b170       ??_C@_1HC@FMDAMFPC@?$AAI?$AAs?$AAs?$AAu?$AAe?$AAB?$AAu?$AAl?$AAk?$AAT?$AAr?$AAa?$AAn?$AAs?$AAf?$AAe?$AAr?$AA?5?$AAC?$AAe?$AAA?$AAl?$AAl?$AAo?$AAc?$AAA?$AAs?$AAy?$AAn?$AAc?$AAh?$AAr@ 1000c170     usbddrv.obj
 0001:0000b1e8       ??_C@_1FE@KIDEMELG@?$AA?9?$AAU?$AAS?$AAB?$AAD?$AA?3?$AAI?$AAs?$AAs?$AAu?$AAe?$AAB?$AAu?$AAl?$AAk?$AAT?$AAr?$AAa?$AAn?$AAs?$AAf?$AAe?$AAr?$AA?0?$AA?5?$AAp?$AAT?$AAr?$AAa?$AAn?$AAs?$AAf@ 1000c1e8     usbddrv.obj
 0001:0000b240       ??_C@_1GA@BAGOEHDC@?$AA?$CB?$AAU?$AAS?$AAB?$AAD?$AA?3?$AAI?$AAs?$AAs?$AAu?$AAe?$AAI?$AAn?$AAt?$AAe?$AAr?$AAr?$AAu?$AAp?$AAt?$AAT?$AAr?$AAa?$AAn?$AAs?$AAf?$AAe?$AAr?$AA?5?$AA?9?$AA?5?$AAI@ 1000c240     usbddrv.obj
 0001:0000b2a0       ??_C@_1LA@BHDEGCAP@?$AA?$CL?$AAU?$AAS?$AAB?$AAD?$AA?3?$AAI?$AAs?$AAs?$AAu?$AAe?$AAI?$AAn?$AAt?$AAe?$AAr?$AAr?$AAu?$AAp?$AAt?$AAT?$AAr?$AAa?$AAn?$AAs?$AAf?$AAe?$AAr?$AA?0?$AA?5?$AAp?$AAi@ 1000c2a0     usbddrv.obj
 0001:0000b350       ??_C@_1HM@NEIAHCFP@?$AAI?$AAs?$AAs?$AAu?$AAe?$AAI?$AAn?$AAt?$AAe?$AAr?$AAr?$AAu?$AAp?$AAt?$AAT?$AAr?$AAa?$AAn?$AAs?$AAf?$AAe?$AAr?$AA?5?$AAC?$AAe?$AAA?$AAl?$AAl?$AAo?$AAc?$AAA?$AAs@ 1000c350     usbddrv.obj
 0001:0000b3d0       ??_C@_1FO@GMDJCDLK@?$AA?9?$AAU?$AAS?$AAB?$AAD?$AA?3?$AAI?$AAs?$AAs?$AAu?$AAe?$AAI?$AAn?$AAt?$AAe?$AAr?$AAr?$AAu?$AAp?$AAt?$AAT?$AAr?$AAa?$AAn?$AAs?$AAf?$AAe?$AAr?$AA?0?$AA?5?$AAp?$AAT@ 1000c3d0     usbddrv.obj
 0001:0000b430       ??_C@_1FI@KBAEGDGM@?$AA?$CB?$AAU?$AAS?$AAB?$AAD?$AA?3?$AAI?$AAs?$AAs?$AAu?$AAe?$AAI?$AAs?$AAo?$AAc?$AAh?$AAT?$AAr?$AAa?$AAn?$AAs?$AAf?$AAe?$AAr?$AA?5?$AA?9?$AA?5?$AAI?$AAn?$AAv?$AAa?$AAl@ 1000c430     usbddrv.obj
 0001:0000b488       ??_C@_1MM@BKFCOJOB@?$AA?$CL?$AAU?$AAS?$AAB?$AAD?$AA?3?$AAI?$AAs?$AAs?$AAu?$AAe?$AAI?$AAs?$AAo?$AAc?$AAh?$AAT?$AAr?$AAa?$AAn?$AAs?$AAf?$AAe?$AAr?$AA?0?$AA?5?$AAp?$AAi?$AAp?$AAe?$AA?3?$AA?$CF@ 1000c488     usbddrv.obj
 0001:0000b558       ??_C@_1HE@KOEEBJPK@?$AAI?$AAs?$AAs?$AAu?$AAe?$AAI?$AAs?$AAo?$AAc?$AAh?$AAT?$AAr?$AAa?$AAn?$AAs?$AAf?$AAe?$AAr?$AA?5?$AAC?$AAe?$AAA?$AAl?$AAl?$AAo?$AAc?$AAA?$AAs?$AAy?$AAn?$AAc?$AAh@ 1000c558     usbddrv.obj
 0001:0000b5d0       ??_C@_1FG@BPNBCJKC@?$AA?9?$AAU?$AAS?$AAB?$AAD?$AA?3?$AAI?$AAs?$AAs?$AAu?$AAe?$AAI?$AAs?$AAo?$AAc?$AAh?$AAT?$AAr?$AAa?$AAn?$AAs?$AAf?$AAe?$AAr?$AA?0?$AA?5?$AAp?$AAT?$AAr?$AAa?$AAn?$AAs@ 1000c5d0     usbddrv.obj
 0001:0000b628       ??_C@_1EM@FCNDDCPC@?$AA?$CB?$AAU?$AAS?$AAB?$AAD?$AA?3?$AAC?$AAl?$AAo?$AAs?$AAe?$AAT?$AAr?$AAa?$AAn?$AAs?$AAf?$AAe?$AAr?$AA?0?$AA?5?$AAi?$AAn?$AAv?$AAa?$AAl?$AAi?$AAd?$AA?5?$AAh?$AAa?$AAn@ 1000c628     usbddrv.obj
 0001:0000b678       ??_C@_1EM@KJIOFIAF@?$AA?$CL?$AAU?$AAS?$AAB?$AAD?$AA?3?$AAC?$AAl?$AAo?$AAs?$AAe?$AAT?$AAr?$AAa?$AAn?$AAs?$AAf?$AAe?$AAr?$AA?0?$AA?5?$AAp?$AAT?$AAr?$AAa?$AAn?$AAs?$AAf?$AAe?$AAr?$AA?3?$AA0@ 1000c678     usbddrv.obj
 0001:0000b6c4       ??_C@_1CM@LIODHCEM@?$AA?9?$AAU?$AAS?$AAB?$AAD?$AA?3?$AAC?$AAl?$AAo?$AAs?$AAe?$AAT?$AAr?$AAa?$AAn?$AAs?$AAf?$AAe?$AAr?$AA?$AN?$AA?6?$AA?$AA@ 1000c6c4     usbddrv.obj
 0001:0000b6f0       ??_C@_1EM@HAIIBFAJ@?$AA?$CB?$AAU?$AAS?$AAB?$AAD?$AA?3?$AAA?$AAb?$AAo?$AAr?$AAt?$AAT?$AAr?$AAa?$AAn?$AAs?$AAf?$AAe?$AAr?$AA?0?$AA?5?$AAi?$AAn?$AAv?$AAa?$AAl?$AAi?$AAd?$AA?5?$AAh?$AAa?$AAn@ 1000c6f0     usbddrv.obj
 0001:0000b740       ??_C@_1FK@NCEOGJOO@?$AA?$CL?$AAU?$AAS?$AAB?$AAD?$AA?3?$AAA?$AAb?$AAo?$AAr?$AAt?$AAT?$AAr?$AAa?$AAn?$AAs?$AAf?$AAe?$AAr?$AA?0?$AA?5?$AAp?$AAT?$AAr?$AAa?$AAn?$AAs?$AAf?$AAe?$AAr?$AA?3?$AA?$CF@ 1000c740     usbddrv.obj
 0001:0000b7a0       ??_C@_1EI@PCFOPDHF@?$AA?$CB?$AAU?$AAS?$AAB?$AAD?$AA?3?$AAA?$AAb?$AAo?$AAr?$AAt?$AAT?$AAr?$AAa?$AAn?$AAs?$AAf?$AAe?$AAr?$AA?5?$AAE?$AAr?$AAr?$AAo?$AAr?$AA?5?$AAi?$AAn?$AA?5?$AAW?$AAF?$AAS@ 1000c7a0     usbddrv.obj
 0001:0000b7e8       ??_C@_1DO@GNMPCOMH@?$AA?9?$AAU?$AAS?$AAB?$AAD?$AA?3?$AAA?$AAb?$AAo?$AAr?$AAt?$AAT?$AAr?$AAa?$AAn?$AAs?$AAf?$AAe?$AAr?$AA?0?$AA?5?$AAf?$AAR?$AAe?$AAt?$AA?3?$AA?$CF?$AAu?$AA?$AN?$AA?6?$AA?$AA@ 1000c7e8     usbddrv.obj
 0001:0000b828       ??_C@_1FA@KMCHLABL@?$AA?9?$AAU?$AAS?$AAB?$AAD?$AA?3?$AAA?$AAb?$AAo?$AAr?$AAt?$AAT?$AAr?$AAa?$AAn?$AAs?$AAf?$AAe?$AAr?$AA?0?$AA?5?$AAa?$AAl?$AAr?$AAe?$AAa?$AAd?$AAy?$AA?5?$AAc?$AAo?$AAm@ 1000c828     usbddrv.obj
 0001:0000b878       ??_C@_1FG@GMOBAADM@?$AA?$CB?$AAU?$AAS?$AAB?$AAD?$AA?3?$AAI?$AAs?$AAT?$AAr?$AAa?$AAn?$AAs?$AAf?$AAe?$AAr?$AAC?$AAo?$AAm?$AAp?$AAl?$AAe?$AAt?$AAe?$AA?0?$AA?5?$AAi?$AAn?$AAv?$AAa?$AAl?$AAi@ 1000c878     usbddrv.obj
 0001:0000b8d0       ??_C@_1EG@PBBOEOPG@?$AA?$CL?$AAU?$AAS?$AAB?$AAD?$AA?3?$AAI?$AAs?$AAT?$AAr?$AAa?$AAn?$AAs?$AAf?$AAe?$AAr?$AAC?$AAo?$AAm?$AAp?$AAl?$AAe?$AAt?$AAe?$AA?0?$AA?5?$AAr?$AAe?$AAt?$AA?5?$AA?$CF?$AAu@ 1000c8d0     usbddrv.obj
 0001:0000b918       ??_C@_1FC@FHHEGEDO@?$AA?$CB?$AAU?$AAS?$AAB?$AAD?$AA?3?$AAG?$AAe?$AAt?$AAT?$AAr?$AAa?$AAn?$AAs?$AAf?$AAe?$AAr?$AAE?$AAr?$AAr?$AAo?$AAr?$AA?0?$AA?5?$AAi?$AAn?$AAv?$AAa?$AAl?$AAi?$AAd?$AA?5@ 1000c918     usbddrv.obj
 0001:0000b96c       ??_C@_1DK@LEDPODJC@?$AA?$CL?$AAU?$AAS?$AAB?$AAD?$AA?3?$AAG?$AAe?$AAt?$AAT?$AAr?$AAa?$AAn?$AAs?$AAf?$AAe?$AAr?$AAE?$AAr?$AAr?$AAo?$AAr?$AA?3?$AA?5?$AA?$CF?$AAu?$AA?$AN?$AA?6?$AA?$AA@ 1000c96c     usbddrv.obj
 0001:0000b9a8       ??_C@_1HI@JGKJFBAK@?$AA?$CB?$AAU?$AAS?$AAB?$AAD?$AA?3?$AAR?$AAe?$AAg?$AAi?$AAs?$AAt?$AAe?$AAr?$AAN?$AAo?$AAt?$AAi?$AAf?$AAi?$AAc?$AAa?$AAt?$AAi?$AAo?$AAn?$AAR?$AAo?$AAu?$AAt?$AAi?$AAn@ 1000c9a8     usbddrv.obj
 0001:0000ba20       ??_C@_1GI@OMDDKFGL@?$AA?$CB?$AAU?$AAS?$AAB?$AAD?$AA?3?$AAR?$AAe?$AAg?$AAi?$AAs?$AAt?$AAe?$AAr?$AAN?$AAo?$AAt?$AAi?$AAf?$AAi?$AAc?$AAa?$AAt?$AAi?$AAo?$AAn?$AAR?$AAo?$AAu?$AAt?$AAi?$AAn@ 1000ca20     usbddrv.obj
 0001:0000ba88       ??_C@_1EI@CHKDGKDB@?$AA?$CL?$AAU?$AAS?$AAB?$AAD?$AA?3?$AAR?$AAe?$AAg?$AAi?$AAs?$AAt?$AAe?$AAr?$AAN?$AAo?$AAt?$AAi?$AAf?$AAi?$AAc?$AAa?$AAt?$AAi?$AAo?$AAn?$AAR?$AAo?$AAu?$AAt?$AAi?$AAn@ 1000ca88     usbddrv.obj
 0001:0000bad0       ??_C@_1EI@HFHKIPML@?$AA?9?$AAU?$AAS?$AAB?$AAD?$AA?3?$AAR?$AAe?$AAg?$AAi?$AAs?$AAt?$AAe?$AAr?$AAN?$AAo?$AAt?$AAi?$AAf?$AAi?$AAc?$AAa?$AAt?$AAi?$AAo?$AAn?$AAR?$AAo?$AAu?$AAt?$AAi?$AAn@ 1000cad0     usbddrv.obj
 0001:0000bb18       ??_C@_1HM@MFLKMBAF@?$AA?$CB?$AAU?$AAS?$AAB?$AAD?$AA?3?$AAU?$AAn?$AAR?$AAe?$AAg?$AAi?$AAs?$AAt?$AAe?$AAr?$AAN?$AAo?$AAt?$AAi?$AAf?$AAi?$AAc?$AAa?$AAt?$AAi?$AAo?$AAn?$AAR?$AAo?$AAu?$AAt@ 1000cb18     usbddrv.obj
 0001:0000bb98       ??_C@_1EM@JCGCPBBK@?$AA?$CL?$AAU?$AAS?$AAB?$AAD?$AA?3?$AAU?$AAn?$AAR?$AAe?$AAg?$AAi?$AAs?$AAt?$AAe?$AAr?$AAN?$AAo?$AAt?$AAi?$AAf?$AAi?$AAc?$AAa?$AAt?$AAi?$AAo?$AAn?$AAR?$AAo?$AAu?$AAt@ 1000cb98     usbddrv.obj
 0001:0000bbe8       ??_C@_1EM@BAPFLBM@?$AA?9?$AAU?$AAS?$AAB?$AAD?$AA?3?$AAU?$AAn?$AAR?$AAe?$AAg?$AAi?$AAs?$AAt?$AAe?$AAr?$AAN?$AAo?$AAt?$AAi?$AAf?$AAi?$AAc?$AAa?$AAt?$AAi?$AAo?$AAn?$AAR?$AAo?$AAu?$AAt@ 1000cbe8     usbddrv.obj
 0001:0000bc38       ??_C@_1FE@POCNFIJO@?$AA?$CB?$AAU?$AAS?$AAB?$AAD?$AA?3?$AAG?$AAe?$AAt?$AAT?$AAr?$AAa?$AAn?$AAs?$AAf?$AAe?$AAr?$AAS?$AAt?$AAa?$AAt?$AAu?$AAs?$AA?0?$AA?5?$AAi?$AAn?$AAv?$AAa?$AAl?$AAi?$AAd@ 1000cc38     usbddrv.obj
 0001:0000bc8c       ??_C@_1DE@OEDAOKGN@?$AA?$CL?$AAU?$AAS?$AAB?$AAD?$AA?3?$AAG?$AAe?$AAt?$AAT?$AAr?$AAa?$AAn?$AAs?$AAf?$AAe?$AAr?$AAS?$AAt?$AAa?$AAt?$AAu?$AAs?$AA?$AN?$AA?6?$AA?$AA@ 1000cc8c     usbddrv.obj
 0001:0000bcc0       ??_C@_1DE@ELOLOEAC@?$AA?9?$AAU?$AAS?$AAB?$AAD?$AA?3?$AAG?$AAe?$AAt?$AAT?$AAr?$AAa?$AAn?$AAs?$AAf?$AAe?$AAr?$AAS?$AAt?$AAa?$AAt?$AAu?$AAs?$AA?$AN?$AA?6?$AA?$AA@ 1000ccc0     usbddrv.obj
 0001:0000bcf8       ??_C@_1FA@NCJCPI@?$AA?$CB?$AAU?$AAS?$AAB?$AAD?$AA?3?$AAG?$AAe?$AAt?$AAI?$AAs?$AAo?$AAc?$AAh?$AAR?$AAe?$AAs?$AAu?$AAl?$AAt?$AAs?$AA?0?$AA?5?$AAi?$AAn?$AAv?$AAa?$AAl?$AAi?$AAd?$AA?5?$AAh@ 1000ccf8     usbddrv.obj
 0001:0000bd48       ??_C@_1DA@OPDFOGD@?$AA?$CL?$AAU?$AAS?$AAB?$AAD?$AA?3?$AAG?$AAe?$AAt?$AAI?$AAs?$AAo?$AAc?$AAh?$AAR?$AAe?$AAs?$AAu?$AAl?$AAt?$AAs?$AA?$AN?$AA?6?$AA?$AA@ 1000cd48     usbddrv.obj
 0001:0000bd78       ??_C@_1FM@BHKEOJKP@?$AA?$CB?$AAU?$AAS?$AAB?$AAD?$AA?3?$AAG?$AAe?$AAt?$AAD?$AAe?$AAv?$AAi?$AAc?$AAe?$AAI?$AAn?$AAf?$AAo?$AA?5?$AA?9?$AA?5?$AAI?$AAn?$AAv?$AAa?$AAl?$AAi?$AAd?$AA?5?$AAd?$AAe@ 1000cd78     usbddrv.obj
 0001:0000bdd4       ??_C@_1CM@IAPFPGNL@?$AA?$CL?$AAU?$AAS?$AAB?$AAD?$AA?3?$AAG?$AAe?$AAt?$AAD?$AAe?$AAv?$AAi?$AAc?$AAe?$AAI?$AAn?$AAf?$AAo?$AA?$AN?$AA?6?$AA?$AA@ 1000cdd4     usbddrv.obj
 0001:0000be00       ??_C@_1EM@EHAKJKHM@?$AA?$CB?$AAU?$AAS?$AAB?$AAD?$AA?3?$AAI?$AAs?$AAP?$AAi?$AAp?$AAe?$AAH?$AAa?$AAl?$AAt?$AAe?$AAd?$AA?5?$AA?9?$AA?5?$AAI?$AAn?$AAv?$AAa?$AAl?$AAi?$AAd?$AA?5?$AAh?$AAa?$AAn@ 1000ce00     usbddrv.obj
 0001:0000be4c       ??_C@_1CK@MENHKKON@?$AA?$CL?$AAU?$AAS?$AAB?$AAD?$AA?3?$AAI?$AAs?$AAP?$AAi?$AAp?$AAe?$AAH?$AAa?$AAl?$AAt?$AAe?$AAd?$AA?$AN?$AA?6?$AA?$AA@ 1000ce4c     usbddrv.obj
 0001:0000be78       ??_C@_1DK@EHFKBMHG@?$AA?9?$AAU?$AAS?$AAB?$AAD?$AA?3?$AAI?$AAs?$AAP?$AAi?$AAp?$AAe?$AAH?$AAa?$AAl?$AAt?$AAe?$AAd?$AA?3?$AA?5?$AAr?$AAe?$AAt?$AA?5?$AA?$CF?$AAu?$AA?$AN?$AA?6?$AA?$AA@ 1000ce78     usbddrv.obj
 0001:0000beb8       ??_C@_1GI@NNFHHBJO@?$AA?$CB?$AAU?$AAS?$AAB?$AAD?$AA?3?$AAI?$AAs?$AAD?$AAe?$AAf?$AAa?$AAu?$AAl?$AAt?$AAP?$AAi?$AAp?$AAe?$AAH?$AAa?$AAl?$AAt?$AAe?$AAd?$AA?5?$AA?9?$AA?5?$AAI?$AAn?$AAv?$AAa@ 1000ceb8     usbddrv.obj
 0001:0000bf20       ??_C@_1FM@MBLBIGIK@?$AA?$CB?$AAU?$AAS?$AAB?$AAD?$AA?3?$AAD?$AAi?$AAs?$AAa?$AAb?$AAl?$AAe?$AAD?$AAe?$AAv?$AAi?$AAc?$AAe?$AA?5?$AA?9?$AA?5?$AAI?$AAn?$AAv?$AAa?$AAl?$AAi?$AAd?$AA?5?$AAd?$AAe@ 1000cf20     usbddrv.obj
 0001:0000bf7c       ??_C@_1CM@FINLMMKG@?$AA?$CL?$AAU?$AAS?$AAB?$AAD?$AA?3?$AAD?$AAi?$AAs?$AAa?$AAb?$AAl?$AAe?$AAD?$AAe?$AAv?$AAi?$AAc?$AAe?$AA?$AN?$AA?6?$AA?$AA@ 1000cf7c     usbddrv.obj
 0001:0000bfa8       ??_C@_1EG@JFPALODL@?$AA?9?$AAU?$AAS?$AAB?$AAD?$AA?3?$AAD?$AAi?$AAs?$AAa?$AAb?$AAl?$AAe?$AAD?$AAe?$AAv?$AAi?$AAc?$AAe?$AA?$CI?$AAb?$AAR?$AAe?$AAt?$AAu?$AAr?$AAn?$AA?5?$AA?$DN?$AA?5?$AA?$CF?$AAd@ 1000cfa8     usbddrv.obj
 0001:0000bff0       ??_C@_1FM@PFCPPLKK@?$AA?$CB?$AAU?$AAS?$AAB?$AAD?$AA?3?$AAS?$AAu?$AAs?$AAp?$AAe?$AAn?$AAd?$AAD?$AAe?$AAv?$AAi?$AAc?$AAe?$AA?5?$AA?9?$AA?5?$AAI?$AAn?$AAv?$AAa?$AAl?$AAi?$AAd?$AA?5?$AAd?$AAe@ 1000cff0     usbddrv.obj
 0001:0000c04c       ??_C@_1CM@HDGOCGKH@?$AA?$CL?$AAU?$AAS?$AAB?$AAD?$AA?3?$AAS?$AAu?$AAs?$AAp?$AAe?$AAn?$AAd?$AAD?$AAe?$AAv?$AAi?$AAc?$AAe?$AA?$AN?$AA?6?$AA?$AA@ 1000d04c     usbddrv.obj
 0001:0000c078       ??_C@_1EI@CHDAPGJB@?$AA?9?$AAU?$AAS?$AAB?$AAD?$AA?3?$AAS?$AAu?$AAs?$AAp?$AAe?$AAn?$AAd?$AAD?$AAe?$AAv?$AAi?$AAc?$AAe?$AA?5?$AA?$CI?$AAb?$AAR?$AAe?$AAt?$AAu?$AAr?$AAn?$AA?5?$AA?$DN?$AA?5?$AA?$CF@ 1000d078     usbddrv.obj
 0001:0000c0c0       ??_C@_1FK@FOFKLEPM@?$AA?$CB?$AAU?$AAS?$AAB?$AAD?$AA?3?$AAR?$AAe?$AAs?$AAu?$AAm?$AAe?$AAD?$AAe?$AAv?$AAi?$AAc?$AAe?$AA?5?$AA?9?$AA?5?$AAI?$AAn?$AAv?$AAa?$AAl?$AAi?$AAd?$AA?5?$AAd?$AAe?$AAv@ 1000d0c0     usbddrv.obj
 0001:0000c11c       ??_C@_1CK@BLJOCGMN@?$AA?$CL?$AAU?$AAS?$AAB?$AAD?$AA?3?$AAR?$AAe?$AAs?$AAu?$AAm?$AAe?$AAD?$AAe?$AAv?$AAi?$AAc?$AAe?$AA?$AN?$AA?6?$AA?$AA@ 1000d11c     usbddrv.obj
 0001:0000c148       ??_C@_1EG@LIFIHABN@?$AA?9?$AAU?$AAS?$AAB?$AAD?$AA?3?$AAR?$AAe?$AAs?$AAu?$AAm?$AAe?$AAD?$AAe?$AAv?$AAi?$AAc?$AAe?$AA?5?$AA?$CI?$AAb?$AAR?$AAe?$AAt?$AAu?$AAr?$AAn?$AA?5?$AA?$DN?$AA?5?$AA?$CF?$AAd@ 1000d148     usbddrv.obj
 0001:0000c190       ??_C@_1BI@NIBKFDCC@?$AAD?$AAr?$AAi?$AAv?$AAe?$AAr?$AAs?$AA?2?$AAU?$AAS?$AAB?$AA?$AA@ 1000d190     usbd.obj
 0001:0000c1a8       ??_C@_1BM@EKFDCEJD@?$AAC?$AAl?$AAi?$AAe?$AAn?$AAt?$AAD?$AAr?$AAi?$AAv?$AAe?$AAr?$AAs?$AA?$AA@ 1000d1a8     usbd.obj
 0001:0000c1c4       ??_C@_1BI@PGFBCHEP@?$AAL?$AAo?$AAa?$AAd?$AAC?$AAl?$AAi?$AAe?$AAn?$AAt?$AAs?$AA?$AA@ 1000d1c4     usbd.obj
 0001:0000c1dc       ??_C@_1BA@GHOECOCL@?$AAD?$AAe?$AAf?$AAa?$AAu?$AAl?$AAt?$AA?$AA@ 1000d1dc     usbd.obj
 0001:0000c1ec       ??_C@_17JOFCMBBD@?$AAD?$AAL?$AAL?$AA?$AA@ 1000d1ec     usbd.obj
 0001:0000c1f4       ??_C@_1CA@PKLHEOKA@?$AAU?$AAS?$AAB?$AAD?$AAe?$AAv?$AAi?$AAc?$AAe?$AAA?$AAt?$AAt?$AAa?$AAc?$AAh?$AA?$AA@ 1000d1f4     usbd.obj
 0001:0000c214       ??_C@_1CC@BDLJNJJG@?$AAU?$AAS?$AAB?$AAI?$AAn?$AAs?$AAt?$AAa?$AAl?$AAl?$AAD?$AAr?$AAi?$AAv?$AAe?$AAr?$AA?$AA@ 1000d214     usbd.obj
 0001:0000c238       ??_C@_17ODMKMPCC@?$AA?$CF?$AAu?$AA_?$AA?$AA@ 1000d238     usbd.obj
 0001:0000c240       ??_C@_1HI@CPHFIHAD@?$AAc?$AA?3?$AA?2?$AAw?$AAi?$AAn?$AAc?$AAe?$AA8?$AA0?$AA0?$AA?2?$AAo?$AAs?$AAd?$AAe?$AAs?$AAi?$AAg?$AAn?$AAs?$AA?2?$AAv?$AAc?$AAp?$AAo?$AAs?$AAc?$AAe?$AAp?$AAc?$AA?2@ 1000d240     usbd.obj
 0001:0000c2b8       ??_C@_1BC@OCIMDPHE@?$AA?$CF?$AAu?$AA_?$AA?$CF?$AAu?$AA_?$AA?$CF?$AAu?$AA?$AA@ 1000d2b8     usbd.obj
 0001:0000c2cc       ??_C@_1M@JDFOPOOF@?$AA?$CF?$AAu?$AA_?$AA?$CF?$AAu?$AA?$AA@ 1000d2cc     usbd.obj
 0001:0000c2d8       ??_C@_15EFLNJKHH@?$AA?$CF?$AAu?$AA?$AA@ 1000d2d8     usbd.obj
 0001:0000c2e0       ??_C@_1HO@CEFJPPL@?$AAU?$AAS?$AAB?$AAD?$AA?3?$AAI?$AAn?$AAs?$AAt?$AAa?$AAl?$AAl?$AAC?$AAl?$AAi?$AAe?$AAn?$AAt?$AAD?$AAr?$AAi?$AAv?$AAe?$AAr?$AA?$CI?$AA?$CF?$AAs?$AA?$CJ?$AA?0?$AA?5?$AAI?$AAn@ 1000d2e0     usbd.obj
 0001:0000c360       ??_C@_1IA@LIBMGBDK@?$AA?$CB?$AAU?$AAS?$AAB?$AAD?$AA?3?$AAI?$AAn?$AAs?$AAt?$AAa?$AAl?$AAl?$AAC?$AAl?$AAi?$AAe?$AAn?$AAt?$AAD?$AAr?$AAi?$AAv?$AAe?$AAr?$AA?$CI?$AA?$CF?$AAs?$AA?$CJ?$AA?0?$AA?5?$AAe@ 1000d360     usbd.obj
 0001:0000c3e0       ??_C@_1EG@PPCHDFHJ@?$AA?$CB?$AAU?$AAS?$AAB?$AAD?$AA?3?$AA?5?$AAE?$AAx?$AAc?$AAe?$AAp?$AAt?$AAi?$AAo?$AAn?$AA?5?$AAi?$AAn?$AA?5?$AAi?$AAn?$AAs?$AAt?$AAa?$AAl?$AAl?$AA?5?$AAp?$AAr?$AAo?$AAc@ 1000d3e0     usbd.obj
 0001:0000c428       ??_C@_1HG@NAJFJBKD@?$AA?$CB?$AAU?$AAS?$AAB?$AAD?$AA?3?$AAI?$AAn?$AAs?$AAt?$AAa?$AAl?$AAl?$AAC?$AAl?$AAi?$AAe?$AAn?$AAt?$AAD?$AAr?$AAi?$AAv?$AAe?$AAr?$AA?0?$AA?5?$AAG?$AAe?$AAt?$AAP?$AAr@ 1000d428     usbd.obj
 0001:0000c4a0       ??_C@_1HE@NBMMIAPO@?$AA?$CB?$AAU?$AAS?$AAB?$AAD?$AA?3?$AAI?$AAn?$AAs?$AAt?$AAa?$AAl?$AAl?$AAC?$AAl?$AAi?$AAe?$AAn?$AAt?$AAD?$AAr?$AAi?$AAv?$AAe?$AAr?$AA?0?$AA?5?$AAe?$AAr?$AAr?$AAo?$AAr@ 1000d4a0     usbd.obj
 0001:0000c518       ??_C@_1FE@LEPBAHBK@?$AAU?$AAS?$AAB?$AAD?$AA?3?$AA?5?$AAC?$AAa?$AAl?$AAl?$AAi?$AAn?$AAg?$AA?5?$AAc?$AAl?$AAi?$AAe?$AAn?$AAt?$AA?5?$AAa?$AAt?$AAt?$AAa?$AAc?$AAh?$AA?5?$AAp?$AAr?$AAo?$AAc@ 1000d518     usbd.obj
 0001:0000c570       ??_C@_1EE@DKHKGIDJ@?$AA?$CB?$AAU?$AAS?$AAB?$AAD?$AA?3?$AA?5?$AAE?$AAx?$AAc?$AAe?$AAp?$AAt?$AAi?$AAo?$AAn?$AA?5?$AAi?$AAn?$AA?5?$AAa?$AAt?$AAt?$AAa?$AAc?$AAh?$AA?5?$AAp?$AAr?$AAo?$AAc?$AA?$AN@ 1000d570     usbd.obj
 0001:0000c5b4       ??_C@_1BC@PCJHCCND@?$AAa?$AAc?$AAc?$AAe?$AAp?$AAt?$AAe?$AAd?$AA?$AA@ 1000d5b4     usbd.obj
 0001:0000c5c8       ??_C@_1BO@DDELADIO@?$AAd?$AAi?$AAd?$AA?5?$AAn?$AAo?$AAt?$AA?5?$AAa?$AAc?$AAc?$AAe?$AAp?$AAt?$AA?$AA@ 1000d5c8     usbd.obj
 0001:0000c5e8       ??_C@_1EI@KLADJMEF@?$AAU?$AAS?$AAB?$AAD?$AA?3?$AA?5?$AAC?$AAl?$AAi?$AAe?$AAn?$AAt?$AA?5?$AA?$CF?$AAs?$AA?5?$AAc?$AAo?$AAn?$AAt?$AAr?$AAo?$AAl?$AA?5?$AAo?$AAf?$AA?5?$AAd?$AAe?$AAv?$AAi?$AAc@ 1000d5e8     usbd.obj
 0001:0000c630       ??_C@_1HK@GKEKEGBP@?$AA?$CB?$AAL?$AAo?$AAa?$AAd?$AAR?$AAe?$AAg?$AAi?$AAs?$AAt?$AAe?$AAr?$AAe?$AAd?$AAD?$AAr?$AAi?$AAv?$AAe?$AAr?$AA?3?$AA?5?$AAN?$AAo?$AA?5?$AAa?$AAt?$AAt?$AAa?$AAc?$AAh@ 1000d630     usbd.obj
 0001:0000c6b0       ??_C@_1EK@OAKCOIMK@?$AA?$CB?$AAU?$AAS?$AAB?$AAD?$AA?3?$AA?5?$AAE?$AAr?$AAr?$AAo?$AAr?$AA?5?$AAi?$AAn?$AA?5?$AAL?$AAo?$AAa?$AAd?$AAD?$AAr?$AAi?$AAv?$AAe?$AAr?$AA?$CI?$AA?$CF?$AAs?$AA?$CJ?$AA?3?$AA?5@ 1000d6b0     usbd.obj
 0001:0000c700       ??_C@_1IG@DPCAOLLM@?$AAU?$AAS?$AAB?$AAD?$AA?3?$AAC?$AAo?$AAn?$AAv?$AAe?$AAr?$AAt?$AAT?$AAo?$AAC?$AAl?$AAi?$AAe?$AAn?$AAt?$AAR?$AAe?$AAg?$AAi?$AAs?$AAt?$AAr?$AAy?$AA?5?$AAf?$AAo?$AAr@ 1000d700     usbd.obj
 0001:0000c788       ??_C@_1BO@LBHFGNBG@?$AA?$CF?$AAs?$AA?2?$AA?$CF?$AAs?$AA?2?$AA?$CF?$AAs?$AA?2?$AA?$CF?$AAs?$AA?2?$AA?$CF?$AAs?$AA?$AA@ 1000d788     usbd.obj
 0001:0000c7a8       ??_C@_1GK@LKNCDFHB@?$AAU?$AAS?$AAB?$AAD?$AA?3?$AAC?$AAo?$AAn?$AAv?$AAe?$AAr?$AAt?$AAT?$AAo?$AAC?$AAl?$AAi?$AAe?$AAn?$AAt?$AAR?$AAe?$AAg?$AAi?$AAs?$AAt?$AAr?$AAy?$AA?0?$AA?5?$AAR?$AAe@ 1000d7a8     usbd.obj
 0001:0000c818       ??_C@_1HC@GOCKJFPL@?$AAU?$AAS?$AAB?$AAD?$AA?3?$AAC?$AAo?$AAn?$AAv?$AAe?$AAr?$AAt?$AAT?$AAo?$AAC?$AAl?$AAi?$AAe?$AAn?$AAt?$AAR?$AAe?$AAg?$AAi?$AAs?$AAt?$AAr?$AAy?$AA?0?$AA?5?$AAR?$AAe@ 1000d818     usbd.obj
 0001:0000c890       ??_C@_1GO@HGPDPHKP@?$AA?9?$AAU?$AAS?$AAB?$AAD?$AA?3?$AAC?$AAo?$AAn?$AAv?$AAe?$AAr?$AAt?$AAT?$AAo?$AAC?$AAl?$AAi?$AAe?$AAn?$AAt?$AAR?$AAe?$AAg?$AAi?$AAs?$AAt?$AAr?$AAy?$AA?0?$AA?5?$AAC@ 1000d890     usbd.obj
 0001:0000c900       ??_C@_1GA@IGELGLDD@?$AAU?$AAS?$AAB?$AAD?$AA?3?$AAL?$AAo?$AAa?$AAd?$AAG?$AAr?$AAo?$AAu?$AAp?$AAD?$AAr?$AAi?$AAv?$AAe?$AAr?$AA?$CI?$AA?$CJ?$AA?3?$AA?5?$AAn?$AAo?$AA?5?$AAk?$AAe?$AAy?$AA?5?$AAL@ 1000d900     usbd.obj
 0001:0000c960       ??_C@_1JG@HGHFHKIA@?$AAU?$AAS?$AAB?$AAD?$AA?3?$AAL?$AAo?$AAa?$AAd?$AAD?$AAe?$AAv?$AAi?$AAc?$AAe?$AAD?$AAr?$AAi?$AAv?$AAe?$AAr?$AAs?$AA?5?$AA?9?$AA?5?$AAD?$AAe?$AAv?$AAi?$AAc?$AAe?$AA?5@ 1000d960     usbd.obj
 0001:0000c9f8       ??_C@_1HC@MKNJFLBB@?$AAU?$AAS?$AAB?$AAD?$AA?3?$AAL?$AAo?$AAa?$AAd?$AAD?$AAe?$AAv?$AAi?$AAc?$AAe?$AAD?$AAr?$AAi?$AAv?$AAe?$AAr?$AAs?$AA?5?$AAl?$AAo?$AAa?$AAd?$AAi?$AAn?$AAg?$AA?5?$AAd@ 1000d9f8     usbd.obj
 0001:0000ca70       ??_C@_1FE@CHEOICHB@?$AAU?$AAS?$AAB?$AAD?$AA?3?$AA?5?$AAC?$AAa?$AAl?$AAl?$AAi?$AAn?$AAg?$AA?5?$AAc?$AAl?$AAi?$AAe?$AAn?$AAt?$AA?5?$AAd?$AAe?$AAv?$AAi?$AAc?$AAe?$AA?5?$AAd?$AAe?$AAt?$AAa@ 1000da70     usbd.obj
 0001:0000cac8       ??_C@_1GA@EJJHKKJC@?$AAU?$AAS?$AAB?$AAD?$AA?3?$AA?5?$AAR?$AAe?$AAt?$AAu?$AAr?$AAn?$AAe?$AAd?$AA?5?$AAf?$AAr?$AAo?$AAm?$AA?5?$AAc?$AAl?$AAi?$AAe?$AAn?$AAt?$AA?5?$AAd?$AAe?$AAv?$AAi?$AAc@ 1000dac8     usbd.obj
 0001:0000cb28       ??_C@_1DG@JMOAGCMN@?$AA?$CB?$AAU?$AAS?$AAB?$AAD?$AA?3?$AA?5?$AAN?$AAU?$AAL?$AAL?$AA?5?$AAP?$AAi?$AAp?$AAe?$AA?5?$AAh?$AAa?$AAn?$AAd?$AAl?$AAe?$AA?4?$AA?$AN?$AA?6?$AA?$AA@ 1000db28     usbd.obj
 0001:0000cb60       ??_C@_1FK@KIKDCPLI@?$AA?$CB?$AAU?$AAS?$AAB?$AAD?$AA?3?$AA?5?$AAI?$AAn?$AAv?$AAa?$AAl?$AAi?$AAd?$AA?5?$AAP?$AAi?$AAp?$AAe?$AA?5?$AAh?$AAa?$AAn?$AAd?$AAl?$AAe?$AA?5?$AA0?$AAx?$AA?$CF?$AAX?$AA?5@ 1000db60     usbd.obj
 0001:0000cbc0       ??_C@_1FK@JKGEFOCF@?$AA?$CB?$AAU?$AAS?$AAB?$AAD?$AA?3?$AA?5?$AAE?$AAx?$AAc?$AAe?$AAp?$AAt?$AAi?$AAo?$AAn?$AA?5?$AAc?$AAh?$AAe?$AAc?$AAk?$AAi?$AAn?$AAg?$AA?5?$AAP?$AAi?$AAp?$AAe?$AA?5?$AAh@ 1000dbc0     usbd.obj
 0001:0000cc1c       ??_C@_1CM@OPGBINKG@?$AAV?$AAD?$AAH?$AA?5?$AAI?$AAn?$AAv?$AAa?$AAl?$AAi?$AAd?$AA?5?$AA?$CF?$AAp?$AA?5?$AA?$CI?$AA?$CF?$AAx?$AA?$CJ?$AA?$AN?$AA?6?$AA?$AA@ 1000dc1c     usbd.obj
 0001:0000cc48       ??_C@_1FO@BPPKPIHP@?$AA?$CB?$AAU?$AAS?$AAB?$AAD?$AA?3?$AA?5?$AAI?$AAn?$AAv?$AAa?$AAl?$AAi?$AAd?$AA?5?$AAd?$AAe?$AAv?$AAi?$AAc?$AAe?$AA?5?$AAh?$AAa?$AAn?$AAd?$AAl?$AAe?$AA?5?$AA0?$AAx?$AA?$CF@ 1000dc48     usbd.obj
 0001:0000cca8       ??_C@_1CG@PAPLOCPN@?$AAV?$AAD?$AAH?$AA?5?$AAE?$AAx?$AAc?$AAe?$AAp?$AAt?$AAi?$AAo?$AAn?$AA?5?$AA?$CF?$AAp?$AA?$AN?$AA?6?$AA?$AA@ 1000dca8     usbd.obj
 0001:0000ccd0       ??_C@_1FO@LADPHGMP@?$AA?$CB?$AAU?$AAS?$AAB?$AAD?$AA?3?$AA?5?$AAE?$AAx?$AAc?$AAe?$AAp?$AAt?$AAi?$AAo?$AAn?$AA?5?$AAc?$AAh?$AAe?$AAc?$AAk?$AAi?$AAn?$AAg?$AA?5?$AAd?$AAe?$AAv?$AAi?$AAc?$AAe@ 1000dcd0     usbd.obj
 0001:0000cd30       ??_C@_1GC@FHDIHFPC@?$AA?$CB?$AAU?$AAS?$AAB?$AAD?$AA?3?$AA?5?$AAI?$AAn?$AAv?$AAa?$AAl?$AAi?$AAd?$AA?5?$AAt?$AAr?$AAa?$AAn?$AAs?$AAf?$AAe?$AAr?$AA?5?$AAh?$AAa?$AAn?$AAd?$AAl?$AAe?$AA?5?$AA0@ 1000dd30     usbd.obj
 0001:0000cd98       ??_C@_1GC@HOJJLIP@?$AA?$CB?$AAU?$AAS?$AAB?$AAD?$AA?3?$AA?5?$AAE?$AAx?$AAc?$AAe?$AAp?$AAt?$AAi?$AAo?$AAn?$AA?5?$AAc?$AAh?$AAe?$AAc?$AAk?$AAi?$AAn?$AAg?$AA?5?$AAt?$AAr?$AAa?$AAn?$AAs?$AAf@ 1000dd98     usbd.obj
 0001:0000ce00       ??_C@_1HG@MANDAPFL@?$AAU?$AAS?$AAB?$AAD?$AA?3?$AAF?$AAr?$AAe?$AAe?$AAP?$AAi?$AAp?$AAe?$AAO?$AAb?$AAj?$AAe?$AAc?$AAt?$AA?$CI?$AA0?$AAx?$AA?$CF?$AAX?$AA?$CJ?$AA?0?$AA?5?$AAw?$AAa?$AAi?$AAt?$AAi@ 1000de00     usbd.obj
 0001:0000ce78       ??_C@_1HG@GADCLNC@?$AA?$CB?$AAU?$AAS?$AAB?$AAD?$AA?3?$AAF?$AAr?$AAe?$AAe?$AAP?$AAi?$AAp?$AAe?$AAO?$AAb?$AAj?$AAe?$AAc?$AAt?$AA?$CI?$AA0?$AAx?$AA?$CF?$AAX?$AA?$CJ?$AA?5?$AAt?$AAi?$AAm?$AAe?$AAd@ 1000de78     usbd.obj
 0001:0000cef0       ??_C@_1HC@EGIJLBJG@?$AAU?$AAS?$AAB?$AAD?$AA?3?$AAF?$AAr?$AAe?$AAe?$AAT?$AAr?$AAa?$AAn?$AAs?$AAf?$AAe?$AAr?$AAO?$AAb?$AAj?$AAe?$AAc?$AAt?$AA?$CI?$AA0?$AAx?$AA?$CF?$AAX?$AA?$CJ?$AA?0?$AA?5?$AAa@ 1000def0     usbd.obj
 0001:0000cf68       ??_C@_1HO@PCAAIKKI@?$AAU?$AAS?$AAB?$AAD?$AA?3?$AAF?$AAr?$AAe?$AAe?$AAT?$AAr?$AAa?$AAn?$AAs?$AAf?$AAe?$AAr?$AAO?$AAb?$AAj?$AAe?$AAc?$AAt?$AA?$CI?$AA0?$AAx?$AA?$CF?$AAX?$AA?$CJ?$AA?0?$AA?5?$AAw@ 1000df68     usbd.obj
 0001:0000cfe8       ??_C@_1HO@NBFBBLIF@?$AA?$CB?$AAU?$AAS?$AAB?$AAD?$AA?3?$AAF?$AAr?$AAe?$AAe?$AAT?$AAr?$AAa?$AAn?$AAs?$AAf?$AAe?$AAr?$AAO?$AAb?$AAj?$AAe?$AAc?$AAt?$AA?$CI?$AA0?$AAx?$AA?$CF?$AAX?$AA?$CJ?$AA?5?$AAt@ 1000dfe8     usbd.obj
 0001:0000d068       ??_C@_1DK@IDLOABHP@?$AA?$CK?$AA?$CK?$AA?$CK?$AA?5?$AAR?$AAe?$AAs?$AAe?$AAt?$AAE?$AAv?$AAe?$AAn?$AAt?$AA?5?$AAE?$AAR?$AAR?$AAO?$AAR?$AA?3?$AA?$CF?$AAd?$AA?5?$AA?$CK?$AA?$CK?$AA?$CK?$AA?6?$AA?$AA@ 1000e068     usbclient.obj
 0001:0000d0a8       ??_C@_1EA@DLNKEDK@?$AA?$CK?$AA?$CK?$AA?$CK?$AA?5?$AAA?$AAb?$AAo?$AAr?$AAt?$AAT?$AAr?$AAa?$AAn?$AAs?$AAf?$AAe?$AAr?$AA?5?$AAE?$AAR?$AAR?$AAO?$AAR?$AA?3?$AA?$CF?$AAd?$AA?5?$AA?$CK?$AA?$CK?$AA?$CK?$AA?6?$AA?$AA@ 1000e0a8     usbclient.obj
 0001:0000d0e8       ??_C@_1EA@OEBLAPPP@?$AA?$CK?$AA?$CK?$AA?$CK?$AA?5?$AAC?$AAl?$AAo?$AAs?$AAe?$AAT?$AAr?$AAa?$AAn?$AAs?$AAf?$AAe?$AAr?$AA?5?$AAE?$AAR?$AAR?$AAO?$AAR?$AA?3?$AA?$CF?$AAd?$AA?5?$AA?$CK?$AA?$CK?$AA?$CK?$AA?6?$AA?$AA@ 1000e0e8     usbclient.obj
 0001:0000d128       ??_C@_1FO@EGDNIMLN@?$AAC?$AAl?$AAe?$AAa?$AAr?$AAO?$AAr?$AAS?$AAe?$AAt?$AAF?$AAe?$AAa?$AAt?$AAu?$AAr?$AAe?$AA?3?$AAW?$AAA?$AAI?$AAT?$AA_?$AAT?$AAI?$AAM?$AAE?$AAO?$AAU?$AAT?$AA?5?$AAo@ 1000e128     usbclient.obj
 0001:0000d188       ??_C@_1EC@JIGPENPP@?$AA?$CK?$AA?$CK?$AA?$CK?$AA?5?$AAU?$AAn?$AAh?$AAa?$AAn?$AAd?$AAl?$AAe?$AAd?$AA?5?$AAW?$AAa?$AAi?$AAt?$AAR?$AAe?$AAa?$AAs?$AAo?$AAn?$AA?3?$AA?$CF?$AAd?$AA?5?$AA?$CK?$AA?$CK?$AA?$CK?$AA?6@ 1000e188     usbclient.obj
 0001:0000d1d0       ??_C@_1GK@NFJEKGG@?$AA?$CK?$AA?$CK?$AA?$CK?$AA?5?$AAC?$AAl?$AAe?$AAa?$AAr?$AAO?$AAr?$AAS?$AAe?$AAt?$AAF?$AAe?$AAa?$AAt?$AAu?$AAr?$AAe?$AA?5?$AAo?$AAn?$AA?5?$AAe?$AAn?$AAd?$AAp?$AAo?$AAi?$AAn@ 1000e1d0     usbclient.obj
 0001:0000d240       ??_C@_1FE@GJFHKKL@?$AA?$CK?$AA?$CK?$AA?$CK?$AA?5?$AAD?$AAe?$AAf?$AAa?$AAu?$AAl?$AAt?$AAT?$AAr?$AAa?$AAn?$AAs?$AAf?$AAe?$AAr?$AAC?$AAo?$AAm?$AAp?$AAl?$AAe?$AAt?$AAe?$AA?5?$AAE?$AAR?$AAR?$AAO@ 1000e240     usbclient.obj
 0001:0000d298       ??_C@_1EO@LLIJNJID@?$AAG?$AAe?$AAt?$AAS?$AAt?$AAa?$AAt?$AAu?$AAs?$AA?3?$AAW?$AAA?$AAI?$AAT?$AA_?$AAT?$AAI?$AAM?$AAE?$AAO?$AAU?$AAT?$AA?5?$AAo?$AAn?$AA?5?$AAb?$AAI?$AAn?$AAd?$AAe?$AAx@ 1000e298     usbclient.obj
 0001:0000d2e8       ??_C@_1HC@OIDPFNDL@?$AA?$CK?$AA?$CK?$AA?$CK?$AA?5?$AAG?$AAe?$AAt?$AAS?$AAt?$AAa?$AAt?$AAu?$AAs?$AA?5?$AAo?$AAn?$AA?5?$AAe?$AAn?$AAd?$AAp?$AAo?$AAi?$AAn?$AAt?$AA?3?$AA0?$AAx?$AA?$CF?$AAx?$AA?5?$AAf@ 1000e2e8     usbclient.obj
 0001:0000d360       ??_C@_1HA@BBDFJFG@?$AAG?$AAe?$AAt?$AAT?$AAr?$AAa?$AAn?$AAs?$AAf?$AAe?$AAr?$AAS?$AAt?$AAa?$AAt?$AAu?$AAs?$AA?5?$AA?$CI?$AAB?$AAy?$AAt?$AAe?$AAs?$AAT?$AAr?$AAa?$AAn?$AAs?$AAf?$AAe?$AAr@ 1000e360     usbclient.obj
 0001:0000d3d0       ??_C@_1EI@EFFJOCFO@?$AA?$CK?$AA?$CK?$AA?$CK?$AA?5?$AAG?$AAe?$AAt?$AAT?$AAr?$AAa?$AAn?$AAs?$AAf?$AAe?$AAr?$AAS?$AAt?$AAa?$AAt?$AAu?$AAs?$AA?5?$AAE?$AAR?$AAR?$AAO?$AAR?$AA?3?$AA?$CF?$AAd?$AA?5?$AA?$CK@ 1000e3d0     usbclient.obj
 0001:0000d418       ??_C@_15BNKBCKPG@?$AAI?$AAN?$AA?$AA@ 1000e418     usbclient.obj
 0001:0000d420       ??_C@_17HCEMPBGG@?$AAO?$AAU?$AAT?$AA?$AA@ 1000e420     usbclient.obj
 0001:0000d428       ??_C@_1DI@EENFKOKJ@?$AA?$CF?$AAs?$AA?3?$AAW?$AAA?$AAI?$AAT?$AA_?$AAT?$AAI?$AAM?$AAE?$AAO?$AAU?$AAT?$AA?5?$AAo?$AAn?$AA?5?$AAh?$AAT?$AA?3?$AA0?$AAx?$AA?$CF?$AAx?$AA?6?$AA?$AA@ 1000e428     usbclient.obj
 0001:0000d460       ??_C@_1FA@COJHPOOL@?$AA?$CK?$AA?$CK?$AA?$CK?$AA?5?$AAI?$AAs?$AAs?$AAu?$AAe?$AAB?$AAu?$AAl?$AAk?$AAT?$AAr?$AAa?$AAn?$AAs?$AAf?$AAe?$AAr?$AA?5?$AAE?$AAR?$AAR?$AAO?$AAR?$AA?$CI?$AA3?$AA?0?$AA?5?$AA?$CF@ 1000e460     usbclient.obj
 0001:0000d4b0       ??_C@_1JK@HKJHGPDC@?$AAI?$AAs?$AAs?$AAu?$AAe?$AAB?$AAu?$AAl?$AAk?$AAT?$AAr?$AAa?$AAn?$AAs?$AAf?$AAe?$AAr?$AA?5?$AAE?$AAR?$AAR?$AAO?$AAR?$AA?$CI?$AA5?$AA?0?$AA?5?$AAB?$AAy?$AAt?$AAe?$AAs@ 1000e4b0     usbclient.obj
 0001:0000d550       ??_C@_1FK@KGMBLFKM@?$AA?$CK?$AA?$CK?$AA?$CK?$AA?5?$AAI?$AAs?$AAs?$AAu?$AAe?$AAI?$AAn?$AAt?$AAe?$AAr?$AAr?$AAu?$AAp?$AAt?$AAT?$AAr?$AAa?$AAn?$AAs?$AAf?$AAe?$AAr?$AA?5?$AAE?$AAR?$AAR?$AAO?$AAR@ 1000e550     usbclient.obj
 0001:0000d5b0       ??_C@_1KE@HEHDFMIE@?$AAI?$AAs?$AAs?$AAu?$AAe?$AAI?$AAn?$AAt?$AAe?$AAr?$AAr?$AAu?$AAp?$AAt?$AAT?$AAr?$AAa?$AAn?$AAs?$AAf?$AAe?$AAr?$AA?5?$AAE?$AAR?$AAR?$AAO?$AAR?$AA?$CI?$AA5?$AA?0?$AA?5@ 1000e5b0     usbclient.obj
 0001:0000d654       ??_C@_1CA@LPNFMIEO@?$AAC?$AAL?$AAI?$AAI?$AAV?$AAT?$AA?5?$AA?$CF?$AAx?$AA?0?$AA?5?$AA?$CF?$AAx?$AA?$AN?$AA?6?$AA?$AA@ 1000e654     usbclient.obj
 0001:0000d678       ??_C@_1FI@ILPCPOCG@?$AA?$CK?$AA?$CK?$AA?$CK?$AA?5?$AAI?$AAs?$AAs?$AAu?$AAe?$AAV?$AAe?$AAn?$AAd?$AAo?$AAr?$AAT?$AAr?$AAa?$AAn?$AAs?$AAf?$AAe?$AAr?$AA?5?$AAE?$AAR?$AAR?$AAO?$AAR?$AA?$CI?$AA3?$AA?0@ 1000e678     usbclient.obj
 0001:0000d6d0       ??_C@_1JO@FNJJOIFN@?$AAI?$AAs?$AAs?$AAu?$AAe?$AAV?$AAe?$AAn?$AAd?$AAo?$AAr?$AAT?$AAr?$AAa?$AAn?$AAs?$AAf?$AAe?$AAr?$AA?5?$AAE?$AAR?$AAR?$AAO?$AAR?$AA?$CI?$AA5?$AA?0?$AA?5?$AAB?$AAy?$AAt@ 1000e6d0     usbclient.obj
 0001:0000d770       ??_C@_1EE@FGLFADDK@?$AA?$CK?$AA?$CK?$AA?$CK?$AA?5?$AAR?$AAe?$AAs?$AAe?$AAt?$AAD?$AAe?$AAf?$AAa?$AAu?$AAl?$AAt?$AAP?$AAi?$AAp?$AAe?$AA?5?$AAf?$AAa?$AAi?$AAl?$AAu?$AAr?$AAe?$AA?5?$AA?$CK?$AA?$CK?$AA?$CK@ 1000e770     usbclient.obj
 0001:0000d7b8       ??_C@_1EM@GADAJNPB@?$AA?$CK?$AA?$CK?$AA?$CK?$AA?5?$AAI?$AAs?$AAD?$AAe?$AAf?$AAa?$AAu?$AAl?$AAt?$AAP?$AAi?$AAp?$AAe?$AAH?$AAa?$AAl?$AAt?$AAe?$AAd?$AA?5?$AAE?$AAR?$AAR?$AAO?$AAR?$AA?3?$AA?$CF?$AAd@ 1000e7b8     usbclient.obj
 0001:0000d804       ??_C@_1DI@CNDBPNKB@?$AAE?$AAn?$AAd?$AAp?$AAo?$AAi?$AAn?$AAt?$AA?3?$AA0?$AAx?$AA?$CF?$AAx?$AA?5?$AAw?$AAS?$AAt?$AAa?$AAt?$AAu?$AAs?$AA?3?$AA0?$AAx?$AA?$CF?$AAx?$AA?6?$AA?$AA@ 1000e804     usbclient.obj
 0001:0000d83c       ??_C@_1DI@MOPNAAFE@?$AA?$CK?$AA?$CK?$AA?$CK?$AA?5?$AAR?$AAe?$AAs?$AAe?$AAt?$AAP?$AAi?$AAp?$AAe?$AA?5?$AAE?$AAR?$AAR?$AAO?$AAR?$AA?3?$AA?$CF?$AAd?$AA?5?$AA?$CK?$AA?$CK?$AA?$CK?$AA?6?$AA?$AA@ 1000e83c     usbclient.obj
 0001:0000d874       ??_C@_03HMFOOINA@r?$CLb?$AA@ 1000e874     MultiPlatformFile.obj
 0001:0000d910       ??_C@_07FCMOEAAJ@VID_?$CFlX?$AA@ 1000e910     INFParse.obj
 0001:0000d918       ??_C@_07JEKBEJIO@PID_?$CFlX?$AA@ 1000e918     INFParse.obj
 0001:0000d920       ??_C@_01OHGJGJJP@?$FL?$AA@ 1000e920     INFParse.obj
 0001:0000d924       ??_C@_02GENKJLAO@?$FN?$AA?$AA@ 1000e924     INFParse.obj
 0001:0000d928       ??_C@_03JALODAI@?$CFld?$AA@ 1000e928     INFParse.obj
 0001:0000d92c       ??_C@_02EMFKHFLK@?$CFX?$AA@ 1000e92c     INFParse.obj
 0001:0000d930       ??_C@_03HEFJANMG@HKR?$AA@  1000e930     INFParse.obj
 0001:0000d934       ??_C@_01IHBHIGKO@?0?$AA@   1000e934     INFParse.obj
 0001:0000d938       ??_C@_03HKPIJKPH@?$CFlX?$AA@ 1000e938     INFParse.obj
 0001:0000d93c       ??_C@_0P@EOLGHOHJ@?$FLManufacturer?$FN?$AA@ 1000e93c     INFParse.obj
 0001:0000d94c       ??_C@_05GCELKHFA@?$FL?$CFs?$CFs?$AA@ 1000e94c     INFParse.obj
 0001:0000d958       ??_C@_1EM@LDNEMOFO@?$AAD?$AAr?$AAi?$AAv?$AAe?$AAr?$AAs?$AA?2?$AAU?$AAS?$AAB?$AA?2?$AAC?$AAl?$AAi?$AAe?$AAn?$AAt?$AAD?$AAr?$AAi?$AAv?$AAe?$AAr?$AAs?$AA?2?$AAF?$AAT?$AAD?$AAI?$AA_?$AAD@ 1000e958     INFParse.obj
 0001:0000d9a4       ??_C@_17KKLPNNMB@?$AAC?$AAO?$AAM?$AA?$AA@ 1000e9a4     INFParse.obj
 0001:0000dc60       ??_C@_1HE@BFNMFKA@?$AAc?$AA?3?$AA?2?$AAw?$AAi?$AAn?$AAc?$AAe?$AA8?$AA0?$AA0?$AA?2?$AAo?$AAs?$AAd?$AAe?$AAs?$AAi?$AAg?$AAn?$AAs?$AA?2?$AAv?$AAc?$AAp?$AAo?$AAs?$AAc?$AAe?$AAp?$AAc?$AA?2@ 1000ec60     EMUL.obj
 0001:0000dcd4       ??_C@_02CJNFGIML@aw?$AA@   1000ecd4     ftdi_debug.obj
 0001:0000dcd8       ??_C@_08KKALHPOF@dbug?4txt?$AA@ 1000ecd8     ftdi_debug.obj
 0001:0000dce8       __load_config_used         1000ece8     ccrt0:loadcfg.obj
 0001:0000dd70       ___safe_se_handler_table   1000ed70     <linker-defined>
 0001:0000dd78       _WaitCommEvent             1000ed78 f   mdd.obj
 0001:0000e044       _EvaluateEventFlag         1000f044 f   mdd.obj
 0001:0000e1b2       _COM_Close                 1000f1b2 f   mdd.obj
 0001:0000e802       _COM_Deinit                1000f802 f   mdd.obj
 0001:0000ea63       _DllEntry                  1000fa63 f   mdd.obj
 0001:0000eb1b       _DoTxData                  1000fb1b f   mdd.obj
 0001:0000ef3e       _SerialEventHandler        1000ff3e f   mdd.obj
 0001:0000f732       _StartDispatchThread       10010732 f   mdd.obj
 0001:0000f847       _StopDispatchThread        10010847 f   mdd.obj
 0001:0000f975       _ApplyDCB                  10010975 f   mdd.obj
 0001:0000fbf1       _COM_Init                  10010bf1 f   mdd.obj
 0001:0001023f       _COM_Open                  1001123f f   mdd.obj
 0001:00010d70       _ProcessExiting            10011d70 f   mdd.obj
 0001:00011060       _COM_Read                  10012060 f   mdd.obj
 0001:000117b3       _COM_Write                 100127b3 f   mdd.obj
 0001:00011eda       _COM_Seek                  10012eda f   mdd.obj
 0001:00011ede       _COM_PowerUp               10012ede f   mdd.obj
 0001:00011f8e       _COM_PowerDown             10012f8e f   mdd.obj
 0001:00011fe7       _SerialGetDroppedByteNumber 10012fe7 f   mdd.obj
 0001:00011ffd       _COM_IOControl             10012ffd f   mdd.obj
 0001:000130da       _CheckListEntry            100140da f i mdd.obj
 0001:0001319e       _GetCurrentThread          1001419e f i mdd.obj
 0001:000131a2       _InitializeListHead        100141a2 f i mdd.obj
 0001:000131af       _InsertEntryList           100141af f i mdd.obj
 0001:00013576       _InsertHeadList            10014576 f i mdd.obj
 0001:0001393a       _PulseEvent                1001493a f i mdd.obj
 0001:0001394b       _RemoveEntryList           1001494b f i mdd.obj
 0001:00013aaa       _ResetEvent                10014aaa f i mdd.obj
 0001:00013abb       _RxBytesAvail              10014abb f i mdd.obj
 0001:00013ae3       _SetEvent                  10014ae3 f i mdd.obj
 0001:00013af4       _GetSerialObject           10014af4 f   ftdi_ser.obj
 0001:000141e1       _SerClearDTR               100151e1 f   ftdi_ser.obj
 0001:000142a8       _SerSetDTR                 100152a8 f   ftdi_ser.obj
 0001:0001436f       _SerClearRTS               1001536f f   ftdi_ser.obj
 0001:00014436       _SerSetRTS                 10015436 f   ftdi_ser.obj
 0001:000144fd       _SerClearBreak             100154fd f   ftdi_ser.obj
 0001:000145c9       _SerSetBreak               100155c9 f   ftdi_ser.obj
 0001:00014698       _SerSetDCB                 10015698 f   ftdi_ser.obj
 0001:000147ff       _SerSetCommTimeouts        100157ff f   ftdi_ser.obj
 0001:000148b0       _SerGetRxBufferSize        100158b0 f   ftdi_ser.obj
 0001:000148b3       _SerGetInterruptType       100158b3 f   ftdi_ser.obj
 0001:000149ea       _SerRxIntr                 100159ea f   ftdi_ser.obj
 0001:00014f0f       _SerTxIntr                 10015f0f f   ftdi_ser.obj
 0001:0001537a       _SerLineIntr               1001637a f   ftdi_ser.obj
 0001:000153e3       _SerModemIntr              100163e3 f   ftdi_ser.obj
 0001:0001551a       _SerGetStatus              1001651a f   ftdi_ser.obj
 0001:00015604       _SerReset                  10016604 f   ftdi_ser.obj
 0001:000156cc       _SerGetModemStatus         100166cc f   ftdi_ser.obj
 0001:00015782       _SerPurgeComm              10016782 f   ftdi_ser.obj
 0001:0001591a       _SerXmitComChar            1001691a f   ftdi_ser.obj
 0001:00015b52       _SerIoctl                  10016b52 f   ftdi_ser.obj
 0001:00016133       _CleanupOpenDevice         10017133 f   ftdi_ser.obj
 0001:000164bd       _ConfigureActiveSyncMonitor 100174bd f   ftdi_ser.obj
 0001:0001666f       _TerminateActiveSyncMonitor 1001766f f   ftdi_ser.obj
 0001:00016701       _FTDIWriteTransferComplete 10017701 f   ftdi_ser.obj
 0001:0001682f       _SetDeviceUnloading        1001782f f   ftdi_ser.obj
 0001:00016860       _SetDeviceLoading          10017860 f   ftdi_ser.obj
 0001:00016a1b       _StartEventThread          10017a1b f   ftdi_ser.obj
 0001:00016b9a       _ActiveSyncMonitor         10017b9a f   ftdi_ser.obj
 0001:00016c8d       _Ser_GetRegistryData       10017c8d f   ftdi_ser.obj
 0001:00016ecc       _myNOP                     10017ecc f   ftdi_ser.obj
 0001:00016ecd       _RegQueryDWORD             10017ecd f   ftdi_ser.obj
 0001:00016ef9       _InitialiseOpenDevice      10017ef9 f   ftdi_ser.obj
 0001:00017921       _RegRemoveDeviceContext    10018921 f   ftdi_ser.obj
 0001:00017a5b       _SerGetRxStart             10018a5b f   ftdi_ser.obj
 0001:00017a5e       _OutRequest                10018a5e f   ftdi_ser.obj
 0001:00017c67       _CheckValidDCB             10018c67 f   ftdi_ser.obj
 0001:00017c6b       _SetFlowParams             10018c6b f   ftdi_ser.obj
 0001:00017cba       _ErrorInvalidArgs          10018cba f   ftdi_ser.obj
 0001:00017cd7       _ErrorSuccess              10018cd7 f   ftdi_ser.obj
 0001:00017cf1       _ErrorFail                 10018cf1 f   ftdi_ser.obj
 0001:00017d10       _FT_VendorRequest          10018d10 f   ftdi_utils.obj
 0001:00017e76       _FT_SetBaudRate            10018e76 f   ftdi_utils.obj
 0001:0001817d       _FT_SetDivisor             1001917d f   ftdi_utils.obj
 0001:000181a1       _FT_SetLineControl         100191a1 f   ftdi_utils.obj
 0001:00018204       _FT_SetFlowControl         10019204 f   ftdi_utils.obj
 0001:0001829e       _FT_SetDtr                 1001929e f   ftdi_utils.obj
 0001:00018358       _FT_ClrDtr                 10019358 f   ftdi_utils.obj
 0001:00018412       _FT_SetRts                 10019412 f   ftdi_utils.obj
 0001:000184cc       _FT_ClrRts                 100194cc f   ftdi_utils.obj
 0001:00018583       _FT_SetChars               10019583 f   ftdi_utils.obj
 0001:000185fe       _FT_GetModemStatus         100195fe f   ftdi_utils.obj
 0001:000186e0       _FT_PurgeInternalBuffer    100196e0 f   ftdi_utils.obj
 0001:00018723       _FT_Purge                  10019723 f   ftdi_utils.obj
 0001:0001879c       _FT_SetBreak               1001979c f   ftdi_utils.obj
 0001:000187cc       _FT_SetLatencyTimer        100197cc f   ftdi_utils.obj
 0001:0001886f       _FT_GetLatencyTimer        1001986f f   ftdi_utils.obj
 0001:00018911       _FT_SetBitMode             10019911 f   ftdi_utils.obj
 0001:000189c6       _FT_GetBitMode             100199c6 f   ftdi_utils.obj
 0001:00018a68       _FT_GetDeviceSerialNumber  10019a68 f   ftdi_utils.obj
 0001:00018a8f       _FT_GetDeviceDescription   10019a8f f   ftdi_utils.obj
 0001:00018ab6       _StringToWchar             10019ab6 f   ftdi_utils.obj
 0001:00018ae2       _FT_SetState               10019ae2 f   ftdi_utils.obj
 0001:00018ae5       _FT_ResetHardware          10019ae5 f   ftdi_utils.obj
 0001:00018c68       _FT_SetDeviceEvent         10019c68 f   ftdi_utils.obj
 0001:00018cf4       _IoErrorHandler            10019cf4 f   ftdi_utils.obj
 0001:00018f57       _FT_RestoreDeviceSettings  10019f57 f   ftdi_utils.obj
 0001:00018fc6       _LResetPipe                10019fc6 f   ftdi_utils.obj
 0001:000190b1       _SoftReset                 1001a0b1 f   ftdi_utils.obj
 0001:0001925d       _FT_ResetPipe              1001a25d f   ftdi_utils.obj
 0001:000192b5       _FT_PurgeRead              1001a2b5 f   ftdi_utils.obj
 0001:000192b6       _FT_ResetDevice            1001a2b6 f   ftdi_utils.obj
 0001:000192b9       _FT_GetStringDescriptor    1001a2b9 f   ftdi_utils.obj
 0001:0001953b       _FT_GetDescriptor          1001a53b f   ftdi_utils.obj
 0001:000195a1       _USBDeviceAttach           1001a5a1 f   ftdi_usb.obj
 0001:0001a218       _USBInstallDriver          1001b218 f   ftdi_usb.obj
 0001:0001a56d       _USBUnInstallDriver        1001b56d f   ftdi_usb.obj
 0001:0001a5c1       _DeviceNotify              1001b5c1 f   ftdi_usb.obj
 0001:0001ab3e       _GetMaxIndex               1001bb3e f   ftdi_usb.obj
 0001:0001abcc       _GetNameIndex              1001bbcc f   ftdi_usb.obj
 0001:0001ac88       _GetRegistryInitialIndex   1001bc88 f   ftdi_usb.obj
 0001:0001b0da       _GetNextAvailableIndex     1001c0da f   ftdi_usb.obj
 0001:0001b4e7       _RemoveDeviceStructure     1001c4e7 f   ftdi_usb.obj
 0001:0001b8d1       _DelayedDeviceDeactivate   1001c8d1 f   ftdi_usb.obj
 0001:0001b9e4       _CreateBulkPipeEvents      1001c9e4 f   ftdi_usb.obj
 0001:0001bb38       _ConfigureBulkTransfers    1001cb38 f   ftdi_usb.obj
 0001:0001bcb0       _CreateUniqueDriverSettings 1001ccb0 f   ftdi_usb.obj
 0001:0001c131       _SetIndexKeyValue          1001d131 f   ftdi_usb.obj
 0001:0001c234       _SetUsbInterface           1001d234 f   ftdi_usb.obj
 0001:0001c95c       _RestoreUSBHandles         1001d95c f   ftdi_usb.obj
 0001:0001c997       _InitialiseDeviceStructure 1001d997 f   ftdi_usb.obj
 0001:0001cc34       _RestoreDeviceInstance     1001dc34 f   ftdi_usb.obj
 0001:0001cda5       _UpdateDriverVersion       1001dda5 f   ftdi_usb.obj
 0001:0001ce07       _lstrlenW                  1001de07 f i ftdi_usb.obj
 0001:0001ce2f       _FT_LocalAlloc             1001de2f f   BUSBDBG.obj
 0001:0001ce92       _FT_LocalFree              1001de92 f   BUSBDBG.obj
 0001:0001cef5       _FT_StrCpy                 1001def5 f   STRING.obj
 0001:0001cf10       _FT_StrLen                 1001df10 f   STRING.obj
 0001:0001cf25       _FT_CopyWStrToStr          1001df25 f   STRING.obj
 0001:0001cf63       _FT_CalcDivisor            1001df63 f   BAUD.obj
 0001:0001d04e       _FT_CalcDivisorHi          1001e04e f   BAUD.obj
 0001:0001d15e       _FT_CalcBaudRate           1001e15e f   BAUD.obj
 0001:0001d1e7       _FT_CalcBaudRateHi         1001e1e7 f   BAUD.obj
 0001:0001d279       _FT_GetDivisor             1001e279 f   BAUD.obj
 0001:0001d36d       _FT_GetDivisorHi           1001e36d f   BAUD.obj
 0001:0001d45a       _FT_ProcessBulkInEx        1001e45a f   BULK_IN.obj
 0001:0001d4d8       _FT_ProcessRead            1001e4d8 f   BULK_IN.obj
 0001:0001d852       _BulkInTask                1001e852 f   BULK_IN.obj
 0001:0001e49a       _FTDIReadTransferComplete  1001f49a f   BULK_IN.obj
 0001:0001e595       _FT_ProcessBulkIn          1001f595 f   BULK_IN.obj
 0001:0001e787       _InRequest                 1001f787 f   BULK_IN.obj
 0001:0001e97f       _FT_GetBytesPerTransfer    1001f97f f   BULK_IN.obj
 0001:0001e99c       _CheckObjectReturnCode     1001f99c f   BULK_IN.obj
 0001:0001e9a9       _FT_CompleteReadIrp        1001f9a9 f   IRPQUEUE.obj
 0001:0001e9c0       _DllMain                   1001f9c0 f   usbddrv.obj
 0001:0001e9fb       _GetUSBDVersion            1001f9fb f   usbddrv.obj
 0001:0001ea0d       _RegisterClientDriverID    1001fa0d f   usbddrv.obj
 0001:0001ea9a       _UnRegisterClientDriverID  1001fa9a f   usbddrv.obj
 0001:0001eb06       _RegisterClientSettings    1001fb06 f   usbddrv.obj
 0001:0001ed33       _UnRegisterClientSettings  1001fd33 f   usbddrv.obj
 0001:0001eff0       _OpenClientRegistryKey     1001fff0 f   usbddrv.obj
 0001:0001f069       _GetClientRegistryPath     10020069 f   usbddrv.obj
 0001:0001f0fa       _HcdAttach                 100200fa f   usbddrv.obj
 0001:0001f17b       _HcdDetach                 1002017b f   usbddrv.obj
 0001:0001f1ba       _HcdDeviceAttached         100201ba f   usbddrv.obj
 0001:0001f487       _HcdDeviceDetached         10020487 f   usbddrv.obj
 0001:0001f5f1       _RegisterNotificationRoutine 100205f1 f   usbddrv.obj
 0001:0001f6b0       _UnRegisterNotificationRoutine 100206b0 f   usbddrv.obj
 0001:0001f75d       _LoadGenericInterfaceDriver 1002075d f   usbddrv.obj
 0001:0001f7ae       _TranslateStringDescr      100207ae f   usbddrv.obj
 0001:0001f7f1       _FindInterface             100207f1 f   usbddrv.obj
 0001:0001f877       _GetFrameNumber            10020877 f   usbddrv.obj
 0001:0001f8ce       _GetFrameLength            100208ce f   usbddrv.obj
 0001:0001f925       _TakeFrameLengthControl    10020925 f   usbddrv.obj
 0001:0001f9ad       _SetFrameLength            100209ad f   usbddrv.obj
 0001:0001fa2e       _ReleaseFrameLengthControl 10020a2e f   usbddrv.obj
 0001:0001faab       _GetDeviceInfo             10020aab f   usbddrv.obj
 0001:0001faf8       _IssueVendorTransfer       10020af8 f   usbddrv.obj
 0001:0001fddd       _GetInterface              10020ddd f   usbddrv.obj
 0001:0001fe34       _SetInterface              10020e34 f   usbddrv.obj
 0001:0001fe8e       _GetDescriptor             10020e8e f   usbddrv.obj
 0001:0001fef8       _SetDescriptor             10020ef8 f   usbddrv.obj
 0001:0001ff62       _SetFeature                10020f62 f   usbddrv.obj
 0001:0001ffdf       _ClearFeature              10020fdf f   usbddrv.obj
 0001:0002005c       _GetStatus                 1002105c f   usbddrv.obj
 0001:000200dd       _SyncFrame                 100210dd f   usbddrv.obj
 0001:0002013a       _OpenPipe                  1002113a f   usbddrv.obj
 0001:000202af       _AbortPipeTransfers        100212af f   usbddrv.obj
 0001:0002036b       _ResetPipe                 1002136b f   usbddrv.obj
 0001:000203e2       _ResetDefaultPipe          100213e2 f   usbddrv.obj
 0001:0002042f       _ClosePipe                 1002142f f   usbddrv.obj
 0001:0002059b       _IsPipeHalted              1002159b f   usbddrv.obj
 0001:0002062e       _IsDefaultPipeHalted       1002162e f   usbddrv.obj
 0001:0002067e       _IssueControlTransfer      1002167e f   usbddrv.obj
 0001:000208da       _IssueBulkTransfer         100218da f   usbddrv.obj
 0001:00020ad5       _IssueInterruptTransfer    10021ad5 f   usbddrv.obj
 0001:00020cd0       _IssueIsochTransfer        10021cd0 f   usbddrv.obj
 0001:00020fa9       _IsTransferComplete        10021fa9 f   usbddrv.obj
 0001:00021000       _GetTransferStatus         10022000 f   usbddrv.obj
 0001:0002109a       _GetIsochResults           1002209a f   usbddrv.obj
 0001:00021178       _AbortTransfer             10022178 f   usbddrv.obj
 0001:00021322       _CloseTransfer             10022322 f   usbddrv.obj
 0001:00021401       _DisableDevice             10022401 f   usbddrv.obj
 0001:0002153c       _SuspendDevice             1002253c f   usbddrv.obj
 0001:00021642       _ResumeDevice              10022642 f   usbddrv.obj
 0001:000217de       _HcdSelectConfiguration    100227de f   usbddrv.obj
 0001:00021a39       ?SignalEventFunc@@YAKPAX@Z 10022a39 f   usbddrv.obj
 0001:00021a4e       _GetTransferError          10022a4e f   usbddrv.obj
 0001:00021abc       ?SetDeviceBit@@YAHPAUSDevice@@EHE@Z 10022abc f   usbddrv.obj
 0001:00021b06       ?IsAllBitSet@@YAHPAUSDevice@@E@Z 10022b06 f   usbddrv.obj
 0001:00021b44       ?IsOneBitSet@@YAHPAUSDevice@@E@Z 10022b44 f   usbddrv.obj
 0001:00021b82       ?CallKGetDriverName@@YAHPAUHWND__@@PAU_GETDRIVERNAMEPARMS@@@Z 10022b82 f i usbddrv.obj
 0001:00021c4d       ?CallKGetNetString@@YAHIPAGH@Z 10022c4d f i usbddrv.obj
 0001:00021d24       ?CallKGetNetStringSize@@YAHI@Z 10022d24 f i usbddrv.obj
 0001:00021d6e       ?CallKVNetMsgBox@@YAHPAUHWND__@@KIPAD@Z 10022d6e f i usbddrv.obj
 0001:00021f21       ?CeCallUserProcWrapper@@YAHPBG0PAXK1KPAK@Z 10022f21 f i usbddrv.obj
 0001:00021f83       ?WaitForAPIReadyWrapper@@YAKKK@Z 10022f83 f i usbddrv.obj
 0001:00021fd7       ?safeIntUAdd@@YAHIIPAI@Z   10022fd7 f i usbddrv.obj
 0001:00021fed       ?safeIntUMul@@YAHIIPAI@Z   10022fed f i usbddrv.obj
 0001:0002200e       _CallGetDriverName         1002300e f i usbddrv.obj
 0001:00022033       _CallNetMsgBox             10023033 f i usbddrv.obj
 0001:00022077       _CallUGetDriverName        10023077 f i usbddrv.obj
 0001:000220b6       _CallUGetNetString         100230b6 f i usbddrv.obj
 0001:000220f9       _CallUNetMsgBox            100230f9 f i usbddrv.obj
 0001:00022203       _CheckAndWaitForGWE        10023203 f i usbddrv.obj
 0001:00022217       _GetNetuiFunction          10023217 f i usbddrv.obj
 0001:000222a3       _IsCeCallUserProcAvailable 100232a3 f i usbddrv.obj
 0001:000222d8       ?AddTransfer@@YAHPAUSPipe@@PAUSTransfer@@@Z 100232d8 f   usbd.obj
 0001:000223b2       ?LoadUSBClient@@YAHPAUSDevice@@PAHPBU_USB_INTERFACE@@@Z 100233b2 f   usbd.obj
 0001:00022441       ?InstallClientDriver@@YAHPBG@Z 10023441 f   usbd.obj
 0001:00022552       ?LoadDeviceDrivers@@YAHPAUSDevice@@PAH@Z 10023552 f   usbd.obj
 0001:000226af       ?CloseUSBDevice@@YAHPAUSDevice@@@Z 100236af f   usbd.obj
 0001:00022726       ?GetSettingString@@YAXPAGKKKK@Z 10023726 f   usbd.obj
 0001:000227c8       ?FindEndpoint@@YAPBU_USB_ENDPOINT@@PBU_USB_INTERFACE@@E@Z 100237c8 f   usbd.obj
 0001:000227f1       ?ReferencePipeHandle@@YAHPAUSPipe@@@Z 100237f1 f   usbd.obj
 0001:0002288d       ?DereferencePipeHandle@@YAXPAUSPipe@@@Z 1002388d f   usbd.obj
 0001:000228c3       ?ValidateDeviceHandle@@YAHPAUSDevice@@@Z 100238c3 f   usbd.obj
 0001:00022958       ?ReferenceTransferHandle@@YAHPAUSTransfer@@@Z 10023958 f   usbd.obj
 0001:000229db       ?DereferenceTransferHandle@@YAXPAUSTransfer@@@Z 100239db f   usbd.obj
 0001:00022a11       ?GetPipeObject@@YAPAUSPipe@@PAUSDevice@@@Z 10023a11 f   usbd.obj
 0001:00022a9d       ?FreePipeObject@@YAXPAUSPipe@@@Z 10023a9d f   usbd.obj
 0001:00022b51       ?FreePipeObjectMem@@YAXPAUSPipe@@@Z 10023b51 f   usbd.obj
 0001:00022b6c       ?GetTransferObject@@YAPAUSTransfer@@PAUSPipe@@K@Z 10023b6c f   usbd.obj
 0001:00022c74       ?FreeTransferObject@@YAXPAUSTransfer@@@Z 10023c74 f   usbd.obj
 0001:00022de5       ?FreeTransferObjectMem@@YAXPAUSTransfer@@@Z 10023de5 f   usbd.obj
 0001:00022e1e       ?GetWaitObject@@YAPAUSWait@@XZ 10023e1e f   usbd.obj
 0001:00022e53       ?FreeWaitObject@@YAHPAUSWait@@@Z 10023e53 f   usbd.obj
 0001:00022e79       ?ConvertToClientRegistry@@YAHPAGKPBU_USB_DEVICE@@PBU_USB_INTERFACE@@HHHPAU_USB_DRIVER_SETTINGS@@@Z 10023e79 f   usbd.obj
 0001:000231b2       ?GetSettingString@@YAXPAGKKK@Z 100241b2 f   usbd.obj
 0001:00023239       ?AddDriverLib@@YAHPAUSDevice@@PAUHINSTANCE__@@@Z 10024239 f   usbd.obj
 0001:0002328b       ?LoadRegisteredDriver@@YAHPAUHKEY__@@PAUSDevice@@PBU_USB_INTERFACE@@PAHPBU_USB_DRIVER_SETTINGS@@@Z 1002428b f   usbd.obj
 0001:000234dc       ?LoadGroupDriver@@YAHPAUSDevice@@PAHPBU_USB_INTERFACE@@HHH@Z 100244dc f   usbd.obj
 0001:000235bd       ?LoadDeviceDrivers@@YAHPAUSDevice@@PAHPAE@Z 100245bd f   usbd.obj
 0001:000236b1       _CLIAbortTransfer          100246b1 f   usbclient.obj
 0001:000236f3       _CLICloseTransferHandle    100246f3 f   usbclient.obj
 0001:00023731       _CLIClearOrSetFeature      10024731 f   usbclient.obj
 0001:00023856       _CLIDefaultTransferComplete 10024856 f   usbclient.obj
 0001:000238b6       _CLIGetStatus              100248b6 f   usbclient.obj
 0001:000239e6       _CLIGetTransferStatus      100249e6 f   usbclient.obj
 0001:00023a66       _CLIIssueBulkTransfer      10024a66 f   usbclient.obj
 0001:00023c05       _CLIIssueInterruptTransfer 10024c05 f   usbclient.obj
 0001:00023da1       _CLIIssueVendorTransfer    10024da1 f   usbclient.obj
 0001:00023f63       _CLIResetDefaultEndpoint   10024f63 f   usbclient.obj
 0001:00023fe4       _CLIResetBulkEndpoint      10024fe4 f   usbclient.obj
 0001:0002407b       _CLIResetPipe              1002507b f   usbclient.obj
 0001:000240cf       __ResetEvent               100250cf f i usbclient.obj
 0001:0002410e       ?Open@MultiPlatformFile@@QAEHPADK@Z 1002510e f   MultiPlatformFile.obj
 0001:00024134       ?IsOpen@MultiPlatformFile@@QAEHXZ 10025134 f   MultiPlatformFile.obj
 0001:0002413c       ?Close@MultiPlatformFile@@QAEHXZ 1002513c f   MultiPlatformFile.obj
 0001:0002414c       ?Read@MultiPlatformFile@@QAEHPAXII@Z 1002514c f   MultiPlatformFile.obj
 0001:00024186       ?Write@MultiPlatformFile@@QAEHPAXII@Z 10025186 f   MultiPlatformFile.obj
 0001:000241a0       ?Access@MultiPlatformFile@@QAEHPADK@Z 100251a0 f   MultiPlatformFile.obj
 0001:000241fd       ?Seek@MultiPlatformFile@@QAEHJH@Z 100251fd f   MultiPlatformFile.obj
 0001:00024218       ?EOFile@MultiPlatformFile@@QAEHXZ 10025218 f   MultiPlatformFile.obj
 0001:00024221       ??0MultiPlatformFile@@QAE@XZ 10025221 f   MultiPlatformFile.obj
 0001:00024227       ??1MultiPlatformFile@@QAE@XZ 10025227 f   MultiPlatformFile.obj
 0001:00024228       ?WcharToString@@YAXPADPAGK@Z 10025228 f   MultiPlatformFile.obj
 0001:00024254       ?StringToWchar@@YAXPAGPADK@Z 10025254 f   MultiPlatformFile.obj
 0001:00024280       ?FindVIDPIDInLine@@YAHPAVMultiPlatformFile@@PAK1@Z 10025280 f   INFParse.obj
 0001:000243f5       ?FindSection@@YAHPAVMultiPlatformFile@@PBD@Z 100253f5 f   INFParse.obj
 0001:0002447b       ?ParseManufacturer@@YAXPAVMultiPlatformFile@@PAK1@Z 1002547b f   INFParse.obj
 0001:000245ab       ?ParseRegSettings@@YAXPAVMultiPlatformFile@@PAG1@Z 100255ab f   INFParse.obj
 0001:00024a11       _GetVIDPID                 10025a11 f   INFParse.obj
 0001:00024a93       _GetNextVIDPID             10025a93 f   INFParse.obj
 0001:00024b6c       _RegisterINFValues         10025b6c f   INFParse.obj
 0001:00024c16       _GetStreamDriverKey        10025c16 f   INFParse.obj
 0001:00024c2d       _GetDevicePrefix           10025c2d f   INFParse.obj
 0001:00024cae       ??_GMultiPlatformFile@@QAEPAXI@Z 10025cae f i INFParse.obj
 0001:00024ccd       _FT_InitEmulMode           10025ccd f   EMUL.obj
 0001:00024d4c       _FT_InitEmulChars          10025d4c f   EMUL.obj
 0001:00024d66       _FT_EmulProcessRxPacket    10025d66 f   EMUL.obj
 0001:00025062       _FT_EmulCopyTxBytes        10026062 f   EMUL.obj
 0001:000250c4       _FT_EmulBuildModemCtrlRequest 100260c4 f   EMUL.obj
 0001:0002510e       _FT_EmulConvertRxChar      1002610e f   EMUL.obj
 0001:00025245       _FT_EmulProcessMSR         10026245 f   EMUL.obj
 0001:0002527d       _FT_EmulProcessLSR         1002627d f   EMUL.obj
 0001:000252a9       _FT_EmulGetNextTxByte      100262a9 f   EMUL.obj
 0001:00025336       _SerialHandleModemUpdate   10026336 f   MODMFLOW.obj
 0001:00025339       _SerialProcessLSR          10026339 f   MODMFLOW.obj
 0001:0002533c       _SerialPutChar             1002633c f   MODMFLOW.obj
 0001:00025378       _WcharToString             10026378 f   ftdi_debug.obj
 0001:000253a4       _WriteToDebugFile          100263a4 f   ftdi_debug.obj
 0001:00025446       _GetVersionExW             10026446 f   coredll:COREDLL.dll
 0001:0002544c       _EnterCriticalSection      1002644c f   coredll:COREDLL.dll
 0001:00025452       _LeaveCriticalSection      10026452 f   coredll:COREDLL.dll
 0001:00025458       _InitializeCriticalSection 10026458 f   coredll:COREDLL.dll
 0001:0002545e       _DeleteCriticalSection     1002645e f   coredll:COREDLL.dll
 0001:00025464       _CreateThread              10026464 f   coredll:COREDLL.dll
 0001:0002546a       _ExitThread                1002646a f   coredll:COREDLL.dll
 0001:00025470       _GetLastError              10026470 f   coredll:COREDLL.dll
 0001:00025476       _GetTickCount              10026476 f   coredll:COREDLL.dll
 0001:0002547c       _CloseHandle               1002647c f   coredll:COREDLL.dll
 0001:00025482       _SetThreadPriority         10026482 f   coredll:COREDLL.dll
 0001:00025488       _CeGetThreadPriority       10026488 f   coredll:COREDLL.dll
 0001:0002548e       _CeSetThreadPriority       1002648e f   coredll:COREDLL.dll
 0001:00025494       _SetLastError              10026494 f   coredll:COREDLL.dll
 0001:0002549a       _Sleep                     1002649a f   coredll:COREDLL.dll
 0001:000254a0       _CreateEventW              100264a0 f   coredll:COREDLL.dll
 0001:000254a6       _WaitForSingleObject       100264a6 f   coredll:COREDLL.dll
 0001:000254ac       _IsBadReadPtr              100264ac f   coredll:COREDLL.dll
 0001:000254b2       _IsBadWritePtr             100264b2 f   coredll:COREDLL.dll
 0001:000254b8       _DisableThreadLibraryCalls 100264b8 f   coredll:COREDLL.dll
 0001:000254be       _NKDbgPrintfW              100264be f   coredll:COREDLL.dll
 0001:000254c4       _RegisterDbgZones          100264c4 f   coredll:COREDLL.dll
 0001:000254ca       _CeAllocAsynchronousBuffer 100264ca f   coredll:COREDLL.dll
 0001:000254d0       _CeFreeAsynchronousBuffer  100264d0 f   coredll:COREDLL.dll
 0001:000254d6       _EventModify               100264d6 f   coredll:COREDLL.dll
 0001:000254dc       _RegCloseKey               100264dc f   coredll:COREDLL.dll
 0001:000254e2       _RegQueryValueExW          100264e2 f   coredll:COREDLL.dll
 0001:000254e8       _OpenDeviceKey             100264e8 f   coredll:COREDLL.dll
 0001:000254ee       _TerminateThread           100264ee f   coredll:COREDLL.dll
 0001:000254f4       _GetThreadPriority         100264f4 f   coredll:COREDLL.dll
 0001:000254fa       _CeSetThreadQuantum        100264fa f   coredll:COREDLL.dll
 0001:00025500       _CreateMutexW              10026500 f   coredll:COREDLL.dll
 0001:00025506       _ReleaseMutex              10026506 f   coredll:COREDLL.dll
 0001:0002550c       _IsAPIReady                1002650c f   coredll:COREDLL.dll
 0001:00025512       _RegOpenKeyExW             10026512 f   coredll:COREDLL.dll
 0001:00025518       _RegSetValueExW            10026518 f   coredll:COREDLL.dll
 0001:0002551e       _CeEventHasOccurred        1002651e f   coredll:COREDLL.dll
 0001:00025524       _CeLogData                 10026524 f   coredll:COREDLL.dll
 0001:0002552a       _GetProcAddressW           1002652a f   coredll:COREDLL.dll
 0001:00025530       _wsprintfW                 10026530 f   coredll:COREDLL.dll
 0001:00025536       _LoadLibraryW              10026536 f   coredll:COREDLL.dll
 0001:0002553c       _FreeLibrary               1002653c f   coredll:COREDLL.dll
 0001:00025542       _ActivateDeviceEx          10026542 f   coredll:COREDLL.dll
 0001:00025548       _DeactivateDevice          10026548 f   coredll:COREDLL.dll
 0001:0002554e       _MessageBoxW               1002654e f   coredll:COREDLL.dll
 0001:00025554       _RegCreateKeyExW           10026554 f   coredll:COREDLL.dll
 0001:0002555a       _RegDeleteKeyW             1002655a f   coredll:COREDLL.dll
 0001:00025560       _RegEnumKeyExW             10026560 f   coredll:COREDLL.dll
 0001:00025566       _LocalAlloc                10026566 f   coredll:COREDLL.dll
 0001:0002556c       _LocalFree                 1002656c f   coredll:COREDLL.dll
 0001:00025572       _WaitForMultipleObjects    10026572 f   coredll:COREDLL.dll
 0001:00025578       _FormatMessageW            10026578 f   coredll:COREDLL.dll
 0001:0002557e       _OpenEventW                1002657e f   coredll:COREDLL.dll
 0001:00025584       _WaitForAPIReady           10026584 f   coredll:COREDLL.dll
 0001:0002558a       _StringCchCopyW            1002658a f   coredll:COREDLL.dll
 0001:00025590       _StringCchCatW             10026590 f   coredll:COREDLL.dll
 0001:00025596       _LoadDriver                10026596 f   coredll:COREDLL.dll
 0001:0002559c       _StringCchPrintfW          1002659c f   coredll:COREDLL.dll
 0001:000255a2       _GetFileAttributesW        100265a2 f   coredll:COREDLL.dll
 0001:000255a8       _timeGetTime               100265a8 f   Mmtimer:MMTimer.dll
 0001:000255ae       ___report_rangecheckfailure 100265ae f   ccrt0:x86secgs.obj
 0001:000255ba       @__security_check_cookie@4 100265ba f   ccrt0:x86secgs.obj
 0001:000255e0       ___security_init_cookie    100265e0 f   ccrt0:seccinit.obj
 0001:0002560c       __SEH_prolog4              1002660c f   ccrt0:sehprolg4.obj
 0001:00025651       __SEH_epilog4              10026651 f   ccrt0:sehprolg4.obj
 0001:00025665       __except_handler4          10026665 f   ccrt0:chandler4gs.obj
 0001:00025688       __SEH_prolog4_GS           10026688 f   ccrt0:sehprolg4gs.obj
 0001:000256d0       __SEH_epilog4_GS           100266d0 f   ccrt0:sehprolg4gs.obj
 0001:000256e0       _memmove                   100266e0 f   msvcrt:MSVCRT.dll
 0001:000256e6       _swprintf_s                100266e6 f   msvcrt:MSVCRT.dll
 0001:000256ec       _memcpy                    100266ec f   msvcrt:MSVCRT.dll
 0001:000256f2       _memset                    100266f2 f   msvcrt:MSVCRT.dll
 0001:000256f8       _mbstowcs                  100266f8 f   msvcrt:MSVCRT.dll
 0001:000256fe       __swprintf                 100266fe f   msvcrt:MSVCRT.dll
 0001:00025704       _wcsncmp                   10026704 f   msvcrt:MSVCRT.dll
 0001:0002570a       _wcsncpy                   1002670a f   msvcrt:MSVCRT.dll
 0001:00025710       _swscanf                   10026710 f   msvcrt:MSVCRT.dll
 0001:00025716       ??2@YAPAXI@Z               10026716 f   msvcrt:MSVCRT.dll
 0001:0002571c       ??3@YAXPAX@Z               1002671c f   msvcrt:MSVCRT.dll
 0001:00025722       _fclose                    10026722 f   msvcrt:MSVCRT.dll
 0001:00025728       _feof                      10026728 f   msvcrt:MSVCRT.dll
 0001:0002572e       _ferror                    1002672e f   msvcrt:MSVCRT.dll
 0001:00025734       _fopen                     10026734 f   msvcrt:MSVCRT.dll
 0001:0002573a       _fread                     1002673a f   msvcrt:MSVCRT.dll
 0001:00025740       _fseek                     10026740 f   msvcrt:MSVCRT.dll
 0001:00025746       _fwrite                    10026746 f   msvcrt:MSVCRT.dll
 0001:0002574c       _strncmp                   1002674c f   msvcrt:MSVCRT.dll
 0001:00025752       _sscanf                    10026752 f   msvcrt:MSVCRT.dll
 0001:00025758       _sprintf                   10026758 f   msvcrt:MSVCRT.dll
 0001:0002575e       __chkstk                   1002675e f   msvcrt:MSVCRT.dll
 0001:00025764       ___report_gsfailure        10026764 f   msvcrt:MSVCRT.dll
 0001:0002576a       ___security_gen_cookie2    1002676a f   msvcrt:MSVCRT.dll
 0001:00025770       __except_handler4_common   10026770 f   msvcrt:MSVCRT.dll
 0001:000258e4       __IMPORT_DESCRIPTOR_COREDLL 100268e4     coredll:COREDLL.dll
 0001:000258f8       __IMPORT_DESCRIPTOR_MMTimer 100268f8     Mmtimer:MMTimer.dll
 0001:0002590c       __IMPORT_DESCRIPTOR_MSVCRT 1002690c     msvcrt:MSVCRT.dll
 0001:00025920       __NULL_IMPORT_DESCRIPTOR   10026920     coredll:COREDLL.dll
 0002:00000000       __imp__GetVersionExW       10027000     coredll:COREDLL.dll
 0002:00000004       __imp__EnterCriticalSection 10027004     coredll:COREDLL.dll
 0002:00000008       __imp__LeaveCriticalSection 10027008     coredll:COREDLL.dll
 0002:0000000c       __imp__InitializeCriticalSection 1002700c     coredll:COREDLL.dll
 0002:00000010       __imp__DeleteCriticalSection 10027010     coredll:COREDLL.dll
 0002:00000014       __imp__CreateThread        10027014     coredll:COREDLL.dll
 0002:00000018       __imp__ExitThread          10027018     coredll:COREDLL.dll
 0002:0000001c       __imp__GetLastError        1002701c     coredll:COREDLL.dll
 0002:00000020       __imp__GetTickCount        10027020     coredll:COREDLL.dll
 0002:00000024       __imp__CloseHandle         10027024     coredll:COREDLL.dll
 0002:00000028       __imp__SetThreadPriority   10027028     coredll:COREDLL.dll
 0002:0000002c       __imp__CeGetThreadPriority 1002702c     coredll:COREDLL.dll
 0002:00000030       __imp__CeSetThreadPriority 10027030     coredll:COREDLL.dll
 0002:00000034       __imp__SetLastError        10027034     coredll:COREDLL.dll
 0002:00000038       __imp__Sleep               10027038     coredll:COREDLL.dll
 0002:0000003c       __imp__CreateEventW        1002703c     coredll:COREDLL.dll
 0002:00000040       __imp__WaitForSingleObject 10027040     coredll:COREDLL.dll
 0002:00000044       __imp__IsBadReadPtr        10027044     coredll:COREDLL.dll
 0002:00000048       __imp__IsBadWritePtr       10027048     coredll:COREDLL.dll
 0002:0000004c       __imp__DisableThreadLibraryCalls 1002704c     coredll:COREDLL.dll
 0002:00000050       __imp__NKDbgPrintfW        10027050     coredll:COREDLL.dll
 0002:00000054       __imp__RegisterDbgZones    10027054     coredll:COREDLL.dll
 0002:00000058       __imp__CeAllocAsynchronousBuffer 10027058     coredll:COREDLL.dll
 0002:0000005c       __imp__CeFreeAsynchronousBuffer 1002705c     coredll:COREDLL.dll
 0002:00000060       __imp__EventModify         10027060     coredll:COREDLL.dll
 0002:00000064       __imp__RegCloseKey         10027064     coredll:COREDLL.dll
 0002:00000068       __imp__RegQueryValueExW    10027068     coredll:COREDLL.dll
 0002:0000006c       __imp__OpenDeviceKey       1002706c     coredll:COREDLL.dll
 0002:00000070       __imp__TerminateThread     10027070     coredll:COREDLL.dll
 0002:00000074       __imp__GetThreadPriority   10027074     coredll:COREDLL.dll
 0002:00000078       __imp__CeSetThreadQuantum  10027078     coredll:COREDLL.dll
 0002:0000007c       __imp__CreateMutexW        1002707c     coredll:COREDLL.dll
 0002:00000080       __imp__ReleaseMutex        10027080     coredll:COREDLL.dll
 0002:00000084       __imp__IsAPIReady          10027084     coredll:COREDLL.dll
 0002:00000088       __imp__RegOpenKeyExW       10027088     coredll:COREDLL.dll
 0002:0000008c       __imp__RegSetValueExW      1002708c     coredll:COREDLL.dll
 0002:00000090       __imp__CeEventHasOccurred  10027090     coredll:COREDLL.dll
 0002:00000094       __imp__CeLogData           10027094     coredll:COREDLL.dll
 0002:00000098       __imp__GetProcAddressW     10027098     coredll:COREDLL.dll
 0002:0000009c       __imp__wsprintfW           1002709c     coredll:COREDLL.dll
 0002:000000a0       __imp__LoadLibraryW        100270a0     coredll:COREDLL.dll
 0002:000000a4       __imp__FreeLibrary         100270a4     coredll:COREDLL.dll
 0002:000000a8       __imp__ActivateDeviceEx    100270a8     coredll:COREDLL.dll
 0002:000000ac       __imp__DeactivateDevice    100270ac     coredll:COREDLL.dll
 0002:000000b0       __imp__MessageBoxW         100270b0     coredll:COREDLL.dll
 0002:000000b4       __imp__RegCreateKeyExW     100270b4     coredll:COREDLL.dll
 0002:000000b8       __imp__RegDeleteKeyW       100270b8     coredll:COREDLL.dll
 0002:000000bc       __imp__RegEnumKeyExW       100270bc     coredll:COREDLL.dll
 0002:000000c0       __imp__LocalAlloc          100270c0     coredll:COREDLL.dll
 0002:000000c4       __imp__LocalFree           100270c4     coredll:COREDLL.dll
 0002:000000c8       __imp__WaitForMultipleObjects 100270c8     coredll:COREDLL.dll
 0002:000000cc       __imp__FormatMessageW      100270cc     coredll:COREDLL.dll
 0002:000000d0       __imp__OpenEventW          100270d0     coredll:COREDLL.dll
 0002:000000d4       __imp__WaitForAPIReady     100270d4     coredll:COREDLL.dll
 0002:000000d8       __imp__StringCchCopyW      100270d8     coredll:COREDLL.dll
 0002:000000dc       __imp__StringCchCatW       100270dc     coredll:COREDLL.dll
 0002:000000e0       __imp__LoadDriver          100270e0     coredll:COREDLL.dll
 0002:000000e4       __imp__StringCchPrintfW    100270e4     coredll:COREDLL.dll
 0002:000000e8       __imp__GetFileAttributesW  100270e8     coredll:COREDLL.dll
 0002:000000ec       \177COREDLL_NULL_THUNK_DATA 100270ec     coredll:COREDLL.dll
 0002:000000f0       __imp__timeGetTime         100270f0     Mmtimer:MMTimer.dll
 0002:000000f4       \177MMTimer_NULL_THUNK_DATA 100270f4     Mmtimer:MMTimer.dll
 0002:000000f8       __imp__memmove             100270f8     msvcrt:MSVCRT.dll
 0002:000000fc       __imp__swprintf_s          100270fc     msvcrt:MSVCRT.dll
 0002:00000100       __imp__memcpy              10027100     msvcrt:MSVCRT.dll
 0002:00000104       __imp__memset              10027104     msvcrt:MSVCRT.dll
 0002:00000108       __imp__mbstowcs            10027108     msvcrt:MSVCRT.dll
 0002:0000010c       __imp___swprintf           1002710c     msvcrt:MSVCRT.dll
 0002:00000110       __imp__wcsncmp             10027110     msvcrt:MSVCRT.dll
 0002:00000114       __imp__wcsncpy             10027114     msvcrt:MSVCRT.dll
 0002:00000118       __imp__swscanf             10027118     msvcrt:MSVCRT.dll
 0002:0000011c       __imp_??2@YAPAXI@Z         1002711c     msvcrt:MSVCRT.dll
 0002:00000120       __imp_??3@YAXPAX@Z         10027120     msvcrt:MSVCRT.dll
 0002:00000124       __imp__fclose              10027124     msvcrt:MSVCRT.dll
 0002:00000128       __imp__feof                10027128     msvcrt:MSVCRT.dll
 0002:0000012c       __imp__ferror              1002712c     msvcrt:MSVCRT.dll
 0002:00000130       __imp__fopen               10027130     msvcrt:MSVCRT.dll
 0002:00000134       __imp__fread               10027134     msvcrt:MSVCRT.dll
 0002:00000138       __imp__fseek               10027138     msvcrt:MSVCRT.dll
 0002:0000013c       __imp__fwrite              1002713c     msvcrt:MSVCRT.dll
 0002:00000140       __imp__strncmp             10027140     msvcrt:MSVCRT.dll
 0002:00000144       __imp__sscanf              10027144     msvcrt:MSVCRT.dll
 0002:00000148       __imp__sprintf             10027148     msvcrt:MSVCRT.dll
 0002:0000014c       __imp___chkstk             1002714c     msvcrt:MSVCRT.dll
 0002:00000150       __imp____report_gsfailure  10027150     msvcrt:MSVCRT.dll
 0002:00000154       __imp____security_gen_cookie2 10027154     msvcrt:MSVCRT.dll
 0002:00000158       __imp___except_handler4_common 10027158     msvcrt:MSVCRT.dll
 0002:0000015c       \177MSVCRT_NULL_THUNK_DATA 1002715c     msvcrt:MSVCRT.dll
 0002:00000160       _dpCurSettings             10027160     mdd.obj
 0002:000005d4       _gpDbg                     100275d4     BUSBDBG.obj
 0002:000005e8       ?gcszUsbConfigureEntry@@3PBGB 100275e8     usbddrv.obj
 0002:000005f0       ?gcszUsbRegKey@@3PBGB      100275f0     usbd.obj
 0002:000005f4       ?gcszDriverIDs@@3PBGB      100275f4     usbd.obj
 0002:000005f8       ?gcszLoadClients@@3PBGB    100275f8     usbd.obj
 0002:000005fc       ?gcszDllName@@3PBGB        100275fc     usbd.obj
 0002:00000600       ?gcszDefaultDriver@@3PBGB  10027600     usbd.obj
 0002:00000604       ?gcszUSBDeviceAttach@@3PBGB 10027604     usbd.obj
 0002:00000608       ?gcszUSBInstallDriver@@3PBGB 10027608     usbd.obj
 0002:000006c0       ___security_cookie         100276c0     ccrt0:seccinit.obj
 0002:000006c4       ___security_cookie_complement 100276c4     ccrt0:seccinit.obj
 0002:000006e4       _gbAttached                100276e4     mdd.obj
 0002:000006f4       _gDbgBuf                   100276f4     BUSBDBG.obj
 0002:00000b20       _gszStreamDriverKey        10027b20     <common>
 0002:00000d40       _gtcBufTime                10027d40     <common>
 0002:00001540       _gtcBuf                    10028540     <common>
 0002:00001d40       _osv                       10028d40     <common>
 0002:00001e54       _t                         10028e54     <common>

 entry point at        0001:0000ea63

 Static symbols

 0000:fffd2000       .debug$S                   10000000     coredll:COREDLL.dll
 0000:fffd2000       .debug$S                   10000000     msvcrt:MSVCRT.dll
 0000:fffd2000       .debug$S                   10000000     msvcrt:MSVCRT.dll
 0000:fffd2000       .debug$S                   10000000     msvcrt:MSVCRT.dll
 0000:fffd2000       .debug$S                   10000000     msvcrt:MSVCRT.dll
 0000:fffd2000       .debug$S                   10000000     msvcrt:MSVCRT.dll
 0000:fffd2000       .debug$S                   10000000     msvcrt:MSVCRT.dll
 0000:fffd2000       .debug$S                   10000000     msvcrt:MSVCRT.dll
 0000:fffd2000       .debug$S                   10000000     msvcrt:MSVCRT.dll
 0000:fffd2000       .debug$S                   10000000     msvcrt:MSVCRT.dll
 0000:fffd2000       .debug$S                   10000000     msvcrt:MSVCRT.dll
 0000:fffd2000       .debug$S                   10000000     msvcrt:MSVCRT.dll
 0000:fffd2000       .debug$S                   10000000     msvcrt:MSVCRT.dll
 0000:fffd2000       .debug$S                   10000000     msvcrt:MSVCRT.dll
 0000:fffd2000       .debug$S                   10000000     msvcrt:MSVCRT.dll
 0000:fffd2000       .debug$S                   10000000     msvcrt:MSVCRT.dll
 0000:fffd2000       .debug$S                   10000000     msvcrt:MSVCRT.dll
 0000:fffd2000       .debug$S                   10000000     msvcrt:MSVCRT.dll
 0000:fffd2000       .debug$S                   10000000     msvcrt:MSVCRT.dll
 0000:fffd2000       .debug$S                   10000000     msvcrt:MSVCRT.dll
 0000:fffd2000       .debug$S                   10000000     coredll:COREDLL.dll
 0000:fffd2000       .debug$S                   10000000     coredll:COREDLL.dll
 0000:fffd2000       .debug$S                   10000000     coredll:COREDLL.dll
 0000:fffd2000       .debug$S                   10000000     coredll:COREDLL.dll
 0000:fffd2000       .debug$S                   10000000     coredll:COREDLL.dll
 0000:fffd2000       .debug$S                   10000000     coredll:COREDLL.dll
 0000:fffd2000       .debug$S                   10000000     msvcrt:MSVCRT.dll
 0000:fffd2000       .debug$S                   10000000     msvcrt:MSVCRT.dll
 0000:fffd2000       .debug$S                   10000000     msvcrt:MSVCRT.dll
 0000:fffd2000       .debug$S                   10000000     coredll:COREDLL.dll
 0000:fffd2000       .debug$S                   10000000     coredll:COREDLL.dll
 0000:fffd2000       .debug$S                   10000000     coredll:COREDLL.dll
 0000:fffd2000       .debug$S                   10000000     coredll:COREDLL.dll
 0000:fffd2000       .debug$S                   10000000     coredll:COREDLL.dll
 0000:fffd2000       .debug$S                   10000000     msvcrt:MSVCRT.dll
 0000:fffd2000       .debug$S                   10000000     coredll:COREDLL.dll
 0000:fffd2000       .debug$S                   10000000     coredll:COREDLL.dll
 0000:fffd2000       .debug$S                   10000000     coredll:COREDLL.dll
 0000:fffd2000       .debug$S                   10000000     coredll:COREDLL.dll
 0000:fffd2000       .debug$S                   10000000     coredll:COREDLL.dll
 0000:fffd2000       .debug$S                   10000000     coredll:COREDLL.dll
 0000:fffd2000       .debug$S                   10000000     coredll:COREDLL.dll
 0000:fffd2000       .debug$S                   10000000     coredll:COREDLL.dll
 0000:fffd2000       .debug$S                   10000000     coredll:COREDLL.dll
 0000:fffd2000       .debug$S                   10000000     coredll:COREDLL.dll
 0000:fffd2000       .debug$S                   10000000     coredll:COREDLL.dll
 0000:fffd2000       .debug$S                   10000000     msvcrt:MSVCRT.dll
 0000:fffd2000       .debug$S                   10000000     msvcrt:MSVCRT.dll
 0000:fffd2000       .debug$S                   10000000     coredll:COREDLL.dll
 0000:fffd2000       .debug$S                   10000000     coredll:COREDLL.dll
 0000:fffd2000       .debug$S                   10000000     coredll:COREDLL.dll
 0000:fffd2000       .debug$S                   10000000     coredll:COREDLL.dll
 0000:fffd2000       .debug$S                   10000000     coredll:COREDLL.dll
 0000:fffd2000       .debug$S                   10000000     coredll:COREDLL.dll
 0000:fffd2000       .debug$S                   10000000     Mmtimer:MMTimer.dll
 0000:fffd2000       .debug$S                   10000000     coredll:COREDLL.dll
 0000:fffd2000       .debug$S                   10000000     coredll:COREDLL.dll
 0000:fffd2000       .debug$S                   10000000     coredll:COREDLL.dll
 0000:fffd2000       .debug$S                   10000000     coredll:COREDLL.dll
 0000:fffd2000       .debug$S                   10000000     coredll:COREDLL.dll
 0000:fffd2000       .debug$S                   10000000     coredll:COREDLL.dll
 0000:fffd2000       .debug$S                   10000000     coredll:COREDLL.dll
 0000:fffd2000       .debug$S                   10000000     coredll:COREDLL.dll
 0000:fffd2000       .debug$S                   10000000     coredll:COREDLL.dll
 0000:fffd2000       .debug$S                   10000000     coredll:COREDLL.dll
 0000:fffd2000       .debug$S                   10000000     coredll:COREDLL.dll
 0000:fffd2000       .debug$S                   10000000     coredll:COREDLL.dll
 0000:fffd2000       .debug$S                   10000000     coredll:COREDLL.dll
 0000:fffd2000       .debug$S                   10000000     coredll:COREDLL.dll
 0000:fffd2000       .debug$S                   10000000     coredll:COREDLL.dll
 0000:fffd2000       .debug$S                   10000000     coredll:COREDLL.dll
 0000:fffd2000       .debug$S                   10000000     coredll:COREDLL.dll
 0000:fffd2000       .debug$S                   10000000     coredll:COREDLL.dll
 0000:fffd2000       .debug$S                   10000000     coredll:COREDLL.dll
 0000:fffd2000       .debug$S                   10000000     coredll:COREDLL.dll
 0000:fffd2000       .debug$S                   10000000     coredll:COREDLL.dll
 0000:fffd2000       .debug$S                   10000000     coredll:COREDLL.dll
 0000:fffd2000       .debug$S                   10000000     coredll:COREDLL.dll
 0000:fffd2000       .debug$S                   10000000     coredll:COREDLL.dll
 0000:fffd2000       .debug$S                   10000000     coredll:COREDLL.dll
 0000:fffd2000       .debug$S                   10000000     coredll:COREDLL.dll
 0000:fffd2000       .debug$S                   10000000     coredll:COREDLL.dll
 0000:fffd2000       .debug$S                   10000000     coredll:COREDLL.dll
 0000:fffd2000       .debug$S                   10000000     coredll:COREDLL.dll
 0000:fffd2000       .debug$S                   10000000     coredll:COREDLL.dll
 0001:00000038       _szIrpMajFuncDesc          10001038     mdd.obj
 0001:000000a8       _szPnpMnFuncDesc           100010a8     mdd.obj
 0001:00000108       _szSystemPowerState        10001108     mdd.obj
 0001:00000128       _szDevicePowerState        10001128     mdd.obj
 0001:00000140       _szIoctlDesc               10001140     mdd.obj
 0001:00003f58       _szIrpMajFuncDesc          10004f58     ftdi_ser.obj
 0001:00003fc8       _szPnpMnFuncDesc           10004fc8     ftdi_ser.obj
 0001:00004028       _szSystemPowerState        10005028     ftdi_ser.obj
 0001:00004048       _szDevicePowerState        10005048     ftdi_ser.obj
 0001:00004060       _szIoctlDesc               10005060     ftdi_ser.obj
 0001:000061f0       _szIrpMajFuncDesc          100071f0     ftdi_utils.obj
 0001:00006260       _szPnpMnFuncDesc           10007260     ftdi_utils.obj
 0001:000062c0       _szSystemPowerState        100072c0     ftdi_utils.obj
 0001:000062e0       _szDevicePowerState        100072e0     ftdi_utils.obj
 0001:000062f8       _szIoctlDesc               100072f8     ftdi_utils.obj
 0001:000069b0       _szIrpMajFuncDesc          100079b0     ftdi_usb.obj
 0001:00006a20       _szPnpMnFuncDesc           10007a20     ftdi_usb.obj
 0001:00006a80       _szSystemPowerState        10007a80     ftdi_usb.obj
 0001:00006aa0       _szDevicePowerState        10007aa0     ftdi_usb.obj
 0001:00006ab8       _szIoctlDesc               10007ab8     ftdi_usb.obj
 0001:00008678       _szIrpMajFuncDesc          10009678     BUSBDBG.obj
 0001:000086e8       _szPnpMnFuncDesc           100096e8     BUSBDBG.obj
 0001:00008748       _szSystemPowerState        10009748     BUSBDBG.obj
 0001:00008768       _szDevicePowerState        10009768     BUSBDBG.obj
 0001:00008780       _szIoctlDesc               10009780     BUSBDBG.obj
 0001:000089d8       _szIrpMajFuncDesc          100099d8     BULK_IN.obj
 0001:00008a48       _szPnpMnFuncDesc           10009a48     BULK_IN.obj
 0001:00008aa8       _szSystemPowerState        10009aa8     BULK_IN.obj
 0001:00008ac8       _szDevicePowerState        10009ac8     BULK_IN.obj
 0001:00008ae0       _szIoctlDesc               10009ae0     BULK_IN.obj
 0001:0000d878       _acSections                1000e878     INFParse.obj
 0001:0000d9b0       _szIrpMajFuncDesc          1000e9b0     EMUL.obj
 0001:0000da20       _szPnpMnFuncDesc           1000ea20     EMUL.obj
 0001:0000da80       _szSystemPowerState        1000ea80     EMUL.obj
 0001:0000daa0       _szDevicePowerState        1000eaa0     EMUL.obj
 0001:0000dab8       _szIoctlDesc               1000eab8     EMUL.obj
 0001:0000f5c5       _SerialDispatchThread      100105c5 f   mdd.obj
 0001:00013021       $LN248                     10014021     mdd.obj
 0001:00013081       $LN214                     10014081     mdd.obj
 0001:00013b4a       _SerInit                   10014b4a f   ftdi_ser.obj
 0001:00013dad       _SerPostInit               10014dad f   ftdi_ser.obj
 0001:00013dbe       _SerDeinit                 10014dbe f   ftdi_ser.obj
 0001:00013e9d       _SerOpen                   10014e9d f   ftdi_ser.obj
 0001:00013f7b       _SerClose                  10014f7b f   ftdi_ser.obj
 0001:00015af8       _SerPowerOn                10016af8 f   ftdi_ser.obj
 0001:00015afc       _SerPowerOff               10016afc f   ftdi_ser.obj
 0001:0001688e       _FTDIEventThread           1001788e f   ftdi_ser.obj
 0001:00017c45       _SerEnableIR               10018c45 f   ftdi_ser.obj
 0001:00017c49       _SerDisableIR              10018c49 f   ftdi_ser.obj
 0001:00017c4d       _SerGetCommProperties      10018c4d f   ftdi_ser.obj
 0001:00021736       ?GetClientDriverName@@YAHPAGH@Z 10022736 f   usbddrv.obj
 0001:00025778       __sehtable$_SerXmitComChar 10026778     ftdi_ser.obj
 0001:00025798       __sehtable$_SerPurgeComm   10026798     ftdi_ser.obj
 0001:000257b8       __sehtable$_SerRxIntr      100267b8     ftdi_ser.obj
 0001:000257d8       __sehtable$_SerIoctl       100267d8     ftdi_ser.obj
 0001:00025848       __sehtable$?LoadRegisteredDriver@@YAHPAUHKEY__@@PAUSDevice@@PBU_USB_INTERFACE@@PAHPBU_USB_DRIVER_SETTINGS@@@Z 10026848     usbd.obj
 0001:00025868       __sehtable$?ReferenceTransferHandle@@YAHPAUSTransfer@@@Z 10026868     usbd.obj
 0001:00025888       __sehtable$?ValidateDeviceHandle@@YAHPAUSDevice@@@Z 10026888     usbd.obj
 0001:000258a8       __sehtable$?ReferencePipeHandle@@YAHPAUSPipe@@@Z 100268a8     usbd.obj
 0001:000258c8       __sehtable$?InstallClientDriver@@YAHPBG@Z 100268c8     usbd.obj
 0001:00025a94       .idata$6                   10026a94     coredll:COREDLL.dll
 0001:00025aae       .idata$6                   10026aae     Mmtimer:MMTimer.dll
 0001:00025aba       .idata$6                   10026aba     msvcrt:MSVCRT.dll
 0001:00025ad0       .edata                     10026ad0     ftdi_ser.exp
 0001:00025af8       rgpv                       10026af8     ftdi_ser.exp
 0001:00025b2c       rgszName                   10026b2c     ftdi_ser.exp
 0001:00025b60       rgwOrd                     10026b60     ftdi_ser.exp
 0001:00025b7a       szName                     10026b7a     ftdi_ser.exp
 0001:00025b87       $N00001                    10026b87     ftdi_ser.exp
 0001:00025b91       $N00002                    10026b91     ftdi_ser.exp
 0001:00025b9c       $N00003                    10026b9c     ftdi_ser.exp
 0001:00025baa       $N00004                    10026baa     ftdi_ser.exp
 0001:00025bb3       $N00005                    10026bb3     ftdi_ser.exp
 0001:00025bbc       $N00006                    10026bbc     ftdi_ser.exp
 0001:00025bca       $N00007                    10026bca     ftdi_ser.exp
 0001:00025bd6       $N00008                    10026bd6     ftdi_ser.exp
 0001:00025bdf       $N00009                    10026bdf     ftdi_ser.exp
 0001:00025be8       $N00010                    10026be8     ftdi_ser.exp
 0001:00025bf2       $N00011                    10026bf2     ftdi_ser.exp
 0001:00025c02       $N00012                    10026c02     ftdi_ser.exp
 0001:00025c13       $N00013                    10026c13     ftdi_ser.exp
 0002:000005a4       _gszDriverPrefix           100275a4     ftdi_usb.obj
 0002:000005ac       _g_DriverSettings          100275ac     ftdi_usb.obj
 0002:000005d8       _aszTypeStrings            100275d8     usbddrv.obj
 0002:00000610       _gc_UsbFuncs               10027610     usbd.obj
 0002:000006e0       _GlobalSerialHeadNumber    100276e0     mdd.obj
 0002:000006e8       _GlobalSerialHeadNumber    100276e8     ftdi_ser.obj
 0002:000006ec       _GlobalSerialHeadNumber    100276ec     ftdi_usb.obj
 0002:000006f0       _gLocalAllocCount          100276f0     BUSBDBG.obj
 0002:00000708       _gcPortName                10027708     INFParse.obj
 0002:00000b08       ?pmpf@?1??GetNextVIDPID@@9@4PAVMultiPlatformFile@@A 10027b08     INFParse.obj
 0002:00000b0c       ?bUsed@?1??WriteToDebugFile@@9@9 10027b0c     ftdi_debug.obj
 0003:00000060       $R000000                   10029060     ftdi_ser.res
